 usbfn

 Timestamp is 4fb05c6f (Mon May 14 13:14:23 2012)

 Preferred load address is 10000000

 Start         Length     Name                   Class
 0001:00000000 00000004H .CRT$XCA                CODE
 0001:00000004 00000004H .CRT$XCU                CODE
 0001:00000008 00000004H .CRT$XCZ                CODE
 0001:0000000c 00000004H .CRT$XIA                CODE
 0001:00000010 00000004H .CRT$XIZ                CODE
 0001:00000014 00000004H .CRT$XPA                CODE
 0001:00000018 00000004H .CRT$XPZ                CODE
 0001:0000001c 00000004H .CRT$XTA                CODE
 0001:00000020 00000004H .CRT$XTZ                CODE
 0001:00000030 0000cc5eH .rdata                  CODE
 0001:0000cc90 00000022H .rdata$debug            CODE
 0001:0000ccb4 000394dcH .text                   CODE
 0001:00046190 00000090H .text$yc                CODE
 0001:00046220 00000018H .text$yd                CODE
 0001:00046238 00000134H .xdata                  CODE
 0001:0004636c 0000003cH .idata$2                CODE
 0001:000463a8 00000014H .idata$3                CODE
 0001:000463bc 000001ccH .idata$4                CODE
 0001:00046588 00000068H .idata$6                CODE
 0001:000465f0 000000f6H .edata                  CODE
 0002:00000000 000001ccH .idata$5                DATA
 0002:000001d0 0000045cH .data                   DATA
 0002:00000640 000000a0H .bss                    DATA
 0003:00000000 000018c8H .pdata                  DATA

  Address         Publics by Value              Rva+Base       Lib:Object

 0000:00000000       ___safe_se_handler_count   00000000     <absolute>
 0000:00000000       ___safe_se_handler_table   00000000     <absolute>
 0001:00000000       __xc_a                     10001000     corelib0:crt0init.obj
 0001:00000008       __xc_z                     10001008     corelib0:crt0init.obj
 0001:0000000c       __xi_a                     1000100c     corelib0:crt0init.obj
 0001:00000010       __xi_z                     10001010     corelib0:crt0init.obj
 0001:00000014       __xp_a                     10001014     corelib0:crt0init.obj
 0001:00000018       __xp_z                     10001018     corelib0:crt0init.obj
 0001:0000001c       __xt_a                     1000101c     corelib0:crt0init.obj
 0001:00000020       __xt_z                     10001020     corelib0:crt0init.obj
 0001:000000e0       ??_C@_1DA@DCCNOILH@?$AAH?$AAi?$AAg?$AAh?$AA?5?$AAs?$AAp?$AAe?$AAe?$AAd?$AA?5?$AAU?$AAS?$AAB?$AA?5?$AAc?$AAl?$AAi?$AAe?$AAn?$AAt?$AA?$AN?$AA?6?$AA?$AA@ 100010e0     hwinit.obj
 0001:00000110       ??_C@_1DK@PNDOGEED@?$AAI?$AAn?$AAi?$AAt?$AAi?$AAa?$AAl?$AAi?$AAz?$AAe?$AAT?$AAr?$AAa?$AAn?$AAs?$AAc?$AAe?$AAi?$AAv?$AAe?$AAr?$AA?5?$AAd?$AAo?$AAn?$AAe?$AA?$AN?$AA?6?$AA?$AA@ 10001110     hwinit.obj
 0001:00000150       ??_C@_1FK@FNONLNGN@?$AA?$CF?$AAs?$AA?3?$AA?5?$AAD?$AAE?$AAB?$AAU?$AAG?$AAC?$AAH?$AAK?$AA?5?$AAf?$AAa?$AAi?$AAl?$AAe?$AAd?$AA?5?$AAi?$AAn?$AA?5?$AAf?$AAi?$AAl?$AAe?$AA?5?$AA?$CF?$AAs?$AA?5?$AAa@ 10001150     hwinit.obj
 0001:000001b0       ??_C@_1JA@JMHFFEM@?$AAC?$AA?3?$AA?2?$AAW?$AAI?$AAN?$AAC?$AAE?$AAR?$AAO?$AAO?$AAT?$AAS?$AA?2?$AAT?$AAo?$AAp?$AAa?$AAz?$AA?2?$AAW?$AAI?$AAN?$AAC?$AAE?$AA6?$AA0?$AA0?$AA?2?$AAP?$AAL?$AAA@ 100011b0     hwinit.obj
 0001:00000240       ??_C@_1FA@IDGNLIJP@?$AAI?$AAS?$AAP?$AA1?$AA3?$AA0?$AA1?$AA?5?$AAF?$AAu?$AAl?$AAl?$AA?5?$AAS?$AAp?$AAe?$AAe?$AAd?$AA?5?$AAi?$AAs?$AA?5?$AAn?$AAo?$AAt?$AA?5?$AAi?$AAm?$AAp?$AAl?$AAe?$AAm@ 10001240     hwinit.obj
 0001:00000320       ??_C@_1GM@KKEMFHME@?$AA?9?$AAP?$AAo?$AAr?$AAt?$AA?$CI?$AA?$CF?$AAd?$AA?$CJ?$AA?3?$AAB?$AAS?$AAP?$AAU?$AAS?$AAB?$AAC?$AAl?$AAo?$AAc?$AAk?$AAC?$AAr?$AAe?$AAa?$AAt?$AAe?$AAF?$AAi?$AAl?$AAe?$AAM@ 10001320     i_usbclock.obj
 0001:00000390       ??_C@_1GO@KPNBKEAO@?$AAP?$AAo?$AAr?$AAt?$AA?$CI?$AA?$CF?$AAd?$AA?$CJ?$AA?3?$AAB?$AAS?$AAP?$AAU?$AAS?$AAB?$AAC?$AAl?$AAo?$AAc?$AAk?$AAC?$AAr?$AAe?$AAa?$AAt?$AAe?$AAF?$AAi?$AAl?$AAe?$AAM?$AAa@ 10001390     i_usbclock.obj
 0001:00000400       ??_C@_1FE@GNDFGBM@?$AAP?$AAo?$AAr?$AAt?$AA?$CI?$AA?$CF?$AAd?$AA?$CJ?$AA?5?$AAO?$AAp?$AAe?$AAn?$AA?5?$AAe?$AAx?$AAi?$AAs?$AAt?$AAi?$AAn?$AAg?$AA?5?$AAU?$AAS?$AAB?$AA_?$AAC?$AAL?$AAO?$AAC?$AAK@ 10001400     i_usbclock.obj
 0001:00000458       ??_C@_1FI@ECFJDMMH@?$AAP?$AAo?$AAr?$AAt?$AA?$CI?$AA?$CF?$AAd?$AA?$CJ?$AA?3?$AAF?$AAi?$AAr?$AAs?$AAt?$AA?5?$AAt?$AAo?$AA?5?$AAc?$AAr?$AAe?$AAa?$AAt?$AAe?$AA?5?$AAU?$AAS?$AAB?$AA_?$AAC?$AAL?$AAO@ 10001458     i_usbclock.obj
 0001:000004b0       ??_C@_1FC@NEMMIEIK@?$AAF?$AAa?$AAi?$AAl?$AAu?$AAr?$AAe?$AA?5?$AAt?$AAo?$AA?5?$AAC?$AAr?$AAe?$AAa?$AAt?$AAe?$AA?5?$AAF?$AAi?$AAl?$AAe?$AA?5?$AAM?$AAa?$AAp?$AAp?$AAi?$AAn?$AAg?$AA?5?$AAf@ 100014b0     i_usbclock.obj
 0001:00000504       ??_C@_1CC@BJPGGDNC@?$AAU?$AAS?$AAB?$AA_?$AAC?$AAL?$AAO?$AAC?$AAK?$AA_?$AAG?$AAA?$AAT?$AAI?$AAN?$AAG?$AA?$AA@ 10001504     i_usbclock.obj
 0001:00000528       ??_C@_1EG@CGIBPELK@?$AAP?$AAo?$AAr?$AAt?$AA?$CI?$AA?$CF?$AAd?$AA?$CJ?$AA?3?$AAB?$AAS?$AAP?$AAU?$AAS?$AAB?$AAC?$AAr?$AAe?$AAa?$AAt?$AAe?$AAF?$AAi?$AAl?$AAe?$AAM?$AAa?$AAp?$AAp?$AAi?$AAn?$AAg@ 10001528     i_usbclock.obj
 0001:00000570       ??_C@_1IC@FDNBOOON@?$AAP?$AAo?$AAr?$AAt?$AA?$CI?$AA?$CF?$AAd?$AA?$CJ?$AA?5?$AA?9?$AA?5?$AAU?$AAS?$AAB?$AAC?$AAl?$AAo?$AAc?$AAk?$AAC?$AAa?$AAn?$AAC?$AAl?$AAo?$AAc?$AAk?$AAG?$AAa?$AAt?$AAi?$AAn@ 10001570     i_usbclock.obj
 0001:000005f4       ??_C@_1DA@CLIJDNJA@?$AAU?$AAS?$AAB?$AAC?$AAl?$AAo?$AAc?$AAk?$AA?5?$AA?$CF?$AAs?$AA?5?$AAr?$AAe?$AAt?$AAu?$AAr?$AAn?$AA?5?$AA?$CF?$AAd?$AA?$AN?$AA?6?$AA?$AA@ 100015f4     i_usbclock.obj
 0001:00000624       ??_C@_1M@HCOOECOK@?$AAF?$AAA?$AAL?$AAS?$AAE?$AA?$AA@ 10001624     i_usbclock.obj
 0001:00000630       ??_C@_19ELAAHEEL@?$AAT?$AAR?$AAU?$AAE?$AA?$AA@ 10001630     i_usbclock.obj
 0001:00000640       ??_C@_1FM@HIIFJIHO@?$AAD?$AAi?$AAs?$AAa?$AAb?$AAl?$AAe?$AA?5?$AAF?$AAa?$AAi?$AAl?$AA?0?$AA?5?$AAN?$AAe?$AAe?$AAd?$AA?5?$AAt?$AAo?$AA?5?$AAc?$AAh?$AAe?$AAc?$AAk?$AA?0?$AA?5?$AAc?$AAu?$AAr@ 10001640     i_usbclock.obj
 0001:000006a0       ??_C@_1FK@HJNHKCPL@?$AAE?$AAn?$AAa?$AAb?$AAl?$AAe?$AA?5?$AAF?$AAa?$AAi?$AAl?$AA?0?$AA?5?$AAN?$AAe?$AAe?$AAd?$AA?5?$AAt?$AAo?$AA?5?$AAc?$AAh?$AAe?$AAc?$AAk?$AA?0?$AA?5?$AAc?$AAu?$AAr?$AAr@ 100016a0     i_usbclock.obj
 0001:00000700       ??_C@_1FI@MBIBGPGK@?$AAU?$AAS?$AAB?$AAC?$AAl?$AAo?$AAc?$AAk?$AAS?$AAe?$AAt?$AA?3?$AA?5?$AAD?$AAD?$AAK?$AAC?$AAl?$AAo?$AAc?$AAk?$AAS?$AAe?$AAt?$AAG?$AAa?$AAt?$AAi?$AAn?$AAg?$AAM?$AAo@ 10001700     i_usbclock.obj
 0001:00000758       ??_C@_1FC@PCOPMCOB@?$AAU?$AAS?$AAB?$AAC?$AAl?$AAo?$AAc?$AAk?$AAS?$AAe?$AAt?$AA?3?$AA?5?$AAD?$AAD?$AAK?$AAC?$AAl?$AAo?$AAc?$AAk?$AAC?$AAo?$AAn?$AAf?$AAi?$AAg?$AAB?$AAa?$AAu?$AAd?$AA?5@ 10001758     i_usbclock.obj
 0001:00000840       ??_C@_1EK@IBIELIGM@?$AAC?$AAa?$AAn?$AAn?$AAo?$AAt?$AA?5?$AAo?$AAb?$AAt?$AAa?$AAi?$AAn?$AA?5?$AAt?$AAh?$AAe?$AA?5?$AAs?$AAi?$AAl?$AAi?$AAc?$AAo?$AAn?$AA?5?$AAv?$AAe?$AAr?$AAs?$AAi?$AAo@ 10001840     i_usbutils.obj
 0001:0000088c       ??_C@_1CI@OHCJFJPM@?$AAE?$AAR?$AAR?$AAO?$AAR?$AA?3?$AA?5?$AA?$CF?$AAs?$AA?5?$AAl?$AAi?$AAn?$AAe?$AA?5?$AA?$CF?$AAd?$AA?3?$AA?5?$AA?$AA@ 1000188c     i_usbutils.obj
 0001:000008b4       ??_C@_1DE@DKKKIJG@?$AA?4?$AA?2?$AA?4?$AA?4?$AA?2?$AAU?$AAS?$AAB?$AAC?$AAo?$AAm?$AAm?$AAo?$AAn?$AA?2?$AAU?$AAs?$AAb?$AAU?$AAt?$AAi?$AAl?$AAs?$AA?4?$AAc?$AA?$AA@ 100018b4     i_usbutils.obj
 0001:000008e8       ??_C@_1NE@HMEFNKHG@?$AAC?$AA?3?$AA?2?$AAW?$AAI?$AAN?$AAC?$AAE?$AAR?$AAO?$AAO?$AAT?$AAS?$AA?2?$AAT?$AAo?$AAp?$AAa?$AAz?$AA?2?$AAW?$AAI?$AAN?$AAC?$AAE?$AA6?$AA0?$AA0?$AA?2?$AAP?$AAL?$AAA@ 100018e8     usb_ufnmddbase_common_topaz_v1:ufnmdd.obj
 0001:000009bc       ??_C@_19PKICIIJD@?$AAh?$AAi?$AAg?$AAh?$AA?$AA@ 100019bc     usb_ufnmddbase_common_topaz_v1:ufnmdd.obj
 0001:000009c8       ??_C@_19CKPKPLNA@?$AAf?$AAu?$AAl?$AAl?$AA?$AA@ 100019c8     usb_ufnmddbase_common_topaz_v1:ufnmdd.obj
 0001:000009d4       ??_C@_1BA@KDMGPDJH@?$AAu?$AAn?$AAk?$AAn?$AAo?$AAw?$AAn?$AA?$AA@ 100019d4     usb_ufnmddbase_common_topaz_v1:ufnmdd.obj
 0001:000009e4       ??_C@_1BA@PLOOFDPK@?$AA?$CF?$AAs?$AA?5?$AA?9?$AA?9?$AA?$AN?$AA?6?$AA?$AA@ 100019e4     usb_ufnmddbase_common_topaz_v1:ufnmdd.obj
 0001:000009f4       ??_C@_1CA@DHEHDNOA@?$AA?$CF?$AAs?$AA?5?$AAE?$AAx?$AAc?$AAe?$AAp?$AAt?$AAi?$AAo?$AAn?$AA?$CB?$AA?$AN?$AA?6?$AA?$AA@ 100019f4     usb_ufnmddbase_common_topaz_v1:ufnmdd.obj
 0001:00000a14       ??_C@_1CO@ICJCBGDC@?$AA?$CF?$AAs?$AA?5?$AAD?$AAe?$AAv?$AAi?$AAc?$AAe?$AA?5?$AAr?$AAe?$AAg?$AAi?$AAs?$AAt?$AAe?$AAr?$AAe?$AAd?$AA?$AN?$AA?6?$AA?$AA@ 10001a14     usb_ufnmddbase_common_topaz_v1:ufnmdd.obj
 0001:00000a48       ??_C@_1IE@OJIPOPM@?$AAR?$AAe?$AAg?$AAi?$AAs?$AAt?$AAe?$AAr?$AAD?$AAe?$AAv?$AAi?$AAc?$AAe?$AA?5?$AAf?$AAa?$AAi?$AAl?$AAe?$AAd?$AA?5?$AAt?$AAo?$AA?5?$AAa?$AAl?$AAl?$AAo?$AAc?$AAa?$AAt@ 10001a48     usb_ufnmddbase_common_topaz_v1:ufnmdd.obj
 0001:00000ad0       ??_C@_1EA@DBPBMCMC@?$AA?$CF?$AAs?$AA?5?$AAD?$AAe?$AAv?$AAi?$AAc?$AAe?$AA?5?$AAi?$AAs?$AA?5?$AAs?$AAt?$AAi?$AAl?$AAl?$AA?5?$AAr?$AAe?$AAg?$AAi?$AAs?$AAt?$AAe?$AAr?$AAe?$AAd?$AA?$AN?$AA?6?$AA?$AA@ 10001ad0     usb_ufnmddbase_common_topaz_v1:ufnmdd.obj
 0001:00000b10       ??_C@_1DK@BCODDEFN@?$AA?$CF?$AAs?$AA?5?$AAD?$AAe?$AAv?$AAi?$AAc?$AAe?$AA?5?$AAi?$AAs?$AA?5?$AAs?$AAt?$AAi?$AAl?$AAl?$AA?5?$AAr?$AAu?$AAn?$AAn?$AAi?$AAn?$AAg?$AA?$AN?$AA?6?$AA?$AA@ 10001b10     usb_ufnmddbase_common_topaz_v1:ufnmdd.obj
 0001:00000b4c       ??_C@_1CO@HCBPDHLK@?$AA?$CF?$AAs?$AA?5?$AAI?$AAn?$AAv?$AAa?$AAl?$AAi?$AAd?$AA?5?$AAp?$AAa?$AAr?$AAa?$AAm?$AAe?$AAt?$AAe?$AAr?$AA?$AN?$AA?6?$AA?$AA@ 10001b4c     usb_ufnmddbase_common_topaz_v1:ufnmdd.obj
 0001:00000b7c       ??_C@_1DG@OBEFBEAF@?$AA?$CF?$AAs?$AA?5?$AAI?$AAn?$AAv?$AAa?$AAl?$AAi?$AAd?$AA?5?$AAd?$AAe?$AAv?$AAi?$AAc?$AAe?$AA?5?$AAh?$AAa?$AAn?$AAd?$AAl?$AAe?$AA?$AN?$AA?6?$AA?$AA@ 10001b7c     usb_ufnmddbase_common_topaz_v1:ufnmdd.obj
 0001:00000bb4       ??_C@_1BA@DAJPCKDK@?$AA?$CF?$AAs?$AA?5?$AA?$CL?$AA?$CL?$AA?$AN?$AA?6?$AA?$AA@ 10001bb4     usb_ufnmddbase_common_topaz_v1:ufnmdd.obj
 0001:00000bc8       ??_C@_1EA@JFAPMBLB@?$AAU?$AAs?$AAb?$AAF?$AAn?$AAM?$AAd?$AAd?$AA?$CB?$AAU?$AAf?$AAn?$AAM?$AAd?$AAd?$AA_?$AAR?$AAe?$AAg?$AAi?$AAs?$AAt?$AAe?$AAr?$AAD?$AAe?$AAv?$AAi?$AAc?$AAe?$AA?3?$AA?$AA@ 10001bc8     usb_ufnmddbase_common_topaz_v1:ufnmdd.obj
 0001:00000c08       ??_C@_1DO@IHPGBGBD@?$AAU?$AAs?$AAb?$AAF?$AAn?$AAM?$AAd?$AAd?$AA?$CB?$AAR?$AAe?$AAs?$AAe?$AAt?$AAP?$AAi?$AAp?$AAe?$AAS?$AAt?$AAa?$AAt?$AAu?$AAs?$AAT?$AAa?$AAb?$AAl?$AAe?$AA?3?$AA?$AA@ 10001c08     usb_ufnmddbase_common_topaz_v1:ufnmdd.obj
 0001:00000c48       ??_C@_1EC@NLLFBLEO@?$AA?$CF?$AAs?$AA?5?$AAF?$AAu?$AAn?$AAc?$AAt?$AAi?$AAo?$AAn?$AA?5?$AAc?$AAo?$AAn?$AAt?$AAr?$AAo?$AAl?$AAl?$AAe?$AAr?$AA?5?$AAr?$AAu?$AAn?$AAn?$AAi?$AAn?$AAg?$AA?$AN?$AA?6@ 10001c48     usb_ufnmddbase_common_topaz_v1:ufnmdd.obj
 0001:00000c8c       ??_C@_1DO@IKKDOHHI@?$AA?$CF?$AAs?$AA?5?$AAC?$AAo?$AAu?$AAl?$AAd?$AA?5?$AAn?$AAo?$AAt?$AA?5?$AAi?$AAn?$AAi?$AAt?$AA?5?$AAe?$AAn?$AAd?$AAp?$AAo?$AAi?$AAn?$AAt?$AA?5?$AA0?$AA?$AN?$AA?6?$AA?$AA@ 10001c8c     usb_ufnmddbase_common_topaz_v1:ufnmdd.obj
 0001:00000cd0       ??_C@_1EI@NFLGNK@?$AA?$CF?$AAs?$AA?5?$AAD?$AAe?$AAv?$AAi?$AAc?$AAe?$AA?5?$AAh?$AAa?$AAs?$AA?5?$AAn?$AAo?$AAt?$AA?5?$AAb?$AAe?$AAe?$AAn?$AA?5?$AAr?$AAe?$AAg?$AAi?$AAs?$AAt?$AAe?$AAr?$AAe@ 10001cd0     usb_ufnmddbase_common_topaz_v1:ufnmdd.obj
 0001:00000d18       ??_C@_1CO@CJALBPBG@?$AAU?$AAs?$AAb?$AAF?$AAn?$AAM?$AAd?$AAd?$AA?$CB?$AAU?$AAf?$AAn?$AAM?$AAd?$AAd?$AA_?$AAS?$AAt?$AAa?$AAr?$AAt?$AA?3?$AA?$AA@ 10001d18     usb_ufnmddbase_common_topaz_v1:ufnmdd.obj
 0001:00000d48       ??_C@_1BA@LEPJIIOK@?$AAU?$AAn?$AAk?$AAn?$AAo?$AAw?$AAn?$AA?$AA@ 10001d48     usb_ufnmddbase_common_topaz_v1:ufnmdd.obj
 0001:00000d58       ??_C@_1CC@DAFIFOLF@?$AAU?$AAs?$AAb?$AAF?$AAn?$AAM?$AAd?$AAd?$AA?$CB?$AAD?$AAo?$AAS?$AAt?$AAo?$AAp?$AA?3?$AA?$AA@ 10001d58     usb_ufnmddbase_common_topaz_v1:ufnmdd.obj
 0001:00000d7c       ??_C@_1DG@PFKKLBEK@?$AA?$CF?$AAs?$AA?5?$AAD?$AAe?$AAv?$AAi?$AAc?$AAe?$AA?5?$AAi?$AAs?$AA?5?$AAn?$AAo?$AAt?$AA?5?$AAr?$AAu?$AAn?$AAn?$AAi?$AAn?$AAg?$AA?$AN?$AA?6?$AA?$AA@ 10001d7c     usb_ufnmddbase_common_topaz_v1:ufnmdd.obj
 0001:00000db4       ??_C@_1CM@NNCLMGGI@?$AAU?$AAs?$AAb?$AAF?$AAn?$AAM?$AAd?$AAd?$AA?$CB?$AAU?$AAf?$AAn?$AAM?$AAd?$AAd?$AA_?$AAS?$AAt?$AAo?$AAp?$AA?3?$AA?$AA@ 10001db4     usb_ufnmddbase_common_topaz_v1:ufnmdd.obj
 0001:00000de0       ??_C@_1DM@BMJFBOJB@?$AA?$CF?$AAs?$AA?5?$AAD?$AAe?$AAv?$AAi?$AAc?$AAe?$AA?5?$AAi?$AAs?$AA?5?$AAn?$AAo?$AAt?$AA?5?$AAr?$AAe?$AAg?$AAi?$AAs?$AAt?$AAe?$AAr?$AAe?$AAd?$AA?$AN?$AA?6?$AA?$AA@ 10001de0     usb_ufnmddbase_common_topaz_v1:ufnmdd.obj
 0001:00000e1c       ??_C@_1DK@DMIOHJGN@?$AAU?$AAs?$AAb?$AAF?$AAn?$AAM?$AAd?$AAd?$AA?$CB?$AAD?$AAo?$AAD?$AAe?$AAr?$AAe?$AAg?$AAi?$AAs?$AAt?$AAe?$AAr?$AAD?$AAe?$AAv?$AAi?$AAc?$AAe?$AA?3?$AA?$AA@ 10001e1c     usb_ufnmddbase_common_topaz_v1:ufnmdd.obj
 0001:00000e58       ??_C@_1EE@DDOEBEJP@?$AAU?$AAs?$AAb?$AAF?$AAn?$AAM?$AAd?$AAd?$AA?$CB?$AAU?$AAf?$AAn?$AAM?$AAd?$AAd?$AA_?$AAD?$AAe?$AAr?$AAe?$AAg?$AAi?$AAs?$AAt?$AAe?$AAr?$AAD?$AAe?$AAv?$AAi?$AAc?$AAe@ 10001e58     usb_ufnmddbase_common_topaz_v1:ufnmdd.obj
 0001:00000e9c       ??_C@_1DE@KNEPIHAP@?$AA?$CF?$AAs?$AA?5?$AAO?$AAp?$AAe?$AAn?$AAe?$AAd?$AA?5?$AAe?$AAn?$AAd?$AAp?$AAo?$AAi?$AAn?$AAt?$AA?5?$AA0?$AAx?$AA?$CF?$AAx?$AA?$AN?$AA?6?$AA?$AA@ 10001e9c     usb_ufnmddbase_common_topaz_v1:ufnmdd.obj
 0001:00000ed0       ??_C@_1EC@GJMJADBJ@?$AA?$CF?$AAs?$AA?5?$AAE?$AAr?$AAr?$AAo?$AAr?$AA?5?$AAo?$AAp?$AAe?$AAn?$AAi?$AAn?$AAg?$AA?5?$AAe?$AAn?$AAd?$AAp?$AAo?$AAi?$AAn?$AAt?$AA?5?$AA0?$AAx?$AA?$CF?$AAx?$AA?$AN?$AA?6@ 10001ed0     usb_ufnmddbase_common_topaz_v1:ufnmdd.obj
 0001:00000f18       ??_C@_1EK@NMABJOCF@?$AA?$CF?$AAs?$AA?5?$AAI?$AAn?$AAv?$AAa?$AAl?$AAi?$AAd?$AA?5?$AAe?$AAn?$AAd?$AAp?$AAo?$AAi?$AAn?$AAt?$AA?5?$AAa?$AAd?$AAd?$AAr?$AAe?$AAs?$AAs?$AA?5?$AA?$DN?$AA?5?$AA0?$AAx@ 10001f18     usb_ufnmddbase_common_topaz_v1:ufnmdd.obj
 0001:00000f64       ??_C@_1DG@JAIKGGKD@?$AA?$CF?$AAs?$AA?5?$AAD?$AAe?$AAv?$AAi?$AAc?$AAe?$AA?5?$AAn?$AAo?$AAt?$AA?5?$AAr?$AAe?$AAg?$AAi?$AAs?$AAt?$AAe?$AAr?$AAe?$AAd?$AA?$AN?$AA?6?$AA?$AA@ 10001f64     usb_ufnmddbase_common_topaz_v1:ufnmdd.obj
 0001:00000f9c       ??_C@_1DE@FFGHHBMF@?$AAU?$AAs?$AAb?$AAF?$AAn?$AAM?$AAd?$AAd?$AA?$CB?$AAU?$AAf?$AAn?$AAM?$AAd?$AAd?$AA_?$AAO?$AAp?$AAe?$AAn?$AAP?$AAi?$AAp?$AAe?$AA?3?$AA?$AA@ 10001f9c     usb_ufnmddbase_common_topaz_v1:ufnmdd.obj
 0001:00000fd0       ??_C@_1FG@KPDPELLH@?$AA?$CF?$AAs?$AA?5?$AAC?$AAa?$AAn?$AAn?$AAo?$AAt?$AA?5?$AAc?$AAl?$AAo?$AAs?$AAe?$AA?5?$AAe?$AAn?$AAd?$AAp?$AAo?$AAi?$AAn?$AAt?$AA?5?$AA0?$AA?5?$AAp?$AAi?$AAp?$AAe?$AA?5@ 10001fd0     usb_ufnmddbase_common_topaz_v1:ufnmdd.obj
 0001:00001028       ??_C@_1DG@JBCOLMIG@?$AAU?$AAs?$AAb?$AAF?$AAn?$AAM?$AAd?$AAd?$AA?$CB?$AAU?$AAf?$AAn?$AAM?$AAd?$AAd?$AA_?$AAC?$AAl?$AAo?$AAs?$AAe?$AAP?$AAi?$AAp?$AAe?$AA?3?$AA?$AA@ 10002028     usb_ufnmddbase_common_topaz_v1:ufnmdd.obj
 0001:00001060       ??_C@_1CG@FFEEFBAB@?$AA?$CF?$AAs?$AA?5?$AAB?$AAa?$AAd?$AA?5?$AAp?$AAa?$AAr?$AAa?$AAm?$AAe?$AAt?$AAe?$AAr?$AA?$AN?$AA?6?$AA?$AA@ 10002060     usb_ufnmddbase_common_topaz_v1:ufnmdd.obj
 0001:00001088       ??_C@_1EG@BBBNGFOC@?$AAU?$AAs?$AAb?$AAF?$AAn?$AAM?$AAd?$AAd?$AA?$CB?$AAU?$AAf?$AAn?$AAM?$AAd?$AAd?$AA_?$AAG?$AAe?$AAt?$AAT?$AAr?$AAa?$AAn?$AAs?$AAf?$AAe?$AAr?$AAS?$AAt?$AAa?$AAt?$AAu@ 10002088     usb_ufnmddbase_common_topaz_v1:ufnmdd.obj
 0001:000010d0       ??_C@_1DO@EGMDBLDE@?$AAU?$AAs?$AAb?$AAF?$AAn?$AAM?$AAd?$AAd?$AA?$CB?$AAU?$AAf?$AAn?$AAM?$AAd?$AAd?$AA_?$AAA?$AAb?$AAo?$AAr?$AAt?$AAT?$AAr?$AAa?$AAn?$AAs?$AAf?$AAe?$AAr?$AA?3?$AA?$AA@ 100020d0     usb_ufnmddbase_common_topaz_v1:ufnmdd.obj
 0001:00001110       ??_C@_1DO@JOLHACE@?$AAU?$AAs?$AAb?$AAF?$AAn?$AAM?$AAd?$AAd?$AA?$CB?$AAU?$AAf?$AAn?$AAM?$AAd?$AAd?$AA_?$AAC?$AAl?$AAo?$AAs?$AAe?$AAT?$AAr?$AAa?$AAn?$AAs?$AAf?$AAe?$AAr?$AA?3?$AA?$AA@ 10002110     usb_ufnmddbase_common_topaz_v1:ufnmdd.obj
 0001:00001150       ??_C@_1DO@DOHHNABE@?$AAU?$AAs?$AAb?$AAF?$AAn?$AAM?$AAd?$AAd?$AA?$CB?$AAU?$AAf?$AAn?$AAM?$AAd?$AAd?$AA_?$AAI?$AAs?$AAs?$AAu?$AAe?$AAT?$AAr?$AAa?$AAn?$AAs?$AAf?$AAe?$AAr?$AA?3?$AA?$AA@ 10002150     usb_ufnmddbase_common_topaz_v1:ufnmdd.obj
 0001:00001190       ??_C@_1DG@JKHCDPDN@?$AAU?$AAs?$AAb?$AAF?$AAn?$AAM?$AAd?$AAd?$AA?$CB?$AAU?$AAf?$AAn?$AAM?$AAd?$AAd?$AA_?$AAS?$AAt?$AAa?$AAl?$AAl?$AAP?$AAi?$AAp?$AAe?$AA?3?$AA?$AA@ 10002190     usb_ufnmddbase_common_topaz_v1:ufnmdd.obj
 0001:000011c8       ??_C@_1EA@EDKBMKBA@?$AAU?$AAs?$AAb?$AAF?$AAn?$AAM?$AAd?$AAd?$AA?$CB?$AAU?$AAf?$AAn?$AAM?$AAd?$AAd?$AA_?$AAC?$AAl?$AAe?$AAa?$AAr?$AAP?$AAi?$AAp?$AAe?$AAS?$AAt?$AAa?$AAl?$AAl?$AA?3?$AA?$AA@ 100021c8     usb_ufnmddbase_common_topaz_v1:ufnmdd.obj
 0001:00001208       ??_C@_1GI@ODIGBJML@?$AA?$CF?$AAs?$AA?5?$AAR?$AAe?$AAm?$AAo?$AAt?$AAe?$AA?5?$AAw?$AAa?$AAk?$AAe?$AAu?$AAp?$AA?5?$AAh?$AAa?$AAs?$AA?5?$AAn?$AAo?$AAt?$AA?5?$AAb?$AAe?$AAe?$AAn?$AA?5?$AAe?$AAn@ 10002208     usb_ufnmddbase_common_topaz_v1:ufnmdd.obj
 0001:00001270       ??_C@_1EM@HCEGCNMH@?$AAU?$AAs?$AAb?$AAF?$AAn?$AAM?$AAd?$AAd?$AA?$CB?$AAU?$AAf?$AAn?$AAM?$AAd?$AAd?$AA_?$AAI?$AAn?$AAi?$AAt?$AAi?$AAa?$AAt?$AAe?$AAR?$AAe?$AAm?$AAo?$AAt?$AAe?$AAW?$AAa@ 10002270     usb_ufnmddbase_common_topaz_v1:ufnmdd.obj
 0001:000012c0       ??_C@_1FI@EMKCEFGA@?$AAU?$AAs?$AAb?$AAF?$AAn?$AAM?$AAd?$AAd?$AA?$CB?$AAU?$AAf?$AAn?$AAM?$AAd?$AAd?$AA_?$AAS?$AAe?$AAn?$AAd?$AAC?$AAo?$AAn?$AAt?$AAr?$AAo?$AAl?$AAS?$AAt?$AAa?$AAt?$AAu@ 100022c0     usb_ufnmddbase_common_topaz_v1:ufnmdd.obj
 0001:00001318       ??_C@_1EI@NAJPOCMO@?$AA?$CF?$AAs?$AA?5?$AAP?$AAD?$AAD?$AA?5?$AAi?$AAn?$AAt?$AAe?$AAr?$AAf?$AAa?$AAc?$AAe?$AA?5?$AAi?$AAn?$AAf?$AAo?$AA?5?$AAi?$AAs?$AA?5?$AAi?$AAn?$AAv?$AAa?$AAl?$AAi?$AAd@ 10002318     usb_ufnmddbase_common_topaz_v1:ufnmdd.obj
 0001:00001360       ??_C@_1DM@DNLIINMN@?$AA?$CF?$AAs?$AA?5?$AAP?$AAD?$AAD?$AA?5?$AAs?$AAu?$AAp?$AAp?$AAo?$AAr?$AAt?$AAs?$AA?5?$AAs?$AAp?$AAe?$AAe?$AAd?$AAs?$AA?5?$AA0?$AAx?$AA?$CF?$AAx?$AA?$AN?$AA?6?$AA?$AA@ 10002360     usb_ufnmddbase_common_topaz_v1:ufnmdd.obj
 0001:0000139c       ??_C@_1DE@DLKCNCJA@?$AA?$CF?$AAs?$AA?5?$AAP?$AAD?$AAD?$AA?5?$AAh?$AAa?$AAs?$AA?5?$AA?$CF?$AAu?$AA?5?$AAe?$AAn?$AAd?$AAp?$AAo?$AAi?$AAn?$AAt?$AAs?$AA?$AN?$AA?6?$AA?$AA@ 1000239c     usb_ufnmddbase_common_topaz_v1:ufnmdd.obj
 0001:000013d0       ??_C@_1EA@HGEMGKJF@?$AA?$CF?$AAs?$AA?5?$AAP?$AAD?$AAD?$AA?5?$AAi?$AAn?$AAi?$AAt?$AAi?$AAa?$AAl?$AAi?$AAz?$AAa?$AAt?$AAi?$AAo?$AAn?$AA?5?$AAf?$AAa?$AAi?$AAl?$AAe?$AAd?$AA?4?$AA?$AN?$AA?6?$AA?$AA@ 100023d0     usb_ufnmddbase_common_topaz_v1:ufnmdd.obj
 0001:00001410       ??_C@_1GA@GILHOPKB@?$AA?$CF?$AAs?$AA?5?$AAF?$AAa?$AAi?$AAl?$AAe?$AAd?$AA?5?$AAt?$AAo?$AA?5?$AAo?$AAp?$AAe?$AAn?$AA?5?$AAd?$AAe?$AAv?$AAi?$AAc?$AAe?$AA?5?$AAk?$AAe?$AAy?$AA?5?$AA?$CC?$AA?$CF?$AAs@ 10002410     usb_ufnmddbase_common_topaz_v1:ufnmdd.obj
 0001:00001470       ??_C@_1FA@NPBIEJNM@?$AA?$CF?$AAs?$AA?5?$AAF?$AAa?$AAi?$AAl?$AAe?$AAd?$AA?5?$AAt?$AAo?$AA?5?$AAc?$AAr?$AAe?$AAa?$AAt?$AAe?$AA?5?$AAe?$AAv?$AAe?$AAn?$AAt?$AA?4?$AA?5?$AAE?$AAr?$AAr?$AAo?$AAr@ 10002470     usb_ufnmddbase_common_topaz_v1:ufnmdd.obj
 0001:000014c0       ??_C@_1DG@DLKFAJJC@?$AA?$CF?$AAs?$AA?5?$AAn?$AAe?$AAw?$AA?5?$AAf?$AAa?$AAi?$AAl?$AAe?$AAd?$AA?4?$AA?5?$AAE?$AAr?$AAr?$AAo?$AAr?$AA?3?$AA?5?$AA?$CF?$AAd?$AA?$AN?$AA?6?$AA?$AA@ 100024c0     usb_ufnmddbase_common_topaz_v1:ufnmdd.obj
 0001:000014f8       ??_C@_1EE@EDPBGAAJ@?$AA?$CF?$AAs?$AA?5?$AAL?$AAo?$AAc?$AAa?$AAl?$AAA?$AAl?$AAl?$AAo?$AAc?$AA?5?$AAf?$AAa?$AAi?$AAl?$AAe?$AAd?$AA?4?$AA?5?$AAE?$AAr?$AAr?$AAo?$AAr?$AA?3?$AA?5?$AA?$CF?$AAd?$AA?$AN@ 100024f8     usb_ufnmddbase_common_topaz_v1:ufnmdd.obj
 0001:0000153c       ??_C@_1DO@MHFAFBD@?$AA?$CF?$AAs?$AA?5?$AAF?$AAa?$AAi?$AAl?$AAe?$AAd?$AA?5?$AAt?$AAo?$AA?5?$AAo?$AAp?$AAe?$AAn?$AA?5?$AAa?$AAc?$AAt?$AAi?$AAv?$AAe?$AA?5?$AAk?$AAe?$AAy?$AA?$AN?$AA?6?$AA?$AA@ 1000253c     usb_ufnmddbase_common_topaz_v1:ufnmdd.obj
 0001:0000157c       ??_C@_1CG@EPAHDJNK@?$AAU?$AAs?$AAb?$AAF?$AAn?$AAM?$AAd?$AAd?$AA?$CB?$AAU?$AAF?$AAN?$AA_?$AAI?$AAn?$AAi?$AAt?$AA?3?$AA?$AA@ 1000257c     usb_ufnmddbase_common_topaz_v1:ufnmdd.obj
 0001:000015a8       ??_C@_1HI@COPKOFIP@?$AAC?$AA?3?$AA?2?$AAW?$AAI?$AAN?$AAC?$AAE?$AAR?$AAO?$AAO?$AAT?$AAS?$AA?2?$AAT?$AAo?$AAp?$AAa?$AAz?$AA?2?$AAW?$AAI?$AAN?$AAC?$AAE?$AA6?$AA0?$AA0?$AA?2?$AAp?$AAu?$AAb@ 100025a8     usb_ufnmddbase_common_topaz_v1:ufnmdd.obj
 0001:00001620       ??_C@_1CM@NBPACNN@?$AAU?$AAs?$AAb?$AAF?$AAn?$AAM?$AAd?$AAd?$AA?$CB?$AAF?$AAr?$AAe?$AAe?$AAC?$AAo?$AAn?$AAt?$AAe?$AAx?$AAt?$AA?3?$AA?$AA@ 10002620     usb_ufnmddbase_common_topaz_v1:ufnmdd.obj
 0001:00001650       ??_C@_1NA@OPKIGHKO@?$AAc?$AA?3?$AA?2?$AAw?$AAi?$AAn?$AAc?$AAe?$AAr?$AAo?$AAo?$AAt?$AAs?$AA?2?$AAt?$AAo?$AAp?$AAa?$AAz?$AA?2?$AAw?$AAi?$AAn?$AAc?$AAe?$AA6?$AA0?$AA0?$AA?2?$AAp?$AAl?$AAa@ 10002650     usb_ufnmddbase_common_topaz_v1:ufnmdd.obj
 0001:00001720       ??_C@_1DA@GAGBDGJF@?$AAU?$AAs?$AAb?$AAF?$AAn?$AAM?$AAd?$AAd?$AA?$CB?$AAU?$AAF?$AAN?$AA_?$AAP?$AAr?$AAe?$AAD?$AAe?$AAi?$AAn?$AAi?$AAt?$AA?3?$AA?$AA@ 10002720     usb_ufnmddbase_common_topaz_v1:ufnmdd.obj
 0001:00001750       ??_C@_1CK@GJADIGIG@?$AAU?$AAs?$AAb?$AAF?$AAn?$AAM?$AAd?$AAd?$AA?$CB?$AAU?$AAF?$AAN?$AA_?$AAD?$AAe?$AAi?$AAn?$AAi?$AAt?$AA?3?$AA?$AA@ 10002750     usb_ufnmddbase_common_topaz_v1:ufnmdd.obj
 0001:0000177c       ??_C@_1CG@GMLPBJND@?$AAU?$AAs?$AAb?$AAF?$AAn?$AAM?$AAd?$AAd?$AA?$CB?$AAU?$AAF?$AAN?$AA_?$AAO?$AAp?$AAe?$AAn?$AA?3?$AA?$AA@ 1000277c     usb_ufnmddbase_common_topaz_v1:ufnmdd.obj
 0001:000017a4       ??_C@_1CO@DIEDJLEE@?$AAU?$AAs?$AAb?$AAF?$AAn?$AAM?$AAd?$AAd?$AA?$CB?$AAU?$AAF?$AAN?$AA_?$AAP?$AAr?$AAe?$AAC?$AAl?$AAo?$AAs?$AAe?$AA?3?$AA?$AA@ 100027a4     usb_ufnmddbase_common_topaz_v1:ufnmdd.obj
 0001:000017d4       ??_C@_1CI@HPELHFCH@?$AAU?$AAs?$AAb?$AAF?$AAn?$AAM?$AAd?$AAd?$AA?$CB?$AAU?$AAF?$AAN?$AA_?$AAC?$AAl?$AAo?$AAs?$AAe?$AA?3?$AA?$AA@ 100027d4     usb_ufnmddbase_common_topaz_v1:ufnmdd.obj
 0001:000017fc       ??_C@_1DK@GMGAOFND@?$AAU?$AAs?$AAb?$AAF?$AAn?$AAM?$AAd?$AAd?$AA?$CB?$AAG?$AAe?$AAt?$AAC?$AAl?$AAi?$AAe?$AAn?$AAt?$AAF?$AAu?$AAn?$AAc?$AAt?$AAi?$AAo?$AAn?$AAs?$AA?3?$AA?$AA@ 100027fc     usb_ufnmddbase_common_topaz_v1:ufnmdd.obj
 0001:00001838       ??_C@_1DA@PMLPKIAK@?$AAU?$AAs?$AAb?$AAF?$AAn?$AAM?$AAd?$AAd?$AA?$CB?$AAU?$AAF?$AAN?$AA_?$AAI?$AAO?$AAC?$AAo?$AAn?$AAt?$AAr?$AAo?$AAl?$AA?3?$AA?$AA@ 10002838     usb_ufnmddbase_common_topaz_v1:ufnmdd.obj
 0001:00001868       ??_C@_1FA@GICEAEIA@?$AA?$CF?$AAs?$AA?5?$AAE?$AAx?$AAc?$AAe?$AAp?$AAt?$AAi?$AAo?$AAn?$AA?5?$AAi?$AAn?$AA?5?$AAn?$AAo?$AAt?$AAi?$AAf?$AAi?$AAc?$AAa?$AAt?$AAi?$AAo?$AAn?$AA?5?$AAr?$AAo?$AAu@ 10002868     usb_ufnmddbase_common_topaz_v1:ufnmdd.obj
 0001:000018b8       ??_C@_1EC@FCGHHPGF@?$AAU?$AAs?$AAb?$AAF?$AAn?$AAM?$AAd?$AAd?$AA?$CB?$AAS?$AAe?$AAn?$AAd?$AAD?$AAe?$AAv?$AAi?$AAc?$AAe?$AAN?$AAo?$AAt?$AAi?$AAf?$AAi?$AAc?$AAa?$AAt?$AAi?$AAo?$AAn?$AA?3@ 100028b8     usb_ufnmddbase_common_topaz_v1:ufnmdd.obj
 0001:000018fc       ??_C@_1BI@NKJNCKNK@?$AA?$CF?$AAs?$AA?5?$AAD?$AAe?$AAt?$AAa?$AAc?$AAh?$AA?$AN?$AA?6?$AA?$AA@ 100028fc     usb_ufnmddbase_common_topaz_v1:ufnmdd.obj
 0001:00001914       ??_C@_1BI@HGCIOEDC@?$AA?$CF?$AAs?$AA?5?$AAA?$AAt?$AAt?$AAa?$AAc?$AAh?$AA?$AN?$AA?6?$AA?$AA@ 10002914     usb_ufnmddbase_common_topaz_v1:ufnmdd.obj
 0001:0000192c       ??_C@_1CG@GABFHBBK@?$AAU?$AAs?$AAb?$AAF?$AAn?$AAM?$AAd?$AAd?$AA?$CB?$AAD?$AAl?$AAl?$AAE?$AAn?$AAt?$AAr?$AAy?$AA?3?$AA?$AA@ 1000292c     usb_ufnmddbase_common_topaz_v1:ufnmdd.obj
 0001:00001958       ??_C@_1NC@LINEONCP@?$AAc?$AA?3?$AA?2?$AAw?$AAi?$AAn?$AAc?$AAe?$AAr?$AAo?$AAo?$AAt?$AAs?$AA?2?$AAt?$AAo?$AAp?$AAa?$AAz?$AA?2?$AAw?$AAi?$AAn?$AAc?$AAe?$AA6?$AA0?$AA0?$AA?2?$AAp?$AAl?$AAa@ 10002958     usb_ufnmddbase_common_topaz_v1:ufnmdd.obj
 0001:00001a30       ??_C@_1PG@KOFPIMHL@?$AA?$AN?$AA?6?$AA?$CK?$AA?$CK?$AA?$CK?$AA?5?$AAA?$AAS?$AAS?$AAE?$AAR?$AAT?$AAI?$AAO?$AAN?$AA?5?$AAF?$AAA?$AAI?$AAL?$AAE?$AAD?$AA?5?$AAi?$AAn?$AA?5?$AAc?$AA?3?$AA?2?$AAw?$AAi?$AAn@ 10002a30     usb_ufnmddbase_common_topaz_v1:ufnmdd.obj
 0001:00001b28       ??_C@_1PG@NJODDJJH@?$AA?$AN?$AA?6?$AA?$CK?$AA?$CK?$AA?$CK?$AA?5?$AAA?$AAS?$AAS?$AAE?$AAR?$AAT?$AAI?$AAO?$AAN?$AA?5?$AAF?$AAA?$AAI?$AAL?$AAE?$AAD?$AA?5?$AAi?$AAn?$AA?5?$AAc?$AA?3?$AA?2?$AAw?$AAi?$AAn@ 10002b28     usb_ufnmddbase_common_topaz_v1:ufnmdd.obj
 0001:00001c20       ??_C@_1IO@IFFBAMNB@?$AAC?$AA?3?$AA?2?$AAW?$AAI?$AAN?$AAC?$AAE?$AAR?$AAO?$AAO?$AAT?$AAS?$AA?2?$AAT?$AAo?$AAp?$AAa?$AAz?$AA?2?$AAW?$AAI?$AAN?$AAC?$AAE?$AA6?$AA0?$AA0?$AA?2?$AAp?$AAu?$AAb@ 10002c20     usb_ufnmddbase_common_topaz_v1:ufnmdd.obj
 0001:00001cb0       ??_C@_1OA@CLKFJDEL@?$AA?$AN?$AA?6?$AA?$CK?$AA?$CK?$AA?$CK?$AA?5?$AAA?$AAS?$AAS?$AAE?$AAR?$AAT?$AAI?$AAO?$AAN?$AA?5?$AAF?$AAA?$AAI?$AAL?$AAE?$AAD?$AA?5?$AAi?$AAn?$AA?5?$AAc?$AA?3?$AA?2?$AAw?$AAi?$AAn@ 10002cb0     usb_ufnmddbase_common_topaz_v1:ufnmdd.obj
 0001:00001d90       ??_C@_1OA@NFCDPJJI@?$AA?$AN?$AA?6?$AA?$CK?$AA?$CK?$AA?$CK?$AA?5?$AAA?$AAS?$AAS?$AAE?$AAR?$AAT?$AAI?$AAO?$AAN?$AA?5?$AAF?$AAA?$AAI?$AAL?$AAE?$AAD?$AA?5?$AAi?$AAn?$AA?5?$AAc?$AA?3?$AA?2?$AAw?$AAi?$AAn@ 10002d90     usb_ufnmddbase_common_topaz_v1:ufnmdd.obj
 0001:00001e70       ??_C@_1NC@JCDBHFFH@?$AA?$AN?$AA?6?$AA?$CK?$AA?$CK?$AA?$CK?$AA?5?$AAA?$AAS?$AAS?$AAE?$AAR?$AAT?$AAI?$AAO?$AAN?$AA?5?$AAF?$AAA?$AAI?$AAL?$AAE?$AAD?$AA?5?$AAi?$AAn?$AA?5?$AAc?$AA?3?$AA?2?$AAw?$AAi?$AAn@ 10002e70     usb_ufnmddbase_common_topaz_v1:ufnmdd.obj
 0001:00001f48       ??_C@_1NM@CNLIIAJN@?$AA?$AN?$AA?6?$AA?$CK?$AA?$CK?$AA?$CK?$AA?5?$AAA?$AAS?$AAS?$AAE?$AAR?$AAT?$AAI?$AAO?$AAN?$AA?5?$AAF?$AAA?$AAI?$AAL?$AAE?$AAD?$AA?5?$AAi?$AAn?$AA?5?$AAc?$AA?3?$AA?2?$AAw?$AAi?$AAn@ 10002f48     usb_ufnmddbase_common_topaz_v1:ufnmdd.obj
 0001:00002028       ??_C@_1OA@FGLJACBN@?$AA?$AN?$AA?6?$AA?$CK?$AA?$CK?$AA?$CK?$AA?5?$AAA?$AAS?$AAS?$AAE?$AAR?$AAT?$AAI?$AAO?$AAN?$AA?5?$AAF?$AAA?$AAI?$AAL?$AAE?$AAD?$AA?5?$AAi?$AAn?$AA?5?$AAc?$AA?3?$AA?2?$AAw?$AAi?$AAn@ 10003028     usb_ufnmddbase_common_topaz_v1:ufnmdd.obj
 0001:00002108       ??_C@_1NC@LGAMOIND@?$AA?$AN?$AA?6?$AA?$CK?$AA?$CK?$AA?$CK?$AA?5?$AAA?$AAS?$AAS?$AAE?$AAR?$AAT?$AAI?$AAO?$AAN?$AA?5?$AAF?$AAA?$AAI?$AAL?$AAE?$AAD?$AA?5?$AAi?$AAn?$AA?5?$AAc?$AA?3?$AA?2?$AAw?$AAi?$AAn@ 10003108     usb_ufnmddbase_common_topaz_v1:ufnmdd.obj
 0001:000021e0       ??_C@_1NA@IAFCNGEC@?$AAC?$AA?3?$AA?2?$AAW?$AAI?$AAN?$AAC?$AAE?$AAR?$AAO?$AAO?$AAT?$AAS?$AA?2?$AAT?$AAo?$AAp?$AAa?$AAz?$AA?2?$AAW?$AAI?$AAN?$AAC?$AAE?$AA6?$AA0?$AA0?$AA?2?$AAP?$AAL?$AAA@ 100031e0     usb_ufnmddbase_common_topaz_v1:pipe.obj
 0001:000022b0       ??_7CPipeBase@@6B@         100032b0     usb_ufnmddbase_common_topaz_v1:pipe.obj
 0001:000022d0       ??_7CStaticPipe@@6B@       100032d0     usb_ufnmddbase_common_topaz_v1:pipe.obj
 0001:000022f0       ??_7CDynamicPipe@@6B@      100032f0     usb_ufnmddbase_common_topaz_v1:pipe.obj
 0001:00002310       ??_C@_1NA@MLFEOHPP@?$AAc?$AA?3?$AA?2?$AAw?$AAi?$AAn?$AAc?$AAe?$AAr?$AAo?$AAo?$AAt?$AAs?$AA?2?$AAt?$AAo?$AAp?$AAa?$AAz?$AA?2?$AAw?$AAi?$AAn?$AAc?$AAe?$AA6?$AA0?$AA0?$AA?2?$AAp?$AAl?$AAa@ 10003310     usb_ufnmddbase_common_topaz_v1:pipe.obj
 0001:000023e0       ??_C@_1JG@CGDPEAOM@?$AA?$CF?$AAs?$AA?5?$AAF?$AAa?$AAi?$AAl?$AAe?$AAd?$AA?5?$AAt?$AAo?$AA?5?$AAo?$AAp?$AAe?$AAn?$AA?5?$AAp?$AAi?$AAp?$AAe?$AA?5?$AA?$CI?$AA0?$AAx?$AA?$CF?$AA0?$AA8?$AAx?$AA?$CJ?$AA?3@ 100033e0     usb_ufnmddbase_common_topaz_v1:pipe.obj
 0001:00002478       ??_C@_1IG@EAFBPNCG@?$AA?$CF?$AAs?$AA?5?$AAO?$AAp?$AAe?$AAn?$AAe?$AAd?$AA?5?$AAp?$AAi?$AAp?$AAe?$AA?5?$AA?$CI?$AA0?$AAx?$AA?$CF?$AA0?$AA8?$AAx?$AA?$CJ?$AA?3?$AA?5?$AAp?$AAh?$AAy?$AAs?$AAi?$AAc?$AAa@ 10003478     usb_ufnmddbase_common_topaz_v1:pipe.obj
 0001:00002500       ??_C@_1EK@FNLNBPAG@?$AA?$CF?$AAs?$AA?5?$AAP?$AAi?$AAp?$AAe?$AA?5?$AA?$CI?$AA0?$AAx?$AA?$CF?$AA0?$AA8?$AAx?$AA?$CJ?$AA?5?$AAi?$AAs?$AA?5?$AAa?$AAl?$AAr?$AAe?$AAa?$AAd?$AAy?$AA?5?$AAo?$AAp?$AAe?$AAn@ 10003500     usb_ufnmddbase_common_topaz_v1:pipe.obj
 0001:0000254c       ??_C@_1DE@HELBLJGB@?$AAU?$AAs?$AAb?$AAF?$AAn?$AAM?$AAd?$AAd?$AA?$CB?$AAC?$AAP?$AAi?$AAp?$AAe?$AAB?$AAa?$AAs?$AAe?$AA?3?$AA?3?$AAO?$AAp?$AAe?$AAn?$AA?3?$AA?$AA@ 1000354c     usb_ufnmddbase_common_topaz_v1:pipe.obj
 0001:00002580       ??_C@_1JI@NACFLCAI@?$AA?$CF?$AAs?$AA?5?$AAF?$AAa?$AAi?$AAl?$AAe?$AAd?$AA?5?$AAt?$AAo?$AA?5?$AAc?$AAl?$AAo?$AAs?$AAe?$AA?5?$AAp?$AAi?$AAp?$AAe?$AA?5?$AA?$CI?$AA0?$AAx?$AA?$CF?$AA0?$AA8?$AAx?$AA?$CJ@ 10003580     usb_ufnmddbase_common_topaz_v1:pipe.obj
 0001:00002618       ??_C@_1IG@GGGGEHKN@?$AA?$CF?$AAs?$AA?5?$AAC?$AAl?$AAo?$AAs?$AAe?$AAd?$AA?5?$AAp?$AAi?$AAp?$AAe?$AA?5?$AA?$CI?$AA0?$AAx?$AA?$CF?$AA0?$AA8?$AAx?$AA?$CJ?$AA?3?$AA?5?$AAp?$AAh?$AAy?$AAs?$AAi?$AAc?$AAa@ 10003618     usb_ufnmddbase_common_topaz_v1:pipe.obj
 0001:000026a0       ??_C@_1GI@IAOGBPIC@?$AA?$CF?$AAs?$AA?5?$AAP?$AAi?$AAp?$AAe?$AA?5?$AA?$CI?$AA0?$AAx?$AA?$CF?$AA0?$AA8?$AAx?$AA?$CJ?$AA?3?$AA?5?$AAp?$AAh?$AAy?$AAs?$AAi?$AAc?$AAa?$AAl?$AA?5?$AAa?$AAd?$AAd?$AAr?$AAe@ 100036a0     usb_ufnmddbase_common_topaz_v1:pipe.obj
 0001:00002708       ??_C@_1DG@HPGOACPL@?$AAU?$AAs?$AAb?$AAF?$AAn?$AAM?$AAd?$AAd?$AA?$CB?$AAC?$AAP?$AAi?$AAp?$AAe?$AAB?$AAa?$AAs?$AAe?$AA?3?$AA?3?$AAC?$AAl?$AAo?$AAs?$AAe?$AA?3?$AA?$AA@ 10003708     usb_ufnmddbase_common_topaz_v1:pipe.obj
 0001:00002740       ??_C@_1EO@NFJDCPE@?$AAU?$AAs?$AAb?$AAF?$AAn?$AAM?$AAd?$AAd?$AA?$CB?$AAC?$AAP?$AAi?$AAp?$AAe?$AAB?$AAa?$AAs?$AAe?$AA?3?$AA?3?$AAA?$AAb?$AAo?$AAr?$AAt?$AAA?$AAl?$AAl?$AAT?$AAr?$AAa?$AAn@ 10003740     usb_ufnmddbase_common_topaz_v1:pipe.obj
 0001:00002790       ??_C@_1NA@KJGPOIOG@?$AAc?$AA?3?$AA?2?$AAw?$AAi?$AAn?$AAc?$AAe?$AAr?$AAo?$AAo?$AAt?$AAs?$AA?2?$AAt?$AAo?$AAp?$AAa?$AAz?$AA?2?$AAw?$AAi?$AAn?$AAc?$AAe?$AA6?$AA0?$AA0?$AA?2?$AAp?$AAl?$AAa@ 10003790     usb_ufnmddbase_common_topaz_v1:pipe.obj
 0001:00002860       ??_C@_1EK@ECEMMANF@?$AA?$CF?$AAs?$AA?5?$AAC?$AAo?$AAu?$AAl?$AAd?$AA?5?$AAn?$AAo?$AAt?$AA?5?$AAs?$AAt?$AAa?$AAr?$AAt?$AA?5?$AAt?$AAr?$AAa?$AAn?$AAs?$AAf?$AAe?$AAr?$AA?5?$AA0?$AAx?$AA?$CF?$AA0@ 10003860     usb_ufnmddbase_common_topaz_v1:pipe.obj
 0001:000028b0       ??_C@_1IC@HOCHNMII@?$AA?$CF?$AAs?$AA?5?$AAI?$AAs?$AAs?$AAu?$AAi?$AAn?$AAg?$AA?5?$AA?$CF?$AAs?$AA?5?$AAt?$AAr?$AAa?$AAn?$AAs?$AAf?$AAe?$AAr?$AA?5?$AA?$CI?$AA0?$AAx?$AA?$CF?$AA0?$AA8?$AAx?$AA?$CJ?$AA?5@ 100038b0     usb_ufnmddbase_common_topaz_v1:pipe.obj
 0001:00002934       ??_C@_17HCEMPBGG@?$AAO?$AAU?$AAT?$AA?$AA@ 10003934     usb_ufnmddbase_common_topaz_v1:pipe.obj
 0001:0000293c       ??_C@_15BNKBCKPG@?$AAI?$AAN?$AA?$AA@ 1000393c     usb_ufnmddbase_common_topaz_v1:pipe.obj
 0001:00002948       ??_C@_1GA@DDLMCCCM@?$AA?$CF?$AAs?$AA?5?$AAF?$AAa?$AAi?$AAl?$AAe?$AAd?$AA?5?$AAt?$AAo?$AA?5?$AAa?$AAl?$AAl?$AAo?$AAc?$AAa?$AAt?$AAe?$AA?5?$AAn?$AAe?$AAw?$AA?5?$AAt?$AAr?$AAa?$AAn?$AAs?$AAf@ 10003948     usb_ufnmddbase_common_topaz_v1:pipe.obj
 0001:000029a8       ??_C@_1EG@HIONKIAE@?$AAU?$AAs?$AAb?$AAF?$AAn?$AAM?$AAd?$AAd?$AA?$CB?$AAC?$AAP?$AAi?$AAp?$AAe?$AAB?$AAa?$AAs?$AAe?$AA?3?$AA?3?$AAI?$AAs?$AAs?$AAu?$AAe?$AAT?$AAr?$AAa?$AAn?$AAs?$AAf?$AAe@ 100039a8     usb_ufnmddbase_common_topaz_v1:pipe.obj
 0001:000029f0       ??_C@_1HK@CBMHIKE@?$AA?$CF?$AAs?$AA?5?$AAA?$AAb?$AAo?$AAr?$AAt?$AAi?$AAn?$AAg?$AA?5?$AAt?$AAr?$AAa?$AAn?$AAs?$AAf?$AAe?$AAr?$AA?5?$AA0?$AAx?$AA?$CF?$AA0?$AA8?$AAx?$AA?5?$AAo?$AAn?$AA?5?$AAp@ 100039f0     usb_ufnmddbase_common_topaz_v1:pipe.obj
 0001:00002a70       ??_C@_1EG@FJGDCE@?$AAU?$AAs?$AAb?$AAF?$AAn?$AAM?$AAd?$AAd?$AA?$CB?$AAC?$AAP?$AAi?$AAp?$AAe?$AAB?$AAa?$AAs?$AAe?$AA?3?$AA?3?$AAA?$AAb?$AAo?$AAr?$AAt?$AAT?$AAr?$AAa?$AAn?$AAs?$AAf?$AAe@ 10003a70     usb_ufnmddbase_common_topaz_v1:pipe.obj
 0001:00002ab8       ??_C@_1EO@NJGPFCEJ@?$AAU?$AAs?$AAb?$AAF?$AAn?$AAM?$AAd?$AAd?$AA?$CB?$AAC?$AAP?$AAi?$AAp?$AAe?$AAB?$AAa?$AAs?$AAe?$AA?3?$AA?3?$AAG?$AAe?$AAt?$AAT?$AAr?$AAa?$AAn?$AAs?$AAf?$AAe?$AAr?$AAS@ 10003ab8     usb_ufnmddbase_common_topaz_v1:pipe.obj
 0001:00002b08       ??_C@_1HI@FLHMHEAB@?$AA?$CF?$AAs?$AA?5?$AAC?$AAl?$AAo?$AAs?$AAi?$AAn?$AAg?$AA?5?$AAt?$AAr?$AAa?$AAn?$AAs?$AAf?$AAe?$AAr?$AA?5?$AA0?$AAx?$AA?$CF?$AA0?$AA8?$AAx?$AA?5?$AAo?$AAn?$AA?5?$AAp?$AAi@ 10003b08     usb_ufnmddbase_common_topaz_v1:pipe.obj
 0001:00002b80       ??_C@_1EG@EPHBAIDE@?$AAU?$AAs?$AAb?$AAF?$AAn?$AAM?$AAd?$AAd?$AA?$CB?$AAC?$AAP?$AAi?$AAp?$AAe?$AAB?$AAa?$AAs?$AAe?$AA?3?$AA?3?$AAC?$AAl?$AAo?$AAs?$AAe?$AAT?$AAr?$AAa?$AAn?$AAs?$AAf?$AAe@ 10003b80     usb_ufnmddbase_common_topaz_v1:pipe.obj
 0001:00002bc8       ??_C@_1FE@GEBNAGPN@?$AA?$CF?$AAs?$AA?5?$AAP?$AAl?$AAa?$AAc?$AAi?$AAn?$AAg?$AA?5?$AAt?$AAr?$AAa?$AAn?$AAs?$AAf?$AAe?$AAr?$AA?5?$AA0?$AAx?$AA?$CF?$AA0?$AA8?$AAx?$AA?5?$AAo?$AAn?$AA?5?$AAf?$AAr@ 10003bc8     usb_ufnmddbase_common_topaz_v1:pipe.obj
 0001:00002c20       ??_C@_1EE@NBICGMBG@?$AAU?$AAs?$AAb?$AAF?$AAn?$AAM?$AAd?$AAd?$AA?$CB?$AAC?$AAP?$AAi?$AAp?$AAe?$AAB?$AAa?$AAs?$AAe?$AA?3?$AA?3?$AAF?$AAr?$AAe?$AAe?$AAT?$AAr?$AAa?$AAn?$AAs?$AAf?$AAe?$AAr@ 10003c20     usb_ufnmddbase_common_topaz_v1:pipe.obj
 0001:00002c68       ??_C@_1BCK@IPBHCAK@?$AA?$AN?$AA?6?$AA?$CK?$AA?$CK?$AA?$CK?$AA?5?$AAA?$AAS?$AAS?$AAE?$AAR?$AAT?$AAI?$AAO?$AAN?$AA?5?$AAF?$AAA?$AAI?$AAL?$AAE?$AAD?$AA?5?$AAi?$AAn?$AA?5?$AAc?$AA?3?$AA?2?$AAw?$AAi?$AAn@ 10003c68     usb_ufnmddbase_common_topaz_v1:pipe.obj
 0001:00002d98       ??_C@_1FE@JHADALKD@?$AA?$CF?$AAs?$AA?5?$AAC?$AAo?$AAu?$AAl?$AAd?$AA?5?$AAn?$AAo?$AAt?$AA?5?$AAs?$AAt?$AAa?$AAr?$AAt?$AA?5?$AAn?$AAe?$AAx?$AAt?$AA?5?$AAt?$AAr?$AAa?$AAn?$AAs?$AAf?$AAe?$AAr@ 10003d98     usb_ufnmddbase_common_topaz_v1:pipe.obj
 0001:00002df0       ??_C@_1HO@POIGLOBC@?$AA?$CF?$AAs?$AA?5?$AAC?$AAo?$AAm?$AAp?$AAl?$AAe?$AAt?$AAi?$AAn?$AAg?$AA?5?$AAt?$AAr?$AAa?$AAn?$AAs?$AAf?$AAe?$AAr?$AA?5?$AA0?$AAx?$AA?$CF?$AA0?$AA8?$AAx?$AA?5?$AAo?$AAn@ 10003df0     usb_ufnmddbase_common_topaz_v1:pipe.obj
 0001:00002e70       ??_C@_1EM@LJHMPH@?$AAU?$AAs?$AAb?$AAF?$AAn?$AAM?$AAd?$AAd?$AA?$CB?$AAC?$AAP?$AAi?$AAp?$AAe?$AAB?$AAa?$AAs?$AAe?$AA?3?$AA?3?$AAT?$AAr?$AAa?$AAn?$AAs?$AAf?$AAe?$AAr?$AAC?$AAo?$AAm?$AAp@ 10003e70     usb_ufnmddbase_common_topaz_v1:pipe.obj
 0001:00002ec0       ??_C@_1FA@LENIMDKE@?$AA?$CF?$AAs?$AA?5?$AAS?$AAt?$AAa?$AAl?$AAl?$AAi?$AAn?$AAg?$AA?5?$AAe?$AAn?$AAd?$AAp?$AAo?$AAi?$AAn?$AAt?$AA?5?$AA?$CF?$AAu?$AA?5?$AAp?$AAi?$AAp?$AAe?$AA?5?$AA?$CI?$AA0?$AAx@ 10003ec0     usb_ufnmddbase_common_topaz_v1:pipe.obj
 0001:00002f10       ??_C@_1CM@LFPJLPKB@?$AA?$CF?$AAs?$AA?5?$AAP?$AAi?$AAp?$AAe?$AA?5?$AAi?$AAs?$AA?5?$AAn?$AAo?$AAt?$AA?5?$AAo?$AAp?$AAe?$AAn?$AA?$AN?$AA?6?$AA?$AA@ 10003f10     usb_ufnmddbase_common_topaz_v1:pipe.obj
 0001:00002f3c       ??_C@_1DG@IPJFOHGJ@?$AAU?$AAs?$AAb?$AAF?$AAn?$AAM?$AAd?$AAd?$AA?$CB?$AAC?$AAP?$AAi?$AAp?$AAe?$AAB?$AAa?$AAs?$AAe?$AA?3?$AA?3?$AAS?$AAt?$AAa?$AAl?$AAl?$AA?3?$AA?$AA@ 10003f3c     usb_ufnmddbase_common_topaz_v1:pipe.obj
 0001:00002f78       ??_C@_1GC@FIJKAPIA@?$AA?$CF?$AAs?$AA?5?$AAC?$AAl?$AAe?$AAa?$AAr?$AAi?$AAn?$AAg?$AA?5?$AAs?$AAt?$AAa?$AAl?$AAl?$AA?5?$AAo?$AAn?$AA?5?$AAe?$AAn?$AAd?$AAp?$AAo?$AAi?$AAn?$AAt?$AA?5?$AA?$CF?$AAu@ 10003f78     usb_ufnmddbase_common_topaz_v1:pipe.obj
 0001:00002fe0       ??_C@_1EA@CCKBNLFB@?$AAU?$AAs?$AAb?$AAF?$AAn?$AAM?$AAd?$AAd?$AA?$CB?$AAC?$AAP?$AAi?$AAp?$AAe?$AAB?$AAa?$AAs?$AAe?$AA?3?$AA?3?$AAC?$AAl?$AAe?$AAa?$AAr?$AAS?$AAt?$AAa?$AAl?$AAl?$AA?3?$AA?$AA@ 10003fe0     usb_ufnmddbase_common_topaz_v1:pipe.obj
 0001:00003020       ??_C@_1EM@MBJHNODD@?$AA?$CF?$AAs?$AA?5?$AAS?$AAe?$AAn?$AAd?$AAi?$AAn?$AAg?$AA?5?$AAC?$AAo?$AAn?$AAt?$AAr?$AAo?$AAl?$AA?5?$AAS?$AAt?$AAa?$AAt?$AAu?$AAs?$AA?5?$AAH?$AAa?$AAn?$AAd?$AAs?$AAh@ 10004020     usb_ufnmddbase_common_topaz_v1:pipe.obj
 0001:00003070       ??_C@_1GA@EIALGOEI@?$AAU?$AAs?$AAb?$AAF?$AAn?$AAM?$AAd?$AAd?$AA?$CB?$AAC?$AAP?$AAi?$AAp?$AAe?$AAB?$AAa?$AAs?$AAe?$AA?3?$AA?3?$AAS?$AAe?$AAn?$AAd?$AAC?$AAo?$AAn?$AAt?$AAr?$AAo?$AAl?$AAS@ 10004070     usb_ufnmddbase_common_topaz_v1:pipe.obj
 0001:000030d0       ??_C@_1FG@NCPIOAIE@?$AA?$CF?$AAs?$AA?5?$AAE?$AAx?$AAc?$AAe?$AAp?$AAt?$AAi?$AAo?$AAn?$AA?5?$AAc?$AAh?$AAe?$AAc?$AAk?$AAi?$AAn?$AAg?$AA?5?$AAP?$AAi?$AAp?$AAe?$AA?5?$AAh?$AAa?$AAn?$AAd?$AAl@ 100040d0     usb_ufnmddbase_common_topaz_v1:pipe.obj
 0001:00003128       ??_C@_1FG@JAGLEFOD@?$AA?$CF?$AAs?$AA?5?$AAI?$AAn?$AAv?$AAa?$AAl?$AAi?$AAd?$AA?5?$AAP?$AAi?$AAp?$AAe?$AA?5?$AAh?$AAa?$AAn?$AAd?$AAl?$AAe?$AA?5?$AA0?$AAx?$AA?$CF?$AA0?$AA8?$AAx?$AA?5?$AA?$CI?$AAs@ 10004128     usb_ufnmddbase_common_topaz_v1:pipe.obj
 0001:00003180       ??_C@_1EA@KHIBPCBC@?$AA?$CF?$AAs?$AA?5?$AAI?$AAn?$AAv?$AAa?$AAl?$AAi?$AAd?$AA?5?$AAP?$AAi?$AAp?$AAe?$AA?5?$AAh?$AAa?$AAn?$AAd?$AAl?$AAe?$AA?5?$AA0?$AAx?$AA?$CF?$AA0?$AA8?$AAx?$AA?$AN?$AA?6?$AA?$AA@ 10004180     usb_ufnmddbase_common_topaz_v1:pipe.obj
 0001:000031c0       ??_C@_1FA@BKIGJOKK@?$AAU?$AAs?$AAb?$AAF?$AAn?$AAM?$AAd?$AAd?$AA?$CB?$AAC?$AAP?$AAi?$AAp?$AAe?$AAB?$AAa?$AAs?$AAe?$AA?3?$AA?3?$AAV?$AAa?$AAl?$AAi?$AAd?$AAa?$AAt?$AAe?$AAP?$AAi?$AAp?$AAe@ 100041c0     usb_ufnmddbase_common_topaz_v1:pipe.obj
 0001:00003210       ??_C@_1BBM@IEIHDAJN@?$AA?$AN?$AA?6?$AA?$CK?$AA?$CK?$AA?$CK?$AA?5?$AAA?$AAS?$AAS?$AAE?$AAR?$AAT?$AAI?$AAO?$AAN?$AA?5?$AAF?$AAA?$AAI?$AAL?$AAE?$AAD?$AA?5?$AAi?$AAn?$AA?5?$AAc?$AA?3?$AA?2?$AAw?$AAi?$AAn@ 10004210     usb_ufnmddbase_common_topaz_v1:pipe.obj
 0001:00003330       ??_C@_1BBM@KKNHPJBN@?$AA?$AN?$AA?6?$AA?$CK?$AA?$CK?$AA?$CK?$AA?5?$AAA?$AAS?$AAS?$AAE?$AAR?$AAT?$AAI?$AAO?$AAN?$AA?5?$AAF?$AAA?$AAI?$AAL?$AAE?$AAD?$AA?5?$AAi?$AAn?$AA?5?$AAc?$AA?3?$AA?2?$AAw?$AAi?$AAn@ 10004330     usb_ufnmddbase_common_topaz_v1:pipe.obj
 0001:00003450       ??_C@_1BBM@GOHHKFDA@?$AA?$AN?$AA?6?$AA?$CK?$AA?$CK?$AA?$CK?$AA?5?$AAA?$AAS?$AAS?$AAE?$AAR?$AAT?$AAI?$AAO?$AAN?$AA?5?$AAF?$AAA?$AAI?$AAL?$AAE?$AAD?$AA?5?$AAi?$AAn?$AA?5?$AAc?$AA?3?$AA?2?$AAw?$AAi?$AAn@ 10004450     usb_ufnmddbase_common_topaz_v1:pipe.obj
 0001:00003570       ??_C@_1BEI@EMELIHOJ@?$AA?$AN?$AA?6?$AA?$CK?$AA?$CK?$AA?$CK?$AA?5?$AAA?$AAS?$AAS?$AAE?$AAR?$AAT?$AAI?$AAO?$AAN?$AA?5?$AAF?$AAA?$AAI?$AAL?$AAE?$AAD?$AA?5?$AAi?$AAn?$AA?5?$AAc?$AA?3?$AA?2?$AAw?$AAi?$AAn@ 10004570     usb_ufnmddbase_common_topaz_v1:pipe.obj
 0001:000036b8       ??_C@_1NA@GGGMIAJ@?$AAc?$AA?3?$AA?2?$AAw?$AAi?$AAn?$AAc?$AAe?$AAr?$AAo?$AAo?$AAt?$AAs?$AA?2?$AAt?$AAo?$AAp?$AAa?$AAz?$AA?2?$AAw?$AAi?$AAn?$AAc?$AAe?$AA6?$AA0?$AA0?$AA?2?$AAp?$AAl?$AAa@ 100046b8     usb_ufnmddbase_common_topaz_v1:pipe.obj
 0001:00003788       ??_C@_1BEI@BEINIMBF@?$AA?$AN?$AA?6?$AA?$CK?$AA?$CK?$AA?$CK?$AA?5?$AAA?$AAS?$AAS?$AAE?$AAR?$AAT?$AAI?$AAO?$AAN?$AA?5?$AAF?$AAA?$AAI?$AAL?$AAE?$AAD?$AA?5?$AAi?$AAn?$AA?5?$AAc?$AA?3?$AA?2?$AAw?$AAi?$AAn@ 10004788     usb_ufnmddbase_common_topaz_v1:pipe.obj
 0001:000038d0       ??_C@_1NM@NGJEHHEF@?$AA?$AN?$AA?6?$AA?$CK?$AA?$CK?$AA?$CK?$AA?5?$AAA?$AAS?$AAS?$AAE?$AAR?$AAT?$AAI?$AAO?$AAN?$AA?5?$AAF?$AAA?$AAI?$AAL?$AAE?$AAD?$AA?5?$AAi?$AAn?$AA?5?$AAC?$AA?3?$AA?2?$AAW?$AAI?$AAN@ 100048d0     usb_ufnmddbase_common_topaz_v1:pipe.obj
 0001:000039b0       ??_C@_1PA@NOFBDKCC@?$AA?$AN?$AA?6?$AA?$CK?$AA?$CK?$AA?$CK?$AA?5?$AAA?$AAS?$AAS?$AAE?$AAR?$AAT?$AAI?$AAO?$AAN?$AA?5?$AAF?$AAA?$AAI?$AAL?$AAE?$AAD?$AA?5?$AAi?$AAn?$AA?5?$AAC?$AA?3?$AA?2?$AAW?$AAI?$AAN@ 100049b0     usb_ufnmddbase_common_topaz_v1:pipe.obj
 0001:00003aa0       ??_C@_1NA@NEEIGIEK@?$AA?$AN?$AA?6?$AA?$CK?$AA?$CK?$AA?$CK?$AA?5?$AAA?$AAS?$AAS?$AAE?$AAR?$AAT?$AAI?$AAO?$AAN?$AA?5?$AAF?$AAA?$AAI?$AAL?$AAE?$AAD?$AA?5?$AAi?$AAn?$AA?5?$AAC?$AA?3?$AA?2?$AAW?$AAI?$AAN@ 10004aa0     usb_ufnmddbase_common_topaz_v1:pipe.obj
 0001:00003b70       ??_C@_1NG@DPFMNOON@?$AA?$AN?$AA?6?$AA?$CK?$AA?$CK?$AA?$CK?$AA?5?$AAA?$AAS?$AAS?$AAE?$AAR?$AAT?$AAI?$AAO?$AAN?$AA?5?$AAF?$AAA?$AAI?$AAL?$AAE?$AAD?$AA?5?$AAi?$AAn?$AA?5?$AAC?$AA?3?$AA?2?$AAW?$AAI?$AAN@ 10004b70     usb_ufnmddbase_common_topaz_v1:pipe.obj
 0001:00003c48       ??_C@_1NG@BDFJKOEH@?$AA?$AN?$AA?6?$AA?$CK?$AA?$CK?$AA?$CK?$AA?5?$AAA?$AAS?$AAS?$AAE?$AAR?$AAT?$AAI?$AAO?$AAN?$AA?5?$AAF?$AAA?$AAI?$AAL?$AAE?$AAD?$AA?5?$AAi?$AAn?$AA?5?$AAC?$AA?3?$AA?2?$AAW?$AAI?$AAN@ 10004c48     usb_ufnmddbase_common_topaz_v1:pipe.obj
 0001:00003d20       ??_C@_1BBM@KBHKODJI@?$AA?$AN?$AA?6?$AA?$CK?$AA?$CK?$AA?$CK?$AA?5?$AAA?$AAS?$AAS?$AAE?$AAR?$AAT?$AAI?$AAO?$AAN?$AA?5?$AAF?$AAA?$AAI?$AAL?$AAE?$AAD?$AA?5?$AAi?$AAn?$AA?5?$AAc?$AA?3?$AA?2?$AAw?$AAi?$AAn@ 10004d20     usb_ufnmddbase_common_topaz_v1:pipe.obj
 0001:00003e40       ??_C@_1BCG@INAJHCPN@?$AA?$AN?$AA?6?$AA?$CK?$AA?$CK?$AA?$CK?$AA?5?$AAA?$AAS?$AAS?$AAE?$AAR?$AAT?$AAI?$AAO?$AAN?$AA?5?$AAF?$AAA?$AAI?$AAL?$AAE?$AAD?$AA?5?$AAi?$AAn?$AA?5?$AAc?$AA?3?$AA?2?$AAw?$AAi?$AAn@ 10004e40     usb_ufnmddbase_common_topaz_v1:pipe.obj
 0001:00003f68       ??_C@_1BBM@IAOEOLNI@?$AA?$AN?$AA?6?$AA?$CK?$AA?$CK?$AA?$CK?$AA?5?$AAA?$AAS?$AAS?$AAE?$AAR?$AAT?$AAI?$AAO?$AAN?$AA?5?$AAF?$AAA?$AAI?$AAL?$AAE?$AAD?$AA?5?$AAi?$AAn?$AA?5?$AAc?$AA?3?$AA?2?$AAw?$AAi?$AAn@ 10004f68     usb_ufnmddbase_common_topaz_v1:pipe.obj
 0001:00004088       ??_C@_1PG@LCJIKPDJ@?$AA?$AN?$AA?6?$AA?$CK?$AA?$CK?$AA?$CK?$AA?5?$AAA?$AAS?$AAS?$AAE?$AAR?$AAT?$AAI?$AAO?$AAN?$AA?5?$AAF?$AAA?$AAI?$AAL?$AAE?$AAD?$AA?5?$AAi?$AAn?$AA?5?$AAc?$AA?3?$AA?2?$AAw?$AAi?$AAn@ 10005088     usb_ufnmddbase_common_topaz_v1:pipe.obj
 0001:00004180       ??_C@_1PG@FNJFJKJB@?$AA?$AN?$AA?6?$AA?$CK?$AA?$CK?$AA?$CK?$AA?5?$AAA?$AAS?$AAS?$AAE?$AAR?$AAT?$AAI?$AAO?$AAN?$AA?5?$AAF?$AAA?$AAI?$AAL?$AAE?$AAD?$AA?5?$AAi?$AAn?$AA?5?$AAc?$AA?3?$AA?2?$AAw?$AAi?$AAn@ 10005180     usb_ufnmddbase_common_topaz_v1:pipe.obj
 0001:00004278       ??_C@_1NG@JCMKMAKN@?$AA?$AN?$AA?6?$AA?$CK?$AA?$CK?$AA?$CK?$AA?5?$AAA?$AAS?$AAS?$AAE?$AAR?$AAT?$AAI?$AAO?$AAN?$AA?5?$AAF?$AAA?$AAI?$AAL?$AAE?$AAD?$AA?5?$AAi?$AAn?$AA?5?$AAC?$AA?3?$AA?2?$AAW?$AAI?$AAN@ 10005278     usb_ufnmddbase_common_topaz_v1:pipe.obj
 0001:00004350       ??_C@_1OO@IBENPIBC@?$AA?$AN?$AA?6?$AA?$CK?$AA?$CK?$AA?$CK?$AA?5?$AAA?$AAS?$AAS?$AAE?$AAR?$AAT?$AAI?$AAO?$AAN?$AA?5?$AAF?$AAA?$AAI?$AAL?$AAE?$AAD?$AA?5?$AAi?$AAn?$AA?5?$AAC?$AA?3?$AA?2?$AAW?$AAI?$AAN@ 10005350     usb_ufnmddbase_common_topaz_v1:pipe.obj
 0001:00004440       ??_C@_1OO@MPEKDFHJ@?$AA?$AN?$AA?6?$AA?$CK?$AA?$CK?$AA?$CK?$AA?5?$AAA?$AAS?$AAS?$AAE?$AAR?$AAT?$AAI?$AAO?$AAN?$AA?5?$AAF?$AAA?$AAI?$AAL?$AAE?$AAD?$AA?5?$AAi?$AAn?$AA?5?$AAC?$AA?3?$AA?2?$AAW?$AAI?$AAN@ 10005440     usb_ufnmddbase_common_topaz_v1:pipe.obj
 0001:00004530       ??_C@_1BCA@EHHJJLKF@?$AA?$AN?$AA?6?$AA?$CK?$AA?$CK?$AA?$CK?$AA?5?$AAA?$AAS?$AAS?$AAE?$AAR?$AAT?$AAI?$AAO?$AAN?$AA?5?$AAF?$AAA?$AAI?$AAL?$AAE?$AAD?$AA?5?$AAi?$AAn?$AA?5?$AAC?$AA?3?$AA?2?$AAW?$AAI?$AAN@ 10005530     usb_ufnmddbase_common_topaz_v1:pipe.obj
 0001:00004650       ??_C@_1BAE@CIDAGNOA@?$AA?$AN?$AA?6?$AA?$CK?$AA?$CK?$AA?$CK?$AA?5?$AAA?$AAS?$AAS?$AAE?$AAR?$AAT?$AAI?$AAO?$AAN?$AA?5?$AAF?$AAA?$AAI?$AAL?$AAE?$AAD?$AA?5?$AAi?$AAn?$AA?5?$AAC?$AA?3?$AA?2?$AAW?$AAI?$AAN@ 10005650     usb_ufnmddbase_common_topaz_v1:pipe.obj
 0001:00004758       ??_C@_1NK@MKEEHJPB@?$AA?$AN?$AA?6?$AA?$CK?$AA?$CK?$AA?$CK?$AA?5?$AAA?$AAS?$AAS?$AAE?$AAR?$AAT?$AAI?$AAO?$AAN?$AA?5?$AAF?$AAA?$AAI?$AAL?$AAE?$AAD?$AA?5?$AAi?$AAn?$AA?5?$AAc?$AA?3?$AA?2?$AAw?$AAi?$AAn@ 10005758     usb_ufnmddbase_common_topaz_v1:pipe.obj
 0001:00004838       ??_C@_1NO@NOCCODEO@?$AA?$AN?$AA?6?$AA?$CK?$AA?$CK?$AA?$CK?$AA?5?$AAA?$AAS?$AAS?$AAE?$AAR?$AAT?$AAI?$AAO?$AAN?$AA?5?$AAF?$AAA?$AAI?$AAL?$AAE?$AAD?$AA?5?$AAi?$AAn?$AA?5?$AAc?$AA?3?$AA?2?$AAw?$AAi?$AAn@ 10005838     usb_ufnmddbase_common_topaz_v1:pipe.obj
 0001:00004918       ??_C@_1NE@JGLMIENF@?$AA?$AN?$AA?6?$AA?$CK?$AA?$CK?$AA?$CK?$AA?5?$AAA?$AAS?$AAS?$AAE?$AAR?$AAT?$AAI?$AAO?$AAN?$AA?5?$AAF?$AAA?$AAI?$AAL?$AAE?$AAD?$AA?5?$AAi?$AAn?$AA?5?$AAc?$AA?3?$AA?2?$AAw?$AAi?$AAn@ 10005918     usb_ufnmddbase_common_topaz_v1:pipe.obj
 0001:000049f0       ??_C@_1NE@OKJNOBGL@?$AA?$AN?$AA?6?$AA?$CK?$AA?$CK?$AA?$CK?$AA?5?$AAA?$AAS?$AAS?$AAE?$AAR?$AAT?$AAI?$AAO?$AAN?$AA?5?$AAF?$AAA?$AAI?$AAL?$AAE?$AAD?$AA?5?$AAi?$AAn?$AA?5?$AAc?$AA?3?$AA?2?$AAw?$AAi?$AAn@ 100059f0     usb_ufnmddbase_common_topaz_v1:pipe.obj
 0001:00004ac8       ??_C@_1NE@CJPEKLJL@?$AA?$AN?$AA?6?$AA?$CK?$AA?$CK?$AA?$CK?$AA?5?$AAA?$AAS?$AAS?$AAE?$AAR?$AAT?$AAI?$AAO?$AAN?$AA?5?$AAF?$AAA?$AAI?$AAL?$AAE?$AAD?$AA?5?$AAi?$AAn?$AA?5?$AAc?$AA?3?$AA?2?$AAw?$AAi?$AAn@ 10005ac8     usb_ufnmddbase_common_topaz_v1:pipe.obj
 0001:00004ba0       ??_C@_1PM@MIEOKFGM@?$AA?$AN?$AA?6?$AA?$CK?$AA?$CK?$AA?$CK?$AA?5?$AAA?$AAS?$AAS?$AAE?$AAR?$AAT?$AAI?$AAO?$AAN?$AA?5?$AAF?$AAA?$AAI?$AAL?$AAE?$AAD?$AA?5?$AAi?$AAn?$AA?5?$AAc?$AA?3?$AA?2?$AAw?$AAi?$AAn@ 10005ba0     usb_ufnmddbase_common_topaz_v1:pipe.obj
 0001:00004ca0       ??_C@_1PM@PHNIPBMH@?$AA?$AN?$AA?6?$AA?$CK?$AA?$CK?$AA?$CK?$AA?5?$AAA?$AAS?$AAS?$AAE?$AAR?$AAT?$AAI?$AAO?$AAN?$AA?5?$AAF?$AAA?$AAI?$AAL?$AAE?$AAD?$AA?5?$AAi?$AAn?$AA?5?$AAc?$AA?3?$AA?2?$AAw?$AAi?$AAn@ 10005ca0     usb_ufnmddbase_common_topaz_v1:pipe.obj
 0001:00004da0       ??_C@_1PM@LHEPLEOC@?$AA?$AN?$AA?6?$AA?$CK?$AA?$CK?$AA?$CK?$AA?5?$AAA?$AAS?$AAS?$AAE?$AAR?$AAT?$AAI?$AAO?$AAN?$AA?5?$AAF?$AAA?$AAI?$AAL?$AAE?$AAD?$AA?5?$AAi?$AAn?$AA?5?$AAc?$AA?3?$AA?2?$AAw?$AAi?$AAn@ 10005da0     usb_ufnmddbase_common_topaz_v1:pipe.obj
 0001:00004ea0       ??_C@_1OC@EBJOOINM@?$AA?$AN?$AA?6?$AA?$CK?$AA?$CK?$AA?$CK?$AA?5?$AAA?$AAS?$AAS?$AAE?$AAR?$AAT?$AAI?$AAO?$AAN?$AA?5?$AAF?$AAA?$AAI?$AAL?$AAE?$AAD?$AA?5?$AAi?$AAn?$AA?5?$AAc?$AA?3?$AA?2?$AAw?$AAi?$AAn@ 10005ea0     usb_ufnmddbase_common_topaz_v1:pipe.obj
 0001:00004f88       ??_C@_1OG@MHLKEBPK@?$AA?$AN?$AA?6?$AA?$CK?$AA?$CK?$AA?$CK?$AA?5?$AAA?$AAS?$AAS?$AAE?$AAR?$AAT?$AAI?$AAO?$AAN?$AA?5?$AAF?$AAA?$AAI?$AAL?$AAE?$AAD?$AA?5?$AAi?$AAn?$AA?5?$AAc?$AA?3?$AA?2?$AAw?$AAi?$AAn@ 10005f88     usb_ufnmddbase_common_topaz_v1:pipe.obj
 0001:00005070       ??_C@_1NE@HMGLIKCB@?$AA?$AN?$AA?6?$AA?$CK?$AA?$CK?$AA?$CK?$AA?5?$AAA?$AAS?$AAS?$AAE?$AAR?$AAT?$AAI?$AAO?$AAN?$AA?5?$AAF?$AAA?$AAI?$AAL?$AAE?$AAD?$AA?5?$AAi?$AAn?$AA?5?$AAc?$AA?3?$AA?2?$AAw?$AAi?$AAn@ 10006070     usb_ufnmddbase_common_topaz_v1:pipe.obj
 0001:00005148       ??_C@_1NC@MMKFMMCH@?$AA?$AN?$AA?6?$AA?$CK?$AA?$CK?$AA?$CK?$AA?5?$AAA?$AAS?$AAS?$AAE?$AAR?$AAT?$AAI?$AAO?$AAN?$AA?5?$AAF?$AAA?$AAI?$AAL?$AAE?$AAD?$AA?5?$AAi?$AAn?$AA?5?$AAc?$AA?3?$AA?2?$AAw?$AAi?$AAn@ 10006148     usb_ufnmddbase_common_topaz_v1:pipe.obj
 0001:00005220       ??_C@_1NE@JBCKAMFN@?$AA?$AN?$AA?6?$AA?$CK?$AA?$CK?$AA?$CK?$AA?5?$AAA?$AAS?$AAS?$AAE?$AAR?$AAT?$AAI?$AAO?$AAN?$AA?5?$AAF?$AAA?$AAI?$AAL?$AAE?$AAD?$AA?5?$AAi?$AAn?$AA?5?$AAc?$AA?3?$AA?2?$AAw?$AAi?$AAn@ 10006220     usb_ufnmddbase_common_topaz_v1:pipe.obj
 0001:000052f8       ??_C@_1PA@IHLKMBID@?$AA?$AN?$AA?6?$AA?$CK?$AA?$CK?$AA?$CK?$AA?5?$AAA?$AAS?$AAS?$AAE?$AAR?$AAT?$AAI?$AAO?$AAN?$AA?5?$AAF?$AAA?$AAI?$AAL?$AAE?$AAD?$AA?5?$AAi?$AAn?$AA?5?$AAc?$AA?3?$AA?2?$AAw?$AAi?$AAn@ 100062f8     usb_ufnmddbase_common_topaz_v1:pipe.obj
 0001:000053e8       ??_C@_1PA@JKPJBDBB@?$AA?$AN?$AA?6?$AA?$CK?$AA?$CK?$AA?$CK?$AA?5?$AAA?$AAS?$AAS?$AAE?$AAR?$AAT?$AAI?$AAO?$AAN?$AA?5?$AAF?$AAA?$AAI?$AAL?$AAE?$AAD?$AA?5?$AAi?$AAn?$AA?5?$AAc?$AA?3?$AA?2?$AAw?$AAi?$AAn@ 100063e8     usb_ufnmddbase_common_topaz_v1:pipe.obj
 0001:000054d8       ??_C@_1PK@LJKAAONG@?$AA?$AN?$AA?6?$AA?$CK?$AA?$CK?$AA?$CK?$AA?5?$AAA?$AAS?$AAS?$AAE?$AAR?$AAT?$AAI?$AAO?$AAN?$AA?5?$AAF?$AAA?$AAI?$AAL?$AAE?$AAD?$AA?5?$AAi?$AAn?$AA?5?$AAc?$AA?3?$AA?2?$AAw?$AAi?$AAn@ 100064d8     usb_ufnmddbase_common_topaz_v1:pipe.obj
 0001:000055d8       ??_C@_1PM@MLFKMHMN@?$AA?$AN?$AA?6?$AA?$CK?$AA?$CK?$AA?$CK?$AA?5?$AAA?$AAS?$AAS?$AAE?$AAR?$AAT?$AAI?$AAO?$AAN?$AA?5?$AAF?$AAA?$AAI?$AAL?$AAE?$AAD?$AA?5?$AAi?$AAn?$AA?5?$AAc?$AA?3?$AA?2?$AAw?$AAi?$AAn@ 100065d8     usb_ufnmddbase_common_topaz_v1:pipe.obj
 0001:000056d8       ??_C@_1PM@NJBEGHBC@?$AA?$AN?$AA?6?$AA?$CK?$AA?$CK?$AA?$CK?$AA?5?$AAA?$AAS?$AAS?$AAE?$AAR?$AAT?$AAI?$AAO?$AAN?$AA?5?$AAF?$AAA?$AAI?$AAL?$AAE?$AAD?$AA?5?$AAi?$AAn?$AA?5?$AAc?$AA?3?$AA?2?$AAw?$AAi?$AAn@ 100066d8     usb_ufnmddbase_common_topaz_v1:pipe.obj
 0001:000057d8       ??_C@_1NI@MFBCFIBE@?$AAC?$AA?3?$AA?2?$AAW?$AAI?$AAN?$AAC?$AAE?$AAR?$AAO?$AAO?$AAT?$AAS?$AA?2?$AAT?$AAo?$AAp?$AAa?$AAz?$AA?2?$AAW?$AAI?$AAN?$AAC?$AAE?$AA6?$AA0?$AA0?$AA?2?$AAP?$AAL?$AAA@ 100067d8     usb_ufnmddbase_common_topaz_v1:descript.obj
 0001:000058b0       ??_C@_1FE@FBCNDEDD@?$AA?$CF?$AAs?$AA?5?$AAI?$AAn?$AAv?$AAa?$AAl?$AAi?$AAd?$AA?5?$AAS?$AAt?$AAr?$AAi?$AAn?$AAg?$AA?5?$AAS?$AAe?$AAt?$AA?5?$AAf?$AAo?$AAr?$AA?5?$AAL?$AAa?$AAn?$AAg?$AAI?$AAD@ 100068b0     usb_ufnmddbase_common_topaz_v1:descript.obj
 0001:00005904       ??_C@_1DC@DNKCNEFL@?$AA?$CF?$AAs?$AA?5?$AAI?$AAn?$AAv?$AAa?$AAl?$AAi?$AAd?$AA?5?$AAS?$AAt?$AAr?$AAi?$AAn?$AAg?$AA?5?$AAS?$AAe?$AAt?$AAs?$AA?$AN?$AA?6?$AA?$AA@ 10006904     usb_ufnmddbase_common_topaz_v1:descript.obj
 0001:00005938       ??_C@_1FG@IIFFPMAK@?$AAU?$AAs?$AAb?$AAF?$AAn?$AAM?$AAd?$AAd?$AA?$CB?$AAC?$AAD?$AAe?$AAs?$AAc?$AAr?$AAi?$AAp?$AAt?$AAo?$AAr?$AAs?$AA?3?$AA?3?$AAV?$AAa?$AAl?$AAi?$AAd?$AAa?$AAt?$AAe?$AAD@ 10006938     usb_ufnmddbase_common_topaz_v1:descript.obj
 0001:00005990       ??_C@_1DM@NNOKJKLJ@?$AAU?$AAs?$AAb?$AAF?$AAn?$AAM?$AAd?$AAd?$AA?$CB?$AAC?$AAD?$AAe?$AAs?$AAc?$AAr?$AAi?$AAp?$AAt?$AAo?$AAr?$AAs?$AA?3?$AA?3?$AAC?$AAl?$AAo?$AAn?$AAe?$AA?3?$AA?$AA@ 10006990     usb_ufnmddbase_common_topaz_v1:descript.obj
 0001:000059d0       ??_C@_1EO@EMKBDIEA@?$AA?$CF?$AAs?$AA?5?$AAC?$AAo?$AAu?$AAl?$AAd?$AA?5?$AAn?$AAo?$AAt?$AA?5?$AAR?$AAe?$AAg?$AAi?$AAs?$AAt?$AAe?$AAr?$AAD?$AAe?$AAv?$AAi?$AAc?$AAe?$AA?5?$AAw?$AAi?$AAt?$AAh@ 100069d0     usb_ufnmddbase_common_topaz_v1:descript.obj
 0001:00005a20       ??_C@_1EO@KBHNPCNG@?$AAU?$AAs?$AAb?$AAF?$AAn?$AAM?$AAd?$AAd?$AA?$CB?$AAC?$AAD?$AAe?$AAs?$AAc?$AAr?$AAi?$AAp?$AAt?$AAo?$AAr?$AAs?$AA?3?$AA?3?$AAR?$AAe?$AAg?$AAi?$AAs?$AAt?$AAe?$AAr?$AAD@ 10006a20     usb_ufnmddbase_common_topaz_v1:descript.obj
 0001:00005a70       ??_C@_1EA@JJLFNNAH@?$AA?$CF?$AAs?$AA?5?$AAB?$AAu?$AAf?$AAf?$AAe?$AAr?$AA?5?$AAl?$AAe?$AAn?$AAg?$AAt?$AAh?$AA?5?$AAi?$AAs?$AA?5?$AAt?$AAo?$AAo?$AA?5?$AAs?$AAh?$AAo?$AAr?$AAt?$AA?$AN?$AA?6?$AA?$AA@ 10006a70     usb_ufnmddbase_common_topaz_v1:descript.obj
 0001:00005ab0       ??_C@_1CK@IGLELJIC@?$AAU?$AAs?$AAb?$AAF?$AAn?$AAM?$AAd?$AAd?$AA?$CB?$AAF?$AAi?$AAl?$AAl?$AAB?$AAu?$AAf?$AAf?$AAe?$AAr?$AA?3?$AA?$AA@ 10006ab0     usb_ufnmddbase_common_topaz_v1:descript.obj
 0001:00005adc       ??_C@_1DG@OEECILGP@?$AA?$CF?$AAs?$AA?5?$AAS?$AAt?$AAr?$AAi?$AAn?$AAg?$AA?5?$AA?$CF?$AAs?$AA?5?$AAi?$AAs?$AA?5?$AAt?$AAo?$AAo?$AA?5?$AAl?$AAo?$AAn?$AAg?$AA?$AN?$AA?6?$AA?$AA@ 10006adc     usb_ufnmddbase_common_topaz_v1:descript.obj
 0001:00005b18       ??_C@_1FM@PMFBNJCI@?$AA?$CF?$AAs?$AA?5?$AAS?$AAt?$AAr?$AAi?$AAn?$AAg?$AA?5?$AAc?$AAo?$AAu?$AAn?$AAt?$AA?5?$AAa?$AAc?$AAr?$AAo?$AAs?$AAs?$AA?5?$AAl?$AAo?$AAc?$AAa?$AAl?$AAe?$AAs?$AA?5?$AAd@ 10006b18     usb_ufnmddbase_common_topaz_v1:descript.obj
 0001:00005b78       ??_C@_1EK@GDONALFB@?$AAU?$AAs?$AAb?$AAF?$AAn?$AAM?$AAd?$AAd?$AA?$CB?$AAC?$AAD?$AAe?$AAs?$AAc?$AAr?$AAi?$AAp?$AAt?$AAo?$AAr?$AAs?$AA?3?$AA?3?$AAC?$AAl?$AAo?$AAn?$AAe?$AAS?$AAt?$AAr?$AAi@ 10006b78     usb_ufnmddbase_common_topaz_v1:descript.obj
 0001:00005bc8       ??_C@_1EM@MPABGIFO@?$AAU?$AAs?$AAb?$AAF?$AAn?$AAM?$AAd?$AAd?$AA?$CB?$AAC?$AAD?$AAe?$AAs?$AAc?$AAr?$AAi?$AAp?$AAt?$AAo?$AAr?$AAs?$AA?3?$AA?3?$AAI?$AAs?$AAS?$AAu?$AAp?$AAp?$AAo?$AAr?$AAt@ 10006bc8     usb_ufnmddbase_common_topaz_v1:descript.obj
 0001:00005c18       ??_C@_1MM@PEMIACJK@?$AAc?$AA?3?$AA?2?$AAw?$AAi?$AAn?$AAc?$AAe?$AAr?$AAo?$AAo?$AAt?$AAs?$AA?2?$AAt?$AAo?$AAp?$AAa?$AAz?$AA?2?$AAw?$AAi?$AAn?$AAc?$AAe?$AA6?$AA0?$AA0?$AA?2?$AAp?$AAl?$AAa@ 10006c18     usb_ufnmddbase_common_topaz_v1:descript.obj
 0001:00005ce8       ??_C@_1EG@PEOBIFPJ@?$AA?$CF?$AAs?$AA?5?$AAI?$AAn?$AAv?$AAa?$AAl?$AAi?$AAd?$AA?5?$AAG?$AAe?$AAt?$AAD?$AAe?$AAs?$AAc?$AAr?$AAi?$AAp?$AAt?$AAo?$AAr?$AA?5?$AAr?$AAe?$AAq?$AAu?$AAe?$AAs?$AAt@ 10006ce8     usb_ufnmddbase_common_topaz_v1:descript.obj
 0001:00005d30       ??_C@_1GK@NAANGNEK@?$AA?$CF?$AAs?$AA?5?$AAR?$AAe?$AAq?$AAu?$AAe?$AAs?$AAt?$AA?5?$AAf?$AAo?$AAr?$AA?5?$AAs?$AAt?$AAr?$AAi?$AAn?$AAg?$AAs?$AA?0?$AA?5?$AAb?$AAu?$AAt?$AA?5?$AAM?$AAD?$AAD?$AA?5@ 10006d30     usb_ufnmddbase_common_topaz_v1:descript.obj
 0001:00005d9c       ??_C@_1DK@FOGHCLJO@?$AA?$CF?$AAs?$AA?5?$AAI?$AAn?$AAv?$AAa?$AAl?$AAi?$AAd?$AA?5?$AAs?$AAt?$AAr?$AAi?$AAn?$AAg?$AA?5?$AAi?$AAn?$AAd?$AAe?$AAx?$AA?5?$AA?$CF?$AAu?$AA?$AN?$AA?6?$AA?$AA@ 10006d9c     usb_ufnmddbase_common_topaz_v1:descript.obj
 0001:00005dd8       ??_C@_1EA@PKLEDDMG@?$AA?$CF?$AAs?$AA?5?$AAI?$AAn?$AAv?$AAa?$AAl?$AAi?$AAd?$AA?5?$AAl?$AAa?$AAn?$AAg?$AAu?$AAa?$AAg?$AAe?$AA?5?$AAi?$AAd?$AA?5?$AA0?$AAx?$AA?$CF?$AA0?$AA4?$AAx?$AA?$AN?$AA?6?$AA?$AA@ 10006dd8     usb_ufnmddbase_common_topaz_v1:descript.obj
 0001:00005e18       ??_C@_1GO@NJIKODDH@?$AA?$CF?$AAs?$AA?5?$AAG?$AAe?$AAt?$AA?5?$AAs?$AAt?$AAr?$AAi?$AAn?$AAg?$AA?5?$AAd?$AAe?$AAs?$AAc?$AAr?$AAi?$AAp?$AAt?$AAo?$AAr?$AA?5?$AAr?$AAe?$AAq?$AAu?$AAe?$AAs?$AAt@ 10006e18     usb_ufnmddbase_common_topaz_v1:descript.obj
 0001:00005e88       ??_C@_1EI@MBHMMNKN@?$AA?$CF?$AAs?$AA?5?$AAI?$AAn?$AAv?$AAa?$AAl?$AAi?$AAd?$AA?5?$AAc?$AAo?$AAn?$AAf?$AAi?$AAg?$AAu?$AAr?$AAa?$AAt?$AAi?$AAo?$AAn?$AA?5?$AAi?$AAn?$AAd?$AAe?$AAx?$AA?5?$AA?$CF@ 10006e88     usb_ufnmddbase_common_topaz_v1:descript.obj
 0001:00005ed0       ??_C@_1GE@FJFGADOB@?$AA?$CF?$AAs?$AA?5?$AAG?$AAe?$AAt?$AA?$CF?$AAs?$AA?5?$AAc?$AAo?$AAn?$AAf?$AAi?$AAg?$AAu?$AAr?$AAa?$AAt?$AAi?$AAo?$AAn?$AA?5?$AAd?$AAe?$AAs?$AAc?$AAr?$AAi?$AAp?$AAt?$AAo@ 10006ed0     usb_ufnmddbase_common_topaz_v1:descript.obj
 0001:00005f34       ??_C@_1BK@KGPJHBHL@?$AA?5?$AAo?$AAt?$AAh?$AAe?$AAr?$AA?5?$AAs?$AAp?$AAe?$AAe?$AAd?$AA?$AA@ 10006f34     usb_ufnmddbase_common_topaz_v1:descript.obj
 0001:00005f50       ??_C@_11LOCGONAA@?$AA?$AA@ 10006f50     usb_ufnmddbase_common_topaz_v1:descript.obj
 0001:00005f58       ??_C@_1FM@FFOCBCJM@?$AA?$CF?$AAs?$AA?5?$AAG?$AAe?$AAt?$AA?5?$AAd?$AAe?$AAv?$AAi?$AAc?$AAe?$AA?5?$AAq?$AAu?$AAa?$AAl?$AAi?$AAf?$AAi?$AAe?$AAr?$AA?5?$AAd?$AAe?$AAs?$AAc?$AAr?$AAi?$AAp?$AAt@ 10006f58     usb_ufnmddbase_common_topaz_v1:descript.obj
 0001:00005fb8       ??_C@_1EI@JANJLCOJ@?$AA?$CF?$AAs?$AA?5?$AAG?$AAe?$AAt?$AA?5?$AAd?$AAe?$AAv?$AAi?$AAc?$AAe?$AA?5?$AAd?$AAe?$AAs?$AAc?$AAr?$AAi?$AAp?$AAt?$AAo?$AAr?$AA?5?$AAr?$AAe?$AAq?$AAu?$AAe?$AAs?$AAt@ 10006fb8     usb_ufnmddbase_common_topaz_v1:descript.obj
 0001:00006000       ??_C@_1DK@DKFCOOOF@?$AA?$CF?$AAs?$AA?5?$AAI?$AAn?$AAv?$AAa?$AAl?$AAi?$AAd?$AA?5?$AAw?$AAI?$AAn?$AAd?$AAe?$AAx?$AA?5?$AAv?$AAa?$AAl?$AAu?$AAe?$AA?5?$AA?$CF?$AAu?$AA?$AN?$AA?6?$AA?$AA@ 10007000     usb_ufnmddbase_common_topaz_v1:descript.obj
 0001:00006040       ??_C@_1FK@ILPBFMNK@?$AAU?$AAs?$AAb?$AAF?$AAn?$AAM?$AAd?$AAd?$AA?$CB?$AAC?$AAD?$AAe?$AAs?$AAc?$AAr?$AAi?$AAp?$AAt?$AAo?$AAr?$AAs?$AA?3?$AA?3?$AAP?$AAr?$AAo?$AAc?$AAe?$AAs?$AAs?$AAG?$AAe@ 10007040     usb_ufnmddbase_common_topaz_v1:descript.obj
 0001:0000609c       ??_C@_1CC@EEBNEEGK@?$AA?$CF?$AAs?$AA?5?$AAn?$AAe?$AAw?$AA?5?$AAf?$AAa?$AAi?$AAl?$AAe?$AAd?$AA?4?$AA?$AN?$AA?6?$AA?$AA@ 1000709c     usb_ufnmddbase_common_topaz_v1:descript.obj
 0001:000060c0       ??_C@_1DA@IDBJIGIL@?$AAU?$AAs?$AAb?$AAF?$AAn?$AAM?$AAd?$AAd?$AA?$CB?$AAC?$AAD?$AAe?$AAv?$AAi?$AAc?$AAe?$AA?3?$AA?3?$AAI?$AAn?$AAi?$AAt?$AA?3?$AA?$AA@ 100070c0     usb_ufnmddbase_common_topaz_v1:descript.obj
 0001:000060f0       ??_C@_1DC@GAILFPML@?$AAU?$AAs?$AAb?$AAF?$AAn?$AAM?$AAd?$AAd?$AA?$CB?$AAC?$AAD?$AAe?$AAv?$AAi?$AAc?$AAe?$AA?3?$AA?3?$AAC?$AAl?$AAo?$AAn?$AAe?$AA?3?$AA?$AA@ 100070f0     usb_ufnmddbase_common_topaz_v1:descript.obj
 0001:00006128       ??_C@_1GO@ENFIBCBE@?$AA?$CF?$AAs?$AA?5?$AAT?$AAh?$AAi?$AAs?$AA?5?$AAP?$AAD?$AAD?$AA?5?$AAd?$AAo?$AAe?$AAs?$AA?5?$AAn?$AAo?$AAt?$AA?5?$AAs?$AAu?$AAp?$AAp?$AAo?$AAr?$AAt?$AA?5?$AAm?$AAu?$AAl@ 10007128     usb_ufnmddbase_common_topaz_v1:descript.obj
 0001:00006198       ??_C@_1EC@NBNBANHA@?$AAU?$AAs?$AAb?$AAF?$AAn?$AAM?$AAd?$AAd?$AA?$CB?$AAC?$AAD?$AAe?$AAv?$AAi?$AAc?$AAe?$AA?3?$AA?3?$AAI?$AAs?$AAS?$AAu?$AAp?$AAp?$AAo?$AAr?$AAt?$AAa?$AAb?$AAl?$AAe?$AA?3@ 10007198     usb_ufnmddbase_common_topaz_v1:descript.obj
 0001:000061e0       ??_C@_1GO@LKEJBJIG@?$AA?$CF?$AAs?$AA?5?$AAb?$AAC?$AAo?$AAn?$AAf?$AAi?$AAg?$AAu?$AAr?$AAa?$AAt?$AAi?$AAo?$AAn?$AAV?$AAa?$AAl?$AAu?$AAe?$AA?5?$AA0?$AAx?$AA?$CF?$AA0?$AA2?$AAx?$AA?5?$AAi?$AAs@ 100071e0     usb_ufnmddbase_common_topaz_v1:descript.obj
 0001:00006250       ??_C@_1GC@LMIHPMAO@?$AAU?$AAs?$AAb?$AAF?$AAn?$AAM?$AAd?$AAd?$AA?$CB?$AAC?$AAD?$AAe?$AAv?$AAi?$AAc?$AAe?$AA?3?$AA?3?$AAV?$AAa?$AAl?$AAi?$AAd?$AAa?$AAt?$AAe?$AAD?$AAe?$AAs?$AAc?$AAr?$AAi@ 10007250     usb_ufnmddbase_common_topaz_v1:descript.obj
 0001:000062b4       ??_C@_1DA@OEFEGMN@?$AA?$CF?$AAs?$AA?5?$AAN?$AAo?$AA?5?$AAc?$AAo?$AAn?$AAf?$AAi?$AAg?$AAu?$AAr?$AAa?$AAt?$AAi?$AAo?$AAn?$AAs?$AA?$CB?$AA?$AN?$AA?6?$AA?$AA@ 100072b4     usb_ufnmddbase_common_topaz_v1:descript.obj
 0001:000062e8       ??_C@_1EM@POMJJKAN@?$AAU?$AAs?$AAb?$AAF?$AAn?$AAM?$AAd?$AAd?$AA?$CB?$AAC?$AAD?$AAe?$AAv?$AAi?$AAc?$AAe?$AA?3?$AA?3?$AAV?$AAa?$AAl?$AAi?$AAd?$AAa?$AAt?$AAe?$AAD?$AAe?$AAs?$AAc?$AAr?$AAi@ 100072e8     usb_ufnmddbase_common_topaz_v1:descript.obj
 0001:00006334       ??_C@_1DO@PFCLCDIA@?$AAU?$AAs?$AAb?$AAF?$AAn?$AAM?$AAd?$AAd?$AA?$CB?$AAC?$AAC?$AAo?$AAn?$AAf?$AAi?$AAg?$AAu?$AAr?$AAa?$AAt?$AAi?$AAo?$AAn?$AA?3?$AA?3?$AAI?$AAn?$AAi?$AAt?$AA?3?$AA?$AA@ 10007334     usb_ufnmddbase_common_topaz_v1:descript.obj
 0001:00006378       ??_C@_1EK@JPNOEGGH@?$AA?$CF?$AAs?$AA?5?$AAN?$AAo?$AAt?$AA?5?$AAe?$AAn?$AAo?$AAu?$AAg?$AAh?$AA?5?$AAe?$AAn?$AAd?$AAp?$AAo?$AAi?$AAn?$AAt?$AAs?$AA?5?$AAf?$AAo?$AAr?$AA?5?$AAc?$AAl?$AAi?$AAe@ 10007378     usb_ufnmddbase_common_topaz_v1:descript.obj
 0001:000063c8       ??_C@_1FE@DMLHBHKB@?$AA?$CF?$AAs?$AA?5?$AAP?$AAD?$AAD?$AA?5?$AAc?$AAa?$AAn?$AAn?$AAo?$AAt?$AA?5?$AAs?$AAu?$AAp?$AAp?$AAo?$AAr?$AAt?$AA?5?$AAt?$AAh?$AAe?$AA?5?$AAc?$AAo?$AAn?$AAf?$AAi?$AAg@ 100073c8     usb_ufnmddbase_common_topaz_v1:descript.obj
 0001:00006420       ??_C@_1FA@BOJJAFFO@?$AAU?$AAs?$AAb?$AAF?$AAn?$AAM?$AAd?$AAd?$AA?$CB?$AAC?$AAC?$AAo?$AAn?$AAf?$AAi?$AAg?$AAu?$AAr?$AAa?$AAt?$AAi?$AAo?$AAn?$AA?3?$AA?3?$AAI?$AAs?$AAS?$AAu?$AAp?$AAp?$AAo@ 10007420     usb_ufnmddbase_common_topaz_v1:descript.obj
 0001:00006470       ??_C@_1KE@HFOIEBFH@?$AA?$CF?$AAs?$AA?5?$AAI?$AAn?$AAt?$AAe?$AAr?$AAf?$AAa?$AAc?$AAe?$AA?$CI?$AA?$CF?$AAu?$AA?$CJ?$AA?5?$AAh?$AAa?$AAs?$AA?5?$AAi?$AAn?$AAv?$AAa?$AAl?$AAi?$AAd?$AA?5?$AAa?$AAl?$AAt@ 10007470     usb_ufnmddbase_common_topaz_v1:descript.obj
 0001:00006518       ??_C@_1HO@DGMAOALD@?$AA?$CF?$AAs?$AA?5?$AAI?$AAn?$AAt?$AAe?$AAr?$AAf?$AAa?$AAc?$AAe?$AA?5?$AAn?$AAu?$AAm?$AAb?$AAe?$AAr?$AA?5?$AA?$CF?$AAu?$AA?5?$AAi?$AAs?$AA?5?$AAi?$AAn?$AAv?$AAa?$AAl?$AAi@ 10007518     usb_ufnmddbase_common_topaz_v1:descript.obj
 0001:00006598       ??_C@_1JA@NPAIKCBA@?$AA?$CF?$AAs?$AA?5?$AAI?$AAn?$AAt?$AAe?$AAr?$AAf?$AAa?$AAc?$AAe?$AA?$CI?$AA?$CF?$AAu?$AA?$CJ?$AA?5?$AAh?$AAa?$AAs?$AA?5?$AAi?$AAn?$AAv?$AAa?$AAl?$AAi?$AAd?$AA?5?$AAa?$AAl?$AAt@ 10007598     usb_ufnmddbase_common_topaz_v1:descript.obj
 0001:00006628       ??_C@_1FC@FECGJLHK@?$AA?$CF?$AAs?$AA?5?$AAI?$AAn?$AAv?$AAa?$AAl?$AAi?$AAd?$AA?5?$AAc?$AAb?$AAE?$AAx?$AAt?$AAe?$AAn?$AAd?$AAe?$AAd?$AA?1?$AAp?$AAv?$AAE?$AAx?$AAt?$AAe?$AAn?$AAd?$AAe?$AAd@ 10007628     usb_ufnmddbase_common_topaz_v1:descript.obj
 0001:0000667c       ??_C@_1DM@IOJGGAHK@?$AA?$CF?$AAs?$AA?5?$AAN?$AAo?$AA?5?$AAi?$AAn?$AAt?$AAe?$AAr?$AAf?$AAa?$AAc?$AAe?$AAs?$AA?5?$AAi?$AAn?$AA?5?$AAc?$AAo?$AAn?$AAf?$AAi?$AAg?$AA?$CB?$AA?$AN?$AA?6?$AA?$AA@ 1000767c     usb_ufnmddbase_common_topaz_v1:descript.obj
 0001:000066b8       ??_C@_1FK@NEKIDNEM@?$AAU?$AAs?$AAb?$AAF?$AAn?$AAM?$AAd?$AAd?$AA?$CB?$AAC?$AAC?$AAo?$AAn?$AAf?$AAi?$AAg?$AAu?$AAr?$AAa?$AAt?$AAi?$AAo?$AAn?$AA?3?$AA?3?$AAV?$AAa?$AAl?$AAi?$AAd?$AAa?$AAt@ 100076b8     usb_ufnmddbase_common_topaz_v1:descript.obj
 0001:00006718       ??_C@_1HA@FOKIDKGO@?$AAU?$AAs?$AAb?$AAF?$AAn?$AAM?$AAd?$AAd?$AA?$CB?$AAC?$AAC?$AAo?$AAn?$AAf?$AAi?$AAg?$AAu?$AAr?$AAa?$AAt?$AAi?$AAo?$AAn?$AA?3?$AA?3?$AAG?$AAe?$AAn?$AAe?$AAr?$AAa?$AAt@ 10007718     usb_ufnmddbase_common_topaz_v1:descript.obj
 0001:00006788       ??_C@_1FI@OBADPFDH@?$AAU?$AAs?$AAb?$AAF?$AAn?$AAM?$AAd?$AAd?$AA?$CB?$AAC?$AAC?$AAo?$AAn?$AAf?$AAi?$AAg?$AAu?$AAr?$AAa?$AAt?$AAi?$AAo?$AAn?$AA?3?$AA?3?$AAC?$AAo?$AAp?$AAy?$AAU?$AAf?$AAn@ 10007788     usb_ufnmddbase_common_topaz_v1:descript.obj
 0001:000067e0       ??_C@_1FO@IMCIAINH@?$AA?$CF?$AAs?$AA?5?$AAC?$AAo?$AAp?$AAi?$AAe?$AAd?$AA?5?$AA?$CF?$AAd?$AA?5?$AAb?$AAy?$AAt?$AAe?$AAs?$AA?5?$AAo?$AAf?$AA?5?$AAe?$AAx?$AAt?$AAe?$AAn?$AAd?$AAe?$AAd?$AA?5?$AAd@ 100077e0     usb_ufnmddbase_common_topaz_v1:descript.obj
 0001:00006840       ??_C@_1DG@ILOBAOFA@?$AAU?$AAs?$AAb?$AAF?$AAn?$AAM?$AAd?$AAd?$AA?$CB?$AAC?$AAo?$AAp?$AAy?$AAE?$AAx?$AAt?$AAe?$AAn?$AAd?$AAe?$AAd?$AAD?$AAe?$AAs?$AAc?$AA?3?$AA?$AA@ 10007840     usb_ufnmddbase_common_topaz_v1:descript.obj
 0001:00006878       ??_C@_1FI@BHAAOGDE@?$AAU?$AAs?$AAb?$AAF?$AAn?$AAM?$AAd?$AAd?$AA?$CB?$AAC?$AAC?$AAo?$AAn?$AAf?$AAi?$AAg?$AAu?$AAr?$AAa?$AAt?$AAi?$AAo?$AAn?$AA?3?$AA?3?$AAF?$AAr?$AAe?$AAe?$AAU?$AAf?$AAn@ 10007878     usb_ufnmddbase_common_topaz_v1:descript.obj
 0001:000068d0       ??_C@_1DG@LDPNGGJO@?$AAU?$AAs?$AAb?$AAF?$AAn?$AAM?$AAd?$AAd?$AA?$CB?$AAC?$AAI?$AAn?$AAt?$AAe?$AAr?$AAf?$AAa?$AAc?$AAe?$AA?3?$AA?3?$AAI?$AAn?$AAi?$AAt?$AA?3?$AA?$AA@ 100078d0     usb_ufnmddbase_common_topaz_v1:descript.obj
 0001:00006908       ??_C@_1EI@KFGAMAKC@?$AA?$CF?$AAs?$AA?5?$AAN?$AAo?$AA?5?$AAe?$AAn?$AAd?$AAp?$AAo?$AAi?$AAn?$AAt?$AA?5?$AAs?$AAt?$AAr?$AAu?$AAc?$AAt?$AAu?$AAr?$AAe?$AA?5?$AAp?$AAr?$AAo?$AAv?$AAi?$AAd?$AAe@ 10007908     usb_ufnmddbase_common_topaz_v1:descript.obj
 0001:00006950       ??_C@_1FC@LJOPAPJJ@?$AAU?$AAs?$AAb?$AAF?$AAn?$AAM?$AAd?$AAd?$AA?$CB?$AAC?$AAI?$AAn?$AAt?$AAe?$AAr?$AAf?$AAa?$AAc?$AAe?$AA?3?$AA?3?$AAV?$AAa?$AAl?$AAi?$AAd?$AAa?$AAt?$AAe?$AAD?$AAe?$AAs@ 10007950     usb_ufnmddbase_common_topaz_v1:descript.obj
 0001:000069a8       ??_C@_1GA@MLGFBDPO@?$AA?$CF?$AAs?$AA?5?$AAC?$AAa?$AAn?$AAn?$AAo?$AAt?$AA?5?$AAs?$AAu?$AAp?$AAp?$AAo?$AAr?$AAt?$AA?5?$AAp?$AAr?$AAo?$AAv?$AAi?$AAd?$AAe?$AAd?$AA?5?$AA?$CF?$AAs?$AA?5?$AAs?$AAp@ 100079a8     usb_ufnmddbase_common_topaz_v1:descript.obj
 0001:00006a08       ??_C@_1EI@KPMLCBEM@?$AAU?$AAs?$AAb?$AAF?$AAn?$AAM?$AAd?$AAd?$AA?$CB?$AAC?$AAI?$AAn?$AAt?$AAe?$AAr?$AAf?$AAa?$AAc?$AAe?$AA?3?$AA?3?$AAI?$AAs?$AAS?$AAu?$AAp?$AAp?$AAo?$AAr?$AAt?$AAa?$AAb@ 10007a08     usb_ufnmddbase_common_topaz_v1:descript.obj
 0001:00006a50       ??_C@_1FK@FDIFNHFI@?$AA?$CF?$AAs?$AA?5?$AAE?$AAn?$AAd?$AAp?$AAo?$AAi?$AAn?$AAt?$AA?5?$AAd?$AAe?$AAs?$AAc?$AAr?$AAi?$AAp?$AAt?$AAo?$AAr?$AA?5?$AAc?$AAa?$AAn?$AAn?$AAo?$AAt?$AA?5?$AAb?$AAe@ 10007a50     usb_ufnmddbase_common_topaz_v1:descript.obj
 0001:00006ab0       ??_C@_1GO@CLABJPCH@?$AA?$CF?$AAs?$AA?5?$AAE?$AAn?$AAd?$AAp?$AAo?$AAi?$AAn?$AAt?$AA?5?$AAc?$AAa?$AAn?$AA?5?$AAb?$AAe?$AA?5?$AAs?$AAu?$AAp?$AAp?$AAo?$AAr?$AAt?$AAe?$AAd?$AA?5?$AAb?$AAy?$AA?5@ 10007ab0     usb_ufnmddbase_common_topaz_v1:descript.obj
 0001:00006b20       ??_C@_1EM@ONCAAMBK@?$AAU?$AAs?$AAb?$AAF?$AAn?$AAM?$AAd?$AAd?$AA?$CB?$AAC?$AAM?$AAd?$AAd?$AAE?$AAn?$AAd?$AAp?$AAo?$AAi?$AAn?$AAt?$AA?3?$AA?3?$AAI?$AAs?$AAS?$AAu?$AAp?$AAp?$AAo?$AAr?$AAt@ 10007b20     usb_ufnmddbase_common_topaz_v1:descript.obj
 0001:00006b70       ??_C@_1FG@EPFGBDLJ@?$AA?$CF?$AAs?$AA?5?$AAI?$AAn?$AAv?$AAa?$AAl?$AAi?$AAd?$AA?5?$AAp?$AAa?$AAc?$AAk?$AAe?$AAt?$AA?5?$AAs?$AAi?$AAz?$AAe?$AA?5?$AAf?$AAo?$AAr?$AA?5?$AAe?$AAn?$AAd?$AAp?$AAo@ 10007b70     usb_ufnmddbase_common_topaz_v1:descript.obj
 0001:00006bc8       ??_C@_1FG@HDHFMBAF@?$AAU?$AAs?$AAb?$AAF?$AAn?$AAM?$AAd?$AAd?$AA?$CB?$AAC?$AAM?$AAd?$AAd?$AAE?$AAn?$AAd?$AAp?$AAo?$AAi?$AAn?$AAt?$AA?3?$AA?3?$AAV?$AAa?$AAl?$AAi?$AAd?$AAa?$AAt?$AAe?$AAD@ 10007bc8     usb_ufnmddbase_common_topaz_v1:descript.obj
 0001:00006c20       ??_C@_1HO@LFFCPBPL@?$AA?$CF?$AAs?$AA?5?$AAC?$AAa?$AAn?$AAn?$AAo?$AAt?$AA?5?$AAs?$AAa?$AAt?$AAi?$AAs?$AAf?$AAy?$AA?5?$AA?$CF?$AAs?$AA?5?$AAs?$AAp?$AAe?$AAe?$AAd?$AA?5?$AAE?$AAP?$AA0?$AA?5?$AAp@ 10007c20     usb_ufnmddbase_common_topaz_v1:descript.obj
 0001:00006ca0       ??_C@_1GE@FLBJHEFO@?$AAU?$AAs?$AAb?$AAF?$AAn?$AAM?$AAd?$AAd?$AA?$CB?$AAC?$AAM?$AAd?$AAd?$AAE?$AAn?$AAd?$AAp?$AAo?$AAi?$AAn?$AAt?$AA?3?$AA?3?$AAI?$AAs?$AAE?$AAn?$AAd?$AAp?$AAo?$AAi?$AAn@ 10007ca0     usb_ufnmddbase_common_topaz_v1:descript.obj
 0001:00006d04       ??_C@_1DK@HCGGINKD@?$AA?$CF?$AAs?$AA?5?$AAR?$AAe?$AAf?$AAe?$AAr?$AAe?$AAn?$AAc?$AAe?$AAd?$AA?5?$AA0?$AAx?$AA?$CF?$AA0?$AA8?$AAx?$AA?5?$AAt?$AAo?$AA?5?$AA?$CF?$AAx?$AA?$AN?$AA?6?$AA?$AA@ 10007d04     usb_ufnmddbase_common_topaz_v1:transfer.obj
 0001:00006d40       ??_C@_1NI@HMFBOIHA@?$AAC?$AA?3?$AA?2?$AAW?$AAI?$AAN?$AAC?$AAE?$AAR?$AAO?$AAO?$AAT?$AAS?$AA?2?$AAT?$AAo?$AAp?$AAa?$AAz?$AA?2?$AAW?$AAI?$AAN?$AAC?$AAE?$AA6?$AA0?$AA0?$AA?2?$AAP?$AAL?$AAA@ 10007d40     usb_ufnmddbase_common_topaz_v1:transfer.obj
 0001:00006e18       ??_C@_1EE@CMPAPJAH@?$AAU?$AAs?$AAb?$AAF?$AAn?$AAM?$AAd?$AAd?$AA?$CB?$AAC?$AAU?$AAf?$AAn?$AAM?$AAd?$AAd?$AAT?$AAr?$AAa?$AAn?$AAs?$AAf?$AAe?$AAr?$AA?3?$AA?3?$AAA?$AAd?$AAd?$AAR?$AAe?$AAf@ 10007e18     usb_ufnmddbase_common_topaz_v1:transfer.obj
 0001:00006e5c       ??_C@_1DO@BGOLBBCP@?$AA?$CF?$AAs?$AA?5?$AAD?$AAe?$AAr?$AAe?$AAf?$AAe?$AAr?$AAe?$AAn?$AAc?$AAe?$AAd?$AA?5?$AA0?$AAx?$AA?$CF?$AA0?$AA8?$AAx?$AA?5?$AAt?$AAo?$AA?5?$AA?$CF?$AAx?$AA?$AN?$AA?6?$AA?$AA@ 10007e5c     usb_ufnmddbase_common_topaz_v1:transfer.obj
 0001:00006ea0       ??_C@_1EG@ONHLBMAL@?$AAU?$AAs?$AAb?$AAF?$AAn?$AAM?$AAd?$AAd?$AA?$CB?$AAC?$AAU?$AAf?$AAn?$AAM?$AAd?$AAd?$AAT?$AAr?$AAa?$AAn?$AAs?$AAf?$AAe?$AAr?$AA?3?$AA?3?$AAR?$AAe?$AAl?$AAe?$AAa?$AAs@ 10007ea0     usb_ufnmddbase_common_topaz_v1:transfer.obj
 0001:00006ee8       ??_C@_1GC@LPBPDPBE@?$AAU?$AAs?$AAb?$AAF?$AAn?$AAM?$AAd?$AAd?$AA?$CB?$AAC?$AAU?$AAf?$AAn?$AAM?$AAd?$AAd?$AAT?$AAr?$AAa?$AAn?$AAs?$AAf?$AAe?$AAr?$AA?3?$AA?3?$AAC?$AAa?$AAl?$AAl?$AAC?$AAo@ 10007ee8     usb_ufnmddbase_common_topaz_v1:transfer.obj
 0001:00006f50       ??_C@_1FO@BLHFBLJN@?$AA?$CF?$AAs?$AA?5?$AAE?$AAx?$AAc?$AAe?$AAp?$AAt?$AAi?$AAo?$AAn?$AA?5?$AAc?$AAh?$AAe?$AAc?$AAk?$AAi?$AAn?$AAg?$AA?5?$AAt?$AAr?$AAa?$AAn?$AAs?$AAf?$AAe?$AAr?$AA?5?$AAh@ 10007f50     usb_ufnmddbase_common_topaz_v1:transfer.obj
 0001:00006fb0       ??_C@_1FO@MGPCLFKM@?$AA?$CF?$AAs?$AA?5?$AAI?$AAn?$AAv?$AAa?$AAl?$AAi?$AAd?$AA?5?$AAt?$AAr?$AAa?$AAn?$AAs?$AAf?$AAe?$AAr?$AA?5?$AAh?$AAa?$AAn?$AAd?$AAl?$AAe?$AA?5?$AA0?$AAx?$AA?$CF?$AA0?$AA8@ 10007fb0     usb_ufnmddbase_common_topaz_v1:transfer.obj
 0001:00007010       ??_C@_1EI@BPMEBILK@?$AA?$CF?$AAs?$AA?5?$AAI?$AAn?$AAv?$AAa?$AAl?$AAi?$AAd?$AA?5?$AAt?$AAr?$AAa?$AAn?$AAs?$AAf?$AAe?$AAr?$AA?5?$AAh?$AAa?$AAn?$AAd?$AAl?$AAe?$AA?5?$AA0?$AAx?$AA?$CF?$AA0?$AA8@ 10008010     usb_ufnmddbase_common_topaz_v1:transfer.obj
 0001:00007058       ??_C@_1GG@LAEGOPOI@?$AAU?$AAs?$AAb?$AAF?$AAn?$AAM?$AAd?$AAd?$AA?$CB?$AAC?$AAU?$AAf?$AAn?$AAM?$AAd?$AAd?$AAT?$AAr?$AAa?$AAn?$AAs?$AAf?$AAe?$AAr?$AA?3?$AA?3?$AAR?$AAe?$AAf?$AAe?$AAr?$AAe@ 10008058     usb_ufnmddbase_common_topaz_v1:transfer.obj
 0001:000070c0       ??_C@_1NE@HBJCGECF@?$AAC?$AA?3?$AA?2?$AAW?$AAI?$AAN?$AAC?$AAE?$AAR?$AAO?$AAO?$AAT?$AAS?$AA?2?$AAT?$AAo?$AAp?$AAa?$AAz?$AA?2?$AAW?$AAI?$AAN?$AAC?$AAE?$AA6?$AA0?$AA0?$AA?2?$AAP?$AAL?$AAA@ 100080c0     usb_ufnmddbase_common_topaz_v1:ufnbus.obj
 0001:00007194       ??_7CUfnBusDevice@@6B@     10008194     usb_ufnmddbase_common_topaz_v1:ufnbus.obj
 0001:000071b8       ??_7CUfnBus@@6B@           100081b8     usb_ufnmddbase_common_topaz_v1:ufnbus.obj
 0001:00007218       ??_C@_1BA@FGOFGFHE@?$AA?$CF?$AAs?$AA_?$AA?$CF?$AAd?$AA_?$AA0?$AA?$AA@ 10008218     usb_ufnmddbase_common_topaz_v1:ufnbus.obj
 0001:00007228       ??_C@_1M@LLKDCKCI@?$AAU?$AAS?$AAB?$AAF?$AAN?$AA?$AA@ 10008228     usb_ufnmddbase_common_topaz_v1:ufnbus.obj
 0001:00007238       ??_C@_1GE@HNFCJCHJ@?$AA?$CF?$AAs?$AA?5?$AAC?$AAo?$AAu?$AAl?$AAd?$AA?5?$AAn?$AAo?$AAt?$AA?5?$AAg?$AAe?$AAt?$AA?5?$AAd?$AAe?$AAv?$AAi?$AAc?$AAe?$AA?5?$AAi?$AAn?$AAf?$AAo?$AAr?$AAm?$AAa?$AAt@ 10008238     usb_ufnmddbase_common_topaz_v1:ufnbus.obj
 0001:0000729c       ??_C@_1DA@IKFMMLND@?$AAU?$AAs?$AAb?$AAF?$AAn?$AAM?$AAd?$AAd?$AA?$CB?$AAC?$AAU?$AAf?$AAn?$AAB?$AAu?$AAs?$AA?3?$AA?3?$AAI?$AAn?$AAi?$AAt?$AA?3?$AA?$AA@ 1000829c     usb_ufnmddbase_common_topaz_v1:ufnbus.obj
 0001:000072d0       ??_C@_1EE@FEBCNOJ@?$AA?$CF?$AAs?$AA?5?$AAU?$AAs?$AAi?$AAn?$AAg?$AA?5?$AAc?$AAl?$AAi?$AAe?$AAn?$AAt?$AA?5?$AAd?$AAr?$AAi?$AAv?$AAe?$AAr?$AA?5?$AAk?$AAe?$AAy?$AA?5?$AA?$CC?$AA?$CF?$AAs?$AA?$CC?$AA?$AN@ 100082d0     usb_ufnmddbase_common_topaz_v1:ufnbus.obj
 0001:00007318       ??_C@_1FG@MMNPAHCA@?$AA?$CF?$AAs?$AA?5?$AAR?$AAe?$AAg?$AA?5?$AAp?$AAa?$AAt?$AAh?$AA?5?$AAt?$AAo?$AAo?$AA?5?$AAl?$AAo?$AAn?$AAg?$AA?5?$AAf?$AAo?$AAr?$AA?5?$AAb?$AAu?$AAf?$AAf?$AAe?$AAr?$AA?4@ 10008318     usb_ufnmddbase_common_topaz_v1:ufnbus.obj
 0001:00007370       ??_C@_1M@DFKENGJN@?$AA?$CF?$AAs?$AA?2?$AA?$CF?$AAs?$AA?$AA@ 10008370     usb_ufnmddbase_common_topaz_v1:ufnbus.obj
 0001:0000737c       ??_C@_1DK@HJDLAGJ@?$AA?2?$AAD?$AAr?$AAi?$AAv?$AAe?$AAr?$AAs?$AA?2?$AAU?$AAS?$AAB?$AA?2?$AAF?$AAu?$AAn?$AAc?$AAt?$AAi?$AAo?$AAn?$AAD?$AAr?$AAi?$AAv?$AAe?$AAr?$AAs?$AA?$AA@ 1000837c     usb_ufnmddbase_common_topaz_v1:ufnbus.obj
 0001:000073b8       ??_C@_1DO@HBNODAHL@?$AAU?$AAs?$AAb?$AAF?$AAn?$AAM?$AAd?$AAd?$AA?$CB?$AAC?$AAU?$AAf?$AAn?$AAB?$AAu?$AAs?$AA?3?$AA?3?$AAC?$AAr?$AAe?$AAa?$AAt?$AAe?$AAC?$AAh?$AAi?$AAl?$AAd?$AA?3?$AA?$AA@ 100083b8     usb_ufnmddbase_common_topaz_v1:ufnbus.obj
 0001:000073f8       ??_C@_1HC@FKJDOKIB@?$AA?$CF?$AAs?$AA?5?$AAF?$AAa?$AAi?$AAl?$AAe?$AAd?$AA?5?$AAt?$AAo?$AA?5?$AAo?$AAp?$AAe?$AAn?$AA?5?$AAf?$AAu?$AAn?$AAc?$AAt?$AAi?$AAo?$AAn?$AA?5?$AAc?$AAl?$AAi?$AAe?$AAn@ 100083f8     usb_ufnmddbase_common_topaz_v1:ufnbus.obj
 0001:00007470       ??_C@_1EG@HEKJEEOM@?$AAU?$AAs?$AAb?$AAF?$AAn?$AAM?$AAd?$AAd?$AA?$CB?$AAC?$AAU?$AAf?$AAn?$AAB?$AAu?$AAs?$AA?3?$AA?3?$AAO?$AAp?$AAe?$AAn?$AAF?$AAu?$AAn?$AAc?$AAt?$AAi?$AAo?$AAn?$AAK?$AAe@ 10008470     usb_ufnmddbase_common_topaz_v1:ufnbus.obj
 0001:000074b8       ??_C@_1DG@NLGCFDOF@?$AA?$CF?$AAs?$AA?5?$AAA?$AAc?$AAt?$AAi?$AAv?$AAa?$AAt?$AAe?$AAC?$AAh?$AAi?$AAl?$AAd?$AA?5?$AAf?$AAa?$AAi?$AAl?$AAe?$AAd?$AA?4?$AA?$AN?$AA?6?$AA?$AA@ 100084b8     usb_ufnmddbase_common_topaz_v1:ufnbus.obj
 0001:000074f0       ??_C@_1DC@IMHJCHBH@?$AA?$CF?$AAs?$AA?5?$AAI?$AAn?$AAs?$AAe?$AAr?$AAt?$AAC?$AAh?$AAi?$AAl?$AAd?$AA?5?$AAf?$AAa?$AAi?$AAl?$AAe?$AAd?$AA?4?$AA?$AN?$AA?6?$AA?$AA@ 100084f0     usb_ufnmddbase_common_topaz_v1:ufnbus.obj
 0001:00007524       ??_C@_1DC@JDBLPGOM@?$AA?$CF?$AAs?$AA?5?$AAC?$AAr?$AAe?$AAa?$AAt?$AAe?$AAC?$AAh?$AAi?$AAl?$AAd?$AA?5?$AAf?$AAa?$AAi?$AAl?$AAe?$AAd?$AA?4?$AA?$AN?$AA?6?$AA?$AA@ 10008524     usb_ufnmddbase_common_topaz_v1:ufnbus.obj
 0001:00007558       ??_C@_1DI@HPFFCFPG@?$AAU?$AAs?$AAb?$AAF?$AAn?$AAM?$AAd?$AAd?$AA?$CB?$AAC?$AAU?$AAf?$AAn?$AAB?$AAu?$AAs?$AA?3?$AA?3?$AAP?$AAo?$AAs?$AAt?$AAI?$AAn?$AAi?$AAt?$AA?3?$AA?$AA@ 10008558     usb_ufnmddbase_common_topaz_v1:ufnbus.obj
 0001:00007590       ??_C@_1EE@KGBCBCHF@?$AA?$CF?$AAs?$AA?5?$AAA?$AAc?$AAt?$AAi?$AAv?$AAa?$AAt?$AAe?$AAd?$AA?5?$AAc?$AAl?$AAi?$AAe?$AAn?$AAt?$AA?5?$AAd?$AAr?$AAi?$AAv?$AAe?$AAr?$AA?5?$AA?$CC?$AA?$CF?$AAs?$AA?$CC?$AA?$AN@ 10008590     usb_ufnmddbase_common_topaz_v1:ufnbus.obj
 0001:000075d8       ??_C@_1EM@NAAJILDL@?$AA?$CF?$AAs?$AA?5?$AAF?$AAa?$AAi?$AAl?$AAe?$AAd?$AA?5?$AAt?$AAo?$AA?5?$AAc?$AAr?$AAe?$AAa?$AAt?$AAe?$AA?5?$AAp?$AAi?$AAp?$AAe?$AAs?$AA?4?$AA?5?$AAE?$AAr?$AAr?$AAo?$AAr@ 100085d8     usb_ufnmddbase_common_topaz_v1:ufnbus.obj
 0001:00007628       ??_C@_1GG@KBPJNJGG@?$AA?$CF?$AAs?$AA?5?$AAF?$AAa?$AAi?$AAl?$AAe?$AAd?$AA?5?$AAt?$AAo?$AA?5?$AAc?$AAr?$AAe?$AAa?$AAt?$AAe?$AA?5?$AAf?$AAr?$AAe?$AAe?$AA?5?$AAt?$AAr?$AAa?$AAn?$AAs?$AAf?$AAe@ 10008628     usb_ufnmddbase_common_topaz_v1:ufnbus.obj
 0001:00007690       ??_C@_1EC@NAKIHDDC@?$AAU?$AAs?$AAb?$AAF?$AAn?$AAM?$AAd?$AAd?$AA?$CB?$AAC?$AAU?$AAf?$AAn?$AAB?$AAu?$AAs?$AA?3?$AA?3?$AAA?$AAc?$AAt?$AAi?$AAv?$AAa?$AAt?$AAe?$AAC?$AAh?$AAi?$AAl?$AAd?$AA?3@ 10008690     usb_ufnmddbase_common_topaz_v1:ufnbus.obj
 0001:000076d4       ??_C@_1DA@OPANNIOF@?$AA?$CF?$AAs?$AA?5?$AAL?$AAo?$AAc?$AAa?$AAl?$AAA?$AAl?$AAl?$AAo?$AAc?$AA?5?$AAf?$AAa?$AAi?$AAl?$AAe?$AAd?$AA?$CB?$AA?$AN?$AA?6?$AA?$AA@ 100086d4     usb_ufnmddbase_common_topaz_v1:ufnbus.obj
 0001:00007704       ??_C@_1DI@HALOHOPK@?$AA?$CF?$AAs?$AA?5?$AAT?$AAo?$AAo?$AA?5?$AAm?$AAa?$AAn?$AAy?$AA?5?$AAe?$AAn?$AAd?$AAp?$AAo?$AAi?$AAn?$AAt?$AAs?$AA?3?$AA?5?$AA?$CF?$AAu?$AA?$AN?$AA?6?$AA?$AA@ 10008704     usb_ufnmddbase_common_topaz_v1:ufnbus.obj
 0001:0000773c       ??_C@_1DC@KJHMBJGO@?$AAU?$AAs?$AAb?$AAF?$AAn?$AAM?$AAd?$AAd?$AA?$CB?$AAA?$AAl?$AAl?$AAo?$AAc?$AAE?$AAn?$AAd?$AAp?$AAo?$AAi?$AAn?$AAt?$AAs?$AA?3?$AA?$AA@ 1000873c     usb_ufnmddbase_common_topaz_v1:ufnbus.obj
 0001:00007770       ??_C@_1EG@OKPNAFGG@?$AAU?$AAs?$AAb?$AAF?$AAn?$AAM?$AAd?$AAd?$AA?$CB?$AAC?$AAU?$AAf?$AAn?$AAB?$AAu?$AAs?$AA?3?$AA?3?$AAD?$AAe?$AAa?$AAc?$AAt?$AAi?$AAv?$AAa?$AAt?$AAe?$AAC?$AAh?$AAi?$AAl@ 10008770     usb_ufnmddbase_common_topaz_v1:ufnbus.obj
 0001:000077b8       ??_C@_17DJMMGLBL@?$AAD?$AAl?$AAl?$AA?$AA@ 100087b8     usb_ufnmddbase_common_topaz_v1:ufnbus.obj
 0001:000077c0       ??_C@_1EK@IHNFENMC@?$AA?$CF?$AAs?$AA?5?$AA?$CC?$AA?$CF?$AAs?$AA?$CC?$AA?5?$AAi?$AAs?$AA?5?$AAn?$AAo?$AAt?$AA?5?$AAa?$AAn?$AA?5?$AAa?$AAv?$AAa?$AAi?$AAl?$AAa?$AAb?$AAl?$AAe?$AA?5?$AAc?$AAl?$AAi?$AAe@ 100087c0     usb_ufnmddbase_common_topaz_v1:ufnbus.obj
 0001:00007810       ??_C@_1HC@MLFIPIAN@?$AA?$CF?$AAs?$AA?5?$AAF?$AAa?$AAi?$AAl?$AAu?$AAr?$AAe?$AA?5?$AAc?$AAh?$AAa?$AAn?$AAg?$AAi?$AAn?$AAg?$AA?5?$AAd?$AAe?$AAf?$AAa?$AAu?$AAl?$AAt?$AA?5?$AAc?$AAl?$AAi?$AAe@ 10008810     usb_ufnmddbase_common_topaz_v1:ufnbus.obj
 0001:00007888       ??_C@_1EI@OMAIAIBG@?$AA?$CF?$AAs?$AA?5?$AAC?$AAh?$AAa?$AAn?$AAg?$AAe?$AAd?$AA?5?$AAd?$AAe?$AAf?$AAa?$AAu?$AAl?$AAt?$AA?5?$AAc?$AAl?$AAi?$AAe?$AAn?$AAt?$AA?5?$AAt?$AAo?$AA?5?$AA?$CC?$AA?$CF?$AAs@ 10008888     usb_ufnmddbase_common_topaz_v1:ufnbus.obj
 0001:000078d0       ??_C@_1DK@COMDDHGA@?$AAU?$AAs?$AAb?$AAF?$AAn?$AAM?$AAd?$AAd?$AA?$CB?$AAC?$AAU?$AAf?$AAn?$AAB?$AAu?$AAs?$AA?3?$AA?3?$AAI?$AAO?$AAC?$AAo?$AAn?$AAt?$AAr?$AAo?$AAl?$AA?3?$AA?$AA@ 100088d0     usb_ufnmddbase_common_topaz_v1:ufnbus.obj
 0001:00007910       ??_C@_1EO@CMHPLHOA@?$AA?$CF?$AAs?$AA?5?$AAN?$AAo?$AA?5?$AAf?$AAr?$AAi?$AAe?$AAn?$AAd?$AAl?$AAy?$AA?5?$AAn?$AAa?$AAm?$AAe?$AA?5?$AAg?$AAi?$AAv?$AAe?$AAn?$AA?5?$AAf?$AAo?$AAr?$AA?5?$AAc?$AAl@ 10008910     usb_ufnmddbase_common_topaz_v1:ufnbus.obj
 0001:00007960       ??_C@_1BK@BFIEKNFP@?$AAF?$AAr?$AAi?$AAe?$AAn?$AAd?$AAl?$AAy?$AAN?$AAa?$AAm?$AAe?$AA?$AA@ 10008960     usb_ufnmddbase_common_topaz_v1:ufnbus.obj
 0001:0000797c       ??_C@_1DI@BFGINDMC@?$AAU?$AAs?$AAb?$AAF?$AAn?$AAM?$AAd?$AAd?$AA?$CB?$AAG?$AAe?$AAt?$AAU?$AAf?$AAn?$AAD?$AAe?$AAs?$AAc?$AAr?$AAi?$AAp?$AAt?$AAi?$AAo?$AAn?$AA?3?$AA?$AA@ 1000897c     usb_ufnmddbase_common_topaz_v1:ufnbus.obj
 0001:000079b8       ??_C@_1EI@MBENLCCN@?$AA?$CF?$AAs?$AA?5?$AAD?$AAe?$AAa?$AAc?$AAt?$AAi?$AAv?$AAa?$AAt?$AAe?$AAd?$AA?5?$AAc?$AAl?$AAi?$AAe?$AAn?$AAt?$AA?5?$AAd?$AAr?$AAi?$AAv?$AAe?$AAr?$AA?5?$AA?$CC?$AA?$CF?$AAs@ 100089b8     usb_ufnmddbase_common_topaz_v1:ufnbus.obj
 0001:00007a00       ??_C@_1EK@KOMOKBJB@?$AA?$CF?$AAs?$AA?5?$AAD?$AAe?$AAa?$AAc?$AAt?$AAi?$AAv?$AAa?$AAt?$AAe?$AAD?$AAe?$AAv?$AAi?$AAc?$AAe?$AA?5?$AAo?$AAn?$AA?5?$AA?$CC?$AA?$CF?$AAs?$AA?$CC?$AA?5?$AAf?$AAa?$AAi?$AAl@ 10008a00     usb_ufnmddbase_common_topaz_v1:ufnbus.obj
 0001:00007a50       ??_C@_1EM@CGJKPIII@?$AAU?$AAs?$AAb?$AAF?$AAn?$AAM?$AAd?$AAd?$AA?$CB?$AAC?$AAU?$AAf?$AAn?$AAB?$AAu?$AAs?$AA?3?$AA?3?$AAC?$AAl?$AAe?$AAa?$AAn?$AAU?$AAp?$AAA?$AAf?$AAt?$AAe?$AAr?$AAC?$AAl@ 10008a50     usb_ufnmddbase_common_topaz_v1:ufnbus.obj
 0001:00007a9c       ??_C@_1DI@OCIPBMKL@?$AA?$CF?$AAs?$AA?5?$AAS?$AAt?$AAa?$AAt?$AAe?$AA?5?$AAc?$AAh?$AAa?$AAn?$AAg?$AAe?$AA?3?$AA?5?$AA?$CF?$AAs?$AA?5?$AA?9?$AA?$DO?$AA?5?$AA?$CF?$AAs?$AA?$AN?$AA?6?$AA?$AA@ 10008a9c     usb_ufnmddbase_common_topaz_v1:ufnbus.obj
 0001:00007ad4       ??_C@_1DI@KNBPDCHJ@?$AAU?$AAs?$AAb?$AAF?$AAn?$AAM?$AAd?$AAd?$AA?$CB?$AAC?$AAh?$AAa?$AAn?$AAg?$AAe?$AAD?$AAe?$AAv?$AAi?$AAc?$AAe?$AAS?$AAt?$AAa?$AAt?$AAe?$AA?3?$AA?$AA@ 10008ad4     usb_ufnmddbase_common_topaz_v1:ufnbus.obj
 0001:00007b0c       ??_C@_1CI@MGKPCHDE@?$AAD?$AAe?$AAf?$AAa?$AAu?$AAl?$AAt?$AAC?$AAl?$AAi?$AAe?$AAn?$AAt?$AAD?$AAr?$AAi?$AAv?$AAe?$AAr?$AA?$AA@ 10008b0c     usb_ufnmddbase_common_topaz_v1:ufnbus.obj
 0001:00007b34       ??_C@_1CC@COLLGMBE@?$AAD?$AAe?$AAf?$AAa?$AAu?$AAl?$AAt?$AAC?$AAl?$AAi?$AAe?$AAn?$AAt?$AAK?$AAe?$AAy?$AA?$AA@ 10008b34     usb_ufnmddbase_common_topaz_v1:ufnbus.obj
 0001:00007b58       ??_C@_1FM@OPKMPGMB@?$AA?$CF?$AAs?$AA?5?$AAN?$AAo?$AA?5?$AAd?$AAe?$AAf?$AAa?$AAu?$AAl?$AAt?$AA?5?$AAc?$AAl?$AAi?$AAe?$AAn?$AAt?$AA?5?$AAd?$AAr?$AAi?$AAv?$AAe?$AAr?$AA?5?$AAl?$AAi?$AAs?$AAt@ 10008b58     usb_ufnmddbase_common_topaz_v1:ufnbus.obj
 0001:00007bb8       ??_C@_1HE@IFMOKDJM@?$AA?$CF?$AAs?$AA?5?$AAF?$AAa?$AAi?$AAl?$AAe?$AAd?$AA?5?$AAt?$AAo?$AA?5?$AAr?$AAe?$AAa?$AAd?$AA?5?$AAt?$AAh?$AAe?$AA?5?$AAc?$AAl?$AAi?$AAe?$AAn?$AAt?$AA?5?$AAd?$AAr?$AAi@ 10008bb8     usb_ufnmddbase_common_topaz_v1:ufnbus.obj
 0001:00007c30       ??_C@_1FC@FPNABGOP@?$AA?$CF?$AAs?$AA?5?$AAU?$AAs?$AAi?$AAn?$AAg?$AA?5?$AAd?$AAe?$AAf?$AAa?$AAu?$AAl?$AAt?$AA?5?$AAc?$AAl?$AAi?$AAe?$AAn?$AAt?$AA?5?$AAk?$AAe?$AAy?$AA?5?$AAn?$AAa?$AAm?$AAe@ 10008c30     usb_ufnmddbase_common_topaz_v1:ufnbus.obj
 0001:00007c88       ??_C@_1FA@LMACGDKI@?$AAU?$AAs?$AAb?$AAF?$AAn?$AAM?$AAd?$AAd?$AA?$CB?$AAC?$AAU?$AAf?$AAn?$AAB?$AAu?$AAs?$AA?3?$AA?3?$AAG?$AAe?$AAt?$AAD?$AAe?$AAf?$AAa?$AAu?$AAl?$AAt?$AAC?$AAl?$AAi?$AAe@ 10008c88     usb_ufnmddbase_common_topaz_v1:ufnbus.obj
 0001:00007cd8       ??_C@_1BEI@CKMFIHBN@?$AA?$AN?$AA?6?$AA?$CK?$AA?$CK?$AA?$CK?$AA?5?$AAA?$AAS?$AAS?$AAE?$AAR?$AAT?$AAI?$AAO?$AAN?$AA?5?$AAF?$AAA?$AAI?$AAL?$AAE?$AAD?$AA?5?$AAi?$AAn?$AA?5?$AAc?$AA?3?$AA?2?$AAw?$AAi?$AAn@ 10008cd8     usb_ufnmddbase_common_topaz_v1:ufnbus.obj
 0001:00007e20       ??_C@_1BDG@OLHMDMAM@?$AA?$AN?$AA?6?$AA?$CK?$AA?$CK?$AA?$CK?$AA?5?$AAA?$AAS?$AAS?$AAE?$AAR?$AAT?$AAI?$AAO?$AAN?$AA?5?$AAF?$AAA?$AAI?$AAL?$AAE?$AAD?$AA?5?$AAi?$AAn?$AA?5?$AAc?$AA?3?$AA?2?$AAw?$AAi?$AAn@ 10008e20     usb_ufnmddbase_common_topaz_v1:ufnbus.obj
 0001:00007f58       ??_C@_1BDG@ODKLBMFN@?$AA?$AN?$AA?6?$AA?$CK?$AA?$CK?$AA?$CK?$AA?5?$AAA?$AAS?$AAS?$AAE?$AAR?$AAT?$AAI?$AAO?$AAN?$AA?5?$AAF?$AAA?$AAI?$AAL?$AAE?$AAD?$AA?5?$AAi?$AAn?$AA?5?$AAc?$AA?3?$AA?2?$AAw?$AAi?$AAn@ 10008f58     usb_ufnmddbase_common_topaz_v1:ufnbus.obj
 0001:00008090       ??_C@_1BE@GGBBEMKG@?$AAs?$AAu?$AAs?$AAp?$AAe?$AAn?$AAd?$AAe?$AAd?$AA?$AA@ 10009090     usb_ufnmddbase_common_topaz_v1:enum.obj
 0001:000080a4       ??_C@_1BG@IHPLDPLP@?$AAc?$AAo?$AAn?$AAf?$AAi?$AAg?$AAu?$AAr?$AAe?$AAd?$AA?$AA@ 100090a4     usb_ufnmddbase_common_topaz_v1:enum.obj
 0001:000080bc       ??_C@_1BE@NDHGELNK@?$AAa?$AAd?$AAd?$AAr?$AAe?$AAs?$AAs?$AAe?$AAd?$AA?$AA@ 100090bc     usb_ufnmddbase_common_topaz_v1:enum.obj
 0001:000080d0       ??_C@_1BA@HANLFFFG@?$AAd?$AAe?$AAf?$AAa?$AAu?$AAl?$AAt?$AA?$AA@ 100090d0     usb_ufnmddbase_common_topaz_v1:enum.obj
 0001:000080e0       ??_C@_1BA@HDHPPDHD@?$AAp?$AAo?$AAw?$AAe?$AAr?$AAe?$AAd?$AA?$AA@ 100090e0     usb_ufnmddbase_common_topaz_v1:enum.obj
 0001:000080f0       ??_C@_1BC@OLNFHGE@?$AAa?$AAt?$AAt?$AAa?$AAc?$AAh?$AAe?$AAd?$AA?$AA@ 100090f0     usb_ufnmddbase_common_topaz_v1:enum.obj
 0001:00008104       ??_C@_1BC@KCAIJJIM@?$AAd?$AAe?$AAt?$AAa?$AAc?$AAh?$AAe?$AAd?$AA?$AA@ 10009104     usb_ufnmddbase_common_topaz_v1:enum.obj
 0001:00008138       ??_C@_1NA@DFFNALFL@?$AAC?$AA?3?$AA?2?$AAW?$AAI?$AAN?$AAC?$AAE?$AAR?$AAO?$AAO?$AAT?$AAS?$AA?2?$AAT?$AAo?$AAp?$AAa?$AAz?$AA?2?$AAW?$AAI?$AAN?$AAC?$AAE?$AA6?$AA0?$AA0?$AA?2?$AAP?$AAL?$AAA@ 10009138     usb_ufnmddbase_common_topaz_v1:enum.obj
 0001:00008208       ??_C@_1FA@JIGGNMLH@?$AA?$CF?$AAs?$AA?3?$AA?5?$AAf?$AAa?$AAi?$AAl?$AAe?$AAd?$AA?5?$AAt?$AAo?$AA?5?$AAS?$AAE?$AAT?$AA_?$AAT?$AAE?$AAS?$AAT?$AA_?$AAM?$AAO?$AAD?$AAE?$AA?5?$AA?$CF?$AAd?$AA?5?$AAo@ 10009208     usb_ufnmddbase_common_topaz_v1:enum.obj
 0001:00008258       ??_C@_1FC@NMKPDANJ@?$AAw?$AAe?$AA?5?$AAc?$AAh?$AAo?$AAo?$AAs?$AAe?$AA?5?$AAn?$AAo?$AAt?$AA?5?$AAt?$AAo?$AA?5?$AAh?$AAa?$AAn?$AAd?$AAs?$AAh?$AAa?$AAk?$AAe?$AA?5?$AAa?$AAf?$AAt?$AAe?$AAr@ 10009258     usb_ufnmddbase_common_topaz_v1:enum.obj
 0001:000082ac       ??_C@_1DK@FHFPJNHH@?$AA?$CF?$AAs?$AA?5?$AAS?$AAe?$AAt?$AA?5?$AAc?$AAo?$AAn?$AAf?$AAi?$AAg?$AAu?$AAr?$AAa?$AAt?$AAi?$AAo?$AAn?$AA?5?$AA?$CI?$AA?$CF?$AAu?$AA?$CJ?$AA?4?$AA?$AN?$AA?6?$AA?$AA@ 100092ac     usb_ufnmddbase_common_topaz_v1:enum.obj
 0001:000082e8       ??_C@_1CO@FEALDAL@?$AA?$CF?$AAs?$AA?5?$AAS?$AAe?$AAt?$AA?5?$AAa?$AAd?$AAd?$AAr?$AAe?$AAs?$AAs?$AA?5?$AA?$CI?$AA?$CF?$AAu?$AA?$CJ?$AA?4?$AA?$AN?$AA?6?$AA?$AA@ 100092e8     usb_ufnmddbase_common_topaz_v1:enum.obj
 0001:00008318       ??_C@_1GE@LKDPEFAC@?$AA?$CF?$AAs?$AA?5?$AAU?$AAn?$AAh?$AAa?$AAn?$AAd?$AAl?$AAe?$AAd?$AA?5?$AAs?$AAe?$AAt?$AAu?$AAp?$AA?5?$AAp?$AAa?$AAc?$AAk?$AAe?$AAt?$AA?4?$AA?5?$AAP?$AAa?$AAs?$AAs?$AAi@ 10009318     usb_ufnmddbase_common_topaz_v1:enum.obj
 0001:00008380       ??_C@_1HA@CBEAJLN@?$AA?$CF?$AAs?$AA?5?$AAR?$AAe?$AAc?$AAe?$AAi?$AAv?$AAe?$AAd?$AA?5?$AA?$CF?$AAs?$AA?5?$AAs?$AAe?$AAt?$AAu?$AAp?$AA?5?$AAp?$AAa?$AAc?$AAk?$AAe?$AAt?$AA?3?$AA?5?$AA?$CF?$AA0?$AA2@ 10009380     usb_ufnmddbase_common_topaz_v1:enum.obj
 0001:000083f0       ??_C@_1BK@OBAIJFOP@?$AAp?$AAr?$AAe?$AAp?$AAr?$AAo?$AAc?$AAe?$AAs?$AAs?$AAe?$AAd?$AA?$AA@ 100093f0     usb_ufnmddbase_common_topaz_v1:enum.obj
 0001:0000840c       ??_C@_1DO@DGGMNOGA@?$AA?$CF?$AAs?$AA?5?$AAA?$AAt?$AAt?$AAa?$AAc?$AAh?$AAe?$AAd?$AA?5?$AAt?$AAo?$AA?5?$AA?$CF?$AAs?$AA?5?$AAs?$AAp?$AAe?$AAe?$AAd?$AA?5?$AAb?$AAu?$AAs?$AA?4?$AA?$AN?$AA?6?$AA?$AA@ 1000940c     usb_ufnmddbase_common_topaz_v1:enum.obj
 0001:0000844c       ??_C@_1BK@OHLNHAMO@?$AA?$CF?$AAs?$AA?5?$AAR?$AAe?$AAs?$AAu?$AAm?$AAe?$AAd?$AA?$AN?$AA?6?$AA?$AA@ 1000944c     usb_ufnmddbase_common_topaz_v1:enum.obj
 0001:00008468       ??_C@_1BO@IJBHLJNP@?$AA?$CF?$AAs?$AA?5?$AAS?$AAu?$AAs?$AAp?$AAe?$AAn?$AAd?$AAe?$AAd?$AA?$AN?$AA?6?$AA?$AA@ 10009468     usb_ufnmddbase_common_topaz_v1:enum.obj
 0001:00008488       ??_C@_1EG@CGPFFPFJ@?$AA?$CF?$AAs?$AA?5?$AAR?$AAe?$AAc?$AAe?$AAi?$AAv?$AAe?$AAd?$AA?5?$AAr?$AAe?$AAs?$AAe?$AAt?$AA?5?$AAw?$AAh?$AAe?$AAn?$AA?5?$AAd?$AAe?$AAt?$AAa?$AAc?$AAh?$AAe?$AAd?$AA?$CB@ 10009488     usb_ufnmddbase_common_topaz_v1:enum.obj
 0001:000084d0       ??_C@_1CK@OEAJAPMF@?$AA?$CF?$AAs?$AA?5?$AAR?$AAo?$AAo?$AAt?$AA?5?$AAp?$AAo?$AAr?$AAt?$AA?5?$AAr?$AAe?$AAs?$AAe?$AAt?$AA?$AN?$AA?6?$AA?$AA@ 100094d0     usb_ufnmddbase_common_topaz_v1:enum.obj
 0001:00008500       ??_C@_1FI@NMAEFNKB@?$AA?$CF?$AAs?$AA?5?$AAR?$AAe?$AAc?$AAe?$AAi?$AAv?$AAe?$AAd?$AA?5?$AAa?$AAt?$AAt?$AAa?$AAc?$AAh?$AA?5?$AAw?$AAh?$AAe?$AAn?$AA?5?$AAa?$AAl?$AAr?$AAe?$AAa?$AAd?$AAy?$AA?5@ 10009500     usb_ufnmddbase_common_topaz_v1:enum.obj
 0001:00008558       ??_C@_1BM@MEIADHEC@?$AA?$CF?$AAs?$AA?5?$AAA?$AAt?$AAt?$AAa?$AAc?$AAh?$AAe?$AAd?$AA?$AN?$AA?6?$AA?$AA@ 10009558     usb_ufnmddbase_common_topaz_v1:enum.obj
 0001:00008578       ??_C@_1FI@FIPANPOF@?$AA?$CF?$AAs?$AA?5?$AAR?$AAe?$AAc?$AAe?$AAi?$AAv?$AAe?$AAd?$AA?5?$AAd?$AAe?$AAt?$AAa?$AAc?$AAh?$AA?5?$AAw?$AAh?$AAe?$AAn?$AA?5?$AAa?$AAl?$AAr?$AAe?$AAa?$AAd?$AAy?$AA?5@ 10009578     usb_ufnmddbase_common_topaz_v1:enum.obj
 0001:000085d0       ??_C@_1BM@KKIFAOB@?$AA?$CF?$AAs?$AA?5?$AAD?$AAe?$AAt?$AAa?$AAc?$AAh?$AAe?$AAd?$AA?$AN?$AA?6?$AA?$AA@ 100095d0     usb_ufnmddbase_common_topaz_v1:enum.obj
 0001:000085f0       ??_C@_1GI@GICILDL@?$AA?$CF?$AAs?$AA?5?$AAI?$AAg?$AAn?$AAo?$AAr?$AAi?$AAn?$AAg?$AA?5?$AAn?$AAo?$AAt?$AAi?$AAf?$AAi?$AAc?$AAa?$AAt?$AAi?$AAo?$AAn?$AA?5?$AA0?$AAx?$AA?$CF?$AA0?$AA8?$AAx?$AA?5@ 100095f0     usb_ufnmddbase_common_topaz_v1:enum.obj
 0001:00008658       ??_C@_1DO@NMCGNLEK@?$AA?$CF?$AAs?$AA?5?$AAP?$AAD?$AAD?$AA?5?$AAp?$AAa?$AAs?$AAs?$AAe?$AAd?$AA?5?$AAa?$AA?5?$AAb?$AAa?$AAd?$AA?5?$AAt?$AAr?$AAa?$AAn?$AAs?$AAf?$AAe?$AAr?$AA?$AN?$AA?6?$AA?$AA@ 10009658     usb_ufnmddbase_common_topaz_v1:enum.obj
 0001:00008698       ??_C@_1DA@DEEGFMMN@?$AAU?$AAs?$AAb?$AAF?$AAn?$AAM?$AAd?$AAd?$AA?$CB?$AAU?$AAf?$AAn?$AAM?$AAd?$AAd?$AA_?$AAN?$AAo?$AAt?$AAi?$AAf?$AAy?$AA?3?$AA?$AA@ 10009698     usb_ufnmddbase_common_topaz_v1:enum.obj
 0001:000086c8       ??_C@_1DC@OGILGLGD@?$AAU?$AAs?$AAb?$AAF?$AAn?$AAM?$AAd?$AAd?$AA?$CB?$AAP?$AAr?$AAo?$AAc?$AAe?$AAs?$AAs?$AAR?$AAe?$AAq?$AAu?$AAe?$AAs?$AAt?$AA?3?$AA?$AA@ 100096c8     usb_ufnmddbase_common_topaz_v1:enum.obj
 0001:000086fc       ??_C@_1DO@LANKMPLO@?$AAU?$AAs?$AAb?$AAF?$AAn?$AAM?$AAd?$AAd?$AA?$CB?$AAP?$AAr?$AAo?$AAc?$AAe?$AAs?$AAs?$AAG?$AAe?$AAt?$AAD?$AAe?$AAs?$AAc?$AAr?$AAi?$AAp?$AAt?$AAo?$AAr?$AA?3?$AA?$AA@ 100096fc     usb_ufnmddbase_common_topaz_v1:enum.obj
 0001:00008740       ??_C@_1GK@KKIKCIO@?$AA?$CF?$AAs?$AA?5?$AAA?$AAs?$AAk?$AAe?$AAd?$AA?5?$AAt?$AAo?$AA?5?$AAs?$AAe?$AAn?$AAd?$AA?5?$AA?$CF?$AAu?$AA?5?$AAo?$AAf?$AA?5?$AA?$CF?$AAu?$AA?5?$AAb?$AAy?$AAt?$AAe?$AAs?$AA?4@ 10009740     usb_ufnmddbase_common_topaz_v1:enum.obj
 0001:000087ac       ??_C@_1CE@GLMMGBBK@?$AAU?$AAs?$AAb?$AAF?$AAn?$AAM?$AAd?$AAd?$AA?$CB?$AAS?$AAe?$AAt?$AAu?$AAp?$AAT?$AAx?$AA?3?$AA?$AA@ 100097ac     usb_ufnmddbase_common_topaz_v1:enum.obj
 0001:000087d0       ??_C@_1CM@DNONHKCD@?$AA?$CF?$AAs?$AA?5?$AA?$CF?$AAu?$AA?5?$AAb?$AAy?$AAt?$AAe?$AAs?$AA?5?$AAw?$AAr?$AAi?$AAt?$AAt?$AAe?$AAn?$AA?$AN?$AA?6?$AA?$AA@ 100097d0     usb_ufnmddbase_common_topaz_v1:enum.obj
 0001:000087fc       ??_C@_1DO@KOFCKPI@?$AAU?$AAs?$AAb?$AAF?$AAn?$AAM?$AAd?$AAd?$AA?$CB?$AAE?$AAn?$AAu?$AAm?$AAT?$AAr?$AAa?$AAn?$AAs?$AAf?$AAe?$AAr?$AAC?$AAo?$AAm?$AAp?$AAl?$AAe?$AAt?$AAe?$AA?3?$AA?$AA@ 100097fc     usb_ufnmddbase_common_topaz_v1:enum.obj
 0001:0000883c       ??_C@_1DA@FNGDGMEF@?$AA?$CF?$AAs?$AA?5?$AAG?$AAe?$AAt?$AA?5?$AAc?$AAo?$AAn?$AAf?$AAi?$AAg?$AAu?$AAr?$AAa?$AAt?$AAi?$AAo?$AAn?$AA?4?$AA?$AN?$AA?6?$AA?$AA@ 1000983c     usb_ufnmddbase_common_topaz_v1:enum.obj
 0001:00008870       ??_C@_1EE@PDHMCHEL@?$AAU?$AAs?$AAb?$AAF?$AAn?$AAM?$AAd?$AAd?$AA?$CB?$AAP?$AAr?$AAo?$AAc?$AAe?$AAs?$AAs?$AAG?$AAe?$AAt?$AAC?$AAo?$AAn?$AAf?$AAi?$AAg?$AAu?$AAr?$AAa?$AAt?$AAi?$AAo?$AAn@ 10009870     usb_ufnmddbase_common_topaz_v1:enum.obj
 0001:000088b4       ??_C@_1DA@EBHDKDEN@?$AA?$CF?$AAs?$AA?5?$AAG?$AAe?$AAt?$AA?5?$AAi?$AAn?$AAt?$AAe?$AAr?$AAf?$AAa?$AAc?$AAe?$AA?$CI?$AA?$CF?$AAu?$AA?$CJ?$AA?4?$AA?$AN?$AA?6?$AA?$AA@ 100098b4     usb_ufnmddbase_common_topaz_v1:enum.obj
 0001:000088e4       ??_C@_1DM@DDCBLEOO@?$AAU?$AAs?$AAb?$AAF?$AAn?$AAM?$AAd?$AAd?$AA?$CB?$AAP?$AAr?$AAo?$AAc?$AAe?$AAs?$AAs?$AAG?$AAe?$AAt?$AAI?$AAn?$AAt?$AAe?$AAr?$AAf?$AAa?$AAc?$AAe?$AA?3?$AA?$AA@ 100098e4     usb_ufnmddbase_common_topaz_v1:enum.obj
 0001:00008920       ??_C@_1DE@OPIPKLFF@?$AA?$CF?$AAs?$AA?5?$AAB?$AAa?$AAd?$AA?5?$AAe?$AAn?$AAd?$AAp?$AAo?$AAi?$AAn?$AAt?$AA?5?$AAr?$AAe?$AAq?$AAu?$AAe?$AAs?$AAt?$AA?$AN?$AA?6?$AA?$AA@ 10009920     usb_ufnmddbase_common_topaz_v1:enum.obj
 0001:00008954       ??_C@_1DG@DHKAHKE@?$AA?$CF?$AAs?$AA?5?$AAB?$AAa?$AAd?$AA?5?$AAi?$AAn?$AAt?$AAe?$AAr?$AAf?$AAa?$AAc?$AAe?$AA?5?$AAr?$AAe?$AAq?$AAu?$AAe?$AAs?$AAt?$AA?$AN?$AA?6?$AA?$AA@ 10009954     usb_ufnmddbase_common_topaz_v1:enum.obj
 0001:0000898c       ??_C@_1DA@FPBOEJGH@?$AA?$CF?$AAs?$AA?5?$AAG?$AAe?$AAt?$AA?5?$AAd?$AAe?$AAv?$AAi?$AAc?$AAe?$AA?5?$AAs?$AAt?$AAa?$AAt?$AAu?$AAs?$AA?4?$AA?$AN?$AA?6?$AA?$AA@ 1000998c     usb_ufnmddbase_common_topaz_v1:enum.obj
 0001:000089bc       ??_C@_1DG@EHCGKNIM@?$AAU?$AAs?$AAb?$AAF?$AAn?$AAM?$AAd?$AAd?$AA?$CB?$AAP?$AAr?$AAo?$AAc?$AAe?$AAs?$AAs?$AAG?$AAe?$AAt?$AAS?$AAt?$AAa?$AAt?$AAu?$AAs?$AA?3?$AA?$AA@ 100099bc     usb_ufnmddbase_common_topaz_v1:enum.obj
 0001:000089f8       ??_C@_1FC@ECJCHNH@?$AAP?$AAr?$AAo?$AAc?$AAe?$AAs?$AAs?$AAS?$AAe?$AAt?$AAA?$AAd?$AAd?$AAr?$AAe?$AAs?$AAs?$AA?3?$AA?5?$AAI?$AAn?$AAc?$AAo?$AAr?$AAr?$AAe?$AAc?$AAt?$AA?5?$AAp?$AAa?$AAr@ 100099f8     usb_ufnmddbase_common_topaz_v1:enum.obj
 0001:00008a4c       ??_C@_1DO@ILNFABEB@?$AA?$CF?$AAs?$AA?5?$AAS?$AAe?$AAt?$AA?5?$AAa?$AAd?$AAd?$AAr?$AAe?$AAs?$AAs?$AA?5?$AA?$CI?$AA?$CF?$AAu?$AA?$CJ?$AA?5?$AAr?$AAe?$AAq?$AAu?$AAe?$AAs?$AAt?$AA?4?$AA?$AN?$AA?6?$AA?$AA@ 10009a4c     usb_ufnmddbase_common_topaz_v1:enum.obj
 0001:00008a8c       ??_C@_1DI@BPJNKOFH@?$AAU?$AAs?$AAb?$AAF?$AAn?$AAM?$AAd?$AAd?$AA?$CB?$AAP?$AAr?$AAo?$AAc?$AAe?$AAs?$AAs?$AAS?$AAe?$AAt?$AAA?$AAd?$AAd?$AAr?$AAe?$AAs?$AAs?$AA?3?$AA?$AA@ 10009a8c     usb_ufnmddbase_common_topaz_v1:enum.obj
 0001:00008ac8       ??_C@_1EK@MPNHENNL@?$AA?$CF?$AAs?$AA?5?$AAS?$AAe?$AAt?$AA?5?$AAc?$AAo?$AAn?$AAf?$AAi?$AAg?$AAu?$AAr?$AAa?$AAt?$AAi?$AAo?$AAn?$AA?5?$AA?$CI?$AA?$CF?$AAu?$AA?$CJ?$AA?5?$AAr?$AAe?$AAq?$AAu?$AAe?$AAs@ 10009ac8     usb_ufnmddbase_common_topaz_v1:enum.obj
 0001:00008b18       ??_C@_1EE@CKGNBNIA@?$AAU?$AAs?$AAb?$AAF?$AAn?$AAM?$AAd?$AAd?$AA?$CB?$AAP?$AAr?$AAo?$AAc?$AAe?$AAs?$AAs?$AAS?$AAe?$AAt?$AAC?$AAo?$AAn?$AAf?$AAi?$AAg?$AAu?$AAr?$AAa?$AAt?$AAi?$AAo?$AAn@ 10009b18     usb_ufnmddbase_common_topaz_v1:enum.obj
 0001:00008b60       ??_C@_1EM@JHJPPAD@?$AA?$CF?$AAs?$AA?5?$AAS?$AAe?$AAt?$AA?5?$AAi?$AAn?$AAt?$AAe?$AAr?$AAf?$AAa?$AAc?$AAe?$AA?5?$AA?$CI?$AA?$CF?$AAu?$AA?5?$AA?9?$AA?5?$AA?$CF?$AAu?$AA?$CJ?$AA?5?$AAr?$AAe?$AAq?$AAu?$AAe@ 10009b60     usb_ufnmddbase_common_topaz_v1:enum.obj
 0001:00008bac       ??_C@_1DM@COKJJBEK@?$AAU?$AAs?$AAb?$AAF?$AAn?$AAM?$AAd?$AAd?$AA?$CB?$AAP?$AAr?$AAo?$AAc?$AAe?$AAs?$AAs?$AAS?$AAe?$AAt?$AAI?$AAn?$AAt?$AAe?$AAr?$AAf?$AAa?$AAc?$AAe?$AA?3?$AA?$AA@ 10009bac     usb_ufnmddbase_common_topaz_v1:enum.obj
 0001:00008be8       ??_C@_1GK@DLMMJONG@?$AA?$CF?$AAs?$AA?5?$AAA?$AAs?$AAk?$AAe?$AAd?$AA?5?$AAt?$AAo?$AA?5?$AAc?$AAl?$AAe?$AAa?$AAr?$AA?5?$AAh?$AAa?$AAl?$AAt?$AA?5?$AAf?$AAo?$AAr?$AA?5?$AAi?$AAn?$AAv?$AAa?$AAl@ 10009be8     usb_ufnmddbase_common_topaz_v1:enum.obj
 0001:00008c58       ??_C@_1FG@FPOCHCFD@?$AA?$CF?$AAs?$AA?5?$AAC?$AAl?$AAe?$AAa?$AAr?$AA?5?$AAe?$AAn?$AAd?$AAp?$AAo?$AAi?$AAn?$AAt?$AA?5?$AA?$CI?$AA0?$AAx?$AA?$CF?$AA0?$AA2?$AAx?$AA?$CJ?$AA?5?$AAh?$AAa?$AAl?$AAt?$AA?5@ 10009c58     usb_ufnmddbase_common_topaz_v1:enum.obj
 0001:00008cb0       ??_C@_1DM@GJDFAGPO@?$AAU?$AAs?$AAb?$AAF?$AAn?$AAM?$AAd?$AAd?$AA?$CB?$AAP?$AAr?$AAo?$AAc?$AAe?$AAs?$AAs?$AAC?$AAl?$AAe?$AAa?$AAr?$AAF?$AAe?$AAa?$AAt?$AAu?$AAr?$AAe?$AA?3?$AA?$AA@ 10009cb0     usb_ufnmddbase_common_topaz_v1:enum.obj
 0001:00008cf0       ??_C@_1FM@EKPJFIFG@?$AA?$CF?$AAs?$AA?3?$AAP?$AAr?$AAo?$AAc?$AAe?$AAs?$AAs?$AAS?$AAe?$AAt?$AAF?$AAe?$AAa?$AAt?$AAu?$AAr?$AAe?$AA?5?$AAr?$AAe?$AAt?$AAu?$AAr?$AAn?$AA?3?$AA?5?$AAr?$AAe?$AAs@ 10009cf0     usb_ufnmddbase_common_topaz_v1:enum.obj
 0001:00008d50       ??_C@_1EM@GCLCFFBC@?$AA?$CF?$AAs?$AA?5?$AAI?$AAn?$AAv?$AAa?$AAl?$AAi?$AAd?$AA?5?$AAt?$AAe?$AAs?$AAt?$AA?5?$AAm?$AAo?$AAd?$AAe?$AA?5?$AAr?$AAe?$AAq?$AAu?$AAe?$AAs?$AAt?$AA?5?$AA0?$AAx?$AA?$CF@ 10009d50     usb_ufnmddbase_common_topaz_v1:enum.obj
 0001:00008da0       ??_C@_1FK@HIIMILMH@?$AAI?$AAn?$AAv?$AAa?$AAl?$AAi?$AAd?$AA?5?$AAT?$AAe?$AAs?$AAt?$AA?5?$AAm?$AAo?$AAd?$AAe?$AA?5?$AAr?$AAe?$AAq?$AAu?$AAe?$AAs?$AAt?$AAe?$AAd?$AA?3?$AA?5?$AAw?$AAI?$AAn@ 10009da0     usb_ufnmddbase_common_topaz_v1:enum.obj
 0001:00008dfc       ??_C@_1DE@PNJDKNNA@?$AAT?$AAe?$AAs?$AAt?$AA?5?$AAm?$AAo?$AAd?$AAe?$AA?5?$AAr?$AAe?$AAq?$AAu?$AAe?$AAs?$AAt?$AAe?$AAd?$AA?3?$AA?5?$AA?$CF?$AAd?$AA?$AN?$AA?6?$AA?$AA@ 10009dfc     usb_ufnmddbase_common_topaz_v1:enum.obj
 0001:00008e30       ??_C@_1NM@BOMDOCFB@?$AA?$CF?$AAs?$AA?5?$AAP?$AAr?$AAo?$AAc?$AAe?$AAs?$AAs?$AAS?$AAe?$AAt?$AAF?$AAe?$AAa?$AAt?$AAu?$AAr?$AAe?$AA?3?$AA?5?$AAS?$AAe?$AAt?$AAF?$AAe?$AAa?$AAt?$AAu?$AAr?$AAe@ 10009e30     usb_ufnmddbase_common_topaz_v1:enum.obj
 0001:00008f10       ??_C@_1FG@DANPFBIH@?$AA?$CF?$AAs?$AA?5?$AAA?$AAs?$AAk?$AAe?$AAd?$AA?5?$AAt?$AAo?$AA?5?$AAh?$AAa?$AAl?$AAt?$AA?5?$AAi?$AAn?$AAv?$AAa?$AAl?$AAi?$AAd?$AA?5?$AAe?$AAn?$AAd?$AAp?$AAo?$AAi?$AAn@ 10009f10     usb_ufnmddbase_common_topaz_v1:enum.obj
 0001:00008f68       ??_C@_1EK@DEPJMKOH@?$AA?$CF?$AAs?$AA?5?$AAH?$AAa?$AAl?$AAt?$AA?5?$AAe?$AAn?$AAd?$AAp?$AAo?$AAi?$AAn?$AAt?$AA?5?$AA?$CI?$AA0?$AAx?$AA?$CF?$AA0?$AA2?$AAx?$AA?$CJ?$AA?5?$AAr?$AAe?$AAq?$AAu?$AAe?$AAs@ 10009f68     usb_ufnmddbase_common_topaz_v1:enum.obj
 0001:00008fb8       ??_C@_1JO@BLOEGMOH@?$AA?$CF?$AAs?$AA?3?$AAP?$AAr?$AAo?$AAc?$AAe?$AAs?$AAs?$AAS?$AAe?$AAt?$AAF?$AAe?$AAa?$AAt?$AAu?$AAr?$AAe?$AA?5?$AAu?$AAd?$AAr?$AA?4?$AAb?$AAm?$AAR?$AAe?$AAq?$AAu?$AAe@ 10009fb8     usb_ufnmddbase_common_topaz_v1:enum.obj
 0001:00009058       ??_C@_1DI@FMOJONP@?$AAU?$AAs?$AAb?$AAF?$AAn?$AAM?$AAd?$AAd?$AA?$CB?$AAP?$AAr?$AAo?$AAc?$AAe?$AAs?$AAs?$AAS?$AAe?$AAt?$AAF?$AAe?$AAa?$AAt?$AAu?$AAr?$AAe?$AA?3?$AA?$AA@ 1000a058     usb_ufnmddbase_common_topaz_v1:enum.obj
 0001:00009090       ??_C@_1FE@KNJHFFDC@?$AAU?$AAs?$AAb?$AAF?$AAn?$AAM?$AAd?$AAd?$AA?$CB?$AAC?$AAl?$AAo?$AAs?$AAe?$AAA?$AAl?$AAl?$AAP?$AAi?$AAp?$AAe?$AAs?$AAE?$AAx?$AAc?$AAe?$AAp?$AAt?$AAE?$AAn?$AAd?$AAp@ 1000a090     usb_ufnmddbase_common_topaz_v1:enum.obj
 0001:00009178       ??_C@_1EE@IOHENOFL@?$AAU?$AAS?$AAB?$AAF?$AAN?$AAP?$AAD?$AAD?$AA?5?$AAS?$AAy?$AAs?$AAI?$AAn?$AAt?$AAr?$AA?3?$AA0?$AAx?$AA?$CF?$AAx?$AA?0?$AA?5?$AAI?$AAr?$AAq?$AA?3?$AA0?$AAx?$AA?$CF?$AAx?$AA?$AN@ 1000a178     usb_usbfn_os_mx25_topaz_v1:i_os.obj
 0001:000091c0       ??_C@_1GM@LHAFDILO@?$AAE?$AAR?$AAR?$AAO?$AAR?$AA?3?$AA?5?$AAU?$AAf?$AAn?$AAP?$AAd?$AAd?$AA_?$AAI?$AAn?$AAi?$AAt?$AA?3?$AA?5?$AAI?$AAn?$AAt?$AAe?$AAr?$AAr?$AAu?$AAp?$AAt?$AA?5?$AAi?$AAn@ 1000a1c0     usb_usbfn_os_mx25_topaz_v1:i_os.obj
 0001:00009230       ??_C@_1GK@FDHKBGCI@?$AAE?$AAR?$AAR?$AAO?$AAR?$AA?3?$AA?5?$AAU?$AAf?$AAn?$AAP?$AAd?$AAd?$AA_?$AAI?$AAn?$AAi?$AAt?$AA?3?$AA?5?$AAE?$AAr?$AAr?$AAo?$AAr?$AA?5?$AAc?$AAr?$AAe?$AAa?$AAt?$AAi@ 1000a230     usb_usbfn_os_mx25_topaz_v1:i_os.obj
 0001:000092a0       ??_C@_1FI@JPEGJOPE@?$AAA?$AAl?$AAl?$AAo?$AAc?$AAa?$AAt?$AAe?$AA?5?$AAD?$AAM?$AAA?$AA?5?$AAm?$AAe?$AAm?$AAo?$AAr?$AAy?$AA?5?$AAf?$AAo?$AAr?$AA?5?$AAB?$AAu?$AAf?$AAf?$AAe?$AAr?$AA_?$AAT@ 1000a2a0     usb_usbfn_os_mx25_topaz_v1:i_os.obj
 0001:000092f8       ??_C@_1FI@KGDODDLE@?$AAA?$AAl?$AAl?$AAo?$AAc?$AAa?$AAt?$AAe?$AA?5?$AAD?$AAM?$AAA?$AA?5?$AAm?$AAe?$AAm?$AAo?$AAr?$AAy?$AA?5?$AAf?$AAo?$AAr?$AA?5?$AAB?$AAu?$AAf?$AAf?$AAe?$AAr?$AA_?$AAT@ 1000a2f8     usb_usbfn_os_mx25_topaz_v1:i_os.obj
 0001:00009350       ??_C@_1GO@BLDDEEAN@?$AAE?$AAR?$AAR?$AAO?$AAR?$AA?3?$AA?5?$AAU?$AAf?$AAn?$AAP?$AAd?$AAd?$AA_?$AAI?$AAn?$AAi?$AAt?$AA?3?$AA?5?$AAI?$AAn?$AAt?$AAe?$AAr?$AAr?$AAu?$AAp?$AAt?$AA?5?$AAt?$AAh@ 1000a350     usb_usbfn_os_mx25_topaz_v1:i_os.obj
 0001:000093c0       ??_C@_1FO@JMHJBPEL@?$AAU?$AAS?$AAB?$AAO?$AAT?$AAG?$AA?5?$AAC?$AAl?$AAi?$AAe?$AAn?$AAt?$AA?5?$AAT?$AAe?$AAs?$AAt?$AA?5?$AAM?$AAo?$AAd?$AAe?$AA?5?$AAs?$AAe?$AAt?$AA?5?$AAa?$AAn?$AAd?$AA?5@ 1000a3c0     usb_usbfn_os_mx25_topaz_v1:i_os.obj
 0001:00009420       ??_C@_1EA@OAPKEJIG@?$AAL?$AAe?$AAa?$AAv?$AAe?$AA?5?$AAC?$AAl?$AAi?$AAe?$AAn?$AAt?$AA?5?$AAb?$AAa?$AAc?$AAk?$AA?5?$AAt?$AAo?$AA?5?$AAX?$AAV?$AAR?$AA?5?$AAm?$AAo?$AAd?$AAe?$AA?$AN?$AA?6?$AA?$AA@ 1000a420     usb_usbfn_os_mx25_topaz_v1:i_os.obj
 0001:00009460       ??_C@_1EO@EJBGAILK@?$AAO?$AAT?$AAG?$AAS?$AAC?$AA?5?$AAI?$AAD?$AAI?$AAE?$AA?$CI?$AA0?$AAx?$AA?$CF?$AAx?$AA?$CJ?$AA?0?$AA?5?$AAI?$AAD?$AAI?$AAS?$AA?$CI?$AA0?$AAx?$AA?$CF?$AAx?$AA?$CJ?$AA?0?$AA?5?$AA?$CI?$AA0@ 1000a460     usb_usbfn_os_mx25_topaz_v1:i_os.obj
 0001:000094b0       ??_C@_1CM@NOLMNJB@?$AAU?$AAf?$AAn?$AAP?$AAd?$AAd?$AA_?$AAS?$AAt?$AAa?$AAr?$AAt?$AA?5?$AAc?$AAa?$AAl?$AAl?$AAe?$AAd?$AA?$AN?$AA?6?$AA?$AA@ 1000a4b0     usb_usbfn_os_mx25_topaz_v1:i_os.obj
 0001:000094e0       ??_C@_1HE@MCANNPIK@?$AAE?$AAR?$AAR?$AAO?$AAR?$AA?3?$AA?5?$AAI?$AAn?$AAt?$AAe?$AAr?$AAr?$AAu?$AAp?$AAt?$AAT?$AAh?$AAr?$AAe?$AAa?$AAd?$AA?3?$AA?5?$AAI?$AAn?$AAt?$AAe?$AAr?$AAr?$AAu?$AAp@ 1000a4e0     usb_usbfn_os_mx25_topaz_v1:i_os.obj
 0001:00009558       ??_C@_1EO@MCGPCLFC@?$AAU?$AAF?$AAN?$AA?3?$AA?5?$AAW?$AAa?$AAi?$AAt?$AAi?$AAn?$AAg?$AA?5?$AAf?$AAo?$AAr?$AA?5?$AAs?$AAi?$AAg?$AAn?$AAa?$AAl?$AA?5?$AAf?$AAr?$AAo?$AAm?$AA?5?$AAX?$AAC?$AAV@ 1000a558     usb_usbfn_os_mx25_topaz_v1:i_os.obj
 0001:000095a8       ??_C@_1EK@KBAJIEHD@?$AAU?$AAF?$AAN?$AA?3?$AA?5?$AAC?$AAr?$AAe?$AAa?$AAt?$AAe?$AA?5?$AAE?$AAv?$AAe?$AAn?$AAt?$AA?5?$AAF?$AAa?$AAi?$AAl?$AAe?$AAd?$AA?5?$AAf?$AAo?$AAr?$AA?5?$AAx?$AAc?$AAv@ 1000a5a8     usb_usbfn_os_mx25_topaz_v1:i_os.obj
 0001:000095f8       ??_C@_1EA@CDEDEFDH@?$AAU?$AAF?$AAN?$AA?3?$AA?5?$AAC?$AAr?$AAe?$AAa?$AAt?$AAe?$AAd?$AA?5?$AAa?$AA?5?$AAn?$AAe?$AAw?$AA?5?$AAX?$AAC?$AAV?$AAR?$AA?5?$AAE?$AAv?$AAe?$AAn?$AAt?$AA?$AN?$AA?6?$AA?$AA@ 1000a5f8     usb_usbfn_os_mx25_topaz_v1:i_os.obj
 0001:00009638       ??_C@_1EK@IADMCEKM@?$AAU?$AAF?$AAN?$AA?3?$AA?5?$AAO?$AAp?$AAe?$AAn?$AAe?$AAd?$AA?5?$AAa?$AAn?$AA?5?$AAe?$AAx?$AAi?$AAs?$AAt?$AAi?$AAn?$AAg?$AA?5?$AAX?$AAC?$AAV?$AAR?$AA?5?$AAE?$AAv?$AAe@ 1000a638     usb_usbfn_os_mx25_topaz_v1:i_os.obj
 0001:00009684       ??_C@_1BA@JAHEEJIA@?$AAU?$AAS?$AAB?$AAX?$AAC?$AAV?$AAR?$AA?$AA@ 1000a684     usb_usbfn_os_mx25_topaz_v1:i_os.obj
 0001:00009698       ??_C@_1EK@DLKEEKEI@?$AAU?$AAF?$AAN?$AA?3?$AA?5?$AAC?$AAr?$AAe?$AAa?$AAt?$AAe?$AA?5?$AAE?$AAv?$AAe?$AAn?$AAt?$AA?5?$AAF?$AAa?$AAi?$AAl?$AAe?$AAd?$AA?5?$AAf?$AAo?$AAr?$AA?5?$AAf?$AAu?$AAn@ 1000a698     usb_usbfn_os_mx25_topaz_v1:i_os.obj
 0001:000096e8       ??_C@_1EA@NFBAADLP@?$AAU?$AAF?$AAN?$AA?3?$AA?5?$AAC?$AAr?$AAe?$AAa?$AAt?$AAe?$AAd?$AA?5?$AAa?$AA?5?$AAn?$AAe?$AAw?$AA?5?$AAF?$AAu?$AAn?$AAc?$AA?5?$AAE?$AAv?$AAe?$AAn?$AAt?$AA?$AN?$AA?6?$AA?$AA@ 1000a6e8     usb_usbfn_os_mx25_topaz_v1:i_os.obj
 0001:00009728       ??_C@_1EK@HGGPGCCE@?$AAU?$AAF?$AAN?$AA?3?$AA?5?$AAO?$AAp?$AAe?$AAn?$AAe?$AAd?$AA?5?$AAa?$AAn?$AA?5?$AAe?$AAx?$AAi?$AAs?$AAt?$AAi?$AAn?$AAg?$AA?5?$AAF?$AAu?$AAn?$AAc?$AA?5?$AAE?$AAv?$AAe@ 1000a728     usb_usbfn_os_mx25_topaz_v1:i_os.obj
 0001:00009774       ??_C@_1DA@LMBIJMBC@?$AAU?$AAS?$AAB?$AAF?$AAN?$AA?3?$AA?5?$AAC?$AAr?$AAe?$AAa?$AAt?$AAe?$AAE?$AAv?$AAe?$AAn?$AAt?$AA?3?$AA?$CF?$AAs?$AA?$AN?$AA?6?$AA?$AA@ 1000a774     usb_usbfn_os_mx25_topaz_v1:i_os.obj
 0001:000097a4       ??_C@_1BA@EKAPLICF@?$AAU?$AAS?$AAB?$AAF?$AAu?$AAn?$AAc?$AA?$AA@ 1000a7a4     usb_usbfn_os_mx25_topaz_v1:i_os.obj
 0001:000097b4       ??_C@_1CG@CAPLKHBA@?$AAI?$AAs?$AAO?$AAT?$AAG?$AAS?$AAu?$AAp?$AAp?$AAo?$AAr?$AAt?$AA?$DP?$AA?5?$AA?$CF?$AAd?$AA?$AN?$AA?6?$AA?$AA@ 1000a7b4     usb_usbfn_os_mx25_topaz_v1:i_os.obj
 0001:000097e0       ??_C@_1HC@CCFLKHGC@?$AAd?$AA?3?$AA?2?$AAy?$AAz?$AAk?$AAi?$AAq?$AAf?$AAe?$AA?2?$AAp?$AAr?$AAi?$AAv?$AAa?$AAt?$AAe?$AA?2?$AAw?$AAi?$AAn?$AAc?$AAe?$AAo?$AAs?$AA?2?$AAC?$AAO?$AAR?$AAE?$AAO@ 1000a7e0     ceosutil:utilmem.obj
 0001:00009858       ??_C@_1HE@MNAIPFCF@?$AAd?$AA?3?$AA?2?$AAy?$AAz?$AAk?$AAi?$AAq?$AAf?$AAe?$AA?2?$AAp?$AAr?$AAi?$AAv?$AAa?$AAt?$AAe?$AA?2?$AAw?$AAi?$AAn?$AAc?$AAe?$AAo?$AAs?$AA?2?$AAC?$AAO?$AAR?$AAE?$AAO@ 1000a858     ceosutil:utilmemf.obj
 0001:000098d0       ??_C@_1FK@OFJPBPFD@?$AAd?$AA?3?$AA?2?$AAy?$AAz?$AAk?$AAi?$AAq?$AAf?$AAe?$AA?2?$AAp?$AAu?$AAb?$AAl?$AAi?$AAc?$AA?2?$AAc?$AAo?$AAm?$AAm?$AAo?$AAn?$AA?2?$AAs?$AAd?$AAk?$AA?2?$AAi?$AAn?$AAc@ 1000a8d0     ceosutil:utilmemf.obj
 0001:0000992c       ??_7SVSTree@@6B@           1000a92c     ceosutil:utilmemf.obj
 0001:0000993c       ??_7SVSEnumClass@@6B@      1000a93c     ceosutil:utilmemf.obj
 0001:0000994c       ??_C@_1DK@DAPDOICG@?$AAA?$AAs?$AAs?$AAe?$AAr?$AAt?$AA?5?$AAb?$AAr?$AAo?$AAk?$AAe?$AAn?$AA?5?$AAi?$AAn?$AA?5?$AA?$CF?$AAs?$AA?5?$AAl?$AAi?$AAn?$AAe?$AA?5?$AA?$CF?$AAd?$AA?6?$AA?$AA@ 1000a94c     ceosutil:svsutil.obj
 0001:00009988       ??_C@_1HE@EELBLLPN@?$AAd?$AA?3?$AA?2?$AAy?$AAz?$AAk?$AAi?$AAq?$AAf?$AAe?$AA?2?$AAp?$AAr?$AAi?$AAv?$AAa?$AAt?$AAe?$AA?2?$AAw?$AAi?$AAn?$AAc?$AAe?$AAo?$AAs?$AA?2?$AAC?$AAO?$AAR?$AAE?$AAO@ 1000a988     ceosutil:utiltree.obj
 0001:000099fc       ??_C@_1M@OAJFFPML@?$AAF?$AAl?$AAa?$AAg?$AAs?$AA?$AA@ 1000a9fc     defbuslib:DefBus.obj
 0001:00009a08       ??_C@_1M@PJMPBMAL@?$AAO?$AAr?$AAd?$AAe?$AAr?$AA?$AA@ 1000aa08     defbuslib:DefBus.obj
 0001:00009a14       ??_C@_1BA@KDCCGFJM@?$AAB?$AAu?$AAs?$AAN?$AAa?$AAm?$AAe?$AA?$AA@ 1000aa14     defbuslib:DefBus.obj
 0001:00009a28       ??_C@_1HO@PECMKLPI@?$AAC?$AA?3?$AA?2?$AAy?$AAm?$AAz?$AAk?$AAi?$AA?2?$AAp?$AAu?$AAb?$AAl?$AAi?$AAc?$AA?2?$AAC?$AAO?$AAM?$AAM?$AAO?$AAN?$AA?2?$AAo?$AAa?$AAk?$AA?2?$AAd?$AAr?$AAi?$AAv?$AAe@ 1000aa28     defbuslib:DefBus.obj
 0001:00009aa8       ??_C@_1BI@CDNKGHCP@?$AA?$CF?$AAs?$AA_?$AA?$CF?$AAd?$AA_?$AA?$CF?$AAd?$AA_?$AA?$CF?$AAd?$AA?$AA@ 1000aaa8     defbuslib:DefBus.obj
 0001:00009ac0       ??_C@_1BM@MHMIAMLB@?$AAI?$AAn?$AAt?$AAe?$AAr?$AAf?$AAa?$AAc?$AAe?$AAT?$AAy?$AAp?$AAe?$AA?$AA@ 1000aac0     defbuslib:DefBus.obj
 0001:00009adc       ??_C@_1BE@PMMIAJMN@?$AAB?$AAu?$AAs?$AAP?$AAa?$AAr?$AAe?$AAn?$AAt?$AA?$AA@ 1000aadc     defbuslib:DefBus.obj
 0001:00009af0       ??_7DeviceFolder@@6B@      1000aaf0     defbuslib:DefBus.obj
 0001:00009b14       ??_7CRefObject@@6B@        1000ab14     defbuslib:DefBus.obj
 0001:00009b18       ??_C@_1FE@EDMNJJKI@?$AAE?$AAn?$AAu?$AAm?$AAe?$AAr?$AAa?$AAt?$AAe?$AA?5?$AAG?$AAe?$AAt?$AAP?$AAr?$AAo?$AAc?$AAA?$AAd?$AAd?$AAr?$AA?$CI?$AA?$CF?$AAs?$AA?0?$AA?5?$AA?$CF?$AAs?$AA?$CJ?$AA?5?$AAf?$AAa@ 1000ab18     defbuslib:DefBus.obj
 0001:00009b70       ??_C@_1FK@BHMAEBH@?$AAE?$AAn?$AAu?$AAm?$AAe?$AAr?$AAa?$AAt?$AAe?$AA?5?$AAL?$AAo?$AAa?$AAd?$AAD?$AAr?$AAi?$AAv?$AAe?$AAr?$AA?1?$AAL?$AAi?$AAb?$AAr?$AAa?$AAr?$AAy?$AA?$CI?$AA?$CF?$AAs?$AA?$CJ@ 1000ab70     defbuslib:DefBus.obj
 0001:00009bd0       ??_C@_1GK@HPNKMNIJ@?$AAD?$AAe?$AAv?$AAi?$AAc?$AAe?$AAF?$AAo?$AAl?$AAd?$AAe?$AAr?$AA?3?$AA?3?$AAL?$AAo?$AAa?$AAd?$AAD?$AAe?$AAv?$AAi?$AAc?$AAe?$AA?$CB?$AAE?$AAn?$AAu?$AAm?$AAe?$AAr?$AAa@ 1000abd0     defbuslib:DefBus.obj
 0001:00009c40       ??_C@_1JE@FEKPHJBG@?$AAD?$AAe?$AAv?$AAi?$AAc?$AAe?$AAF?$AAo?$AAl?$AAd?$AAe?$AAr?$AA?3?$AA?3?$AAL?$AAo?$AAa?$AAd?$AAD?$AAe?$AAv?$AAi?$AAc?$AAe?$AA?$CB?$AAE?$AAn?$AAu?$AAm?$AAe?$AAr?$AAa@ 1000ac40     defbuslib:DefBus.obj
 0001:00009cd8       ??_C@_1FG@PFBMMOFN@?$AAD?$AAe?$AAv?$AAi?$AAc?$AAe?$AAF?$AAo?$AAl?$AAd?$AAe?$AAr?$AA?3?$AA?3?$AAL?$AAo?$AAa?$AAd?$AAD?$AAe?$AAv?$AAi?$AAc?$AAe?$AA?$CI?$AA?$CF?$AAs?$AA?$CJ?$AA?5?$AAl?$AAa?$AAs@ 1000acd8     defbuslib:DefBus.obj
 0001:00009d30       ??_C@_1NG@FJIKCOAJ@?$AAD?$AAe?$AAv?$AAi?$AAc?$AAe?$AAF?$AAo?$AAl?$AAd?$AAe?$AAr?$AA?3?$AA?3?$AAL?$AAo?$AAa?$AAd?$AAD?$AAe?$AAv?$AAi?$AAc?$AAe?$AA?$CB?$AAE?$AAn?$AAu?$AAm?$AAe?$AAr?$AAa@ 1000ad30     defbuslib:DefBus.obj
 0001:00009e08       ??_C@_1M@JLADBBAF@?$AAE?$AAn?$AAt?$AAr?$AAy?$AA?$AA@ 1000ae08     defbuslib:DefBus.obj
 0001:00009e18       ??_C@_1GK@HPKHPFKK@?$AAD?$AAe?$AAv?$AAi?$AAc?$AAe?$AAF?$AAo?$AAl?$AAd?$AAe?$AAr?$AA?$CB?$AAL?$AAo?$AAa?$AAd?$AA?5?$AAR?$AAe?$AAg?$AAO?$AAp?$AAe?$AAn?$AAK?$AAe?$AAy?$AAE?$AAx?$AA?$CI?$AA?$CF@ 1000ae18     defbuslib:DefBus.obj
 0001:00009e88       ??_C@_1HK@KFBBFFHK@?$AAD?$AAe?$AAv?$AAi?$AAc?$AAe?$AAF?$AAo?$AAl?$AAd?$AAe?$AAr?$AA?3?$AA?3?$AAL?$AAo?$AAa?$AAd?$AAD?$AAe?$AAv?$AAi?$AAc?$AAe?$AA?$CB?$AAL?$AAo?$AAa?$AAd?$AAi?$AAn?$AAg@ 1000ae88     defbuslib:DefBus.obj
 0001:00009f08       ??_C@_1JI@MDDKNOEL@?$AAD?$AAe?$AAv?$AAi?$AAc?$AAe?$AAF?$AAo?$AAl?$AAd?$AAe?$AAr?$AA?3?$AA?3?$AAU?$AAn?$AAl?$AAo?$AAa?$AAd?$AAD?$AAe?$AAv?$AAi?$AAc?$AAe?$AA?3?$AA?5?$AAD?$AAe?$AAa?$AAc@ 1000af08     defbuslib:DefBus.obj
 0001:00009fa0       ??_7DefaultBusDriver@@6B@  1000afa0     defbuslib:DefBus.obj
 0001:00009ffc       ??_C@_1BA@HABJOAEE@?$AAU?$AAN?$AAK?$AAN?$AAO?$AAW?$AAN?$AA?$AA@ 1000affc     defbuslib:DefBus.obj
 0001:0000a00c       ??_C@_1M@KCNCFNNL@?$AA$?$AAb?$AAu?$AAs?$AA?2?$AA?$AA@ 1000b00c     defbuslib:DefBus.obj
 0001:0000a018       ??_C@_1BC@GDFGLIEL@?$AAO?$AAT?$AAG?$AAG?$AAr?$AAo?$AAu?$AAp?$AA?$AA@ 1000b018     usb_usbfn_mx25_topaz_v1:i_pdd.obj
 0001:0000a02c       ??_C@_1BG@HHFAGDDC@?$AAO?$AAT?$AAG?$AAS?$AAu?$AAp?$AAp?$AAo?$AAr?$AAt?$AA?$AA@ 1000b02c     usb_usbfn_mx25_topaz_v1:i_pdd.obj
 0001:0000a044       ??_C@_1BI@BHLBGEOK@?$AAP?$AAr?$AAi?$AAo?$AAr?$AAi?$AAt?$AAy?$AA2?$AA5?$AA6?$AA?$AA@ 1000b044     usb_usbfn_mx25_topaz_v1:i_pdd.obj
 0001:0000a05c       ??_C@_17DJGGJCGD@?$AAI?$AAr?$AAq?$AA?$AA@ 1000b05c     usb_usbfn_mx25_topaz_v1:i_pdd.obj
 0001:0000a064       ??_C@_1O@LBBNFMDB@?$AAM?$AAe?$AAm?$AAL?$AAe?$AAn?$AA?$AA@ 1000b064     usb_usbfn_mx25_topaz_v1:i_pdd.obj
 0001:0000a074       ??_C@_1BA@INLDIDEN@?$AAM?$AAe?$AAm?$AAB?$AAa?$AAs?$AAe?$AA?$AA@ 1000b074     usb_usbfn_mx25_topaz_v1:i_pdd.obj
 0001:0000a1a8       ??_C@_1CM@IKIIJOLF@?$AAP?$AAo?$AAw?$AAe?$AAr?$AAD?$AAo?$AAw?$AAn?$AA?5?$AAc?$AAo?$AAm?$AAp?$AAl?$AAe?$AAt?$AAe?$AAd?$AA?$AN?$AA?6?$AA?$AA@ 1000b1a8     usb_usbfn_mx25_topaz_v1:i_pdd.obj
 0001:0000a1d4       ??_C@_1CC@OEGDFOPI@?$AAU?$AAS?$AAB?$AA?5?$AAC?$AAl?$AAo?$AAc?$AAk?$AA?5?$AAs?$AAt?$AAo?$AAp?$AA?$AN?$AA?6?$AA?$AA@ 1000b1d4     usb_usbfn_mx25_topaz_v1:i_pdd.obj
 0001:0000a1f8       ??_C@_1DC@MJCJJIDL@?$AAP?$AAo?$AAw?$AAe?$AAr?$AAD?$AAo?$AAw?$AAn?$AA?5?$AAU?$AAS?$AAB?$AAC?$AAT?$AAR?$AAL?$AA?$DN?$AA0?$AAx?$AA?$CF?$AAx?$AA?$AN?$AA?6?$AA?$AA@ 1000b1f8     usb_usbfn_mx25_topaz_v1:i_pdd.obj
 0001:0000a22c       ??_C@_1DC@NJODNJCA@?$AAP?$AAo?$AAw?$AAe?$AAr?$AAD?$AAo?$AAw?$AAn?$AA?5?$AAP?$AAO?$AAR?$AAT?$AAS?$AAC?$AA?$DN?$AA?5?$AA0?$AAx?$AA?$CF?$AAx?$AA?$AN?$AA?6?$AA?$AA@ 1000b22c     usb_usbfn_mx25_topaz_v1:i_pdd.obj
 0001:0000a260       ??_C@_1DG@NJOCHJMF@?$AAP?$AAo?$AAw?$AAe?$AAr?$AAD?$AAo?$AAw?$AAn?$AA?5?$AAU?$AAS?$AAB?$AAI?$AAN?$AAT?$AAR?$AA?5?$AA?$DN?$AA?5?$AA0?$AAx?$AA?$CF?$AAx?$AA?$AN?$AA?6?$AA?$AA@ 1000b260     usb_usbfn_mx25_topaz_v1:i_pdd.obj
 0001:0000a298       ??_C@_1DE@CFOAAIJP@?$AAP?$AAo?$AAw?$AAe?$AAr?$AAD?$AAo?$AAw?$AAn?$AA?5?$AAU?$AAS?$AAB?$AAC?$AAM?$AAD?$AA?5?$AA?$DN?$AA?5?$AA0?$AAx?$AA?$CF?$AAx?$AA?$AN?$AA?6?$AA?$AA@ 1000b298     usb_usbfn_mx25_topaz_v1:i_pdd.obj
 0001:0000a2d0       ??_C@_1EM@IEDMFFDN@?$AAU?$AAf?$AAn?$AAP?$AAd?$AAd?$AA_?$AAP?$AAo?$AAw?$AAe?$AAr?$AAD?$AAo?$AAw?$AAn?$AA?5?$AAn?$AAo?$AA?5?$AAa?$AAc?$AAt?$AAi?$AAo?$AAn?$AA?5?$AAr?$AAe?$AAq?$AAu?$AAi@ 1000b2d0     usb_usbfn_mx25_topaz_v1:i_pdd.obj
 0001:0000a31c       ??_C@_1CG@OIILOOGO@?$AAU?$AAs?$AAb?$AAP?$AAd?$AAd?$AA_?$AAP?$AAo?$AAw?$AAe?$AAr?$AAD?$AAo?$AAw?$AAn?$AA?$AN?$AA?6?$AA?$AA@ 1000b31c     usb_usbfn_mx25_topaz_v1:i_pdd.obj
 0001:0000a344       ??_C@_1DA@KMOKCFJD@?$AAP?$AAo?$AAw?$AAe?$AAr?$AAU?$AAp?$AA?5?$AAU?$AAS?$AAB?$AAC?$AAM?$AAD?$AA?5?$AA?$DN?$AA?5?$AA0?$AAx?$AA?$CF?$AAx?$AA?$AN?$AA?6?$AA?$AA@ 1000b344     usb_usbfn_mx25_topaz_v1:i_pdd.obj
 0001:0000a378       ??_C@_1EA@HIDFOGGD@?$AAW?$AAa?$AAk?$AAe?$AAu?$AAp?$AA?5?$AAI?$AAn?$AAt?$AAe?$AAr?$AAr?$AAu?$AAp?$AAt?$AA?5?$AAS?$AAe?$AAt?$AAt?$AAi?$AAn?$AAg?$AA?5?$AA0?$AAx?$AA?$CF?$AAx?$AA?$AN?$AA?6?$AA?$AA@ 1000b378     usb_usbfn_mx25_topaz_v1:i_pdd.obj
 0001:0000a3b8       ??_C@_1DA@ODLPFKGM@?$AAP?$AAo?$AAw?$AAe?$AAr?$AAU?$AAp?$AA?5?$AAw?$AAa?$AAk?$AAe?$AAu?$AAp?$AA?5?$AA?$DN?$AA?5?$AA0?$AAx?$AA?$CF?$AAx?$AA?$AN?$AA?6?$AA?$AA@ 1000b3b8     usb_usbfn_mx25_topaz_v1:i_pdd.obj
 0001:0000a3e8       ??_C@_1BO@JBMLODEA@?$AAF?$AAo?$AAr?$AAc?$AAe?$AA?5?$AAr?$AAe?$AAs?$AAu?$AAm?$AAe?$AA?$AN?$AA?6?$AA?$AA@ 1000b3e8     usb_usbfn_mx25_topaz_v1:i_pdd.obj
 0001:0000a408       ??_C@_1EI@LEEJEJNJ@?$AAP?$AAo?$AAw?$AAe?$AAr?$AAU?$AAp?$AA?3?$AAU?$AAS?$AAB?$AAS?$AAT?$AAS?$AA?$CI?$AA0?$AAx?$AA?$CF?$AAx?$AA?$CJ?$AA?5?$AAP?$AAO?$AAR?$AAT?$AAS?$AAC?$AA?$CI?$AA0?$AAx?$AA?$CF?$AAx@ 1000b408     usb_usbfn_mx25_topaz_v1:i_pdd.obj
 0001:0000a450       ??_C@_1CE@HMNFKKGB@?$AAU?$AAS?$AAB?$AA?5?$AAC?$AAl?$AAo?$AAc?$AAk?$AA?5?$AAs?$AAt?$AAa?$AAr?$AAt?$AA?$AN?$AA?6?$AA?$AA@ 1000b450     usb_usbfn_mx25_topaz_v1:i_pdd.obj
 0001:0000a478       ??_C@_1EE@FMEOMODP@?$AAU?$AAs?$AAb?$AAP?$AAd?$AAd?$AA_?$AAP?$AAo?$AAw?$AAe?$AAr?$AAU?$AAp?$AA?5?$AAw?$AAi?$AAt?$AAh?$AA?5?$AAb?$AAI?$AAn?$AAU?$AAS?$AAB?$AAF?$AAN?$AA?5?$AA?$CF?$AAd?$AA?$AN@ 1000b478     usb_usbfn_mx25_topaz_v1:i_pdd.obj
 0001:0000a4c0       ??_C@_1EC@POPMIGGA@?$AAU?$AAp?$AAd?$AAa?$AAt?$AAe?$AAD?$AAe?$AAv?$AAi?$AAc?$AAe?$AAP?$AAo?$AAw?$AAe?$AAr?$AA?5?$AAt?$AAo?$AA?5?$AAp?$AAo?$AAw?$AAe?$AAr?$AAd?$AAo?$AAw?$AAn?$AA?$AN?$AA?6@ 1000b4c0     usb_usbfn_mx25_topaz_v1:i_pdd.obj
 0001:0000a504       ??_C@_1DO@CFDCODDO@?$AAU?$AAp?$AAd?$AAa?$AAt?$AAe?$AAD?$AAe?$AAv?$AAi?$AAc?$AAe?$AAP?$AAo?$AAw?$AAe?$AAr?$AA?5?$AAt?$AAo?$AA?5?$AAp?$AAo?$AAw?$AAe?$AAr?$AAu?$AAp?$AA?$AN?$AA?6?$AA?$AA@ 1000b504     usb_usbfn_mx25_topaz_v1:i_pdd.obj
 0001:0000a548       ??_C@_1FE@DIHLBJLK@?$AAU?$AAp?$AAd?$AAa?$AAt?$AAe?$AAD?$AAe?$AAv?$AAi?$AAc?$AAe?$AAP?$AAo?$AAw?$AAe?$AAr?$AA?5?$AAG?$AAo?$AAi?$AAn?$AAg?$AA?5?$AAf?$AAr?$AAo?$AAm?$AA?5?$AAD?$AA?$CF?$AAd@ 1000b548     usb_usbfn_mx25_topaz_v1:i_pdd.obj
 0001:0000a5a0       ??_C@_1KO@LDNIEBB@?$AAC?$AA?3?$AA?2?$AAW?$AAI?$AAN?$AAC?$AAE?$AAR?$AAO?$AAO?$AAT?$AAS?$AA?2?$AAT?$AAo?$AAp?$AAa?$AAz?$AA?2?$AAW?$AAI?$AAN?$AAC?$AAE?$AA6?$AA0?$AA0?$AA?2?$AAp?$AAl?$AAa@ 1000b5a0     usb_usbfn_mx25_topaz_v1:i_pdd.obj
 0001:0000a650       ??_C@_1BO@LJJCCAKA@?$AAS?$AAe?$AAt?$AAu?$AAp?$AA?3?$AA?5?$AA?$CF?$AAx?$AA?5?$AA?$CF?$AAx?$AA?$AN?$AA?6?$AA?$AA@ 1000b650     usb_usbfn_mx25_topaz_v1:i_pdd.obj
 0001:0000a670       ??_C@_1CA@NAJOELH@?$AAD?$AAe?$AAv?$AAi?$AAc?$AAe?$AA?5?$AAA?$AAt?$AAt?$AAa?$AAc?$AAh?$AA?$AN?$AA?6?$AA?$AA@ 1000b670     usb_usbfn_mx25_topaz_v1:i_pdd.obj
 0001:0000a690       ??_C@_1IE@MBNKMJA@?$AA?$CD?$AA?$CD?$AA?$CD?$AA?$CD?$AA?$CD?$AA?$CD?$AA?$CD?$AA?5?$AAG?$AAe?$AAt?$AAS?$AAe?$AAt?$AAu?$AAp?$AAP?$AAa?$AAc?$AAk?$AAe?$AAt?$AA?3?$AA?5?$AAF?$AAl?$AAu?$AAs?$AAh?$AAi?$AAn?$AAg@ 1000b690     usb_usbfn_mx25_topaz_v1:i_pdd.obj
 0001:0000a718       ??_C@_1KK@KOKNNFID@?$AA?$CD?$AA?$CD?$AA?$CD?$AA?$CD?$AA?$CD?$AA?$CD?$AA?$CD?$AA?5?$AAG?$AAe?$AAt?$AAS?$AAe?$AAt?$AAu?$AAp?$AAP?$AAa?$AAc?$AAk?$AAe?$AAt?$AA?3?$AA?5?$AAT?$AAr?$AAa?$AAn?$AAs?$AAf?$AAe?$AAr@ 1000b718     usb_usbfn_mx25_topaz_v1:i_pdd.obj
 0001:0000a7c4       ??_C@_1DM@JOKNMMI@?$AAG?$AAe?$AAt?$AAS?$AAe?$AAt?$AAu?$AAp?$AAP?$AAa?$AAc?$AAk?$AAe?$AAt?$AA?5?$AA?$CF?$AA8?$AA?4?$AA8?$AAl?$AAx?$AA?$CF?$AA8?$AA?4?$AA8?$AAl?$AAx?$AA?$AN?$AA?6?$AA?$AA@ 1000b7c4     usb_usbfn_mx25_topaz_v1:i_pdd.obj
 0001:0000a800       ??_C@_1DM@PINNGIJL@?$AA?7?$AA?7?$AA?7?$AAS?$AAe?$AAr?$AAi?$AAa?$AAl?$AA?1?$AA1?$AA?4?$AA1?$AA?5?$AAP?$AAH?$AAY?$AA?5?$AA?$CI?$AAF?$AAS?$AA?5?$AAO?$AAn?$AAl?$AAy?$AA?$CJ?$AA?$AN?$AA?6?$AA?$AA@ 1000b800     usb_usbfn_mx25_topaz_v1:i_pdd.obj
 0001:0000a83c       ??_C@_1BE@OHMKGMAA@?$AA?7?$AA?7?$AA?7?$AAU?$AAL?$AAP?$AAI?$AA?$AN?$AA?6?$AA?$AA@ 1000b83c     usb_usbfn_mx25_topaz_v1:i_pdd.obj
 0001:0000a850       ??_C@_1CK@JDCKMGFE@?$AA?7?$AA?7?$AA?7?$AAP?$AAh?$AAi?$AAl?$AAi?$AAp?$AAs?$AA?5?$AAC?$AAl?$AAa?$AAs?$AAs?$AAi?$AAc?$AA?$AN?$AA?6?$AA?$AA@ 1000b850     usb_usbfn_mx25_topaz_v1:i_pdd.obj
 0001:0000a87c       ??_C@_1CA@GIFIBBC@?$AA?7?$AA?7?$AA?7?$AAU?$AAT?$AAM?$AAI?$AA?1?$AAU?$AAT?$AAM?$AAI?$AA?$CL?$AA?$AN?$AA?6?$AA?$AA@ 1000b87c     usb_usbfn_mx25_topaz_v1:i_pdd.obj
 0001:0000a8a0       ??_C@_1EG@GEPPEHI@?$AA?7?$AA?7?$AAP?$AAa?$AAr?$AAa?$AAl?$AAl?$AAe?$AAl?$AA?5?$AAT?$AAr?$AAa?$AAn?$AAs?$AAc?$AAe?$AAi?$AAv?$AAe?$AAr?$AA?5?$AAS?$AAe?$AAl?$AAe?$AAc?$AAt?$AA?3?$AA?$CF?$AAx@ 1000b8a0     usb_usbfn_mx25_topaz_v1:i_pdd.obj
 0001:0000a8e8       ??_C@_1DO@GOALHOBG@?$AA?7?$AA?7?$AAS?$AAe?$AAr?$AAi?$AAa?$AAl?$AA?5?$AAT?$AAr?$AAa?$AAn?$AAs?$AAc?$AAe?$AAi?$AAv?$AAe?$AAr?$AA?5?$AAS?$AAe?$AAl?$AAe?$AAc?$AAt?$AA?5?$AA?$AN?$AA?6?$AA?$AA@ 1000b8e8     usb_usbfn_mx25_topaz_v1:i_pdd.obj
 0001:0000a928       ??_C@_1BI@PMFMKPBN@?$AA?7?$AA?7?$AA?7?$AA8?$AA?5?$AAb?$AAi?$AAt?$AAs?$AA?$AN?$AA?6?$AA?$AA@ 1000b928     usb_usbfn_mx25_topaz_v1:i_pdd.obj
 0001:0000a940       ??_C@_1BK@DMIJGPDB@?$AA?7?$AA?7?$AA?7?$AA1?$AA6?$AA?5?$AAb?$AAi?$AAt?$AAs?$AA?$AN?$AA?6?$AA?$AA@ 1000b940     usb_usbfn_mx25_topaz_v1:i_pdd.obj
 0001:0000a960       ??_C@_1EE@PJPHJMEN@?$AA?7?$AA?7?$AAP?$AAa?$AAr?$AAa?$AAl?$AAl?$AAe?$AAl?$AA?5?$AAT?$AAr?$AAa?$AAn?$AAs?$AAc?$AAe?$AAi?$AAv?$AAe?$AAr?$AA?5?$AAW?$AAi?$AAd?$AAt?$AAh?$AA?3?$AA?$CF?$AAx?$AA?9@ 1000b960     usb_usbfn_mx25_topaz_v1:i_pdd.obj
 0001:0000a9a4       ??_C@_1CA@CFDEDDEG@?$AA?7?$AA?7?$AA?7?$AAH?$AAi?$AAg?$AAh?$AA?5?$AAS?$AAp?$AAe?$AAe?$AAd?$AA?$AN?$AA?6?$AA?$AA@ 1000b9a4     usb_usbfn_mx25_topaz_v1:i_pdd.obj
 0001:0000a9c4       ??_C@_1BO@DONMFABC@?$AA?7?$AA?7?$AA?7?$AAL?$AAo?$AAw?$AA?5?$AAS?$AAp?$AAe?$AAe?$AAd?$AA?$AN?$AA?6?$AA?$AA@ 1000b9c4     usb_usbfn_mx25_topaz_v1:i_pdd.obj
 0001:0000a9e4       ??_C@_1CA@EFHFHOIO@?$AA?7?$AA?7?$AA?7?$AAF?$AAu?$AAl?$AAl?$AA?5?$AAS?$AAp?$AAe?$AAe?$AAd?$AA?$AN?$AA?6?$AA?$AA@ 1000b9e4     usb_usbfn_mx25_topaz_v1:i_pdd.obj
 0001:0000aa04       ??_C@_1CG@DLDJDNPN@?$AA?7?$AA?7?$AAP?$AAo?$AAr?$AAt?$AA?5?$AAS?$AAp?$AAe?$AAe?$AAd?$AA?3?$AA?5?$AA?$CF?$AAx?$AA?9?$AA?$DO?$AA?$AA@ 1000ba04     usb_usbfn_mx25_topaz_v1:i_pdd.obj
 0001:0000aa30       ??_C@_1EG@FLKCNOK@?$AA?7?$AA?7?$AAP?$AAo?$AAr?$AAt?$AA?5?$AAF?$AAo?$AAr?$AAc?$AAe?$AA?5?$AAF?$AAu?$AAl?$AAl?$AA?5?$AAS?$AAp?$AAe?$AAe?$AAd?$AA?5?$AAC?$AAo?$AAn?$AAn?$AAe?$AAc?$AAt?$AA?5@ 1000ba30     usb_usbfn_mx25_topaz_v1:i_pdd.obj
 0001:0000aa78       ??_C@_1GI@HKEGLKNC@?$AA?7?$AA?7?$AAP?$AAH?$AAY?$AA?5?$AAL?$AAo?$AAw?$AA?5?$AAP?$AAo?$AAw?$AAe?$AAr?$AA?5?$AAS?$AAu?$AAs?$AAp?$AAe?$AAn?$AAd?$AA?5?$AA?9?$AA?5?$AAC?$AAl?$AAo?$AAc?$AAk?$AA?5@ 1000ba78     usb_usbfn_mx25_topaz_v1:i_pdd.obj
 0001:0000aae0       ??_C@_1FE@PECIMICA@?$AA?7?$AA?7?$AAW?$AAa?$AAk?$AAe?$AA?5?$AAo?$AAn?$AA?5?$AAO?$AAv?$AAe?$AAr?$AA?9?$AAc?$AAu?$AAr?$AAr?$AAe?$AAn?$AAt?$AA?5?$AAE?$AAn?$AAa?$AAb?$AAl?$AAe?$AA?5?$AA?$CI?$AAW@ 1000bae0     usb_usbfn_mx25_topaz_v1:i_pdd.obj
 0001:0000ab38       ??_C@_1FI@KPMEKFHG@?$AA?7?$AA?7?$AAW?$AAa?$AAk?$AAe?$AA?5?$AAo?$AAn?$AA?5?$AAD?$AAi?$AAs?$AAc?$AAo?$AAn?$AAn?$AAe?$AAc?$AAt?$AA?5?$AAE?$AAn?$AAa?$AAb?$AAl?$AAe?$AA?5?$AA?$CI?$AAW?$AAK?$AAD@ 1000bb38     usb_usbfn_mx25_topaz_v1:i_pdd.obj
 0001:0000ab90       ??_C@_1EM@HPIOFCNI@?$AA?7?$AA?7?$AAW?$AAa?$AAk?$AAe?$AA?5?$AAo?$AAn?$AA?5?$AAC?$AAo?$AAn?$AAn?$AAe?$AAc?$AAt?$AA?5?$AAE?$AAn?$AAa?$AAb?$AAl?$AAe?$AA?5?$AA?$CI?$AAW?$AAK?$AAC?$AAN?$AAN?$AAT@ 1000bb90     usb_usbfn_mx25_topaz_v1:i_pdd.obj
 0001:0000abdc       ??_C@_1DE@NJCPBMGI@?$AA?7?$AA?7?$AAP?$AAo?$AAr?$AAt?$AA?5?$AAT?$AAe?$AAs?$AAt?$AA?5?$AAC?$AAo?$AAn?$AAt?$AAr?$AAo?$AAl?$AA?3?$AA?5?$AA?$CF?$AAx?$AA?$AN?$AA?6?$AA?$AA@ 1000bbdc     usb_usbfn_mx25_topaz_v1:i_pdd.obj
 0001:0000ac10       ??_C@_1BG@LAPJBFLO@?$AA?7?$AA?7?$AA?7?$AAG?$AAr?$AAe?$AAe?$AAn?$AA?$AN?$AA?6?$AA?$AA@ 1000bc10     usb_usbfn_mx25_topaz_v1:i_pdd.obj
 0001:0000ac28       ??_C@_1BG@IMMCDJCL@?$AA?7?$AA?7?$AA?7?$AAA?$AAm?$AAb?$AAe?$AAr?$AA?$AN?$AA?6?$AA?$AA@ 1000bc28     usb_usbfn_mx25_topaz_v1:i_pdd.obj
 0001:0000ac40       ??_C@_1DC@IPGABND@?$AA?7?$AA?7?$AAP?$AAo?$AAr?$AAt?$AA?5?$AAI?$AAn?$AAd?$AAi?$AAc?$AAa?$AAt?$AAo?$AAr?$AA?5?$AAC?$AAo?$AAn?$AAt?$AAr?$AAo?$AAl?$AA?$AA@ 1000bc40     usb_usbfn_mx25_topaz_v1:i_pdd.obj
 0001:0000ac74       ??_C@_1BO@FPLCLNEP@?$AA?7?$AA?7?$AAP?$AAo?$AAr?$AAt?$AA?5?$AAO?$AAw?$AAn?$AAe?$AAr?$AA?$AN?$AA?6?$AA?$AA@ 1000bc74     usb_usbfn_mx25_topaz_v1:i_pdd.obj
 0001:0000ac94       ??_C@_1DO@MCLJLJA@?$AA?7?$AA?7?$AA?$DP?$AA?$DP?$AA?$DP?$AA?5?$AAS?$AAh?$AAo?$AAu?$AAl?$AAd?$AA?5?$AAb?$AAe?$AA?5?$AA0?$AA?5?$AAf?$AAo?$AAr?$AA?5?$AAd?$AAe?$AAv?$AAi?$AAc?$AAe?$AA?$AN?$AA?6?$AA?$AA@ 1000bc94     usb_usbfn_mx25_topaz_v1:i_pdd.obj
 0001:0000acd4       ??_C@_1BO@CGJIBKMJ@?$AA?7?$AA?7?$AA?7?$AAU?$AAn?$AAd?$AAe?$AAf?$AAi?$AAn?$AAe?$AAd?$AA?$AN?$AA?6?$AA?$AA@ 1000bcd4     usb_usbfn_mx25_topaz_v1:i_pdd.obj
 0001:0000acf4       ??_C@_1BK@LEBDPOFP@?$AA?7?$AA?7?$AA?7?$AAK?$AA?9?$AAs?$AAt?$AAa?$AAt?$AAe?$AA?$AN?$AA?6?$AA?$AA@ 1000bcf4     usb_usbfn_mx25_topaz_v1:i_pdd.obj
 0001:0000ad10       ??_C@_1BK@NBHEMFBJ@?$AA?7?$AA?7?$AA?7?$AAJ?$AA?9?$AAs?$AAt?$AAa?$AAt?$AAe?$AA?$AN?$AA?6?$AA?$AA@ 1000bd10     usb_usbfn_mx25_topaz_v1:i_pdd.obj
 0001:0000ad2c       ??_C@_1BC@HGFCDNBO@?$AA?7?$AA?7?$AA?7?$AAS?$AAE?$AA0?$AA?$AN?$AA?6?$AA?$AA@ 1000bd2c     usb_usbfn_mx25_topaz_v1:i_pdd.obj
 0001:0000ad40       ??_C@_1CE@HKBMNK@?$AA?7?$AA?7?$AAL?$AAi?$AAn?$AAe?$AA?5?$AAS?$AAt?$AAa?$AAt?$AAu?$AAs?$AA?3?$AA?5?$AA?$CF?$AAx?$AA?$AA@ 1000bd40     usb_usbfn_mx25_topaz_v1:i_pdd.obj
 0001:0000ad64       ??_C@_1CK@KAKGINHH@?$AA?7?$AA?7?$AAH?$AAi?$AAg?$AAh?$AA?9?$AAS?$AAp?$AAe?$AAe?$AAd?$AA?5?$AAP?$AAo?$AAr?$AAt?$AA?5?$AA?$AN?$AA?6?$AA?$AA@ 1000bd64     usb_usbfn_mx25_topaz_v1:i_pdd.obj
 0001:0000ad90       ??_C@_1BO@GDNLNMNM@?$AA?7?$AA?7?$AAP?$AAo?$AAr?$AAt?$AA?5?$AAR?$AAe?$AAs?$AAe?$AAt?$AA?$AN?$AA?6?$AA?$AA@ 1000bd90     usb_usbfn_mx25_topaz_v1:i_pdd.obj
 0001:0000adb0       ??_C@_1BI@BCOEFLFO@?$AA?7?$AA?7?$AAS?$AAu?$AAs?$AAp?$AAe?$AAn?$AAd?$AA?$AN?$AA?6?$AA?$AA@ 1000bdb0     usb_usbfn_mx25_topaz_v1:i_pdd.obj
 0001:0000adc8       ??_C@_1CM@LOGLIGHF@?$AA?7?$AA?7?$AAF?$AAo?$AAr?$AAc?$AAe?$AA?5?$AAP?$AAo?$AAr?$AAt?$AA?5?$AAR?$AAe?$AAs?$AAu?$AAm?$AAe?$AA?$AN?$AA?6?$AA?$AA@ 1000bdc8     usb_usbfn_mx25_topaz_v1:i_pdd.obj
 0001:0000adf4       ??_C@_1DA@IPBKEGAM@?$AA?7?$AA?7?$AAO?$AAv?$AAe?$AAr?$AA?9?$AAc?$AAu?$AAr?$AAr?$AAe?$AAn?$AAt?$AA?5?$AAC?$AAh?$AAa?$AAn?$AAg?$AAe?$AA?$AN?$AA?6?$AA?$AA@ 1000bdf4     usb_usbfn_mx25_topaz_v1:i_pdd.obj
 0001:0000ae24       ??_C@_1DA@IOPAFHGK@?$AA?7?$AA?7?$AAO?$AAv?$AAe?$AAr?$AA?9?$AAc?$AAu?$AAr?$AAr?$AAe?$AAn?$AAt?$AA?5?$AAA?$AAc?$AAt?$AAi?$AAv?$AAe?$AA?$AN?$AA?6?$AA?$AA@ 1000be24     usb_usbfn_mx25_topaz_v1:i_pdd.obj
 0001:0000ae54       ??_C@_1DO@IDEEGAC@?$AA?7?$AA?7?$AAP?$AAo?$AAr?$AAt?$AA?5?$AAE?$AAn?$AAa?$AAb?$AAl?$AAe?$AA?1?$AAD?$AAi?$AAs?$AAa?$AAb?$AAl?$AAe?$AA?5?$AAC?$AAh?$AAa?$AAn?$AAg?$AAe?$AA?$AN?$AA?6?$AA?$AA@ 1000be54     usb_usbfn_mx25_topaz_v1:i_pdd.obj
 0001:0000ae94       ??_C@_1CC@HIBPLHBD@?$AA?7?$AA?7?$AAP?$AAo?$AAr?$AAt?$AA?5?$AAE?$AAn?$AAa?$AAb?$AAl?$AAe?$AAd?$AA?$AN?$AA?6?$AA?$AA@ 1000be94     usb_usbfn_mx25_topaz_v1:i_pdd.obj
 0001:0000aeb8       ??_C@_1EG@CHIFACHN@?$AA?7?$AA?7?$AAC?$AAo?$AAn?$AAn?$AAe?$AAc?$AAt?$AA?5?$AAS?$AAt?$AAa?$AAt?$AAu?$AAs?$AA?5?$AAC?$AAh?$AAa?$AAn?$AAg?$AAe?$AA?3?$AA?5?$AAC?$AAh?$AAa?$AAn?$AAg?$AAe?$AAd@ 1000beb8     usb_usbfn_mx25_topaz_v1:i_pdd.obj
 0001:0000af00       ??_C@_1EK@CIGPBIFB@?$AA?7?$AA?7?$AAC?$AAu?$AAr?$AAr?$AAe?$AAn?$AAt?$AA?5?$AAC?$AAo?$AAn?$AAn?$AAe?$AAc?$AAt?$AA?5?$AAS?$AAt?$AAa?$AAt?$AAu?$AAs?$AA?3?$AA?5?$AAA?$AAt?$AAt?$AAa?$AAc?$AAh@ 1000bf00     usb_usbfn_mx25_topaz_v1:i_pdd.obj
 0001:0000af50       ??_C@_1EE@NKEDAIOG@?$AA?7?$AAA?$AAs?$AAy?$AAn?$AAc?$AAh?$AAr?$AAo?$AAn?$AAo?$AAu?$AAs?$AA?5?$AAS?$AAc?$AAh?$AAe?$AAd?$AAu?$AAl?$AAe?$AA?5?$AAS?$AAt?$AAa?$AAt?$AAu?$AAs?$AA?4?$AA?5?$AA?$AN@ 1000bf50     usb_usbfn_mx25_topaz_v1:i_pdd.obj
 0001:0000af94       ??_C@_1DM@OLIDMOLB@?$AA?7?$AAP?$AAe?$AAr?$AAi?$AAo?$AAd?$AAi?$AAc?$AA?5?$AAS?$AAc?$AAh?$AAe?$AAd?$AAu?$AAl?$AAe?$AA?5?$AAS?$AAt?$AAa?$AAt?$AAu?$AAs?$AA?4?$AA?5?$AA?$AN?$AA?6?$AA?$AA@ 1000bf94     usb_usbfn_mx25_topaz_v1:i_pdd.obj
 0001:0000afd0       ??_C@_1GE@JMEHEIAD@?$AA?7?$AAR?$AAe?$AAc?$AAl?$AAa?$AAm?$AAa?$AAt?$AAi?$AAo?$AAn?$AA?0?$AAO?$AAn?$AAl?$AAy?$AA?5?$AAu?$AAs?$AAe?$AAd?$AA?5?$AAb?$AAy?$AA?5?$AAt?$AAh?$AAe?$AA?5?$AAh?$AAo@ 1000bfd0     usb_usbfn_mx25_topaz_v1:i_pdd.obj
 0001:0000b034       ??_C@_1BK@HBEGAPL@?$AA?7?$AAH?$AAC?$AAH?$AAa?$AAI?$AAt?$AAe?$AAd?$AA?5?$AA?$AN?$AA?6?$AA?$AA@ 1000c034     usb_usbfn_mx25_topaz_v1:i_pdd.obj
 0001:0000b050       ??_C@_1CE@IIMNHGIF@?$AA?7?$AAU?$AAL?$AAP?$AAI?$AA?5?$AAI?$AAn?$AAt?$AAe?$AAr?$AAr?$AAu?$AAp?$AAt?$AA?$AN?$AA?6?$AA?$AA@ 1000c050     usb_usbfn_mx25_topaz_v1:i_pdd.obj
 0001:0000b074       ??_C@_1BM@JKFMOBOF@?$AA?7?$AAD?$AAC?$AAS?$AAu?$AAs?$AAp?$AAe?$AAn?$AAd?$AA?5?$AA?$AN?$AA?6?$AA?$AA@ 1000c074     usb_usbfn_mx25_topaz_v1:i_pdd.obj
 0001:0000b090       ??_C@_1CC@ILIGGFI@?$AA?7?$AAS?$AAO?$AAF?$AA?5?$AAR?$AAe?$AAc?$AAe?$AAi?$AAv?$AAe?$AAd?$AA?5?$AA?$AN?$AA?6?$AA?$AA@ 1000c090     usb_usbfn_mx25_topaz_v1:i_pdd.obj
 0001:0000b0b4       ??_C@_1CO@KLBBIGDH@?$AA?7?$AAU?$AAS?$AAB?$AA?5?$AAR?$AAe?$AAs?$AAe?$AAt?$AA?5?$AAR?$AAe?$AAc?$AAe?$AAi?$AAv?$AAe?$AAd?$AA?5?$AA?$AN?$AA?6?$AA?$AA@ 1000c0b4     usb_usbfn_mx25_topaz_v1:i_pdd.obj
 0001:0000b0e4       ??_C@_1DM@GMIDHHHN@?$AA?7?$AAI?$AAn?$AAt?$AAe?$AAr?$AAr?$AAu?$AAp?$AAt?$AA?5?$AAo?$AAn?$AA?5?$AAA?$AAs?$AAy?$AAn?$AAc?$AA?5?$AAA?$AAd?$AAv?$AAa?$AAn?$AAc?$AAe?$AA?$AN?$AA?6?$AA?$AA@ 1000c0e4     usb_usbfn_mx25_topaz_v1:i_pdd.obj
 0001:0000b120       ??_C@_1CA@OPJKBAE@?$AA?7?$AAS?$AAy?$AAs?$AAt?$AAe?$AAm?$AA?5?$AAE?$AAr?$AAr?$AAo?$AAr?$AA?$AN?$AA?6?$AA?$AA@ 1000c120     usb_usbfn_mx25_topaz_v1:i_pdd.obj
 0001:0000b140       ??_C@_1CO@ONBPMBE@?$AA?7?$AAF?$AAr?$AAa?$AAm?$AAe?$AA?5?$AAL?$AAi?$AAs?$AAt?$AA?5?$AAR?$AAo?$AAl?$AAl?$AAo?$AAv?$AAe?$AAr?$AA?$AN?$AA?6?$AA?$AA@ 1000c140     usb_usbfn_mx25_topaz_v1:i_pdd.obj
 0001:0000b170       ??_C@_1CM@BOJMIELL@?$AA?7?$AAP?$AAo?$AAr?$AAt?$AA?5?$AAC?$AAh?$AAa?$AAn?$AAg?$AAe?$AA?5?$AAD?$AAe?$AAt?$AAe?$AAc?$AAt?$AA?$AN?$AA?6?$AA?$AA@ 1000c170     usb_usbfn_mx25_topaz_v1:i_pdd.obj
 0001:0000b1a0       ??_C@_1EG@JNFJCNAA@?$AA?7?$AAU?$AAS?$AAB?$AA?5?$AAE?$AAr?$AAr?$AAo?$AAr?$AA?5?$AAI?$AAn?$AAt?$AAe?$AAr?$AAr?$AAu?$AAp?$AAt?$AA?5?$AA?$CI?$AAU?$AAS?$AAB?$AAE?$AAR?$AAR?$AAI?$AAN?$AAT?$AA?$CJ@ 1000c1a0     usb_usbfn_mx25_topaz_v1:i_pdd.obj
 0001:0000b1e8       ??_C@_1DE@KHLIMFPA@?$AA?7?$AAU?$AAS?$AAB?$AA?5?$AAI?$AAn?$AAt?$AAe?$AAr?$AAr?$AAu?$AAp?$AAt?$AA?5?$AA?$CI?$AAU?$AAS?$AAB?$AAI?$AAN?$AAT?$AA?$CJ?$AA?$AN?$AA?6?$AA?$AA@ 1000c1e8     usb_usbfn_mx25_topaz_v1:i_pdd.obj
 0001:0000b21c       ??_C@_1DG@EIGILMMI@?$AAI?$AAN?$AA?5?$AA?$CF?$AAs?$AA?5?$AAC?$AAo?$AAm?$AAp?$AAl?$AAe?$AAt?$AAe?$AAd?$AA?5?$AAa?$AAt?$AA?5?$AAe?$AAp?$AA?5?$AA?$CF?$AAd?$AA?$AN?$AA?6?$AA?$AA@ 1000c21c     usb_usbfn_mx25_topaz_v1:i_pdd.obj
 0001:0000b258       ??_C@_1FA@KBGDHCDA@?$AAS?$AAe?$AAn?$AAd?$AA?5?$AAe?$AAr?$AAr?$AAo?$AAr?$AA?$DP?$AA?$DP?$AA?5?$AAl?$AAe?$AAn?$AA?$DN?$AA?$CF?$AAx?$AA?0?$AA?5?$AAs?$AAt?$AAa?$AAt?$AAu?$AAs?$AA?$DN?$AA?$CF?$AAx?$AA?0?$AA?5@ 1000c258     usb_usbfn_mx25_topaz_v1:i_pdd.obj
 0001:0000b2a8       ??_C@_1EC@ONAPCMHH@?$AAS?$AAt?$AAa?$AAt?$AAu?$AAs?$AA?5?$AAi?$AAs?$AA?5?$AAn?$AAo?$AAt?$AA?5?$AA0?$AA?5?$AAo?$AAn?$AA?5?$AAs?$AAe?$AAn?$AAt?$AA?5?$AA?$CF?$AAx?$AA?5?$AA?$DN?$AA?$CF?$AAx?$AA?$AN?$AA?6@ 1000c2a8     usb_usbfn_mx25_topaz_v1:i_pdd.obj
 0001:0000b2f0       ??_C@_1GI@DMJOJCJK@?$AAC?$AAh?$AAe?$AAc?$AAk?$AAE?$AAn?$AAd?$AAp?$AAo?$AAi?$AAn?$AAt?$AA?3?$AAS?$AAe?$AAt?$AA?5?$AAA?$AAd?$AAd?$AAr?$AAe?$AAs?$AAs?$AA?3?$AA?5?$AA?$CF?$AAx?$AA?$CI?$AA?$CF?$AAx@ 1000c2f0     usb_usbfn_mx25_topaz_v1:i_pdd.obj
 0001:0000b358       ??_C@_1FO@LDFIJMJF@?$AAC?$AAh?$AAe?$AAc?$AAk?$AAE?$AAn?$AAd?$AAp?$AAo?$AAi?$AAn?$AAt?$AA?3?$AAE?$AAP?$AA0?$AA?5?$AAO?$AAU?$AAT?$AA?5?$AAN?$AAU?$AAL?$AAL?$AA?5?$AAt?$AAr?$AAa?$AAn?$AAs@ 1000c358     usb_usbfn_mx25_topaz_v1:i_pdd.obj
 0001:0000b3b8       ??_C@_1FG@MIJKNENI@?$AAC?$AAh?$AAe?$AAc?$AAk?$AAE?$AAn?$AAd?$AAp?$AAo?$AAi?$AAn?$AAt?$AA?3?$AAE?$AAP?$AA0?$AA?5?$AAO?$AAU?$AAT?$AA?5?$AA?$CF?$AAd?$AA?5?$AAb?$AAy?$AAt?$AAe?$AAs?$AA?5?$AAc@ 1000c3b8     usb_usbfn_mx25_topaz_v1:i_pdd.obj
 0001:0000b410       ??_C@_1FK@DOJLLFPC@?$AAC?$AAh?$AAe?$AAc?$AAk?$AAE?$AAn?$AAd?$AAp?$AAo?$AAi?$AAn?$AAt?$AA?3?$AAE?$AAP?$AA0?$AA?5?$AAO?$AAU?$AAT?$AA?5?$AA?$CF?$AAd?$AA?5?$AAb?$AAy?$AAt?$AAe?$AAs?$AA?5?$AAn@ 1000c410     usb_usbfn_mx25_topaz_v1:i_pdd.obj
 0001:0000b470       ??_C@_1GA@IAMKOKAN@?$AA?$CD?$AA?$CD?$AA?$CD?$AA?$CD?$AA?$CD?$AA?5?$AAm?$AAo?$AAr?$AAe?$AA?5?$AAd?$AAa?$AAt?$AAa?$AA?5?$AAt?$AAo?$AA?5?$AAr?$AAe?$AAc?$AAe?$AAi?$AAv?$AAe?$AA?5?$AAo?$AAn?$AA?5?$AAE?$AAP@ 1000c470     usb_usbfn_mx25_topaz_v1:i_pdd.obj
 0001:0000b4d0       ??_C@_1IM@GIGJCFIB@?$AA?$CD?$AA?$CD?$AA?$CD?$AA?$CD?$AA?$CD?$AA?$CD?$AA?$CD?$AA?$CD?$AA?$CD?$AA?$CD?$AA?$CD?$AA?$CD?$AA?$CD?$AA?5?$AAE?$AAN?$AAD?$AAP?$AAT?$AAC?$AAO?$AAM?$AAP?$AAL?$AAE?$AAT?$AAE?$AA?5?$AA?$CF?$AAx?$AA?5?$AAN@ 1000c4d0     usb_usbfn_mx25_topaz_v1:i_pdd.obj
 0001:0000b560       ??_C@_1EG@NDHBBAAH@?$AAO?$AAU?$AAT?$AA?5?$AA?$CF?$AAs?$AA?5?$AAC?$AAo?$AAm?$AAp?$AAl?$AAe?$AAt?$AAe?$AAd?$AA?5?$AAf?$AAo?$AAr?$AA?5?$AAe?$AAn?$AAd?$AAp?$AAo?$AAi?$AAn?$AAt?$AA?5?$AA?$CF?$AAd@ 1000c560     usb_usbfn_mx25_topaz_v1:i_pdd.obj
 0001:0000b5a8       ??_C@_1O@BIOIDBLM@?$AAC?$AAa?$AAn?$AAc?$AAe?$AAl?$AA?$AA@ 1000c5a8     usb_usbfn_mx25_topaz_v1:i_pdd.obj
 0001:0000b5b8       ??_C@_1O@PFKKKDLL@?$AAN?$AAo?$AAr?$AAm?$AAa?$AAl?$AA?$AA@ 1000c5b8     usb_usbfn_mx25_topaz_v1:i_pdd.obj
 0001:0000b5c8       ??_C@_1EK@JNBLLHDF@?$AAC?$AAh?$AAe?$AAc?$AAk?$AAE?$AAn?$AAd?$AAp?$AAo?$AAi?$AAn?$AAt?$AA?$CI?$AAe?$AAp?$AA?$DN?$AA?$CF?$AAd?$AA?$CJ?$AA?3?$AA?5?$AAB?$AAU?$AAF?$AAF?$AAE?$AAR?$AA_?$AAE?$AAR?$AAR@ 1000c5c8     usb_usbfn_mx25_topaz_v1:i_pdd.obj
 0001:0000b614       ??_C@_1CG@FAGAAPBN@?$AAE?$AAN?$AAD?$AAP?$AAT?$AAC?$AAO?$AAM?$AAP?$AAL?$AAE?$AAT?$AAE?$AA?5?$AA?$CF?$AAx?$AA?$AN?$AA?6?$AA?$AA@ 1000c614     usb_usbfn_mx25_topaz_v1:i_pdd.obj
 0001:0000b63c       ??_C@_1DO@LDKDDFPP@?$AAS?$AAt?$AAa?$AAt?$AAu?$AAs?$AA?5?$AAi?$AAs?$AA?5?$AAn?$AAo?$AAt?$AA?5?$AA0?$AA?5?$AAo?$AAn?$AA?5?$AAr?$AAe?$AAc?$AAv?$AA?5?$AA?$CF?$AAx?$AA?5?$AA?$DN?$AA?$CF?$AAx?$AA?$AA@ 1000c63c     usb_usbfn_mx25_topaz_v1:i_pdd.obj
 0001:0000b680       ??_C@_1EO@FDNJCHA@?$AAD?$AAe?$AAv?$AAi?$AAc?$AAe?$AA?5?$AAD?$AAe?$AAt?$AAa?$AAc?$AAh?$AA?0?$AA?5?$AAw?$AAi?$AAt?$AAh?$AA?5?$AAs?$AAu?$AAs?$AAp?$AA?$CI?$AA?$CF?$AAd?$AA?$CJ?$AA?0?$AA?5?$AAi?$AAd@ 1000c680     usb_usbfn_mx25_topaz_v1:i_pdd.obj
 0001:0000b6d0       ??_C@_1BO@PIPKGBKA@?$AA?$CK?$AAt?$AAe?$AAm?$AAp?$AA3?$AA?5?$AA0?$AAx?$AA?$CF?$AAx?$AA?5?$AA?$AN?$AA?6?$AA?$AA@ 1000c6d0     usb_usbfn_mx25_topaz_v1:i_pdd.obj
 0001:0000b6f0       ??_C@_1CI@HKDMKLGF@?$AAD?$AAe?$AAt?$AAa?$AAc?$AAh?$AA?3?$AA?5?$AAP?$AAO?$AAR?$AAT?$AAS?$AAC?$AA?5?$AA0?$AAx?$AA?$CF?$AAx?$AA?$AA@ 1000c6f0     usb_usbfn_mx25_topaz_v1:i_pdd.obj
 0001:0000b718       ??_C@_1CK@LPGMAHKL@?$AA?9?$AAU?$AAF?$AAN?$AA_?$AAD?$AAE?$AAT?$AAA?$AAC?$AAH?$AA?5?$AAc?$AAa?$AAl?$AAl?$AAe?$AAd?$AA?$AN?$AA?6?$AA?$AA@ 1000c718     usb_usbfn_mx25_topaz_v1:i_pdd.obj
 0001:0000b744       ??_C@_1CK@MPBLBBEN@?$AA?$CL?$AAU?$AAF?$AAN?$AA_?$AAD?$AAE?$AAT?$AAA?$AAC?$AAH?$AA?5?$AAc?$AAa?$AAl?$AAl?$AAe?$AAd?$AA?$AN?$AA?6?$AA?$AA@ 1000c744     usb_usbfn_mx25_topaz_v1:i_pdd.obj
 0001:0000b770       ??_C@_1O@BJIMCIMK@?$AAR?$AAe?$AAs?$AAu?$AAm?$AAe?$AA?$AA@ 1000c770     usb_usbfn_mx25_topaz_v1:i_pdd.obj
 0001:0000b780       ??_C@_1BC@MHKABCGD@?$AAB?$AAr?$AAe?$AAa?$AAk?$AA?5?$AA?$AN?$AA?6?$AA?$AA@ 1000c780     usb_usbfn_mx25_topaz_v1:i_pdd.obj
 0001:0000b794       ??_C@_1BE@JNFMNJIM@?$AAI?$AAn?$AAt?$AAr?$AA?3?$AAD?$AAo?$AAn?$AAe?$AA?$AA@ 1000c794     usb_usbfn_mx25_topaz_v1:i_pdd.obj
 0001:0000b7a8       ??_C@_1CC@IFAPINEE@?$AAS?$AAe?$AAt?$AAu?$AAp?$AAE?$AAv?$AAe?$AAn?$AAt?$AA?5?$AA?4?$AA?4?$AA?4?$AA?$AN?$AA?6?$AA?$AA@ 1000c7a8     usb_usbfn_mx25_topaz_v1:i_pdd.obj
 0001:0000b7d0       ??_C@_1EE@JAFGGGNF@?$AAI?$AAn?$AAt?$AAr?$AA?3?$AAU?$AAI?$AA?5?$AAS?$AAE?$AAT?$AAU?$AAP?$AAS?$AAT?$AAA?$AAT?$AA?5?$AA?$CF?$AAx?$AA?5?$AAE?$AAN?$AAD?$AAP?$AAT?$AAC?$AAO?$AAM?$AAP?$AA?5?$AA?$CF@ 1000c7d0     usb_usbfn_mx25_topaz_v1:i_pdd.obj
 0001:0000b814       ??_C@_1BC@MCOFDLFC@?$AAI?$AAn?$AAt?$AAr?$AA?3?$AAS?$AAL?$AAI?$AA?$AA@ 1000c814     usb_usbfn_mx25_topaz_v1:i_pdd.obj
 0001:0000b828       ??_C@_1BO@EGKDOEEI@?$AAI?$AAn?$AAt?$AAr?$AA?3?$AAS?$AAi?$AAg?$AAn?$AAa?$AAl?$AAl?$AAe?$AAd?$AA?$AA@ 1000c828     usb_usbfn_mx25_topaz_v1:i_pdd.obj
 0001:0000b848       ??_C@_1CA@FFAPNJLP@?$AAP?$AAD?$AAD?$AA?5?$AA?9?$AA?5?$AAS?$AAU?$AAS?$AAP?$AAE?$AAN?$AAD?$AA?$AN?$AA?6?$AA?$AA@ 1000c848     usb_usbfn_mx25_topaz_v1:i_pdd.obj
 0001:0000b868       ??_C@_1CC@NCLEKMLF@?$AA?5?$AAs?$AAt?$AAa?$AAt?$AAe?$AA?4?$AAP?$AAS?$AAP?$AAD?$AA?5?$AA?$CF?$AAx?$AA?$AN?$AA?6?$AA?$AA@ 1000c868     usb_usbfn_mx25_topaz_v1:i_pdd.obj
 0001:0000b88c       ??_C@_1CM@GCFNPFKO@?$AA?5?$AAB?$AAS?$AA_?$AAF?$AAU?$AAL?$AAL?$AA_?$AAS?$AAP?$AAE?$AAE?$AAD?$AA?5?$AA?5?$AA?5?$AA?$CF?$AAx?$AA?$AN?$AA?6?$AA?$AA@ 1000c88c     usb_usbfn_mx25_topaz_v1:i_pdd.obj
 0001:0000b8b8       ??_C@_1CM@EIGJNBDN@?$AA?5?$AAB?$AAS?$AA_?$AAH?$AAI?$AAG?$AAH?$AA_?$AAS?$AAP?$AAE?$AAE?$AAD?$AA?5?$AA?5?$AA?5?$AA?$CF?$AAx?$AA?$AN?$AA?6?$AA?$AA@ 1000c8b8     usb_usbfn_mx25_topaz_v1:i_pdd.obj
 0001:0000b8e8       ??_C@_1JI@KKCMHPHI@?$AAH?$AAa?$AAn?$AAd?$AAl?$AAe?$AAU?$AAS?$AAB?$AAR?$AAe?$AAs?$AAe?$AAt?$AA?3?$AA?5?$AAN?$AAo?$AAt?$AA?5?$AAs?$AAt?$AAi?$AAl?$AAl?$AA?5?$AAi?$AAn?$AA?5?$AAr?$AAe?$AAs@ 1000c8e8     usb_usbfn_mx25_topaz_v1:i_pdd.obj
 0001:0000b980       ??_C@_1CA@KBLMCKFP@?$AAD?$AAe?$AAv?$AAi?$AAc?$AAe?$AA?5?$AAD?$AAe?$AAt?$AAa?$AAc?$AAh?$AA?$AN?$AA?6?$AA?$AA@ 1000c980     usb_usbfn_mx25_topaz_v1:i_pdd.obj
 0001:0000b9a0       ??_C@_1FO@DFNLJIPA@?$AAU?$AAS?$AAB?$AAC?$AAo?$AAn?$AAt?$AAr?$AAo?$AAl?$AAl?$AAe?$AAr?$AAR?$AAu?$AAn?$AA?$CI?$AA?$CF?$AAd?$AA?$CJ?$AA?3?$AA?5?$AAf?$AAa?$AAi?$AAl?$AAe?$AAd?$AA?5?$AAt?$AAo?$AA?5@ 1000c9a0     usb_usbfn_mx25_topaz_v1:i_pdd.obj
 0001:0000ba00       ??_C@_1HI@FMJPDAIJ@?$AAU?$AAS?$AAB?$AAC?$AAo?$AAn?$AAt?$AAr?$AAo?$AAl?$AAl?$AAe?$AAr?$AAR?$AAu?$AAn?$AA?$CI?$AA1?$AA?$CJ?$AA?3?$AA?5?$AAE?$AAR?$AAR?$AAO?$AAR?$AA?5?$AA?$CD?$AA?$CD?$AA?$CD?$AA?$CD?$AA?$CD@ 1000ca00     usb_usbfn_mx25_topaz_v1:i_pdd.obj
 0001:0000ba78       ??_C@_1EM@BBPKMFPI@?$AAS?$AAt?$AAo?$AAp?$AA?5?$AAU?$AAS?$AAB?$AA?5?$AAc?$AAo?$AAn?$AAt?$AAr?$AAo?$AAl?$AAl?$AAe?$AAr?$AA?5?$AA?$CI?$AAR?$AAS?$AA?$DN?$AA?$CF?$AAd?$AA?5?$AA?9?$AA?$DO?$AA?5?$AAR?$AAS@ 1000ca78     usb_usbfn_mx25_topaz_v1:i_pdd.obj
 0001:0000bac8       ??_C@_1EO@GGMICPAJ@?$AAS?$AAt?$AAa?$AAr?$AAt?$AA?5?$AAU?$AAS?$AAB?$AA?5?$AAc?$AAo?$AAn?$AAt?$AAr?$AAo?$AAl?$AAl?$AAe?$AAr?$AA?5?$AA?$CI?$AAR?$AAS?$AA?$DN?$AA?$CF?$AAd?$AA?5?$AA?9?$AA?$DO?$AA?5?$AAR@ 1000cac8     usb_usbfn_mx25_topaz_v1:i_pdd.obj
 0001:0000bb18       ??_C@_1IO@CBIPFBFK@?$AA?$CD?$AA?$CD?$AA?$CD?$AA?$CD?$AA?$CD?$AA?$CD?$AA?$CD?$AA?$CD?$AA?$CD?$AA?$CD?$AA?$CD?$AA?$CD?$AA?$CD?$AA?5?$AAP?$AAr?$AAi?$AAm?$AAe?$AA?5?$AAF?$AAa?$AAi?$AAl?$AAe?$AAd?$AA?5?$AAf?$AAo?$AAr?$AA?5?$AAe@ 1000cb18     usb_usbfn_mx25_topaz_v1:i_pdd.obj
 0001:0000bba8       ??_C@_1FO@BKKPAEJB@?$AAI?$AAs?$AAs?$AAu?$AAe?$AAT?$AAr?$AAa?$AAn?$AAs?$AAf?$AAe?$AAr?$AA?5?$AAS?$AAE?$AAT?$AAU?$AAP?$AAS?$AAT?$AAA?$AAT?$AA?5?$AAr?$AAe?$AAc?$AAe?$AAi?$AAv?$AAe?$AAd@ 1000cba8     usb_usbfn_mx25_topaz_v1:i_pdd.obj
 0001:0000bc08       ??_C@_1EK@PGGCKEHJ@?$AAU?$AAf?$AAn?$AAP?$AAd?$AAd?$AA?3?$AA?5?$AAn?$AAe?$AAw?$AA?5?$AAs?$AAe?$AAt?$AAu?$AAp?$AA?5?$AAr?$AAe?$AAq?$AAu?$AAe?$AAs?$AAt?$AA?5?$AAd?$AAe?$AAt?$AAe?$AAc?$AAt@ 1000cc08     usb_usbfn_mx25_topaz_v1:i_pdd.obj
 0001:0000bc58       ??_C@_1HI@CDKGKFCF@?$AAE?$AAR?$AAR?$AAO?$AAR?$AA?3?$AA?5?$AAU?$AAf?$AAn?$AAP?$AAd?$AAd?$AA_?$AAI?$AAs?$AAs?$AAu?$AAe?$AAT?$AAr?$AAa?$AAn?$AAs?$AAf?$AAe?$AAr?$AA?3?$AA?5?$AAC?$AAe?$AAC@ 1000cc58     usb_usbfn_mx25_topaz_v1:i_pdd.obj
 0001:0000bcd0       ??_C@_1FK@CELBMJI@?$AAU?$AAf?$AAn?$AAP?$AAd?$AAd?$AA?3?$AA?5?$AAP?$AAa?$AAg?$AAe?$AA?5?$AAt?$AAr?$AAa?$AAn?$AAs?$AAl?$AAa?$AAt?$AAi?$AAo?$AAn?$AA?5?$AAf?$AAa?$AAi?$AAl?$AAe?$AAd?$AA?4@ 1000ccd0     usb_usbfn_mx25_topaz_v1:i_pdd.obj
 0001:0000bd30       ??_C@_1HA@DFAMLEOB@?$AAU?$AAf?$AAn?$AAP?$AAd?$AAd?$AA_?$AAI?$AAs?$AAs?$AAu?$AAe?$AAT?$AAr?$AAa?$AAn?$AAs?$AAf?$AAe?$AAr?$AA?3?$AA?5?$AAB?$AAu?$AAf?$AAf?$AAe?$AAr?$AA?5?$AAP?$AAa?$AAg@ 1000cd30     usb_usbfn_mx25_topaz_v1:i_pdd.obj
 0001:0000bda0       ??_C@_1KA@JGAAJONG@?$AAU?$AAf?$AAn?$AAP?$AAd?$AAd?$AA_?$AAI?$AAs?$AAs?$AAu?$AAe?$AAT?$AAr?$AAa?$AAn?$AAs?$AAf?$AAe?$AAr?$AA?3?$AA?5?$AAF?$AAa?$AAi?$AAl?$AAe?$AAd?$AA?5?$AAt?$AAo?$AA?5@ 1000cda0     usb_usbfn_mx25_topaz_v1:i_pdd.obj
 0001:0000be40       ??_C@_1HG@OBGGAFFH@?$AAE?$AAR?$AAR?$AAO?$AAR?$AA?3?$AA?5?$AAU?$AAf?$AAn?$AAP?$AAd?$AAd?$AA_?$AAI?$AAs?$AAs?$AAu?$AAe?$AAT?$AAr?$AAa?$AAn?$AAs?$AAf?$AAe?$AAr?$AA?3?$AA?5?$AAC?$AAe?$AAO@ 1000ce40     usb_usbfn_mx25_topaz_v1:i_pdd.obj
 0001:0000beb8       ??_C@_1FA@PGOEGLMA@?$AAU?$AAf?$AAn?$AAP?$AAd?$AAd?$AA_?$AAI?$AAs?$AAs?$AAu?$AAe?$AAT?$AAr?$AAa?$AAn?$AAs?$AAf?$AAe?$AAr?$AA?5?$AAf?$AAi?$AAr?$AAs?$AAt?$AA?5?$AAt?$AAi?$AAm?$AAe?$AA?$CI@ 1000ceb8     usb_usbfn_mx25_topaz_v1:i_pdd.obj
 0001:0000bf08       ??_C@_1JO@PEEOMCDL@?$AAI?$AAs?$AAs?$AAT?$AAr?$AAa?$AAn?$AA?5?$AA?$CI?$AA?$CF?$AAd?$AA?$CJ?$AA?3?$AA?5?$AA?$CF?$AAs?$AA?5?$AA?$CI?$AAp?$AAT?$AAr?$AAa?$AAn?$AAs?$AAf?$AAe?$AAr?$AA?$DN?$AA0?$AAx?$AA?$CF?$AAx@ 1000cf08     usb_usbfn_mx25_topaz_v1:i_pdd.obj
 0001:0000bfa8       ??_C@_1EA@GOCNCOIC@?$AAI?$AAs?$AAs?$AAu?$AAe?$AAT?$AAr?$AAa?$AAn?$AAs?$AAf?$AAe?$AAr?$AA?3?$AA?5?$AA?$CF?$AAs?$AA?5?$AAw?$AAi?$AAt?$AAh?$AA?5?$AA?$CF?$AAd?$AA?5?$AAb?$AAy?$AAt?$AAe?$AAs?$AA?$AA@ 1000cfa8     usb_usbfn_mx25_topaz_v1:i_pdd.obj
 0001:0000bfe8       ??_C@_19CIJIHAKK@?$AAN?$AAU?$AAL?$AAL?$AA?$AA@ 1000cfe8     usb_usbfn_mx25_topaz_v1:i_pdd.obj
 0001:0000bff8       ??_C@_1EG@CKENHIMK@?$AAU?$AAs?$AAb?$AAF?$AAn?$AAP?$AAd?$AAd?$AA_?$AAA?$AAb?$AAo?$AAr?$AAt?$AAT?$AAr?$AAa?$AAn?$AAs?$AAf?$AAe?$AAr?$AA?9?$AA?5?$AA?$CI?$AAE?$AAP?$AA?$DN?$AA?5?$AA?$CF?$AAd?$AA?$CJ@ 1000cff8     usb_usbfn_mx25_topaz_v1:i_pdd.obj
 0001:0000c040       ??_C@_1FA@PHGGDELL@?$AAA?$AAb?$AAo?$AAr?$AAt?$AA?$CI?$AA?$CF?$AAd?$AA?$CJ?$AA?5?$AAs?$AAk?$AAi?$AAp?$AAp?$AAe?$AAd?$AA?5?$AA?$CI?$AAT?$AAr?$AAa?$AAn?$AA?5?$AA0?$AAx?$AA?$CF?$AAx?$AA?5?$AA?$CB?$AA?$DN?$AA?5@ 1000d040     usb_usbfn_mx25_topaz_v1:i_pdd.obj
 0001:0000c090       ??_C@_1FK@ENKBNDBL@?$AA?$CD?$AA?$CD?$AA?$CD?$AA?$CD?$AA?$CD?$AA?$CD?$AA?$CD?$AA?$CD?$AA?$CD?$AA?$CD?$AA?$CD?$AA?5?$AAA?$AAb?$AAo?$AAr?$AAt?$AAT?$AAr?$AAa?$AAn?$AAs?$AAf?$AAe?$AAr?$AA?$CI?$AA?$CF?$AAd?$AA?$CJ?$AA?5?$AAD?$AAe@ 1000d090     usb_usbfn_mx25_topaz_v1:i_pdd.obj
 0001:0000c0f0       ??_C@_1GK@BJNDOLBF@?$AAU?$AAs?$AAb?$AAF?$AAn?$AAP?$AAd?$AAd?$AA_?$AAA?$AAb?$AAo?$AAr?$AAt?$AAT?$AAr?$AAa?$AAn?$AAs?$AAf?$AAe?$AAr?$AA?3?$AA?5?$AAp?$AAT?$AAr?$AAa?$AAn?$AAs?$AAf?$AAe@ 1000d0f0     usb_usbfn_mx25_topaz_v1:i_pdd.obj
 0001:0000c15c       ??_C@_1DA@JMEFNML@?$AAA?$AAb?$AAo?$AAr?$AAt?$AAT?$AAr?$AAa?$AAn?$AAs?$AAf?$AAe?$AAr?$AA?5?$AA?$CI?$AA?$CF?$AAs?$AA?5?$AAE?$AAP?$AA?$CF?$AAd?$AA?$CJ?$AA?$AA@ 1000d15c     usb_usbfn_mx25_topaz_v1:i_pdd.obj
 0001:0000c190       ??_C@_1EG@BFJDKFHL@?$AAU?$AAs?$AAb?$AAF?$AAn?$AAP?$AAd?$AAd?$AA_?$AAA?$AAb?$AAo?$AAr?$AAt?$AAT?$AAr?$AAa?$AAn?$AAs?$AAf?$AAe?$AAr?$AA?$CL?$AA?5?$AA?$CI?$AAE?$AAP?$AA?$DN?$AA?5?$AA?$CF?$AAd?$AA?$CJ@ 1000d190     usb_usbfn_mx25_topaz_v1:i_pdd.obj
 0001:0000c1d8       ??_C@_1DI@FFFNHHBF@?$AAU?$AAs?$AAb?$AAF?$AAn?$AAP?$AAd?$AAd?$AA_?$AAS?$AAt?$AAa?$AAl?$AAl?$AAE?$AAn?$AAd?$AAp?$AAo?$AAi?$AAn?$AAt?$AA?5?$AA?$CF?$AAd?$AA?$AN?$AA?6?$AA?$AA@ 1000d1d8     usb_usbfn_mx25_topaz_v1:i_pdd.obj
 0001:0000c210       ??_C@_1DI@EBJLFADF@?$AAU?$AAs?$AAb?$AAF?$AAn?$AAP?$AAd?$AAd?$AA_?$AAC?$AAl?$AAe?$AAa?$AAr?$AAE?$AAn?$AAd?$AAp?$AAo?$AAi?$AAn?$AAt?$AA?5?$AA?$CF?$AAd?$AA?$AN?$AA?6?$AA?$AA@ 1000d210     usb_usbfn_mx25_topaz_v1:i_pdd.obj
 0001:0000c248       ??_C@_1EA@DIDLDIBI@?$AA?9?$AAU?$AAs?$AAb?$AAF?$AAn?$AAP?$AAd?$AAd?$AA_?$AAI?$AAs?$AAE?$AAn?$AAd?$AAp?$AAo?$AAi?$AAn?$AAt?$AAH?$AAa?$AAl?$AAt?$AAe?$AAd?$AA?5?$AA?$CF?$AAd?$AA?$AN?$AA?6?$AA?$AA@ 1000d248     usb_usbfn_mx25_topaz_v1:i_pdd.obj
 0001:0000c288       ??_C@_1DO@MLIBPKBI@?$AAU?$AAs?$AAb?$AAF?$AAn?$AAP?$AAd?$AAd?$AA_?$AAI?$AAs?$AAE?$AAn?$AAd?$AAp?$AAo?$AAi?$AAn?$AAt?$AAH?$AAa?$AAl?$AAt?$AAe?$AAd?$AA?5?$AA?$CF?$AAd?$AA?$AN?$AA?6?$AA?$AA@ 1000d288     usb_usbfn_mx25_topaz_v1:i_pdd.obj
 0001:0000c2c8       ??_C@_1CA@HMLLGPGC@?$AA?9?$AAS?$AAe?$AAn?$AAd?$AAC?$AAS?$AAH?$AA?5?$AA?$CI?$AAE?$AAP?$AA?$CF?$AAd?$AA?$CJ?$AA?$AA@ 1000d2c8     usb_usbfn_mx25_topaz_v1:i_pdd.obj
 0001:0000c2e8       ??_C@_1CE@MAHEKDJP@?$AAS?$AAe?$AAn?$AAd?$AAC?$AAS?$AAH?$AA?5?$AAI?$AAN?$AA?5?$AA?$CI?$AA?$CF?$AAd?$AA?$CJ?$AA?$AN?$AA?6?$AA?$AA@ 1000d2e8     usb_usbfn_mx25_topaz_v1:i_pdd.obj
 0001:0000c30c       ??_C@_1CG@NAGMKJIL@?$AAS?$AAe?$AAn?$AAd?$AAC?$AAS?$AAH?$AA?5?$AAO?$AAU?$AAT?$AA?5?$AA?$CI?$AA?$CF?$AAd?$AA?$CJ?$AA?$AN?$AA?6?$AA?$AA@ 1000d30c     usb_usbfn_mx25_topaz_v1:i_pdd.obj
 0001:0000c334       ??_C@_1CA@DFPEHIFN@?$AA?$CL?$AAS?$AAe?$AAn?$AAd?$AAC?$AAS?$AAH?$AA?5?$AA?$CI?$AAE?$AAP?$AA?$CF?$AAd?$AA?$CJ?$AA?$AA@ 1000d334     usb_usbfn_mx25_topaz_v1:i_pdd.obj
 0001:0000c358       ??_C@_1FM@FGGEPKIB@?$AA?$CD?$AA?$CD?$AA?$CD?$AA?$CD?$AA?$CD?$AA?$CD?$AA?$CD?$AA?$CD?$AA?$CD?$AA?$CD?$AA?$CD?$AA?$CD?$AA?$CD?$AA?$CD?$AA?$CD?$AA?$CD?$AA?5?$AAF?$AAa?$AAi?$AAl?$AAe?$AAd?$AA?5?$AAt?$AAo?$AA?5?$AAp?$AAr?$AAi?$AAm?$AAe@ 1000d358     usb_usbfn_mx25_topaz_v1:i_pdd.obj
 0001:0000c3b8       ??_C@_1EG@KGILPPEC@?$AAC?$AAa?$AAn?$AA?5?$AAn?$AAo?$AAt?$AA?5?$AAp?$AAr?$AAi?$AAm?$AAe?$AA?5?$AAf?$AAo?$AAr?$AA?5?$AAZ?$AAL?$AAT?$AA?5?$AA?$CI?$AA?$CF?$AAs?$AA?$CJ?$AA?3?$AA?5?$AAb?$AAu?$AAs?$AAy@ 1000d3b8     usb_usbfn_mx25_topaz_v1:i_pdd.obj
 0001:0000c400       ??_C@_1BM@LGGJJGMB@?$AAP?$AAr?$AAi?$AAm?$AAe?$AAF?$AAZ?$AAL?$AAT?$AA?3?$AA?5?$AA?$CF?$AAs?$AA?$AA@ 1000d400     usb_usbfn_mx25_topaz_v1:i_pdd.obj
 0001:0000c420       ??_C@_1EA@KNMJPPBI@?$AAU?$AAs?$AAb?$AAF?$AAn?$AAP?$AAd?$AAd?$AA_?$AAI?$AAn?$AAi?$AAt?$AAi?$AAa?$AAt?$AAe?$AAR?$AAe?$AAm?$AAo?$AAt?$AAe?$AAW?$AAa?$AAk?$AAe?$AAu?$AAp?$AA?$AN?$AA?6?$AA?$AA@ 1000d420     usb_usbfn_mx25_topaz_v1:i_pdd.obj
 0001:0000c460       ??_C@_1CO@LFIHBCKN@?$AAS?$AAe?$AAt?$AAP?$AAo?$AAw?$AAe?$AAr?$AAS?$AAt?$AAa?$AAt?$AAe?$AA?5?$AA?$DN?$AA?5?$AA0?$AAx?$AA?$CF?$AAx?$AA?$AN?$AA?6?$AA?$AA@ 1000d460     usb_usbfn_mx25_topaz_v1:i_pdd.obj
 0001:0000c490       ??_C@_1HC@FEAKGGLP@?$AAP?$AAD?$AAD?$AA?3?$AA?5?$AAS?$AAe?$AAt?$AA?5?$AAF?$AAe?$AAa?$AAt?$AAu?$AAr?$AAe?$AA?5?$AA?$CI?$AAT?$AAE?$AAS?$AAT?$AA?5?$AAM?$AAO?$AAD?$AAE?$AA?$CJ?$AA?5?$AAO?$AAT?$AAG@ 1000d490     usb_usbfn_mx25_topaz_v1:i_pdd.obj
 0001:0000c508       ??_C@_1HC@GBFNHNAG@?$AAI?$AAO?$AAC?$AAT?$AAL?$AA_?$AAB?$AAU?$AAS?$AA_?$AAS?$AAE?$AAT?$AA_?$AAP?$AAO?$AAW?$AAE?$AAR?$AA_?$AAS?$AAT?$AAA?$AAT?$AAE?$AA?3?$AA?5?$AAC?$AAe?$AAO?$AAp?$AAe@ 1000d508     usb_usbfn_mx25_topaz_v1:i_pdd.obj
 0001:0000c580       ??_C@_1HE@NONILAAF@?$AAI?$AAO?$AAC?$AAT?$AAL?$AA_?$AAB?$AAU?$AAS?$AA_?$AAS?$AAE?$AAT?$AA_?$AAP?$AAO?$AAW?$AAE?$AAR?$AA_?$AAS?$AAT?$AAA?$AAT?$AAE?$AA?3?$AA?5?$AAC?$AAe?$AAC?$AAl?$AAo@ 1000d580     usb_usbfn_mx25_topaz_v1:i_pdd.obj
 0001:0000c5f8       ??_C@_1EG@GJIKGHF@?$AAI?$AAO?$AAC?$AAT?$AAL?$AA_?$AAB?$AAU?$AAS?$AA_?$AAS?$AAE?$AAT?$AA_?$AAP?$AAO?$AAW?$AAE?$AAR?$AA_?$AAS?$AAT?$AAA?$AAT?$AAE?$AA?5?$AAc?$AAa?$AAl?$AAl?$AAe?$AAd@ 1000d5f8     usb_usbfn_mx25_topaz_v1:i_pdd.obj
 0001:0000c640       ??_C@_1HC@NPNGJCMK@?$AAI?$AAO?$AAC?$AAT?$AAL?$AA_?$AAB?$AAU?$AAS?$AA_?$AAG?$AAE?$AAT?$AA_?$AAP?$AAO?$AAW?$AAE?$AAR?$AA_?$AAS?$AAT?$AAA?$AAT?$AAE?$AA?3?$AA?5?$AAC?$AAe?$AAO?$AAp?$AAe@ 1000d640     usb_usbfn_mx25_topaz_v1:i_pdd.obj
 0001:0000c6b8       ??_C@_1HE@IJCCGJCF@?$AAI?$AAO?$AAC?$AAT?$AAL?$AA_?$AAB?$AAU?$AAS?$AA_?$AAG?$AAE?$AAT?$AA_?$AAP?$AAO?$AAW?$AAE?$AAR?$AA_?$AAS?$AAT?$AAA?$AAT?$AAE?$AA?3?$AA?5?$AAC?$AAe?$AAC?$AAl?$AAo@ 1000d6b8     usb_usbfn_mx25_topaz_v1:i_pdd.obj
 0001:0000c730       ??_C@_1EG@FFODHJCP@?$AAI?$AAO?$AAC?$AAT?$AAL?$AA_?$AAB?$AAU?$AAS?$AA_?$AAG?$AAE?$AAT?$AA_?$AAP?$AAO?$AAW?$AAE?$AAR?$AA_?$AAS?$AAT?$AAA?$AAT?$AAE?$AA?5?$AAc?$AAa?$AAl?$AAl?$AAe?$AAd@ 1000d730     usb_usbfn_mx25_topaz_v1:i_pdd.obj
 0001:0000c778       ??_C@_1BM@ELBPNMDN@?$AAU?$AAf?$AAn?$AAP?$AAd?$AAd?$AA_?$AAS?$AAt?$AAo?$AAp?$AA?$AN?$AA?6?$AA?$AA@ 1000d778     usb_usbfn_mx25_topaz_v1:i_pdd.obj
 0001:0000c794       ??_C@_1DK@CCAICBIP@?$AA?$CL?$AAU?$AAf?$AAn?$AAP?$AAd?$AAd?$AA_?$AAD?$AAe?$AAi?$AAn?$AAi?$AAt?$AAE?$AAn?$AAd?$AAp?$AAo?$AAi?$AAn?$AAt?$AA?3?$AA?5?$AA?$CF?$AAd?$AA?$AN?$AA?6?$AA?$AA@ 1000d794     usb_usbfn_mx25_topaz_v1:i_pdd.obj
 0001:0000c7d0       ??_C@_1DK@MHIAFBPJ@?$AAI?$AAn?$AAi?$AAt?$AA?5?$AAE?$AAn?$AAd?$AAp?$AAo?$AAi?$AAn?$AAt?$AA?3?$AA?5?$AA?$CF?$AAx?$AA?0?$AA?5?$AAc?$AAt?$AAr?$AAl?$AA?$DN?$AA?$CF?$AAx?$AA?$AN?$AA?6?$AA?$AA@ 1000d7d0     usb_usbfn_mx25_topaz_v1:i_pdd.obj
 0001:0000c810       ??_C@_1EK@HMBFBNAN@?$AAU?$AAf?$AAn?$AAP?$AAd?$AAd?$AA_?$AAI?$AAn?$AAi?$AAt?$AAE?$AAn?$AAd?$AAp?$AAo?$AAi?$AAn?$AAt?$AA?3?$AA?5?$AA?$CF?$AAd?$AA?5?$AAA?$AAt?$AAt?$AAr?$AAi?$AAb?$AA?$CI?$AA?$CF@ 1000d810     usb_usbfn_mx25_topaz_v1:i_pdd.obj
 0001:0000c85c       ??_C@_1CA@IJBGFJAE@?$AA?9?$AAU?$AAf?$AAn?$AAP?$AAd?$AAd?$AA_?$AAS?$AAt?$AAa?$AAr?$AAt?$AA?$AN?$AA?6?$AA?$AA@ 1000d85c     usb_usbfn_mx25_topaz_v1:i_pdd.obj
 0001:0000c87c       ??_C@_1CA@MAFJEODL@?$AA?$CL?$AAU?$AAf?$AAn?$AAP?$AAd?$AAd?$AA_?$AAS?$AAt?$AAa?$AAr?$AAt?$AA?$AN?$AA?6?$AA?$AA@ 1000d87c     usb_usbfn_mx25_topaz_v1:i_pdd.obj
 0001:0000c89c       ??_C@_1DG@EEIHMJOF@?$AAS?$AAt?$AAa?$AAt?$AAu?$AAs?$AA?5?$AAf?$AAo?$AAr?$AA?5?$AAt?$AAd?$AA0?$AA?$DN?$AA?$CF?$AAx?$AA?0?$AA?5?$AAt?$AAb?$AA?$DN?$AA?$CF?$AAx?$AA?$AN?$AA?6?$AA?$AA@ 1000d89c     usb_usbfn_mx25_topaz_v1:i_pdd.obj
 0001:0000c8d4       ??_C@_1CM@FGGAHLIL@?$AAP?$AAR?$AAI?$AAM?$AAE?$AA?5?$AAf?$AAa?$AAi?$AAl?$AAe?$AAd?$AA?5?$AAo?$AAn?$AA?5?$AAE?$AAP?$AA0?$AA?$AN?$AA?6?$AA?$AA@ 1000d8d4     usb_usbfn_mx25_topaz_v1:i_pdd.obj
 0001:0000c900       ??_C@_1FC@FLIFOJB@?$AAN?$AAe?$AAw?$AA?5?$AAs?$AAe?$AAt?$AAu?$AAp?$AA?5?$AAr?$AAe?$AAc?$AAe?$AAi?$AAv?$AAe?$AAd?$AA?5?$AAw?$AAh?$AAe?$AAn?$AA?5?$AAp?$AAr?$AAi?$AAm?$AAi?$AAn?$AAg?$AA?$DN@ 1000d900     usb_usbfn_mx25_topaz_v1:i_pdd.obj
 0001:0000c958       ??_C@_1GC@FCEGAELL@?$AAS?$AAe?$AAt?$AAu?$AAp?$AA?5?$AAn?$AAo?$AAt?$AA?5?$AAp?$AAr?$AAo?$AAc?$AAe?$AAs?$AAs?$AAe?$AAd?$AA?5?$AA?$CI?$AAS?$AAE?$AAT?$AAU?$AAP?$AAS?$AAT?$AAA?$AAT?$AA?$DN?$AA0@ 1000d958     usb_usbfn_mx25_topaz_v1:i_pdd.obj
 0001:0000c9bc       ??_C@_1BI@DKIPBNLN@?$AAI?$AAn?$AAi?$AAt?$AAq?$AAh?$AA0?$AA?0?$AA?5?$AA?$CF?$AAx?$AA?$AA@ 1000d9bc     usb_usbfn_mx25_topaz_v1:i_pdd.obj
 0001:0000c9d4       ??_C@_1BK@PALAPBNH@?$AA?4?$AA?4?$AAc?$AAo?$AAu?$AAn?$AAt?$AA?5?$AA?$CF?$AAd?$AA?$AN?$AA?6?$AA?$AA@ 1000d9d4     usb_usbfn_mx25_topaz_v1:i_pdd.obj
 0001:0000c9f0       ??_C@_1HA@BIGHAGHK@?$AAD?$AAi?$AAs?$AAa?$AAb?$AAl?$AAe?$AA?5?$AAI?$AAn?$AAt?$AAe?$AAr?$AAr?$AAu?$AAp?$AAt?$AA?5?$AAa?$AAn?$AAd?$AA?5?$AAl?$AAe?$AAt?$AA?5?$AAt?$AAh?$AAe?$AA?5?$AAT?$AAr@ 1000d9f0     usb_usbfn_mx25_topaz_v1:i_pdd.obj
 0001:0000ca60       ??_C@_1DC@LGPAELOO@?$AAS?$AAi?$AAz?$AAe?$AAo?$AAf?$AA?5?$AAq?$AAh?$AAb?$AAu?$AAf?$AAf?$AAe?$AAr?$AA?5?$AA?$DN?$AA?5?$AA0?$AAx?$AA?$CF?$AAx?$AA?$AN?$AA?6?$AA?$AA@ 1000da60     usb_usbfn_mx25_topaz_v1:i_pdd.obj
 0001:0000ca98       ??_C@_1HE@JFIJHLAK@?$AAE?$AAR?$AAR?$AAO?$AAR?$AA?3?$AA?5?$AAU?$AAf?$AAn?$AAP?$AAd?$AAd?$AA_?$AAI?$AAn?$AAi?$AAt?$AA?3?$AA?5?$AAC?$AAo?$AAn?$AAt?$AAr?$AAo?$AAl?$AAl?$AAe?$AAr?$AA?5?$AAr@ 1000da98     usb_usbfn_mx25_topaz_v1:i_pdd.obj
 0001:0000cb10       ??_C@_1FK@EMBOCJKF@?$AAE?$AAR?$AAR?$AAO?$AAR?$AA?3?$AA?5?$AAU?$AAf?$AAn?$AAP?$AAd?$AAd?$AA_?$AAI?$AAn?$AAi?$AAt?$AA?3?$AA?5?$AAF?$AAa?$AAi?$AAl?$AAe?$AAd?$AA?5?$AAo?$AAp?$AAe?$AAn?$AA?5@ 1000db10     usb_usbfn_mx25_topaz_v1:i_pdd.obj
 0001:0000cb70       ??_C@_1GM@LIECJJPD@?$AAE?$AAR?$AAR?$AAO?$AAR?$AA?3?$AA?5?$AAU?$AAf?$AAn?$AAP?$AAd?$AAd?$AA_?$AAI?$AAn?$AAi?$AAt?$AA?3?$AA?5?$AAF?$AAa?$AAi?$AAl?$AAe?$AAd?$AA?5?$AAr?$AAe?$AAa?$AAd?$AA?5@ 1000db70     usb_usbfn_mx25_topaz_v1:i_pdd.obj
 0001:0000cbe0       ??_C@_1EG@BDFMMKKK@?$AAU?$AAf?$AAn?$AAP?$AAd?$AAd?$AA_?$AAI?$AAn?$AAi?$AAt?$AA?5?$AAp?$AAP?$AAd?$AAd?$AA?5?$AAa?$AAl?$AAl?$AAo?$AAc?$AAa?$AAt?$AAe?$AA?5?$AAf?$AAa?$AAi?$AAl?$AAe?$AAd@ 1000dbe0     usb_usbfn_mx25_topaz_v1:i_pdd.obj
 0001:0000cc28       ??_C@_1GG@IILKAMAB@?$AAU?$AAS?$AAB?$AA?5?$AAD?$AAr?$AAi?$AAv?$AAe?$AAr?$AA?5?$AAl?$AAo?$AAa?$AAd?$AA?5?$AAf?$AAa?$AAi?$AAl?$AAu?$AAr?$AAe?$AA?5?$AAb?$AAe?$AAc?$AAa?$AAu?$AAs?$AAe?$AA?5@ 1000dc28     usb_usbfn_mx25_topaz_v1:i_pdd.obj
 0001:0000ccb4       BSPGetUSBControllerType    1000dcb4 f   hwinit.obj
 0001:0000cccc       HardwareInitialize         1000dccc f   hwinit.obj
 0001:0000d244       HardwarePullupDP           1000e244 f   hwinit.obj
 0001:0000d3a0       GetSysIntr                 1000e3a0 f   hwinit.obj
 0001:0000d3b8       BSPUsbResetPHY             1000e3b8 f   hwinit.obj
 0001:0000d3cc       USBClockInit               1000e3cc f   i_usbclock.obj
 0001:0000d3f8       USBClockGatingLock         1000e3f8 f   i_usbclock.obj
 0001:0000d454       USBClockGatingUnlock       1000e454 f   i_usbclock.obj
 0001:0000d470       BSPUSBClockCreateFileMapping 1000e470 f   i_usbclock.obj
 0001:0000d6a4       BSPUSBClockDeleteFileMapping 1000e6a4 f   i_usbclock.obj
 0001:0000d708       BSPUSBClockSwitch          1000e708 f   i_usbclock.obj
 0001:0000da3c       PowerDownSchemeExist       1000ea3c f   i_usbutils.obj
 0001:0000dae0       BSPUsbXvrEnableVBUSIntr    1000eae0 f   i_usbutils.obj
 0001:0000db60       BSPUsbXvrEnableIDIntr      1000eb60 f   i_usbutils.obj
 0001:0000dbe0       BSPUsbEnableLowPowerIntr   1000ebe0 f   i_usbutils.obj
 0001:0000dc30       BSPUsbSetBusConfig         1000ec30 f   i_usbutils.obj
 0001:0000dc74       BSPUSBInterruptControl     1000ec74 f   i_usbutils.obj
 0001:0000dce0       BSPPhyShowDevDiscon        1000ece0 f   i_usbutils.obj
 0001:0000dcf8       BSPUsbPhyStartUp           1000ecf8 f   i_usbutils.obj
 0001:0000dcfc       BSPUsbSetCurrentLimitation 1000ecfc f   i_usbutils.obj
 0001:0000dd10       BSPUsbPhyRegDump           1000ed10 f   i_usbutils.obj
 0001:0000dd14       BSPUSBSwitchModulePower    1000ed14 f   i_usbutils.obj
 0001:0000dd28       BSPHostDisconDetect        1000ed28 f   i_usbutils.obj
 0001:0000dd3c       ?ValidateContext@@YAXPAUUFN_MDD_CONTEXT@@@Z 1000ed3c f   usb_ufnmddbase_common_topaz_v1:ufnmdd.obj
 0001:0000dffc       ?GetSpeedString@@YAPBGW4_UFN_BUS_SPEED@@@Z 1000effc f   usb_ufnmddbase_common_topaz_v1:ufnmdd.obj
 0001:0000e064       ?FindPipe@@YAPAVCPipeBase@@PAUUFN_MDD_CONTEXT@@K@Z 1000f064 f   usb_ufnmddbase_common_topaz_v1:ufnmdd.obj
 0001:0000e1ec       ?UfnMdd_RegisterDevice@@YAKPAXPAU_USB_DEVICE_DESCRIPTOR@@PAU_UFN_CONFIGURATION@@12PBU_UFN_STRING_SET@@K@Z 1000f1ec f   usb_ufnmddbase_common_topaz_v1:ufnmdd.obj
 0001:0000eb80       ?UfnMdd_Start@@YAKPAXP6AH0KK@Z0PAPAX@Z 1000fb80 f   usb_ufnmddbase_common_topaz_v1:ufnmdd.obj
 0001:0000f160       ?DoStop@@YAKPAUUFN_MDD_CONTEXT@@@Z 10010160 f   usb_ufnmddbase_common_topaz_v1:ufnmdd.obj
 0001:0000f4bc       ?UfnMdd_Stop@@YAKPAX@Z     100104bc f   usb_ufnmddbase_common_topaz_v1:ufnmdd.obj
 0001:0000f6c0       ?DoDeregisterDevice@@YAKPAUUFN_MDD_CONTEXT@@@Z 100106c0 f   usb_ufnmddbase_common_topaz_v1:ufnmdd.obj
 0001:0000f928       ?UfnMdd_DeregisterDevice@@YAKPAX@Z 10010928 f   usb_ufnmddbase_common_topaz_v1:ufnmdd.obj
 0001:0000faf0       ?UfnMdd_OpenPipe@@YAKPAXKPAPAX@Z 10010af0 f   usb_ufnmddbase_common_topaz_v1:ufnmdd.obj
 0001:000100a8       ?UfnMdd_ClosePipe@@YAKPAX0@Z 100110a8 f   usb_ufnmddbase_common_topaz_v1:ufnmdd.obj
 0001:0001039c       ?UfnMdd_GetTransferStatus@@YAKPAX0PAK1@Z 1001139c f   usb_ufnmddbase_common_topaz_v1:ufnmdd.obj
 0001:000105dc       ?UfnMdd_AbortTransfer@@YAKPAX0@Z 100115dc f   usb_ufnmddbase_common_topaz_v1:ufnmdd.obj
 0001:00010828       ?UfnMdd_CloseTransfer@@YAKPAX0@Z 10011828 f   usb_ufnmddbase_common_topaz_v1:ufnmdd.obj
 0001:000109fc       ?UfnMdd_IssueTransfer@@YAKPAX0P6AK0@Z0KK0K0PAPAX@Z 100119fc f   usb_ufnmddbase_common_topaz_v1:ufnmdd.obj
 0001:00010d0c       ?UfnMdd_StallPipe@@YAKPAX0@Z 10011d0c f   usb_ufnmddbase_common_topaz_v1:ufnmdd.obj
 0001:00010f40       ?UfnMdd_ClearPipeStall@@YAKPAX0@Z 10011f40 f   usb_ufnmddbase_common_topaz_v1:ufnmdd.obj
 0001:00011174       ?UfnMdd_InitiateRemoteWakeup@@YAKPAX@Z 10012174 f   usb_ufnmddbase_common_topaz_v1:ufnmdd.obj
 0001:00011408       ?UfnMdd_SendControlStatusHandshake@@YAKPAX@Z 10012408 f   usb_ufnmddbase_common_topaz_v1:ufnmdd.obj
 0001:00011674       UFN_Init                   10012674 f   usb_ufnmddbase_common_topaz_v1:ufnmdd.obj
 0001:000123f0       UFN_PreDeinit              100133f0 f   usb_ufnmddbase_common_topaz_v1:ufnmdd.obj
 0001:000125b0       UFN_Deinit                 100135b0 f   usb_ufnmddbase_common_topaz_v1:ufnmdd.obj
 0001:00012778       UFN_Open                   10013778 f   usb_ufnmddbase_common_topaz_v1:ufnmdd.obj
 0001:00012ae0       UFN_PreClose               10013ae0 f   usb_ufnmddbase_common_topaz_v1:ufnmdd.obj
 0001:00012c70       UFN_Close                  10013c70 f   usb_ufnmddbase_common_topaz_v1:ufnmdd.obj
 0001:00012e84       UFN_PowerDown              10013e84 f   usb_ufnmddbase_common_topaz_v1:ufnmdd.obj
 0001:00012f5c       UFN_PowerUp                10013f5c f   usb_ufnmddbase_common_topaz_v1:ufnmdd.obj
 0001:00013034       ?GetClientFunctions@@YAKPAU_UFN_FUNCTIONS@@@Z 10014034 f   usb_ufnmddbase_common_topaz_v1:ufnmdd.obj
 0001:000131d4       UFN_IOControl              100141d4 f   usb_ufnmddbase_common_topaz_v1:ufnmdd.obj
 0001:00013484       ?SendDeviceNotification@@YAHP6AHPAXKK@Z0KK@Z 10014484 f   usb_ufnmddbase_common_topaz_v1:ufnmdd.obj
 0001:0001355c       DllEntry                   1001455c f   usb_ufnmddbase_common_topaz_v1:ufnmdd.obj
 0001:000136a0       ?IsClientActive@CUfnBus@@QAAHXZ 100146a0 f i usb_ufnmddbase_common_topaz_v1:ufnmdd.obj
 0001:00013710       ?GetDeviceHandle@DeviceFolder@@QAAPAXXZ 10014710 f i usb_ufnmddbase_common_topaz_v1:ufnmdd.obj
 0001:00013740       ?GetDeviceList@DefaultBusDriver@@QAAPAVDeviceFolder@@XZ 10014740 f i usb_ufnmddbase_common_topaz_v1:ufnmdd.obj
 0001:00013770       ??_GCDescriptors@@QAAPAXI@Z 10014770 f i usb_ufnmddbase_common_topaz_v1:ufnmdd.obj
 0001:000137b4       ?IsOpen@CPipeBase@@QBAHXZ  100147b4 f i usb_ufnmddbase_common_topaz_v1:ufnmdd.obj
 0001:000137e4       ?SetChildDevicePowerState@CUfnBus@@QAAHW4_CEDEVICE_POWER_STATE@@@Z 100147e4 f i usb_ufnmddbase_common_topaz_v1:ufnmdd.obj
 0001:00013850       ?GetPhysicalEndpoint@CPipeBase@@QBAKXZ 10014850 f i usb_ufnmddbase_common_topaz_v1:ufnmdd.obj
 0001:00013880       ?GetPipe@CUfnMddTransfer@@QAAPAVCPipeBase@@XZ 10014880 f i usb_ufnmddbase_common_topaz_v1:ufnmdd.obj
 0001:000138b0       ??0COpenList@@QAA@XZ       100148b0 f i usb_ufnmddbase_common_topaz_v1:ufnmdd.obj
 0001:000138f4       ??0critical_section@ce@@QAA@XZ 100148f4 f i usb_ufnmddbase_common_topaz_v1:ufnmdd.obj
 0001:00013924       ?Open@CReg@@QAAHPAUHKEY__@@PBGK@Z 10014924 f i usb_ufnmddbase_common_topaz_v1:ufnmdd.obj
 0001:00013994       ??0CReg@@QAA@XZ            10014994 f i usb_ufnmddbase_common_topaz_v1:ufnmdd.obj
 0001:000139c4       ?ZeroEntries@CReg@@AAAXXZ  100149c4 f i usb_ufnmddbase_common_topaz_v1:ufnmdd.obj
 0001:00013a14       ??1CReg@@QAA@XZ            10014a14 f i usb_ufnmddbase_common_topaz_v1:ufnmdd.obj
 0001:00013abc       ?Reset@CReg@@QAAXXZ        10014abc f i usb_ufnmddbase_common_topaz_v1:ufnmdd.obj
 0001:00013b08       ??_GCOpenList@@QAAPAXI@Z   10014b08 f i usb_ufnmddbase_common_topaz_v1:ufnmdd.obj
 0001:00013b4c       ??1COpenList@@QAA@XZ       10014b4c f i usb_ufnmddbase_common_topaz_v1:ufnmdd.obj
 0001:00013bec       ??1critical_section@ce@@QAA@XZ 10014bec f i usb_ufnmddbase_common_topaz_v1:ufnmdd.obj
 0001:00013c08       ?AddContext@COpenList@@QAA_NK@Z 10014c08 f i usb_ufnmddbase_common_topaz_v1:ufnmdd.obj
 0001:00013c84       ?RemoveContext@COpenList@@QAAXK@Z 10014c84 f i usb_ufnmddbase_common_topaz_v1:ufnmdd.obj
 0001:00013d9c       ?IsChildPowerManaged@CUfnBus@@QAAHXZ 10014d9c f i usb_ufnmddbase_common_topaz_v1:ufnmdd.obj
 0001:00013dcc       ?InitializeClass@?$CTransferQueue@VCUfnMddTransfer@@@@SAXK@Z 10014dcc f i usb_ufnmddbase_common_topaz_v1:ufnmdd.obj
 0001:00013e90       ??2@YAPAXIPAX@Z            10014e90 f i usb_ufnmddbase_common_topaz_v1:ufnmdd.obj
 0001:00013eb8       ?InitializeClassCalled@?$CTransferQueue@VCUfnMddTransfer@@@@SAHXZ 10014eb8 f i usb_ufnmddbase_common_topaz_v1:ufnmdd.obj
 0001:00013ef8       ?DeinitializeClass@?$CTransferQueue@VCUfnMddTransfer@@@@SAXXZ 10014ef8 f i usb_ufnmddbase_common_topaz_v1:ufnmdd.obj
 0001:00013f78       ??0?$list@KVallocator@ce@@@ce@@QAA@XZ 10014f78 f i usb_ufnmddbase_common_topaz_v1:ufnmdd.obj
 0001:00014054       ??1?$list@KVallocator@ce@@@ce@@QAA@XZ 10015054 f i usb_ufnmddbase_common_topaz_v1:ufnmdd.obj
 0001:00014070       ?begin@?$list@KVallocator@ce@@@ce@@QAA?AViterator@12@XZ 10015070 f i usb_ufnmddbase_common_topaz_v1:ufnmdd.obj
 0001:000140b0       ?end@?$list@KVallocator@ce@@@ce@@QAA?AViterator@12@XZ 100150b0 f i usb_ufnmddbase_common_topaz_v1:ufnmdd.obj
 0001:000140e8       ?size@?$list@KVallocator@ce@@@ce@@QBAIXZ 100150e8 f i usb_ufnmddbase_common_topaz_v1:ufnmdd.obj
 0001:00014118       ?remove@?$list@KVallocator@ce@@@ce@@QAAXABK@Z 10015118 f i usb_ufnmddbase_common_topaz_v1:ufnmdd.obj
 0001:000141cc       ??0?$gate@Vcritical_section@ce@@@ce@@QAA@AAVcritical_section@1@@Z 100151cc f i usb_ufnmddbase_common_topaz_v1:ufnmdd.obj
 0001:0001420c       ?lock@critical_section@ce@@QAAXXZ 1001520c f i usb_ufnmddbase_common_topaz_v1:ufnmdd.obj
 0001:00014228       ??1?$gate@Vcritical_section@ce@@@ce@@QAA@XZ 10015228 f i usb_ufnmddbase_common_topaz_v1:ufnmdd.obj
 0001:00014258       ?unlock@critical_section@ce@@QAAXXZ 10015258 f i usb_ufnmddbase_common_topaz_v1:ufnmdd.obj
 0001:00014274       ??9iterator@?$list@KVallocator@ce@@@ce@@QBA_NABV012@@Z 10015274 f i usb_ufnmddbase_common_topaz_v1:ufnmdd.obj
 0001:000142d0       ??_G?$fixed_block_allocator@$0BE@@ce@@QAAPAXI@Z 100152d0 f i usb_ufnmddbase_common_topaz_v1:ufnmdd.obj
 0001:00014314       ??0?$fixed_block_allocator@$0BE@@ce@@QAA@I@Z 10015314 f i usb_ufnmddbase_common_topaz_v1:ufnmdd.obj
 0001:00014348       ??1?$fixed_block_allocator@$0BE@@ce@@QAA@XZ 10015348 f i usb_ufnmddbase_common_topaz_v1:ufnmdd.obj
 0001:000143f0       ?clear@?$list@KVallocator@ce@@@ce@@QAAXXZ 100153f0 f i usb_ufnmddbase_common_topaz_v1:ufnmdd.obj
 0001:00014458       ?erase@?$list@KVallocator@ce@@@ce@@QAA?AViterator@12@V312@@Z 10015458 f i usb_ufnmddbase_common_topaz_v1:ufnmdd.obj
 0001:000145c0       ??0iterator@?$list@KVallocator@ce@@@ce@@QAA@PAU_Node@12@@Z 100155c0 f i usb_ufnmddbase_common_topaz_v1:ufnmdd.obj
 0001:000145f4       ??Diterator@?$list@KVallocator@ce@@@ce@@QBAAAKXZ 100155f4 f i usb_ufnmddbase_common_topaz_v1:ufnmdd.obj
 0001:00014620       ??Eiterator@?$list@KVallocator@ce@@@ce@@QAAAAV012@XZ 10015620 f i usb_ufnmddbase_common_topaz_v1:ufnmdd.obj
 0001:00014660       ??Eiterator@?$list@KVallocator@ce@@@ce@@QAA?AV012@H@Z 10015660 f i usb_ufnmddbase_common_topaz_v1:ufnmdd.obj
 0001:000146b0       ??8iterator@?$list@KVallocator@ce@@@ce@@QBA_NABV012@@Z 100156b0 f i usb_ufnmddbase_common_topaz_v1:ufnmdd.obj
 0001:00014708       ?_Initialize@?$fixed_block_allocator@$0BE@@ce@@IAAXI@Z 10015708 f i usb_ufnmddbase_common_topaz_v1:ufnmdd.obj
 0001:00014764       ?erase@?$list@KVallocator@ce@@@ce@@QAA?AViterator@12@V312@0@Z 10015764 f i usb_ufnmddbase_common_topaz_v1:ufnmdd.obj
 0001:000147ec       ?_Freenode@?$list@KVallocator@ce@@@ce@@IAAXPAU_Node@12@@Z 100157ec f i usb_ufnmddbase_common_topaz_v1:ufnmdd.obj
 0001:00014810       ?deallocate@allocator@ce@@QBAXPAXI@Z 10015810 f i usb_ufnmddbase_common_topaz_v1:ufnmdd.obj
 0001:0001482c       ??0const_iterator@?$list@KVallocator@ce@@@ce@@QAA@PAU_Node@12@@Z 1001582c f i usb_ufnmddbase_common_topaz_v1:ufnmdd.obj
 0001:00014860       ?_MyNode@const_iterator@?$list@KVallocator@ce@@@ce@@QBAPAU_Node@23@XZ 10015860 f i usb_ufnmddbase_common_topaz_v1:ufnmdd.obj
 0001:0001488c       ??$push_back@K@?$list@KVallocator@ce@@@ce@@QAA_NABK@Z 1001588c f i usb_ufnmddbase_common_topaz_v1:ufnmdd.obj
 0001:00014908       ??$find@Viterator@?$list@KVallocator@ce@@@ce@@K@std@@YA?AViterator@?$list@KVallocator@ce@@@ce@@V123@0ABK@Z 10015908 f i usb_ufnmddbase_common_topaz_v1:ufnmdd.obj
 0001:00014994       ??$PreDeinit@P6AHK@Z@COpenList@@QAAXP6AHK@Z@Z 10015994 f i usb_ufnmddbase_common_topaz_v1:ufnmdd.obj
 0001:00014a34       ??$Deinit@P6AHK@Z@COpenList@@QAAXP6AHK@Z@Z 10015a34 f i usb_ufnmddbase_common_topaz_v1:ufnmdd.obj
 0001:00014ac8       ?empty@?$list@KVallocator@ce@@@ce@@QBA_NXZ 10015ac8 f i usb_ufnmddbase_common_topaz_v1:ufnmdd.obj
 0001:00014b1c       ?front@?$list@KVallocator@ce@@@ce@@QAAAAKXZ 10015b1c f i usb_ufnmddbase_common_topaz_v1:ufnmdd.obj
 0001:00014b60       ??$insert@K@?$list@KVallocator@ce@@@ce@@QAA?AViterator@01@V201@ABK@Z 10015b60 f i usb_ufnmddbase_common_topaz_v1:ufnmdd.obj
 0001:00014c24       ??$for_each@Viterator@?$list@KVallocator@ce@@@ce@@P6AHK@Z@std@@YAP6AHK@ZViterator@?$list@KVallocator@ce@@@ce@@0P6AHK@Z@Z 10015c24 f i usb_ufnmddbase_common_topaz_v1:ufnmdd.obj
 0001:00014c98       ?_Buynode@?$list@KVallocator@ce@@@ce@@IAAPAU_Node@12@PAU312@@Z 10015c98 f i usb_ufnmddbase_common_topaz_v1:ufnmdd.obj
 0001:00014da0       ?allocate@allocator@ce@@QBAPAXI@Z 10015da0 f i usb_ufnmddbase_common_topaz_v1:ufnmdd.obj
 0001:00014dd4       ??0lock_factory@?$singleton@V?$free_list@$0GE@Vallocator@ce@@@ce@@$03V?$static_allocator@V?$free_list@$0GE@Vallocator@ce@@@ce@@$03@2@@ce@@QAA@XZ 10015dd4 f i usb_ufnmddbase_common_topaz_v1:ufnmdd.obj
 0001:00014e00       ?get_lock@?$singleton@V?$free_list@$0GE@Vallocator@ce@@@ce@@$03V?$static_allocator@V?$free_list@$0GE@Vallocator@ce@@@ce@@$03@2@@ce@@KAAAVcritical_section@2@XZ 10015e00 f i usb_ufnmddbase_common_topaz_v1:ufnmdd.obj
 0001:00014e6c       ??0CPipeBase@@QAA@KPAU_UFN_PDD_INTERFACE_INFO@@PAVCFreeTransferList@@PAUUFN_MDD_CONTEXT@@@Z 10015e6c f   usb_ufnmddbase_common_topaz_v1:pipe.obj
 0001:00014fc0       ??1CPipeBase@@UAA@XZ       10015fc0 f   usb_ufnmddbase_common_topaz_v1:pipe.obj
 0001:00015094       ??0CStaticPipe@@QAA@KPAU_UFN_PDD_INTERFACE_INFO@@PAVCFreeTransferList@@PAUUFN_MDD_CONTEXT@@@Z 10016094 f   usb_ufnmddbase_common_topaz_v1:pipe.obj
 0001:000150f4       ??1CStaticPipe@@UAA@XZ     100160f4 f   usb_ufnmddbase_common_topaz_v1:pipe.obj
 0001:00015120       ??0CDynamicPipe@@QAA@KPAU_UFN_PDD_INTERFACE_INFO@@PAVCFreeTransferList@@PAUUFN_MDD_CONTEXT@@@Z 10016120 f   usb_ufnmddbase_common_topaz_v1:pipe.obj
 0001:000151e4       ??1CDynamicPipe@@UAA@XZ    100161e4 f   usb_ufnmddbase_common_topaz_v1:pipe.obj
 0001:0001524c       ?OwningInterface@CStaticPipe@@UBAKW4_UFN_BUS_SPEED@@K@Z 1001624c f   usb_ufnmddbase_common_topaz_v1:pipe.obj
 0001:00015334       ?IsPartOfInterface@CStaticPipe@@UBAHW4_UFN_BUS_SPEED@@KK@Z 10016334 f   usb_ufnmddbase_common_topaz_v1:pipe.obj
 0001:000153e4       ?OwningInterface@CDynamicPipe@@UBAKW4_UFN_BUS_SPEED@@K@Z 100163e4 f   usb_ufnmddbase_common_topaz_v1:pipe.obj
 0001:00015560       ?IsPartOfInterface@CDynamicPipe@@UBAHW4_UFN_BUS_SPEED@@KK@Z 10016560 f   usb_ufnmddbase_common_topaz_v1:pipe.obj
 0001:000156c0       ?GetEndpointDescriptor@CStaticPipe@@UBAPAU_USB_ENDPOINT_DESCRIPTOR@@W4_UFN_BUS_SPEED@@@Z 100166c0 f   usb_ufnmddbase_common_topaz_v1:pipe.obj
 0001:00015714       ?Reset@CStaticPipe@@UAAXXZ 10016714 f   usb_ufnmddbase_common_topaz_v1:pipe.obj
 0001:000158b0       ?IsReserved@CStaticPipe@@UBAHW4_UFN_BUS_SPEED@@KKK@Z 100168b0 f   usb_ufnmddbase_common_topaz_v1:pipe.obj
 0001:00015904       ?Reserve@CStaticPipe@@UAAXW4_UFN_BUS_SPEED@@HKKKPAU_USB_ENDPOINT_DESCRIPTOR@@@Z 10016904 f   usb_ufnmddbase_common_topaz_v1:pipe.obj
 0001:00015a6c       ?Reset@CDynamicPipe@@UAAXXZ 10016a6c f   usb_ufnmddbase_common_topaz_v1:pipe.obj
 0001:00015bbc       ?IsReserved@CDynamicPipe@@UBAHW4_UFN_BUS_SPEED@@KKK@Z 10016bbc f   usb_ufnmddbase_common_topaz_v1:pipe.obj
 0001:00015e0c       ?Reserve@CDynamicPipe@@UAAXW4_UFN_BUS_SPEED@@HKKKPAU_USB_ENDPOINT_DESCRIPTOR@@@Z 10016e0c f   usb_ufnmddbase_common_topaz_v1:pipe.obj
 0001:00016480       ?GetEndpointDescriptor@CDynamicPipe@@UBAPAU_USB_ENDPOINT_DESCRIPTOR@@W4_UFN_BUS_SPEED@@@Z 10017480 f   usb_ufnmddbase_common_topaz_v1:pipe.obj
 0001:000167a4       ?GetEndpointAddress@CPipeBase@@QBAKXZ 100177a4 f   usb_ufnmddbase_common_topaz_v1:pipe.obj
 0001:00016850       ?IsReserved@CPipeBase@@UBAHW4_UFN_BUS_SPEED@@@Z 10017850 f   usb_ufnmddbase_common_topaz_v1:pipe.obj
 0001:00016994       ?Open@CPipeBase@@QAAKW4_UFN_BUS_SPEED@@PAU_USB_ENDPOINT_DESCRIPTOR@@@Z 10017994 f   usb_ufnmddbase_common_topaz_v1:pipe.obj
 0001:00017030       ?Close@CPipeBase@@QAAKXZ   10018030 f   usb_ufnmddbase_common_topaz_v1:pipe.obj
 0001:000172f8       ?AbortAllTransfers@CPipeBase@@QAAXXZ 100182f8 f   usb_ufnmddbase_common_topaz_v1:pipe.obj
 0001:00017460       ?IssueTransfer@CPipeBase@@QAAKP6AKPAX@Z0KK0KPAPAVCUfnMddTransfer@@0@Z 10018460 f   usb_ufnmddbase_common_topaz_v1:pipe.obj
 0001:00017bdc       ?AbortTransfer@CPipeBase@@QAAKPAVCUfnMddTransfer@@@Z 10018bdc f   usb_ufnmddbase_common_topaz_v1:pipe.obj
 0001:00017e7c       ?GetTransferStatus@CPipeBase@@SAKPBVCUfnMddTransfer@@PAK1@Z 10018e7c f   usb_ufnmddbase_common_topaz_v1:pipe.obj
 0001:00018018       ?CloseTransfer@CPipeBase@@QAAKPAVCUfnMddTransfer@@@Z 10019018 f   usb_ufnmddbase_common_topaz_v1:pipe.obj
 0001:00018178       ?FreeTransfer@CPipeBase@@QAAXPAVCUfnMddTransfer@@@Z 10019178 f   usb_ufnmddbase_common_topaz_v1:pipe.obj
 0001:00018258       ?TransferComplete@CPipeBase@@QAAKPAVCUfnMddTransfer@@H@Z 10019258 f   usb_ufnmddbase_common_topaz_v1:pipe.obj
 0001:00018640       ?Stall@CPipeBase@@QAAKXZ   10019640 f   usb_ufnmddbase_common_topaz_v1:pipe.obj
 0001:000187c8       ?ClearStall@CPipeBase@@QAAKXZ 100197c8 f   usb_ufnmddbase_common_topaz_v1:pipe.obj
 0001:00018950       ?SendControlStatusHandshake@CPipeBase@@QAAKXZ 10019950 f   usb_ufnmddbase_common_topaz_v1:pipe.obj
 0001:00018af0       ?ValidatePipeHandle@CPipeBase@@SAKPBV1@@Z 10019af0 f   usb_ufnmddbase_common_topaz_v1:pipe.obj
 0001:00018cd0       ?Validate@CPipeBase@@QAAXXZ 10019cd0 f   usb_ufnmddbase_common_topaz_v1:pipe.obj
 0001:00018e60       ??_GCPipeBase@@UAAPAXI@Z   10019e60 f i usb_ufnmddbase_common_topaz_v1:pipe.obj
 0001:00018e60       ??_ECPipeBase@@UAAPAXI@Z   10019e60 f i usb_ufnmddbase_common_topaz_v1:pipe.obj
 0001:00018ea4       ??_GCStaticPipe@@UAAPAXI@Z 10019ea4 f i usb_ufnmddbase_common_topaz_v1:pipe.obj
 0001:00018ea4       ??_ECStaticPipe@@UAAPAXI@Z 10019ea4 f i usb_ufnmddbase_common_topaz_v1:pipe.obj
 0001:00018ee8       ??_ECDynamicPipe@@UAAPAXI@Z 10019ee8 f i usb_ufnmddbase_common_topaz_v1:pipe.obj
 0001:00018ee8       ??_GCDynamicPipe@@UAAPAXI@Z 10019ee8 f i usb_ufnmddbase_common_topaz_v1:pipe.obj
 0001:00018f2c       ??1?$hash_map@KKU?$hash_traits@K@ce@@Vallocator@2@@ce@@QAA@XZ 10019f2c f i usb_ufnmddbase_common_topaz_v1:pipe.obj
 0001:00018f48       ??1?$hash_map@KPAU_USB_ENDPOINT_DESCRIPTOR@@U?$hash_traits@K@ce@@Vallocator@3@@ce@@QAA@XZ 10019f48 f i usb_ufnmddbase_common_topaz_v1:pipe.obj
 0001:00018f64       ??1?$hash@V?$hash_map_traits@KKU?$hash_traits@K@ce@@Vallocator@2@@details@ce@@@details@ce@@QAA@XZ 10019f64 f i usb_ufnmddbase_common_topaz_v1:pipe.obj
 0001:00018f8c       ??1?$hash@V?$hash_map_traits@KPAU_USB_ENDPOINT_DESCRIPTOR@@U?$hash_traits@K@ce@@Vallocator@3@@details@ce@@@details@ce@@QAA@XZ 10019f8c f i usb_ufnmddbase_common_topaz_v1:pipe.obj
 0001:00018fb4       ?Lock@CPipeBase@@IAAXXZ    10019fb4 f i usb_ufnmddbase_common_topaz_v1:pipe.obj
 0001:00019024       GetCurrentThreadId         1001a024 f i usb_ufnmddbase_common_topaz_v1:pipe.obj
 0001:00019050       ?Unlock@CPipeBase@@IAAXXZ  1001a050 f i usb_ufnmddbase_common_topaz_v1:pipe.obj
 0001:000190b0       ?GetConfiguration@CDescriptors@@QAAKW4_UFN_BUS_SPEED@@@Z 1001a0b0 f i usb_ufnmddbase_common_topaz_v1:pipe.obj
 0001:000190fc       ?GetConfiguration@CDevice@@QBAKXZ 1001a0fc f i usb_ufnmddbase_common_topaz_v1:pipe.obj
 0001:00019198       ?GetConfigurationClass@CDevice@@QBAPAVCConfiguration@@K@Z 1001a198 f i usb_ufnmddbase_common_topaz_v1:pipe.obj
 0001:00019248       ?GetConfigurationValue@CConfiguration@@QBAKXZ 1001a248 f i usb_ufnmddbase_common_topaz_v1:pipe.obj
 0001:0001927c       ?GetConfigurationCount@CDevice@@QBAKXZ 1001a27c f i usb_ufnmddbase_common_topaz_v1:pipe.obj
 0001:000192b0       ?GetInterface@CDescriptors@@QAAKW4_UFN_BUS_SPEED@@KPAK@Z 1001a2b0 f i usb_ufnmddbase_common_topaz_v1:pipe.obj
 0001:00019304       ?GetInterface@CDevice@@QAAKKPAK@Z 1001a304 f i usb_ufnmddbase_common_topaz_v1:pipe.obj
 0001:000193e8       ?GetInterface@CConfiguration@@QAAKKPAK@Z 1001a3e8 f i usb_ufnmddbase_common_topaz_v1:pipe.obj
 0001:00019468       ?GetInterface@CInterface@@QBAKXZ 1001a468 f i usb_ufnmddbase_common_topaz_v1:pipe.obj
 0001:000194e8       ?GetInterfaceClass@CConfiguration@@QAAPAVCInterface@@KK@Z 1001a4e8 f i usb_ufnmddbase_common_topaz_v1:pipe.obj
 0001:000195b0       ?GetInterfaceNumber@CInterface@@QBAKXZ 1001a5b0 f i usb_ufnmddbase_common_topaz_v1:pipe.obj
 0001:000195e4       ?GetAlternateSetting@CInterface@@QBAKXZ 1001a5e4 f i usb_ufnmddbase_common_topaz_v1:pipe.obj
 0001:00019618       ?GetInterfaceCount@CConfiguration@@QBAKXZ 1001a618 f i usb_ufnmddbase_common_topaz_v1:pipe.obj
 0001:0001964c       ?GetDevice@CDescriptors@@AAAPAVCDevice@@W4_UFN_BUS_SPEED@@@Z 1001a64c f i usb_ufnmddbase_common_topaz_v1:pipe.obj
 0001:000196f0       ?IsComplete@CUfnMddTransfer@@QAAHXZ 1001a6f0 f i usb_ufnmddbase_common_topaz_v1:pipe.obj
 0001:0001974c       ?GetDwUsbError@CUfnMddTransfer@@QBAKXZ 1001a74c f i usb_ufnmddbase_common_topaz_v1:pipe.obj
 0001:0001977c       ?Validate@CUfnMddTransfer@@QAAXXZ 1001a77c f i usb_ufnmddbase_common_topaz_v1:pipe.obj
 0001:00019884       ?GetCbBuffer@CUfnMddTransfer@@QBAKXZ 1001a884 f i usb_ufnmddbase_common_topaz_v1:pipe.obj
 0001:000198b4       ?GetPvBuffer@CUfnMddTransfer@@QBAPAXXZ 1001a8b4 f i usb_ufnmddbase_common_topaz_v1:pipe.obj
 0001:000198e4       ?EnteringPdd@CUfnMddTransfer@@QAAXXZ 1001a8e4 f i usb_ufnmddbase_common_topaz_v1:pipe.obj
 0001:00019964       ?LeavingPdd@CUfnMddTransfer@@QAAXXZ 1001a964 f i usb_ufnmddbase_common_topaz_v1:pipe.obj
 0001:000199e4       ?GetDwFlags@CUfnMddTransfer@@QBAKXZ 1001a9e4 f i usb_ufnmddbase_common_topaz_v1:pipe.obj
 0001:00019a14       ?GetPddTransfer@CUfnMddTransfer@@QAAPAU_STransfer@@XZ 1001aa14 f i usb_ufnmddbase_common_topaz_v1:pipe.obj
 0001:00019a40       ?AllocTransfer@CFreeTransferList@@QAAPAVCUfnMddTransfer@@XZ 1001aa40 f i usb_ufnmddbase_common_topaz_v1:pipe.obj
 0001:00019a78       ?IsInPdd@CUfnMddTransfer@@QAAHXZ 1001aa78 f i usb_ufnmddbase_common_topaz_v1:pipe.obj
 0001:00019aa8       ?SetDwUsbError@CUfnMddTransfer@@QAAXK@Z 1001aaa8 f i usb_ufnmddbase_common_topaz_v1:pipe.obj
 0001:00019b24       ?GetCbTransferred@CUfnMddTransfer@@QBAKXZ 1001ab24 f i usb_ufnmddbase_common_topaz_v1:pipe.obj
 0001:00019b54       ?FreeTransfer@CFreeTransferList@@QAAXPAVCUfnMddTransfer@@@Z 1001ab54 f i usb_ufnmddbase_common_topaz_v1:pipe.obj
 0001:00019b94       ?allocate@?$CFreePool@$00V?$fixed_block_allocator@$07@ce@@Utransfer_funcs@@@@QAAPAXI@Z 1001ab94 f i usb_ufnmddbase_common_topaz_v1:pipe.obj
 0001:00019db4       ?create@transfer_funcs@@SAXPAX@Z 1001adb4 f i usb_ufnmddbase_common_topaz_v1:pipe.obj
 0001:00019e64       ??0CUfnMddTransfer@@QAA@XZ 1001ae64 f i usb_ufnmddbase_common_topaz_v1:pipe.obj
 0001:00019eb4       ?ClearMembers@CUfnMddTransfer@@AAAXXZ 1001aeb4 f i usb_ufnmddbase_common_topaz_v1:pipe.obj
 0001:00019edc       ?reuse@transfer_funcs@@SAXPAX@Z 1001aedc f i usb_ufnmddbase_common_topaz_v1:pipe.obj
 0001:00019f4c       ?MarkAsValid@CUfnMddTransfer@@QAAXXZ 1001af4c f i usb_ufnmddbase_common_topaz_v1:pipe.obj
 0001:00019fd8       ?deallocate@?$CFreePool@$00V?$fixed_block_allocator@$07@ce@@Utransfer_funcs@@@@QAAXPAXI@Z 1001afd8 f i usb_ufnmddbase_common_topaz_v1:pipe.obj
 0001:0001a108       ?free@transfer_funcs@@SAXPAX@Z 1001b108 f i usb_ufnmddbase_common_topaz_v1:pipe.obj
 0001:0001a17c       ?MarkAsFree@CUfnMddTransfer@@QAAXXZ 1001b17c f i usb_ufnmddbase_common_topaz_v1:pipe.obj
 0001:0001a280       ??0?$CTransferQueue@VCUfnMddTransfer@@@@QAA@XZ 1001b280 f i usb_ufnmddbase_common_topaz_v1:pipe.obj
 0001:0001a2c0       ??1?$CTransferQueue@VCUfnMddTransfer@@@@QAA@XZ 1001b2c0 f i usb_ufnmddbase_common_topaz_v1:pipe.obj
 0001:0001a334       ?IsEmpty@?$CTransferQueue@VCUfnMddTransfer@@@@QBAHXZ 1001b334 f i usb_ufnmddbase_common_topaz_v1:pipe.obj
 0001:0001a370       ?Front@?$CTransferQueue@VCUfnMddTransfer@@@@QBAPAVCUfnMddTransfer@@XZ 1001b370 f i usb_ufnmddbase_common_topaz_v1:pipe.obj
 0001:0001a3f8       ?Back@?$CTransferQueue@VCUfnMddTransfer@@@@QBAPAVCUfnMddTransfer@@XZ 1001b3f8 f i usb_ufnmddbase_common_topaz_v1:pipe.obj
 0001:0001a480       ?PushBack@?$CTransferQueue@VCUfnMddTransfer@@@@QAAKPAVCUfnMddTransfer@@@Z 1001b480 f i usb_ufnmddbase_common_topaz_v1:pipe.obj
 0001:0001a4d4       ?PopFront@?$CTransferQueue@VCUfnMddTransfer@@@@QAAXXZ 1001b4d4 f i usb_ufnmddbase_common_topaz_v1:pipe.obj
 0001:0001a548       ?PopBack@?$CTransferQueue@VCUfnMddTransfer@@@@QAAXXZ 1001b548 f i usb_ufnmddbase_common_topaz_v1:pipe.obj
 0001:0001a5bc       ??0?$hash_map@KKU?$hash_traits@K@ce@@Vallocator@2@@ce@@QAA@I@Z 1001b5bc f i usb_ufnmddbase_common_topaz_v1:pipe.obj
 0001:0001a5f4       ?insert@?$hash_map@KKU?$hash_traits@K@ce@@Vallocator@2@@ce@@QAA?AViterator@?$list@U?$pair@KK@std@@Vallocator@ce@@@2@ABU?$pair@KK@std@@@Z 1001b5f4 f i usb_ufnmddbase_common_topaz_v1:pipe.obj
 0001:0001a62c       ?end@?$hash@V?$hash_map_traits@KKU?$hash_traits@K@ce@@Vallocator@2@@details@ce@@@details@ce@@QAA?AViterator@?$list@U?$pair@KK@std@@Vallocator@ce@@@3@XZ 1001b62c f i usb_ufnmddbase_common_topaz_v1:pipe.obj
 0001:0001a660       ?end@?$hash@V?$hash_map_traits@KKU?$hash_traits@K@ce@@Vallocator@2@@details@ce@@@details@ce@@QBA?AVconst_iterator@?$list@U?$pair@KK@std@@Vallocator@ce@@@3@XZ 1001b660 f i usb_ufnmddbase_common_topaz_v1:pipe.obj
 0001:0001a694       ?erase@?$hash@V?$hash_map_traits@KKU?$hash_traits@K@ce@@Vallocator@2@@details@ce@@@details@ce@@QAA?AViterator@?$list@U?$pair@KK@std@@Vallocator@ce@@@3@V453@@Z 1001b694 f i usb_ufnmddbase_common_topaz_v1:pipe.obj
 0001:0001a858       ?clear@?$hash@V?$hash_map_traits@KKU?$hash_traits@K@ce@@Vallocator@2@@details@ce@@@details@ce@@QAAXXZ 1001b858 f i usb_ufnmddbase_common_topaz_v1:pipe.obj
 0001:0001a960       ?find@?$hash@V?$hash_map_traits@KKU?$hash_traits@K@ce@@Vallocator@2@@details@ce@@@details@ce@@QAA?AViterator@?$list@U?$pair@KK@std@@Vallocator@ce@@@3@ABK@Z 1001b960 f i usb_ufnmddbase_common_topaz_v1:pipe.obj
 0001:0001aab4       ?find@?$hash@V?$hash_map_traits@KKU?$hash_traits@K@ce@@Vallocator@2@@details@ce@@@details@ce@@QBA?AVconst_iterator@?$list@U?$pair@KK@std@@Vallocator@ce@@@3@ABK@Z 1001bab4 f i usb_ufnmddbase_common_topaz_v1:pipe.obj
 0001:0001ac08       ??1?$list@U?$pair@KK@std@@Vallocator@ce@@@ce@@QAA@XZ 1001bc08 f i usb_ufnmddbase_common_topaz_v1:pipe.obj
 0001:0001ac24       ??1?$vector@U?$pair@Viterator@?$list@U?$pair@KK@std@@Vallocator@ce@@@ce@@I@std@@Vallocator@ce@@U?$incremental_growth@$09@4@@ce@@QAA@XZ 1001bc24 f i usb_ufnmddbase_common_topaz_v1:pipe.obj
 0001:0001ac70       ??0?$hash_map@KPAU_USB_ENDPOINT_DESCRIPTOR@@U?$hash_traits@K@ce@@Vallocator@3@@ce@@QAA@I@Z 1001bc70 f i usb_ufnmddbase_common_topaz_v1:pipe.obj
 0001:0001aca8       ?insert@?$hash_map@KPAU_USB_ENDPOINT_DESCRIPTOR@@U?$hash_traits@K@ce@@Vallocator@3@@ce@@QAA?AViterator@?$list@U?$pair@KPAU_USB_ENDPOINT_DESCRIPTOR@@@std@@Vallocator@ce@@@2@ABU?$pair@KPAU_USB_ENDPOINT_DESCRIPTOR@@@std@@@Z 1001bca8 f i usb_ufnmddbase_common_topaz_v1:pipe.obj
 0001:0001ace0       ?end@?$hash@V?$hash_map_traits@KPAU_USB_ENDPOINT_DESCRIPTOR@@U?$hash_traits@K@ce@@Vallocator@3@@details@ce@@@details@ce@@QAA?AViterator@?$list@U?$pair@KPAU_USB_ENDPOINT_DESCRIPTOR@@@std@@Vallocator@ce@@@3@XZ 1001bce0 f i usb_ufnmddbase_common_topaz_v1:pipe.obj
 0001:0001ad14       ?end@?$hash@V?$hash_map_traits@KPAU_USB_ENDPOINT_DESCRIPTOR@@U?$hash_traits@K@ce@@Vallocator@3@@details@ce@@@details@ce@@QBA?AVconst_iterator@?$list@U?$pair@KPAU_USB_ENDPOINT_DESCRIPTOR@@@std@@Vallocator@ce@@@3@XZ 1001bd14 f i usb_ufnmddbase_common_topaz_v1:pipe.obj
 0001:0001ad48       ?erase@?$hash@V?$hash_map_traits@KPAU_USB_ENDPOINT_DESCRIPTOR@@U?$hash_traits@K@ce@@Vallocator@3@@details@ce@@@details@ce@@QAA?AViterator@?$list@U?$pair@KPAU_USB_ENDPOINT_DESCRIPTOR@@@std@@Vallocator@ce@@@3@V453@@Z 1001bd48 f i usb_ufnmddbase_common_topaz_v1:pipe.obj
 0001:0001af0c       ?clear@?$hash@V?$hash_map_traits@KPAU_USB_ENDPOINT_DESCRIPTOR@@U?$hash_traits@K@ce@@Vallocator@3@@details@ce@@@details@ce@@QAAXXZ 1001bf0c f i usb_ufnmddbase_common_topaz_v1:pipe.obj
 0001:0001b014       ?find@?$hash@V?$hash_map_traits@KPAU_USB_ENDPOINT_DESCRIPTOR@@U?$hash_traits@K@ce@@Vallocator@3@@details@ce@@@details@ce@@QAA?AViterator@?$list@U?$pair@KPAU_USB_ENDPOINT_DESCRIPTOR@@@std@@Vallocator@ce@@@3@ABK@Z 1001c014 f i usb_ufnmddbase_common_topaz_v1:pipe.obj
 0001:0001b168       ?find@?$hash@V?$hash_map_traits@KPAU_USB_ENDPOINT_DESCRIPTOR@@U?$hash_traits@K@ce@@Vallocator@3@@details@ce@@@details@ce@@QBA?AVconst_iterator@?$list@U?$pair@KPAU_USB_ENDPOINT_DESCRIPTOR@@@std@@Vallocator@ce@@@3@ABK@Z 1001c168 f i usb_ufnmddbase_common_topaz_v1:pipe.obj
 0001:0001b2bc       ??1?$list@U?$pair@KPAU_USB_ENDPOINT_DESCRIPTOR@@@std@@Vallocator@ce@@@ce@@QAA@XZ 1001c2bc f i usb_ufnmddbase_common_topaz_v1:pipe.obj
 0001:0001b2d8       ??1?$vector@U?$pair@Viterator@?$list@U?$pair@KPAU_USB_ENDPOINT_DESCRIPTOR@@@std@@Vallocator@ce@@@ce@@I@std@@Vallocator@ce@@U?$incremental_growth@$09@4@@ce@@QAA@XZ 1001c2d8 f i usb_ufnmddbase_common_topaz_v1:pipe.obj
 0001:0001b324       ??0const_iterator@?$list@U?$pair@KK@std@@Vallocator@ce@@@ce@@QAA@XZ 1001c324 f i usb_ufnmddbase_common_topaz_v1:pipe.obj
 0001:0001b34c       ??Cconst_iterator@?$list@U?$pair@KK@std@@Vallocator@ce@@@ce@@QBAPBU?$pair@KK@std@@XZ 1001c34c f i usb_ufnmddbase_common_topaz_v1:pipe.obj
 0001:0001b380       ??8const_iterator@?$list@U?$pair@KK@std@@Vallocator@ce@@@ce@@QBA_NABV012@@Z 1001c380 f i usb_ufnmddbase_common_topaz_v1:pipe.obj
 0001:0001b3d8       ??9const_iterator@?$list@U?$pair@KK@std@@Vallocator@ce@@@ce@@QBA_NABV012@@Z 1001c3d8 f i usb_ufnmddbase_common_topaz_v1:pipe.obj
 0001:0001b434       ??0?$pair@KK@std@@QAA@ABK0@Z 1001c434 f i usb_ufnmddbase_common_topaz_v1:pipe.obj
 0001:0001b480       ??0iterator@?$list@U?$pair@KPAU_USB_ENDPOINT_DESCRIPTOR@@@std@@Vallocator@ce@@@ce@@QAA@XZ 1001c480 f i usb_ufnmddbase_common_topaz_v1:pipe.obj
 0001:0001b4b0       ??9iterator@?$list@U?$pair@KPAU_USB_ENDPOINT_DESCRIPTOR@@@std@@Vallocator@ce@@@ce@@QBA_NABV012@@Z 1001c4b0 f i usb_ufnmddbase_common_topaz_v1:pipe.obj
 0001:0001b50c       ??0const_iterator@?$list@U?$pair@KPAU_USB_ENDPOINT_DESCRIPTOR@@@std@@Vallocator@ce@@@ce@@QAA@XZ 1001c50c f i usb_ufnmddbase_common_topaz_v1:pipe.obj
 0001:0001b534       ??Cconst_iterator@?$list@U?$pair@KPAU_USB_ENDPOINT_DESCRIPTOR@@@std@@Vallocator@ce@@@ce@@QBAPBU?$pair@KPAU_USB_ENDPOINT_DESCRIPTOR@@@std@@XZ 1001c534 f i usb_ufnmddbase_common_topaz_v1:pipe.obj
 0001:0001b568       ??9const_iterator@?$list@U?$pair@KPAU_USB_ENDPOINT_DESCRIPTOR@@@std@@Vallocator@ce@@@ce@@QBA_NABV012@@Z 1001c568 f i usb_ufnmddbase_common_topaz_v1:pipe.obj
 0001:0001b5c4       ??0iterator@?$list@U?$pair@KK@std@@Vallocator@ce@@@ce@@QAA@XZ 1001c5c4 f i usb_ufnmddbase_common_topaz_v1:pipe.obj
 0001:0001b5f4       ??Citerator@?$list@U?$pair@KK@std@@Vallocator@ce@@@ce@@QBAPAU?$pair@KK@std@@XZ 1001c5f4 f i usb_ufnmddbase_common_topaz_v1:pipe.obj
 0001:0001b628       ??8iterator@?$list@U?$pair@KK@std@@Vallocator@ce@@@ce@@QBA_NABV012@@Z 1001c628 f i usb_ufnmddbase_common_topaz_v1:pipe.obj
 0001:0001b680       ??9iterator@?$list@U?$pair@KK@std@@Vallocator@ce@@@ce@@QBA_NABV012@@Z 1001c680 f i usb_ufnmddbase_common_topaz_v1:pipe.obj
 0001:0001b6dc       ??0?$pair@KPAU_USB_ENDPOINT_DESCRIPTOR@@@std@@QAA@ABKABQAU_USB_ENDPOINT_DESCRIPTOR@@@Z 1001c6dc f i usb_ufnmddbase_common_topaz_v1:pipe.obj
 0001:0001b728       ?DeleteElement@?$CFreePool@$00V?$fixed_block_allocator@$07@ce@@Utransfer_funcs@@@@IAAXPAX@Z 1001c728 f i usb_ufnmddbase_common_topaz_v1:pipe.obj
 0001:0001b784       ?destroy@transfer_funcs@@SAXPAX@Z 1001c784 f i usb_ufnmddbase_common_topaz_v1:pipe.obj
 0001:0001b7fc       ??_GCUfnMddTransfer@@QAAPAXI@Z 1001c7fc f i usb_ufnmddbase_common_topaz_v1:pipe.obj
 0001:0001b840       ??1CUfnMddTransfer@@QAA@XZ 1001c840 f i usb_ufnmddbase_common_topaz_v1:pipe.obj
 0001:0001b8d4       ?PopulateCache@?$CFreePool@$00V?$fixed_block_allocator@$07@ce@@Utransfer_funcs@@@@IAAXXZ 1001c8d4 f i usb_ufnmddbase_common_topaz_v1:pipe.obj
 0001:0001ba48       ?allocate@?$fixed_block_allocator@$07@ce@@QBAPAXI@Z 1001ca48 f i usb_ufnmddbase_common_topaz_v1:pipe.obj
 0001:0001bb70       ?push@?$interlocked_stack@PAXV?$fixed_block_allocator@$07@ce@@@@QAA_NABQAX@Z 1001cb70 f i usb_ufnmddbase_common_topaz_v1:pipe.obj
 0001:0001bc04       ?InterlockedPushEntrySingleList@@YAPAU_SINGLE_LIST_ENTRY@@PAU1@0@Z 1001cc04 f i usb_ufnmddbase_common_topaz_v1:pipe.obj
 0001:0001bc78       ?pop@?$interlocked_stack@PAXV?$fixed_block_allocator@$07@ce@@@@QAA_NAAPAX@Z 1001cc78 f i usb_ufnmddbase_common_topaz_v1:pipe.obj
 0001:0001bd0c       ?InterlockedPopEntrySingleList@@YAPAU_SINGLE_LIST_ENTRY@@PAU1@@Z 1001cd0c f i usb_ufnmddbase_common_topaz_v1:pipe.obj
 0001:0001bd90       ??0?$list@PAVCUfnMddTransfer@@V?$fixed_block_allocator@$0BE@@ce@@@ce@@QAA@ABV?$fixed_block_allocator@$0BE@@1@@Z 1001cd90 f i usb_ufnmddbase_common_topaz_v1:pipe.obj
 0001:0001be98       ??1?$list@PAVCUfnMddTransfer@@V?$fixed_block_allocator@$0BE@@ce@@@ce@@QAA@XZ 1001ce98 f i usb_ufnmddbase_common_topaz_v1:pipe.obj
 0001:0001bebc       ?empty@?$list@PAVCUfnMddTransfer@@V?$fixed_block_allocator@$0BE@@ce@@@ce@@QBA_NXZ 1001cebc f i usb_ufnmddbase_common_topaz_v1:pipe.obj
 0001:0001bf10       ?pop_back@?$list@PAVCUfnMddTransfer@@V?$fixed_block_allocator@$0BE@@ce@@@ce@@QAAXXZ 1001cf10 f i usb_ufnmddbase_common_topaz_v1:pipe.obj
 0001:0001bf64       ?pop_front@?$list@PAVCUfnMddTransfer@@V?$fixed_block_allocator@$0BE@@ce@@@ce@@QAAXXZ 1001cf64 f i usb_ufnmddbase_common_topaz_v1:pipe.obj
 0001:0001bfac       ?front@?$list@PAVCUfnMddTransfer@@V?$fixed_block_allocator@$0BE@@ce@@@ce@@QBAABQAVCUfnMddTransfer@@XZ 1001cfac f i usb_ufnmddbase_common_topaz_v1:pipe.obj
 0001:0001bff0       ?back@?$list@PAVCUfnMddTransfer@@V?$fixed_block_allocator@$0BE@@ce@@@ce@@QBAABQAVCUfnMddTransfer@@XZ 1001cff0 f i usb_ufnmddbase_common_topaz_v1:pipe.obj
 0001:0001c040       ??0?$hash@V?$hash_map_traits@KKU?$hash_traits@K@ce@@Vallocator@2@@details@ce@@@details@ce@@QAA@I@Z 1001d040 f i usb_ufnmddbase_common_topaz_v1:pipe.obj
 0001:0001c0ac       ?insert@?$hash@V?$hash_map_traits@KKU?$hash_traits@K@ce@@Vallocator@2@@details@ce@@@details@ce@@QAA?AViterator@?$list@U?$pair@KK@std@@Vallocator@ce@@@3@ABU?$pair@KK@std@@@Z 1001d0ac f i usb_ufnmddbase_common_topaz_v1:pipe.obj
 0001:0001c2fc       ?_get_bucket@?$hash@V?$hash_map_traits@KKU?$hash_traits@K@ce@@Vallocator@2@@details@ce@@@details@ce@@IAAAAU?$pair@Viterator@?$list@U?$pair@KK@std@@Vallocator@ce@@@ce@@I@std@@ABK@Z 1001d2fc f i usb_ufnmddbase_common_topaz_v1:pipe.obj
 0001:0001c394       ?_get_bucket@?$hash@V?$hash_map_traits@KKU?$hash_traits@K@ce@@Vallocator@2@@details@ce@@@details@ce@@IBAABU?$pair@Viterator@?$list@U?$pair@KK@std@@Vallocator@ce@@@ce@@I@std@@ABK@Z 1001d394 f i usb_ufnmddbase_common_topaz_v1:pipe.obj
 0001:0001c42c       ?_bucket_begin@?$hash@V?$hash_map_traits@KKU?$hash_traits@K@ce@@Vallocator@2@@details@ce@@@details@ce@@IAAAAViterator@?$list@U?$pair@KK@std@@Vallocator@ce@@@3@AAU?$pair@Viterator@?$list@U?$pair@KK@std@@Vallocator@ce@@@ce@@I@std@@@Z 1001d42c f i usb_ufnmddbase_common_topaz_v1:pipe.obj
 0001:0001c454       ?_bucket_begin@?$hash@V?$hash_map_traits@KKU?$hash_traits@K@ce@@Vallocator@2@@details@ce@@@details@ce@@IBAABViterator@?$list@U?$pair@KK@std@@Vallocator@ce@@@3@ABU?$pair@Viterator@?$list@U?$pair@KK@std@@Vallocator@ce@@@ce@@I@std@@@Z 1001d454 f i usb_ufnmddbase_common_topaz_v1:pipe.obj
 0001:0001c47c       ?_bucket_size@?$hash@V?$hash_map_traits@KKU?$hash_traits@K@ce@@Vallocator@2@@details@ce@@@details@ce@@IAAAAIAAU?$pair@Viterator@?$list@U?$pair@KK@std@@Vallocator@ce@@@ce@@I@std@@@Z 1001d47c f i usb_ufnmddbase_common_topaz_v1:pipe.obj
 0001:0001c4a8       ?_bucket_size@?$hash@V?$hash_map_traits@KKU?$hash_traits@K@ce@@Vallocator@2@@details@ce@@@details@ce@@IBAABIABU?$pair@Viterator@?$list@U?$pair@KK@std@@Vallocator@ce@@@ce@@I@std@@@Z 1001d4a8 f i usb_ufnmddbase_common_topaz_v1:pipe.obj
 0001:0001c4d4       ?_ready@?$hash@V?$hash_map_traits@KKU?$hash_traits@K@ce@@Vallocator@2@@details@ce@@@details@ce@@IBA_NXZ 1001d4d4 f i usb_ufnmddbase_common_topaz_v1:pipe.obj
 0001:0001c588       ?_key@?$hash_map_traits@KKU?$hash_traits@K@ce@@Vallocator@2@@details@ce@@QBAABKABU?$pair@KK@std@@@Z 1001d588 f i usb_ufnmddbase_common_topaz_v1:pipe.obj
 0001:0001c5b0       ?begin@?$list@U?$pair@KK@std@@Vallocator@ce@@@ce@@QAA?AViterator@12@XZ 1001d5b0 f i usb_ufnmddbase_common_topaz_v1:pipe.obj
 0001:0001c5f0       ?end@?$list@U?$pair@KK@std@@Vallocator@ce@@@ce@@QAA?AViterator@12@XZ 1001d5f0 f i usb_ufnmddbase_common_topaz_v1:pipe.obj
 0001:0001c628       ?end@?$list@U?$pair@KK@std@@Vallocator@ce@@@ce@@QBA?AVconst_iterator@12@XZ 1001d628 f i usb_ufnmddbase_common_topaz_v1:pipe.obj
 0001:0001c660       ?clear@?$list@U?$pair@KK@std@@Vallocator@ce@@@ce@@QAAXXZ 1001d660 f i usb_ufnmddbase_common_topaz_v1:pipe.obj
 0001:0001c6c8       ?erase@?$list@U?$pair@KK@std@@Vallocator@ce@@@ce@@QAA?AViterator@12@V312@@Z 1001d6c8 f i usb_ufnmddbase_common_topaz_v1:pipe.obj
 0001:0001c830       ?erase@?$list@U?$pair@KK@std@@Vallocator@ce@@@ce@@QAA?AViterator@12@V312@0@Z 1001d830 f i usb_ufnmddbase_common_topaz_v1:pipe.obj
 0001:0001c8b8       ?begin@?$vector@U?$pair@Viterator@?$list@U?$pair@KK@std@@Vallocator@ce@@@ce@@I@std@@Vallocator@ce@@U?$incremental_growth@$09@4@@ce@@QAAPAU?$pair@Viterator@?$list@U?$pair@KK@std@@Vallocator@ce@@@ce@@I@std@@XZ 1001d8b8 f i usb_ufnmddbase_common_topaz_v1:pipe.obj
 0001:0001c8e4       ?end@?$vector@U?$pair@Viterator@?$list@U?$pair@KK@std@@Vallocator@ce@@@ce@@I@std@@Vallocator@ce@@U?$incremental_growth@$09@4@@ce@@QAAPAU?$pair@Viterator@?$list@U?$pair@KK@std@@Vallocator@ce@@@ce@@I@std@@XZ 1001d8e4 f i usb_ufnmddbase_common_topaz_v1:pipe.obj
 0001:0001c914       ?clear@?$vector@U?$pair@Viterator@?$list@U?$pair@KK@std@@Vallocator@ce@@@ce@@I@std@@Vallocator@ce@@U?$incremental_growth@$09@4@@ce@@QAAXXZ 1001d914 f i usb_ufnmddbase_common_topaz_v1:pipe.obj
 0001:0001c958       ?capacity@?$vector@U?$pair@Viterator@?$list@U?$pair@KK@std@@Vallocator@ce@@@ce@@I@std@@Vallocator@ce@@U?$incremental_growth@$09@4@@ce@@QBAIXZ 1001d958 f i usb_ufnmddbase_common_topaz_v1:pipe.obj
 0001:0001c998       ??0?$hash@V?$hash_map_traits@KPAU_USB_ENDPOINT_DESCRIPTOR@@U?$hash_traits@K@ce@@Vallocator@3@@details@ce@@@details@ce@@QAA@I@Z 1001d998 f i usb_ufnmddbase_common_topaz_v1:pipe.obj
 0001:0001ca04       ?insert@?$hash@V?$hash_map_traits@KPAU_USB_ENDPOINT_DESCRIPTOR@@U?$hash_traits@K@ce@@Vallocator@3@@details@ce@@@details@ce@@QAA?AViterator@?$list@U?$pair@KPAU_USB_ENDPOINT_DESCRIPTOR@@@std@@Vallocator@ce@@@3@ABU?$pair@KPAU_USB_ENDPOINT_DESCRIPTOR@@@std@@@Z 1001da04 f i usb_ufnmddbase_common_topaz_v1:pipe.obj
 0001:0001cc54       ?_get_bucket@?$hash@V?$hash_map_traits@KPAU_USB_ENDPOINT_DESCRIPTOR@@U?$hash_traits@K@ce@@Vallocator@3@@details@ce@@@details@ce@@IAAAAU?$pair@Viterator@?$list@U?$pair@KPAU_USB_ENDPOINT_DESCRIPTOR@@@std@@Vallocator@ce@@@ce@@I@std@@ABK@Z 1001dc54 f i usb_ufnmddbase_common_topaz_v1:pipe.obj
 0001:0001ccec       ?_get_bucket@?$hash@V?$hash_map_traits@KPAU_USB_ENDPOINT_DESCRIPTOR@@U?$hash_traits@K@ce@@Vallocator@3@@details@ce@@@details@ce@@IBAABU?$pair@Viterator@?$list@U?$pair@KPAU_USB_ENDPOINT_DESCRIPTOR@@@std@@Vallocator@ce@@@ce@@I@std@@ABK@Z 1001dcec f i usb_ufnmddbase_common_topaz_v1:pipe.obj
 0001:0001cd84       ?_bucket_begin@?$hash@V?$hash_map_traits@KPAU_USB_ENDPOINT_DESCRIPTOR@@U?$hash_traits@K@ce@@Vallocator@3@@details@ce@@@details@ce@@IAAAAViterator@?$list@U?$pair@KPAU_USB_ENDPOINT_DESCRIPTOR@@@std@@Vallocator@ce@@@3@AAU?$pair@Viterator@?$list@U?$pair@KPAU_USB_ENDPOINT_DESCRIPTOR@@@std@@Vallocator@ce@@@ce@@I@std@@@Z 1001dd84 f i usb_ufnmddbase_common_topaz_v1:pipe.obj
 0001:0001cdac       ?_bucket_begin@?$hash@V?$hash_map_traits@KPAU_USB_ENDPOINT_DESCRIPTOR@@U?$hash_traits@K@ce@@Vallocator@3@@details@ce@@@details@ce@@IBAABViterator@?$list@U?$pair@KPAU_USB_ENDPOINT_DESCRIPTOR@@@std@@Vallocator@ce@@@3@ABU?$pair@Viterator@?$list@U?$pair@KPAU_USB_ENDPOINT_DESCRIPTOR@@@std@@Vallocator@ce@@@ce@@I@std@@@Z 1001ddac f i usb_ufnmddbase_common_topaz_v1:pipe.obj
 0001:0001cdd4       ?_bucket_size@?$hash@V?$hash_map_traits@KPAU_USB_ENDPOINT_DESCRIPTOR@@U?$hash_traits@K@ce@@Vallocator@3@@details@ce@@@details@ce@@IAAAAIAAU?$pair@Viterator@?$list@U?$pair@KPAU_USB_ENDPOINT_DESCRIPTOR@@@std@@Vallocator@ce@@@ce@@I@std@@@Z 1001ddd4 f i usb_ufnmddbase_common_topaz_v1:pipe.obj
 0001:0001ce00       ?_bucket_size@?$hash@V?$hash_map_traits@KPAU_USB_ENDPOINT_DESCRIPTOR@@U?$hash_traits@K@ce@@Vallocator@3@@details@ce@@@details@ce@@IBAABIABU?$pair@Viterator@?$list@U?$pair@KPAU_USB_ENDPOINT_DESCRIPTOR@@@std@@Vallocator@ce@@@ce@@I@std@@@Z 1001de00 f i usb_ufnmddbase_common_topaz_v1:pipe.obj
 0001:0001ce2c       ?_ready@?$hash@V?$hash_map_traits@KPAU_USB_ENDPOINT_DESCRIPTOR@@U?$hash_traits@K@ce@@Vallocator@3@@details@ce@@@details@ce@@IBA_NXZ 1001de2c f i usb_ufnmddbase_common_topaz_v1:pipe.obj
 0001:0001cee0       ?_key@?$hash_map_traits@KPAU_USB_ENDPOINT_DESCRIPTOR@@U?$hash_traits@K@ce@@Vallocator@3@@details@ce@@QBAABKABU?$pair@KPAU_USB_ENDPOINT_DESCRIPTOR@@@std@@@Z 1001dee0 f i usb_ufnmddbase_common_topaz_v1:pipe.obj
 0001:0001cf08       ?begin@?$list@U?$pair@KPAU_USB_ENDPOINT_DESCRIPTOR@@@std@@Vallocator@ce@@@ce@@QAA?AViterator@12@XZ 1001df08 f i usb_ufnmddbase_common_topaz_v1:pipe.obj
 0001:0001cf48       ?end@?$list@U?$pair@KPAU_USB_ENDPOINT_DESCRIPTOR@@@std@@Vallocator@ce@@@ce@@QAA?AViterator@12@XZ 1001df48 f i usb_ufnmddbase_common_topaz_v1:pipe.obj
 0001:0001cf80       ?end@?$list@U?$pair@KPAU_USB_ENDPOINT_DESCRIPTOR@@@std@@Vallocator@ce@@@ce@@QBA?AVconst_iterator@12@XZ 1001df80 f i usb_ufnmddbase_common_topaz_v1:pipe.obj
 0001:0001cfb8       ?clear@?$list@U?$pair@KPAU_USB_ENDPOINT_DESCRIPTOR@@@std@@Vallocator@ce@@@ce@@QAAXXZ 1001dfb8 f i usb_ufnmddbase_common_topaz_v1:pipe.obj
 0001:0001d020       ?erase@?$list@U?$pair@KPAU_USB_ENDPOINT_DESCRIPTOR@@@std@@Vallocator@ce@@@ce@@QAA?AViterator@12@V312@@Z 1001e020 f i usb_ufnmddbase_common_topaz_v1:pipe.obj
 0001:0001d188       ?erase@?$list@U?$pair@KPAU_USB_ENDPOINT_DESCRIPTOR@@@std@@Vallocator@ce@@@ce@@QAA?AViterator@12@V312@0@Z 1001e188 f i usb_ufnmddbase_common_topaz_v1:pipe.obj
 0001:0001d210       ?begin@?$vector@U?$pair@Viterator@?$list@U?$pair@KPAU_USB_ENDPOINT_DESCRIPTOR@@@std@@Vallocator@ce@@@ce@@I@std@@Vallocator@ce@@U?$incremental_growth@$09@4@@ce@@QAAPAU?$pair@Viterator@?$list@U?$pair@KPAU_USB_ENDPOINT_DESCRIPTOR@@@std@@Vallocator@ce@@@ce@@I@std@@XZ 1001e210 f i usb_ufnmddbase_common_topaz_v1:pipe.obj
 0001:0001d23c       ?end@?$vector@U?$pair@Viterator@?$list@U?$pair@KPAU_USB_ENDPOINT_DESCRIPTOR@@@std@@Vallocator@ce@@@ce@@I@std@@Vallocator@ce@@U?$incremental_growth@$09@4@@ce@@QAAPAU?$pair@Viterator@?$list@U?$pair@KPAU_USB_ENDPOINT_DESCRIPTOR@@@std@@Vallocator@ce@@@ce@@I@std@@XZ 1001e23c f i usb_ufnmddbase_common_topaz_v1:pipe.obj
 0001:0001d26c       ?clear@?$vector@U?$pair@Viterator@?$list@U?$pair@KPAU_USB_ENDPOINT_DESCRIPTOR@@@std@@Vallocator@ce@@@ce@@I@std@@Vallocator@ce@@U?$incremental_growth@$09@4@@ce@@QAAXXZ 1001e26c f i usb_ufnmddbase_common_topaz_v1:pipe.obj
 0001:0001d2b0       ?capacity@?$vector@U?$pair@Viterator@?$list@U?$pair@KPAU_USB_ENDPOINT_DESCRIPTOR@@@std@@Vallocator@ce@@@ce@@I@std@@Vallocator@ce@@U?$incremental_growth@$09@4@@ce@@QBAIXZ 1001e2b0 f i usb_ufnmddbase_common_topaz_v1:pipe.obj
 0001:0001d2f0       ??Dconst_iterator@?$list@U?$pair@KK@std@@Vallocator@ce@@@ce@@QBAABU?$pair@KK@std@@XZ 1001e2f0 f i usb_ufnmddbase_common_topaz_v1:pipe.obj
 0001:0001d31c       ??Econst_iterator@?$list@U?$pair@KK@std@@Vallocator@ce@@@ce@@QAAAAV012@XZ 1001e31c f i usb_ufnmddbase_common_topaz_v1:pipe.obj
 0001:0001d35c       ??Diterator@?$list@U?$pair@KPAU_USB_ENDPOINT_DESCRIPTOR@@@std@@Vallocator@ce@@@ce@@QBAAAU?$pair@KPAU_USB_ENDPOINT_DESCRIPTOR@@@std@@XZ 1001e35c f i usb_ufnmddbase_common_topaz_v1:pipe.obj
 0001:0001d388       ??Eiterator@?$list@U?$pair@KPAU_USB_ENDPOINT_DESCRIPTOR@@@std@@Vallocator@ce@@@ce@@QAAAAV012@XZ 1001e388 f i usb_ufnmddbase_common_topaz_v1:pipe.obj
 0001:0001d3c8       ??8iterator@?$list@U?$pair@KPAU_USB_ENDPOINT_DESCRIPTOR@@@std@@Vallocator@ce@@@ce@@QBA_NABV012@@Z 1001e3c8 f i usb_ufnmddbase_common_topaz_v1:pipe.obj
 0001:0001d420       ??Dconst_iterator@?$list@U?$pair@KPAU_USB_ENDPOINT_DESCRIPTOR@@@std@@Vallocator@ce@@@ce@@QBAABU?$pair@KPAU_USB_ENDPOINT_DESCRIPTOR@@@std@@XZ 1001e420 f i usb_ufnmddbase_common_topaz_v1:pipe.obj
 0001:0001d44c       ??Econst_iterator@?$list@U?$pair@KPAU_USB_ENDPOINT_DESCRIPTOR@@@std@@Vallocator@ce@@@ce@@QAAAAV012@XZ 1001e44c f i usb_ufnmddbase_common_topaz_v1:pipe.obj
 0001:0001d48c       ??8const_iterator@?$list@U?$pair@KPAU_USB_ENDPOINT_DESCRIPTOR@@@std@@Vallocator@ce@@@ce@@QBA_NABV012@@Z 1001e48c f i usb_ufnmddbase_common_topaz_v1:pipe.obj
 0001:0001d4e4       ??Diterator@?$list@U?$pair@KK@std@@Vallocator@ce@@@ce@@QBAAAU?$pair@KK@std@@XZ 1001e4e4 f i usb_ufnmddbase_common_topaz_v1:pipe.obj
 0001:0001d510       ??Eiterator@?$list@U?$pair@KK@std@@Vallocator@ce@@@ce@@QAAAAV012@XZ 1001e510 f i usb_ufnmddbase_common_topaz_v1:pipe.obj
 0001:0001d550       ??0?$fixed_block_allocator@$0BE@@ce@@QAA@ABV01@@Z 1001e550 f i usb_ufnmddbase_common_topaz_v1:pipe.obj
 0001:0001d588       ?deallocate@?$fixed_block_allocator@$07@ce@@QBAXPAXI@Z 1001e588 f i usb_ufnmddbase_common_topaz_v1:pipe.obj
 0001:0001d620       ?_InitializeDescr@?$fixed_block_allocator@$07@ce@@IBA_NI@Z 1001e620 f i usb_ufnmddbase_common_topaz_v1:pipe.obj
 0001:0001d74c       ?begin@?$list@PAVCUfnMddTransfer@@V?$fixed_block_allocator@$0BE@@ce@@@ce@@QAA?AViterator@12@XZ 1001e74c f i usb_ufnmddbase_common_topaz_v1:pipe.obj
 0001:0001d790       ?begin@?$list@PAVCUfnMddTransfer@@V?$fixed_block_allocator@$0BE@@ce@@@ce@@QBA?AVconst_iterator@12@XZ 1001e790 f i usb_ufnmddbase_common_topaz_v1:pipe.obj
 0001:0001d7d4       ?end@?$list@PAVCUfnMddTransfer@@V?$fixed_block_allocator@$0BE@@ce@@@ce@@QAA?AViterator@12@XZ 1001e7d4 f i usb_ufnmddbase_common_topaz_v1:pipe.obj
 0001:0001d810       ?end@?$list@PAVCUfnMddTransfer@@V?$fixed_block_allocator@$0BE@@ce@@@ce@@QBA?AVconst_iterator@12@XZ 1001e810 f i usb_ufnmddbase_common_topaz_v1:pipe.obj
 0001:0001d84c       ?clear@?$list@PAVCUfnMddTransfer@@V?$fixed_block_allocator@$0BE@@ce@@@ce@@QAAXXZ 1001e84c f i usb_ufnmddbase_common_topaz_v1:pipe.obj
 0001:0001d8b4       ?erase@?$list@PAVCUfnMddTransfer@@V?$fixed_block_allocator@$0BE@@ce@@@ce@@QAA?AViterator@12@V312@@Z 1001e8b4 f i usb_ufnmddbase_common_topaz_v1:pipe.obj
 0001:0001da1c       ?_init_hash_table@?$hash@V?$hash_map_traits@KKU?$hash_traits@K@ce@@Vallocator@2@@details@ce@@@details@ce@@IAAXI@Z 1001ea1c f i usb_ufnmddbase_common_topaz_v1:pipe.obj
 0001:0001da9c       ??0?$hash_map_traits@KKU?$hash_traits@K@ce@@Vallocator@2@@details@ce@@QAA@XZ 1001ea9c f i usb_ufnmddbase_common_topaz_v1:pipe.obj
 0001:0001dac4       ?hash_function@?$hash_traits@K@ce@@QBAIABK@Z 1001eac4 f i usb_ufnmddbase_common_topaz_v1:pipe.obj
 0001:0001daf0       ??0?$list@U?$pair@KK@std@@Vallocator@ce@@@ce@@QAA@XZ 1001eaf0 f i usb_ufnmddbase_common_topaz_v1:pipe.obj
 0001:0001dbcc       ?_Freenode@?$list@U?$pair@KK@std@@Vallocator@ce@@@ce@@IAAXPAU_Node@12@@Z 1001ebcc f i usb_ufnmddbase_common_topaz_v1:pipe.obj
 0001:0001dbf0       ??0?$vector@U?$pair@Viterator@?$list@U?$pair@KK@std@@Vallocator@ce@@@ce@@I@std@@Vallocator@ce@@U?$incremental_growth@$09@4@@ce@@QAA@XZ 1001ebf0 f i usb_ufnmddbase_common_topaz_v1:pipe.obj
 0001:0001dc44       ?size@?$vector@U?$pair@Viterator@?$list@U?$pair@KK@std@@Vallocator@ce@@@ce@@I@std@@Vallocator@ce@@U?$incremental_growth@$09@4@@ce@@QBAIXZ 1001ec44 f i usb_ufnmddbase_common_topaz_v1:pipe.obj
 0001:0001dc84       ??A?$vector@U?$pair@Viterator@?$list@U?$pair@KK@std@@Vallocator@ce@@@ce@@I@std@@Vallocator@ce@@U?$incremental_growth@$09@4@@ce@@QBAABU?$pair@Viterator@?$list@U?$pair@KK@std@@Vallocator@ce@@@ce@@I@std@@I@Z 1001ec84 f i usb_ufnmddbase_common_topaz_v1:pipe.obj
 0001:0001dcc0       ??A?$vector@U?$pair@Viterator@?$list@U?$pair@KK@std@@Vallocator@ce@@@ce@@I@std@@Vallocator@ce@@U?$incremental_growth@$09@4@@ce@@QAAAAU?$pair@Viterator@?$list@U?$pair@KK@std@@Vallocator@ce@@@ce@@I@std@@I@Z 1001ecc0 f i usb_ufnmddbase_common_topaz_v1:pipe.obj
 0001:0001dcfc       ?erase@?$vector@U?$pair@Viterator@?$list@U?$pair@KK@std@@Vallocator@ce@@@ce@@I@std@@Vallocator@ce@@U?$incremental_growth@$09@4@@ce@@QAAXPAU?$pair@Viterator@?$list@U?$pair@KK@std@@Vallocator@ce@@@ce@@I@std@@0@Z 1001ecfc f i usb_ufnmddbase_common_topaz_v1:pipe.obj
 0001:0001dde4       ?_init_hash_table@?$hash@V?$hash_map_traits@KPAU_USB_ENDPOINT_DESCRIPTOR@@U?$hash_traits@K@ce@@Vallocator@3@@details@ce@@@details@ce@@IAAXI@Z 1001ede4 f i usb_ufnmddbase_common_topaz_v1:pipe.obj
 0001:0001de64       ??0?$hash_map_traits@KPAU_USB_ENDPOINT_DESCRIPTOR@@U?$hash_traits@K@ce@@Vallocator@3@@details@ce@@QAA@XZ 1001ee64 f i usb_ufnmddbase_common_topaz_v1:pipe.obj
 0001:0001de8c       ??0?$list@U?$pair@KPAU_USB_ENDPOINT_DESCRIPTOR@@@std@@Vallocator@ce@@@ce@@QAA@XZ 1001ee8c f i usb_ufnmddbase_common_topaz_v1:pipe.obj
 0001:0001df68       ?_Freenode@?$list@U?$pair@KPAU_USB_ENDPOINT_DESCRIPTOR@@@std@@Vallocator@ce@@@ce@@IAAXPAU_Node@12@@Z 1001ef68 f i usb_ufnmddbase_common_topaz_v1:pipe.obj
 0001:0001df8c       ??0?$vector@U?$pair@Viterator@?$list@U?$pair@KPAU_USB_ENDPOINT_DESCRIPTOR@@@std@@Vallocator@ce@@@ce@@I@std@@Vallocator@ce@@U?$incremental_growth@$09@4@@ce@@QAA@XZ 1001ef8c f i usb_ufnmddbase_common_topaz_v1:pipe.obj
 0001:0001dfe0       ?size@?$vector@U?$pair@Viterator@?$list@U?$pair@KPAU_USB_ENDPOINT_DESCRIPTOR@@@std@@Vallocator@ce@@@ce@@I@std@@Vallocator@ce@@U?$incremental_growth@$09@4@@ce@@QBAIXZ 1001efe0 f i usb_ufnmddbase_common_topaz_v1:pipe.obj
 0001:0001e020       ??A?$vector@U?$pair@Viterator@?$list@U?$pair@KPAU_USB_ENDPOINT_DESCRIPTOR@@@std@@Vallocator@ce@@@ce@@I@std@@Vallocator@ce@@U?$incremental_growth@$09@4@@ce@@QBAABU?$pair@Viterator@?$list@U?$pair@KPAU_USB_ENDPOINT_DESCRIPTOR@@@std@@Vallocator@ce@@@ce@@I@std@@I@Z 1001f020 f i usb_ufnmddbase_common_topaz_v1:pipe.obj
 0001:0001e05c       ??A?$vector@U?$pair@Viterator@?$list@U?$pair@KPAU_USB_ENDPOINT_DESCRIPTOR@@@std@@Vallocator@ce@@@ce@@I@std@@Vallocator@ce@@U?$incremental_growth@$09@4@@ce@@QAAAAU?$pair@Viterator@?$list@U?$pair@KPAU_USB_ENDPOINT_DESCRIPTOR@@@std@@Vallocator@ce@@@ce@@I@std@@I@Z 1001f05c f i usb_ufnmddbase_common_topaz_v1:pipe.obj
 0001:0001e098       ?erase@?$vector@U?$pair@Viterator@?$list@U?$pair@KPAU_USB_ENDPOINT_DESCRIPTOR@@@std@@Vallocator@ce@@@ce@@I@std@@Vallocator@ce@@U?$incremental_growth@$09@4@@ce@@QAAXPAU?$pair@Viterator@?$list@U?$pair@KPAU_USB_ENDPOINT_DESCRIPTOR@@@std@@Vallocator@ce@@@ce@@I@std@@0@Z 1001f098 f i usb_ufnmddbase_common_topaz_v1:pipe.obj
 0001:0001e180       ??0const_iterator@?$list@U?$pair@KK@std@@Vallocator@ce@@@ce@@QAA@PAU_Node@12@@Z 1001f180 f i usb_ufnmddbase_common_topaz_v1:pipe.obj
 0001:0001e1b4       ?_MyNode@const_iterator@?$list@U?$pair@KK@std@@Vallocator@ce@@@ce@@QBAPAU_Node@23@XZ 1001f1b4 f i usb_ufnmddbase_common_topaz_v1:pipe.obj
 0001:0001e1e0       ??0iterator@?$list@U?$pair@KPAU_USB_ENDPOINT_DESCRIPTOR@@@std@@Vallocator@ce@@@ce@@QAA@PAU_Node@12@@Z 1001f1e0 f i usb_ufnmddbase_common_topaz_v1:pipe.obj
 0001:0001e214       ??Eiterator@?$list@U?$pair@KPAU_USB_ENDPOINT_DESCRIPTOR@@@std@@Vallocator@ce@@@ce@@QAA?AV012@H@Z 1001f214 f i usb_ufnmddbase_common_topaz_v1:pipe.obj
 0001:0001e264       ??Fiterator@?$list@U?$pair@KPAU_USB_ENDPOINT_DESCRIPTOR@@@std@@Vallocator@ce@@@ce@@QAAAAV012@XZ 1001f264 f i usb_ufnmddbase_common_topaz_v1:pipe.obj
 0001:0001e2a4       ??0const_iterator@?$list@U?$pair@KPAU_USB_ENDPOINT_DESCRIPTOR@@@std@@Vallocator@ce@@@ce@@QAA@PAU_Node@12@@Z 1001f2a4 f i usb_ufnmddbase_common_topaz_v1:pipe.obj
 0001:0001e2d8       ?_MyNode@const_iterator@?$list@U?$pair@KPAU_USB_ENDPOINT_DESCRIPTOR@@@std@@Vallocator@ce@@@ce@@QBAPAU_Node@23@XZ 1001f2d8 f i usb_ufnmddbase_common_topaz_v1:pipe.obj
 0001:0001e304       ??0iterator@?$list@U?$pair@KK@std@@Vallocator@ce@@@ce@@QAA@PAU_Node@12@@Z 1001f304 f i usb_ufnmddbase_common_topaz_v1:pipe.obj
 0001:0001e338       ??Eiterator@?$list@U?$pair@KK@std@@Vallocator@ce@@@ce@@QAA?AV012@H@Z 1001f338 f i usb_ufnmddbase_common_topaz_v1:pipe.obj
 0001:0001e388       ??Fiterator@?$list@U?$pair@KK@std@@Vallocator@ce@@@ce@@QAAAAV012@XZ 1001f388 f i usb_ufnmddbase_common_topaz_v1:pipe.obj
 0001:0001e3c8       ??Fiterator@?$list@PAVCUfnMddTransfer@@V?$fixed_block_allocator@$0BE@@ce@@@ce@@QAAAAV012@XZ 1001f3c8 f i usb_ufnmddbase_common_topaz_v1:pipe.obj
 0001:0001e408       ??Dconst_iterator@?$list@PAVCUfnMddTransfer@@V?$fixed_block_allocator@$0BE@@ce@@@ce@@QBAABQAVCUfnMddTransfer@@XZ 1001f408 f i usb_ufnmddbase_common_topaz_v1:pipe.obj
 0001:0001e434       ??Fconst_iterator@?$list@PAVCUfnMddTransfer@@V?$fixed_block_allocator@$0BE@@ce@@@ce@@QAAAAV012@XZ 1001f434 f i usb_ufnmddbase_common_topaz_v1:pipe.obj
 0001:0001e474       ?erase@?$list@PAVCUfnMddTransfer@@V?$fixed_block_allocator@$0BE@@ce@@@ce@@QAA?AViterator@12@V312@0@Z 1001f474 f i usb_ufnmddbase_common_topaz_v1:pipe.obj
 0001:0001e4fc       ?_Freenode@?$list@PAVCUfnMddTransfer@@V?$fixed_block_allocator@$0BE@@ce@@@ce@@IAAXPAU_Node@12@@Z 1001f4fc f i usb_ufnmddbase_common_topaz_v1:pipe.obj
 0001:0001e520       ?_MoveBackward@?$vector@U?$pair@Viterator@?$list@U?$pair@KK@std@@Vallocator@ce@@@ce@@I@std@@Vallocator@ce@@U?$incremental_growth@$09@4@@ce@@IAAXPAU?$pair@Viterator@?$list@U?$pair@KK@std@@Vallocator@ce@@@ce@@I@std@@00@Z 1001f520 f i usb_ufnmddbase_common_topaz_v1:pipe.obj
 0001:0001e6dc       ?_MoveBackward@?$vector@U?$pair@Viterator@?$list@U?$pair@KPAU_USB_ENDPOINT_DESCRIPTOR@@@std@@Vallocator@ce@@@ce@@I@std@@Vallocator@ce@@U?$incremental_growth@$09@4@@ce@@IAAXPAU?$pair@Viterator@?$list@U?$pair@KPAU_USB_ENDPOINT_DESCRIPTOR@@@std@@Vallocator@ce@@@ce@@I@std@@00@Z 1001f6dc f i usb_ufnmddbase_common_topaz_v1:pipe.obj
 0001:0001e898       ??0?$pair@Viterator@?$list@U?$pair@KK@std@@Vallocator@ce@@@ce@@I@std@@QAA@ABViterator@?$list@U?$pair@KK@std@@Vallocator@ce@@@ce@@ABI@Z 1001f898 f i usb_ufnmddbase_common_topaz_v1:pipe.obj
 0001:0001e8e4       ??0?$pair@Viterator@?$list@U?$pair@KPAU_USB_ENDPOINT_DESCRIPTOR@@@std@@Vallocator@ce@@@ce@@I@std@@QAA@ABViterator@?$list@U?$pair@KPAU_USB_ENDPOINT_DESCRIPTOR@@@std@@Vallocator@ce@@@ce@@ABI@Z 1001f8e4 f i usb_ufnmddbase_common_topaz_v1:pipe.obj
 0001:0001e930       ??0iterator@?$list@PAVCUfnMddTransfer@@V?$fixed_block_allocator@$0BE@@ce@@@ce@@QAA@PAU_Node@12@@Z 1001f930 f i usb_ufnmddbase_common_topaz_v1:pipe.obj
 0001:0001e964       ??Eiterator@?$list@PAVCUfnMddTransfer@@V?$fixed_block_allocator@$0BE@@ce@@@ce@@QAA?AV012@H@Z 1001f964 f i usb_ufnmddbase_common_topaz_v1:pipe.obj
 0001:0001e9b4       ??9iterator@?$list@PAVCUfnMddTransfer@@V?$fixed_block_allocator@$0BE@@ce@@@ce@@QBA_NABV012@@Z 1001f9b4 f i usb_ufnmddbase_common_topaz_v1:pipe.obj
 0001:0001ea10       ??0const_iterator@?$list@PAVCUfnMddTransfer@@V?$fixed_block_allocator@$0BE@@ce@@@ce@@QAA@PAU_Node@12@@Z 1001fa10 f i usb_ufnmddbase_common_topaz_v1:pipe.obj
 0001:0001ea44       ?_MyNode@const_iterator@?$list@PAVCUfnMddTransfer@@V?$fixed_block_allocator@$0BE@@ce@@@ce@@QBAPAU_Node@23@XZ 1001fa44 f i usb_ufnmddbase_common_topaz_v1:pipe.obj
 0001:0001ea70       ?deallocate@?$fixed_block_allocator@$0BE@@ce@@QBAXPAXI@Z 1001fa70 f i usb_ufnmddbase_common_topaz_v1:pipe.obj
 0001:0001eb08       ?_Destroy@?$vector@U?$pair@Viterator@?$list@U?$pair@KK@std@@Vallocator@ce@@@ce@@I@std@@Vallocator@ce@@U?$incremental_growth@$09@4@@ce@@IAAXPAU?$pair@Viterator@?$list@U?$pair@KK@std@@Vallocator@ce@@@ce@@I@std@@0@Z 1001fb08 f i usb_ufnmddbase_common_topaz_v1:pipe.obj
 0001:0001eb40       ?_Destroy@?$vector@U?$pair@Viterator@?$list@U?$pair@KPAU_USB_ENDPOINT_DESCRIPTOR@@@std@@Vallocator@ce@@@ce@@I@std@@Vallocator@ce@@U?$incremental_growth@$09@4@@ce@@IAAXPAU?$pair@Viterator@?$list@U?$pair@KPAU_USB_ENDPOINT_DESCRIPTOR@@@std@@Vallocator@ce@@@ce@@I@std@@0@Z 1001fb40 f i usb_ufnmddbase_common_topaz_v1:pipe.obj
 0001:0001eb78       ??Eiterator@?$list@PAVCUfnMddTransfer@@V?$fixed_block_allocator@$0BE@@ce@@@ce@@QAAAAV012@XZ 1001fb78 f i usb_ufnmddbase_common_topaz_v1:pipe.obj
 0001:0001ebb8       ??8iterator@?$list@PAVCUfnMddTransfer@@V?$fixed_block_allocator@$0BE@@ce@@@ce@@QBA_NABV012@@Z 1001fbb8 f i usb_ufnmddbase_common_topaz_v1:pipe.obj
 0001:0001ec10       ??$push_back@PAVCUfnMddTransfer@@@?$list@PAVCUfnMddTransfer@@V?$fixed_block_allocator@$0BE@@ce@@@ce@@QAA_NABQAVCUfnMddTransfer@@@Z 1001fc10 f i usb_ufnmddbase_common_topaz_v1:pipe.obj
 0001:0001ec8c       ??$insert@U?$pair@KK@std@@@?$list@U?$pair@KK@std@@Vallocator@ce@@@ce@@QAA?AViterator@01@V201@ABU?$pair@KK@std@@@Z 1001fc8c f i usb_ufnmddbase_common_topaz_v1:pipe.obj
 0001:0001ed50       ??$insert@U?$pair@KPAU_USB_ENDPOINT_DESCRIPTOR@@@std@@@?$list@U?$pair@KPAU_USB_ENDPOINT_DESCRIPTOR@@@std@@Vallocator@ce@@@ce@@QAA?AViterator@01@V201@ABU?$pair@KPAU_USB_ENDPOINT_DESCRIPTOR@@@std@@@Z 1001fd50 f i usb_ufnmddbase_common_topaz_v1:pipe.obj
 0001:0001ee14       ??$resize@U?$pair@Viterator@?$list@U?$pair@KK@std@@Vallocator@ce@@@ce@@I@std@@@?$vector@U?$pair@Viterator@?$list@U?$pair@KK@std@@Vallocator@ce@@@ce@@I@std@@Vallocator@ce@@U?$incremental_growth@$09@4@@ce@@QAA_NIABU?$pair@Viterator@?$list@U?$pair@KK@std@@Vallocator@ce@@@ce@@I@std@@@Z 1001fe14 f i usb_ufnmddbase_common_topaz_v1:pipe.obj
 0001:0001eef4       ??$resize@U?$pair@Viterator@?$list@U?$pair@KPAU_USB_ENDPOINT_DESCRIPTOR@@@std@@Vallocator@ce@@@ce@@I@std@@@?$vector@U?$pair@Viterator@?$list@U?$pair@KPAU_USB_ENDPOINT_DESCRIPTOR@@@std@@Vallocator@ce@@@ce@@I@std@@Vallocator@ce@@U?$incremental_growth@$09@4@@ce@@QAA_NIABU?$pair@Viterator@?$list@U?$pair@KPAU_USB_ENDPOINT_DESCRIPTOR@@@std@@Vallocator@ce@@@ce@@I@std@@@Z 1001fef4 f i usb_ufnmddbase_common_topaz_v1:pipe.obj
 0001:0001efd4       ?_Buynode@?$list@U?$pair@KK@std@@Vallocator@ce@@@ce@@IAAPAU_Node@12@PAU312@@Z 1001ffd4 f i usb_ufnmddbase_common_topaz_v1:pipe.obj
 0001:0001f0dc       ?_Buynode@?$list@U?$pair@KPAU_USB_ENDPOINT_DESCRIPTOR@@@std@@Vallocator@ce@@@ce@@IAAPAU_Node@12@PAU312@@Z 100200dc f i usb_ufnmddbase_common_topaz_v1:pipe.obj
 0001:0001f1e4       ??$insert@PAVCUfnMddTransfer@@@?$list@PAVCUfnMddTransfer@@V?$fixed_block_allocator@$0BE@@ce@@@ce@@QAA?AViterator@01@V201@ABQAVCUfnMddTransfer@@@Z 100201e4 f i usb_ufnmddbase_common_topaz_v1:pipe.obj
 0001:0001f2a8       ??$insert@U?$pair@Viterator@?$list@U?$pair@KK@std@@Vallocator@ce@@@ce@@I@std@@@?$vector@U?$pair@Viterator@?$list@U?$pair@KK@std@@Vallocator@ce@@@ce@@I@std@@Vallocator@ce@@U?$incremental_growth@$09@4@@ce@@QAA_NPAU?$pair@Viterator@?$list@U?$pair@KK@std@@Vallocator@ce@@@ce@@I@std@@IABU23@@Z 100202a8 f i usb_ufnmddbase_common_topaz_v1:pipe.obj
 0001:0001f650       ??$insert@U?$pair@Viterator@?$list@U?$pair@KPAU_USB_ENDPOINT_DESCRIPTOR@@@std@@Vallocator@ce@@@ce@@I@std@@@?$vector@U?$pair@Viterator@?$list@U?$pair@KPAU_USB_ENDPOINT_DESCRIPTOR@@@std@@Vallocator@ce@@@ce@@I@std@@Vallocator@ce@@U?$incremental_growth@$09@4@@ce@@QAA_NPAU?$pair@Viterator@?$list@U?$pair@KPAU_USB_ENDPOINT_DESCRIPTOR@@@std@@Vallocator@ce@@@ce@@I@std@@IABU23@@Z 10020650 f i usb_ufnmddbase_common_topaz_v1:pipe.obj
 0001:0001f9f8       ?_Buynode@?$list@PAVCUfnMddTransfer@@V?$fixed_block_allocator@$0BE@@ce@@@ce@@IAAPAU_Node@12@PAU312@@Z 100209f8 f i usb_ufnmddbase_common_topaz_v1:pipe.obj
 0001:0001fb00       ?_Copy@?$vector@U?$pair@Viterator@?$list@U?$pair@KK@std@@Vallocator@ce@@@ce@@I@std@@Vallocator@ce@@U?$incremental_growth@$09@4@@ce@@IAAPAU?$pair@Viterator@?$list@U?$pair@KK@std@@Vallocator@ce@@@ce@@I@std@@PBU34@0PAU34@@Z 10020b00 f i usb_ufnmddbase_common_topaz_v1:pipe.obj
 0001:0001fbc0       ?_MoveForward@?$vector@U?$pair@Viterator@?$list@U?$pair@KK@std@@Vallocator@ce@@@ce@@I@std@@Vallocator@ce@@U?$incremental_growth@$09@4@@ce@@IAAXPAU?$pair@Viterator@?$list@U?$pair@KK@std@@Vallocator@ce@@@ce@@I@std@@00@Z 10020bc0 f i usb_ufnmddbase_common_topaz_v1:pipe.obj
 0001:0001fe24       ?_Copy@?$vector@U?$pair@Viterator@?$list@U?$pair@KPAU_USB_ENDPOINT_DESCRIPTOR@@@std@@Vallocator@ce@@@ce@@I@std@@Vallocator@ce@@U?$incremental_growth@$09@4@@ce@@IAAPAU?$pair@Viterator@?$list@U?$pair@KPAU_USB_ENDPOINT_DESCRIPTOR@@@std@@Vallocator@ce@@@ce@@I@std@@PBU34@0PAU34@@Z 10020e24 f i usb_ufnmddbase_common_topaz_v1:pipe.obj
 0001:0001fee4       ?_MoveForward@?$vector@U?$pair@Viterator@?$list@U?$pair@KPAU_USB_ENDPOINT_DESCRIPTOR@@@std@@Vallocator@ce@@@ce@@I@std@@Vallocator@ce@@U?$incremental_growth@$09@4@@ce@@IAAXPAU?$pair@Viterator@?$list@U?$pair@KPAU_USB_ENDPOINT_DESCRIPTOR@@@std@@Vallocator@ce@@@ce@@I@std@@00@Z 10020ee4 f i usb_ufnmddbase_common_topaz_v1:pipe.obj
 0001:00020148       ?get_growth@?$incremental_growth@$09@ce@@SAIIII@Z 10021148 f i usb_ufnmddbase_common_topaz_v1:pipe.obj
 0001:00020174       ?allocate@?$fixed_block_allocator@$0BE@@ce@@QBAPAXI@Z 10021174 f i usb_ufnmddbase_common_topaz_v1:pipe.obj
 0001:0002029c       ?_InitializeDescr@?$fixed_block_allocator@$0BE@@ce@@IBA_NI@Z 1002129c f i usb_ufnmddbase_common_topaz_v1:pipe.obj
 0001:000203c8       ??0CDescriptors@@QAA@XZ    100213c8 f   usb_ufnmddbase_common_topaz_v1:descript.obj
 0001:0002043c       ??1CDescriptors@@QAA@XZ    1002143c f   usb_ufnmddbase_common_topaz_v1:descript.obj
 0001:0002048c       ?Init@CDescriptors@@QAAKPAU_USB_DEVICE_DESCRIPTOR@@PAU_UFN_CONFIGURATION@@01PBU_UFN_STRING_SET@@K@Z 1002148c f   usb_ufnmddbase_common_topaz_v1:descript.obj
 0001:00020590       ?GenerateTotalConfigDescriptors@CDescriptors@@QAAKXZ 10021590 f   usb_ufnmddbase_common_topaz_v1:descript.obj
 0001:000205f4       ?ValidateDescriptorAndChildren@CDescriptors@@SAKPAU_USB_DEVICE_DESCRIPTOR@@PAU_UFN_CONFIGURATION@@01PBU_UFN_STRING_SET@@K@Z 100215f4 f   usb_ufnmddbase_common_topaz_v1:descript.obj
 0001:000206ac       ?ValidateDescriptor@CDescriptors@@SAKPAU_USB_DEVICE_DESCRIPTOR@@PAU_UFN_CONFIGURATION@@01PBU_UFN_STRING_SET@@K@Z 100216ac f   usb_ufnmddbase_common_topaz_v1:descript.obj
 0001:000209d0       ?Clone@CDescriptors@@QAAKPAPAV1@@Z 100219d0 f   usb_ufnmddbase_common_topaz_v1:descript.obj
 0001:00020df8       ?RegisterDevice@CDescriptors@@QAAKPAUUFN_MDD_CONTEXT@@@Z 10021df8 f   usb_ufnmddbase_common_topaz_v1:descript.obj
 0001:00021538       ?GetDeviceDescriptor@CDescriptors@@QAAPBU_USB_DEVICE_DESCRIPTOR@@W4_UFN_BUS_SPEED@@@Z 10022538 f   usb_ufnmddbase_common_topaz_v1:descript.obj
 0001:000215c8       ?CloneStrings@CDescriptors@@SAKPBU_UFN_STRING_SET@@KPAPAU2@@Z 100225c8 f   usb_ufnmddbase_common_topaz_v1:descript.obj
 0001:00021c38       ?IsSupportable@CDescriptors@@QAAKPAUUFN_MDD_CONTEXT@@@Z 10022c38 f   usb_ufnmddbase_common_topaz_v1:descript.obj
 0001:00021e80       ?ProcessGetDescriptor@CDescriptors@@QAA?AW4CONTROL_RESPONSE@@W4_UFN_BUS_SPEED@@U_USB_DEVICE_REQUEST@@KHPAPAXPAK@Z 10022e80 f   usb_ufnmddbase_common_topaz_v1:descript.obj
 0001:00022a14       ??0CDevice@@QAA@XZ         10023a14 f   usb_ufnmddbase_common_topaz_v1:descript.obj
 0001:00022a9c       ??1CDevice@@QAA@XZ         10023a9c f   usb_ufnmddbase_common_topaz_v1:descript.obj
 0001:00022b98       ?Init@CDevice@@QAAKW4_UFN_BUS_SPEED@@PAU_USB_DEVICE_DESCRIPTOR@@PAU_UFN_CONFIGURATION@@@Z 10023b98 f   usb_ufnmddbase_common_topaz_v1:descript.obj
 0001:00022e44       ?Clone@CDevice@@QAAKPAV1@@Z 10023e44 f   usb_ufnmddbase_common_topaz_v1:descript.obj
 0001:00023048       ?GenerateTotalConfigDescriptors@CDevice@@QAAKXZ 10024048 f   usb_ufnmddbase_common_topaz_v1:descript.obj
 0001:00023100       ?IsSupportable@CDevice@@QAAKPAUUFN_MDD_CONTEXT@@W4_UFN_BUS_SPEED@@@Z 10024100 f   usb_ufnmddbase_common_topaz_v1:descript.obj
 0001:0002336c       ?ValidateDescriptorAndChildren@CDevice@@SAKW4_UFN_BUS_SPEED@@PAU_USB_DEVICE_DESCRIPTOR@@PAU_UFN_CONFIGURATION@@@Z 1002436c f   usb_ufnmddbase_common_topaz_v1:descript.obj
 0001:00023534       ?ValidateDescriptor@CDevice@@SAKW4_UFN_BUS_SPEED@@PAU_USB_DEVICE_DESCRIPTOR@@PAU_UFN_CONFIGURATION@@@Z 10024534 f   usb_ufnmddbase_common_topaz_v1:descript.obj
 0001:000235f0       ??0CConfiguration@@QAA@XZ  100245f0 f   usb_ufnmddbase_common_topaz_v1:descript.obj
 0001:00023644       ??1CConfiguration@@QAA@XZ  10024644 f   usb_ufnmddbase_common_topaz_v1:descript.obj
 0001:000236e0       ?Init@CConfiguration@@QAAKW4_UFN_BUS_SPEED@@PAU_UFN_CONFIGURATION@@@Z 100246e0 f   usb_ufnmddbase_common_topaz_v1:descript.obj
 0001:00023980       ?IsSupportable@CConfiguration@@QAAKPAUUFN_MDD_CONTEXT@@W4_UFN_BUS_SPEED@@PAU_USB_DEVICE_DESCRIPTOR@@@Z 10024980 f   usb_ufnmddbase_common_topaz_v1:descript.obj
 0001:00023d70       ?ValidateDescriptorAndChildren@CConfiguration@@SAKW4_UFN_BUS_SPEED@@PAU_UFN_CONFIGURATION@@@Z 10024d70 f   usb_ufnmddbase_common_topaz_v1:descript.obj
 0001:0002405c       ?ValidateDescriptor@CConfiguration@@SAKW4_UFN_BUS_SPEED@@PAU_UFN_CONFIGURATION@@@Z 1002505c f   usb_ufnmddbase_common_topaz_v1:descript.obj
 0001:000241dc       ?Serialize@CConfiguration@@QAAKPAEKPAK@Z 100251dc f   usb_ufnmddbase_common_topaz_v1:descript.obj
 0001:00024444       ?GenerateTotalConfigDescriptor@CConfiguration@@QAAKXZ 10025444 f   usb_ufnmddbase_common_topaz_v1:descript.obj
 0001:000246dc       ?CopyUfnConfigTree@CConfiguration@@SAKPAU_UFN_CONFIGURATION@@0@Z 100256dc f   usb_ufnmddbase_common_topaz_v1:descript.obj
 0001:00025008       ?FreeUfnConfigTree@CConfiguration@@SAXPAU_UFN_CONFIGURATION@@@Z 10026008 f   usb_ufnmddbase_common_topaz_v1:descript.obj
 0001:000252ac       ??0CInterface@@QAA@XZ      100262ac f   usb_ufnmddbase_common_topaz_v1:descript.obj
 0001:00025300       ??1CInterface@@QAA@XZ      10026300 f   usb_ufnmddbase_common_topaz_v1:descript.obj
 0001:00025378       ?CountInterfaces@CInterface@@SAKPAU_UFN_CONFIGURATION@@@Z 10026378 f   usb_ufnmddbase_common_topaz_v1:descript.obj
 0001:0002544c       ?Init@CInterface@@QAAKW4_UFN_BUS_SPEED@@PAU_UFN_INTERFACE@@@Z 1002644c f   usb_ufnmddbase_common_topaz_v1:descript.obj
 0001:000256d8       ?ValidateDescriptorAndChildren@CInterface@@SAKW4_UFN_BUS_SPEED@@PAU_UFN_INTERFACE@@@Z 100266d8 f   usb_ufnmddbase_common_topaz_v1:descript.obj
 0001:000257a8       ?ValidateDescriptor@CInterface@@SAKW4_UFN_BUS_SPEED@@PAU_UFN_INTERFACE@@@Z 100267a8 f   usb_ufnmddbase_common_topaz_v1:descript.obj
 0001:00025928       ?Serialize@CInterface@@QAAKPAEKPAK@Z 10026928 f   usb_ufnmddbase_common_topaz_v1:descript.obj
 0001:00025b2c       ?IsSupportable@CInterface@@QAAKPAUUFN_MDD_CONTEXT@@W4_UFN_BUS_SPEED@@E@Z 10026b2c f   usb_ufnmddbase_common_topaz_v1:descript.obj
 0001:00025dc4       ??0CMddEndpoint@@QAA@XZ    10026dc4 f   usb_ufnmddbase_common_topaz_v1:descript.obj
 0001:00025df8       ??1CMddEndpoint@@QAA@XZ    10026df8 f   usb_ufnmddbase_common_topaz_v1:descript.obj
 0001:00025e0c       ?Init@CMddEndpoint@@QAAKW4_UFN_BUS_SPEED@@PAU_UFN_ENDPOINT@@@Z 10026e0c f   usb_ufnmddbase_common_topaz_v1:descript.obj
 0001:00025e98       ?IsSupportable@CMddEndpoint@@QAAKPAUUFN_MDD_CONTEXT@@W4_UFN_BUS_SPEED@@EEE@Z 10026e98 f   usb_ufnmddbase_common_topaz_v1:descript.obj
 0001:000261b8       ?ValidateDescriptorAndChildren@CMddEndpoint@@SAKW4_UFN_BUS_SPEED@@PAU_UFN_ENDPOINT@@@Z 100271b8 f   usb_ufnmddbase_common_topaz_v1:descript.obj
 0001:000261f0       ?ValidateDescriptor@CMddEndpoint@@SAKW4_UFN_BUS_SPEED@@PAU_UFN_ENDPOINT@@@Z 100271f0 f   usb_ufnmddbase_common_topaz_v1:descript.obj
 0001:00026380       ?ValidatePacketSize@CMddEndpoint@@CAHW4_UFN_BUS_SPEED@@PAU_USB_ENDPOINT_DESCRIPTOR@@@Z 10027380 f   usb_ufnmddbase_common_topaz_v1:descript.obj
 0001:00026620       ?Serialize@CMddEndpoint@@QAAKPAEKPAK@Z 10027620 f   usb_ufnmddbase_common_topaz_v1:descript.obj
 0001:00026758       ?IsEndpointZeroSupportable@CMddEndpoint@@SAKPAUUFN_MDD_CONTEXT@@W4_UFN_BUS_SPEED@@PAU_USB_DEVICE_DESCRIPTOR@@@Z 10027758 f   usb_ufnmddbase_common_topaz_v1:descript.obj
 0001:000269c0       ?InitializeEndpointZeroDescriptor@CMddEndpoint@@SAXEPAU_USB_ENDPOINT_DESCRIPTOR@@@Z 100279c0 f   usb_ufnmddbase_common_topaz_v1:descript.obj
 0001:00026a60       ?GetTotalConfigurationDescriptorByIndex@CDevice@@QAAPAU_USB_CONFIGURATION_DESCRIPTOR@@K@Z 10027a60 f i usb_ufnmddbase_common_topaz_v1:descript.obj
 0001:00026adc       ?PddSupportsHighSpeed@@YAHPAUUFN_MDD_CONTEXT@@@Z 10027adc f i usb_ufnmddbase_common_topaz_v1:descript.obj
 0001:00026b78       ?GetTotalConfigurationDescriptorByIndex@CDescriptors@@QAAPAU_USB_CONFIGURATION_DESCRIPTOR@@W4_UFN_BUS_SPEED@@K@Z 10027b78 f i usb_ufnmddbase_common_topaz_v1:descript.obj
 0001:00026bd0       ??_ECConfiguration@@QAAPAXI@Z 10027bd0 f i usb_ufnmddbase_common_topaz_v1:descript.obj
 0001:00026c68       ??_I@YAXPAXIHP6AX0@Z@Z     10027c68 f i usb_ufnmddbase_common_topaz_v1:descript.obj
 0001:00026cd0       ??_H@YAXPAXIHP6APAX0@Z@Z   10027cd0 f i usb_ufnmddbase_common_topaz_v1:descript.obj
 0001:00026d20       ?PddSupportsMultipleConfigurations@@YAHPAUUFN_MDD_CONTEXT@@@Z 10027d20 f i usb_ufnmddbase_common_topaz_v1:descript.obj
 0001:00026dbc       ??_ECInterface@@QAAPAXI@Z  10027dbc f i usb_ufnmddbase_common_topaz_v1:descript.obj
 0001:00026e54       ??_ECMddEndpoint@@QAAPAXI@Z 10027e54 f i usb_ufnmddbase_common_topaz_v1:descript.obj
 0001:00026eec       ?GetEndpointCount@CInterface@@QBAKXZ 10027eec f i usb_ufnmddbase_common_topaz_v1:descript.obj
 0001:00026f20       ?PddSupportsAlternateInterfaces@@YAHPAUUFN_MDD_CONTEXT@@@Z 10027f20 f i usb_ufnmddbase_common_topaz_v1:descript.obj
 0001:00026fbc       ?AddRef@CUfnMddTransfer@@QAAXXZ 10027fbc f   usb_ufnmddbase_common_topaz_v1:transfer.obj
 0001:000271e0       ?Release@CUfnMddTransfer@@QAAXXZ 100281e0 f   usb_ufnmddbase_common_topaz_v1:transfer.obj
 0001:00027378       ?Init@CUfnMddTransfer@@QAAXKPAXKK0P6AK0@Z0PAVCPipeBase@@@Z 10028378 f   usb_ufnmddbase_common_topaz_v1:transfer.obj
 0001:00027530       ?CallCompletionRoutine@CUfnMddTransfer@@QAAXXZ 10028530 f   usb_ufnmddbase_common_topaz_v1:transfer.obj
 0001:0002760c       ?ReferenceTransferHandle@CUfnMddTransfer@@SAKPAV1@@Z 1002860c f   usb_ufnmddbase_common_topaz_v1:transfer.obj
 0001:000277d4       ?ConvertFromPddTransfer@CUfnMddTransfer@@SAPAV1@PAU_STransfer@@@Z 100287d4 f   usb_ufnmddbase_common_topaz_v1:transfer.obj
 0001:00027808       ??0CUfnBusDevice@@QAA@PBG000KPAX@Z 10028808 f   usb_ufnmddbase_common_topaz_v1:ufnbus.obj
 0001:00027920       ??0CUfnBus@@QAA@PBGPAUUFN_MDD_CONTEXT@@@Z 10028920 f   usb_ufnmddbase_common_topaz_v1:ufnbus.obj
 0001:00027a1c       ?Init@CUfnBus@@UAAHXZ      10028a1c f   usb_ufnmddbase_common_topaz_v1:ufnbus.obj
 0001:00027cc0       ??1CUfnBus@@UAA@XZ         10028cc0 f   usb_ufnmddbase_common_topaz_v1:ufnbus.obj
 0001:00027d24       ?CreateChild@CUfnBus@@IAAKPBGPAPAVCUfnBusDevice@@@Z 10028d24 f   usb_ufnmddbase_common_topaz_v1:ufnbus.obj
 0001:00027f94       ?OpenFunctionKey@CUfnBus@@SAKPAPAUHKEY__@@@Z 10028f94 f   usb_ufnmddbase_common_topaz_v1:ufnbus.obj
 0001:000280b0       ?PostInit@CUfnBus@@UAAHXZ  100290b0 f   usb_ufnmddbase_common_topaz_v1:ufnbus.obj
 0001:00028408       ?ActivateChild@CUfnBus@@UAAHPBG@Z 10029408 f   usb_ufnmddbase_common_topaz_v1:ufnbus.obj
 0001:00028cdc       ?DeactivateChild@CUfnBus@@UAAHPBG@Z 10029cdc f   usb_ufnmddbase_common_topaz_v1:ufnbus.obj
 0001:00028e90       ?TranslateChildBusAddr@CUfnBus@@UAAHPAU_CE_BUS_TRANSLATE_BUS_ADDR@@@Z 10029e90 f   usb_ufnmddbase_common_topaz_v1:ufnbus.obj
 0001:000290ac       ?TranslateChildSystemAddr@CUfnBus@@UAAHPAU_CE_BUS_TRANSLATE_SYSTEM_ADDR@@@Z 1002a0ac f   usb_ufnmddbase_common_topaz_v1:ufnbus.obj
 0001:00029288       ?SetChildDevicePowerState@CUfnBus@@UAAHPAU_CE_BUS_POWER_STATE@@PAPAVDeviceFolder@@@Z 1002a288 f   usb_ufnmddbase_common_topaz_v1:ufnbus.obj
 0001:000294a4       ?GetChildDevicePowerState@CUfnBus@@UAAHPAU_CE_BUS_POWER_STATE@@PAPAVDeviceFolder@@@Z 1002a4a4 f   usb_ufnmddbase_common_topaz_v1:ufnbus.obj
 0001:00029680       ?SetChildDeviceConfigurationData@CUfnBus@@UAAHPAU_CE_BUS_DEVICE_CONFIGURATION_DATA@@PAPAVDeviceFolder@@@Z 1002a680 f   usb_ufnmddbase_common_topaz_v1:ufnbus.obj
 0001:00029858       ?GetChildDeviceConfigurationData@CUfnBus@@UAAHPAU_CE_BUS_DEVICE_CONFIGURATION_DATA@@PAPAVDeviceFolder@@@Z 1002a858 f   usb_ufnmddbase_common_topaz_v1:ufnbus.obj
 0001:00029a38       ?IOControl@CUfnBus@@UAAHPAUUFN_MDD_BUS_OPEN_CONTEXT@@KPAEK1KPAK@Z 1002aa38 f   usb_ufnmddbase_common_topaz_v1:ufnbus.obj
 0001:0002a9e8       ?GetBusNamePrefix@CUfnBus@@UAAKPAGK@Z 1002b9e8 f   usb_ufnmddbase_common_topaz_v1:ufnbus.obj
 0001:0002aa34       ?CleanUpAfterClient@CUfnBus@@IAAKXZ 1002ba34 f   usb_ufnmddbase_common_topaz_v1:ufnbus.obj
 0001:0002b060       ?GetDefaultClientKey@CUfnBus@@QAAXPAGK@Z 1002c060 f   usb_ufnmddbase_common_topaz_v1:ufnbus.obj
 0001:0002b16c       ?GetDefaultClientName@CUfnBus@@QAAKPAGK@Z 1002c16c f   usb_ufnmddbase_common_topaz_v1:ufnbus.obj
 0001:0002b404       ?SetPowerState@DeviceFolder@@UAAHW4_CEDEVICE_POWER_STATE@@@Z 1002c404 f i usb_ufnmddbase_common_topaz_v1:ufnbus.obj
 0001:0002b43c       ?GetPowerState@DeviceFolder@@UAA?AW4_CEDEVICE_POWER_STATE@@XZ 1002c43c f i usb_ufnmddbase_common_topaz_v1:ufnbus.obj
 0001:0002b46c       ?Init@CUfnBusDevice@@UAAHXZ 1002c46c f i usb_ufnmddbase_common_topaz_v1:ufnbus.obj
 0001:0002b4d4       ?Init@DeviceFolder@@UAAHXZ 1002c4d4 f i usb_ufnmddbase_common_topaz_v1:ufnbus.obj
 0001:0002b524       ??_ECUfnBusDevice@@UAAPAXI@Z 1002c524 f i usb_ufnmddbase_common_topaz_v1:ufnbus.obj
 0001:0002b524       ??_GCUfnBusDevice@@UAAPAXI@Z 1002c524 f i usb_ufnmddbase_common_topaz_v1:ufnbus.obj
 0001:0002b568       ??1CUfnBusDevice@@UAA@XZ   1002c568 f i usb_ufnmddbase_common_topaz_v1:ufnbus.obj
 0001:0002b594       ?PowerUp@DefaultBusDriver@@UAAHXZ 1002c594 f i usb_ufnmddbase_common_topaz_v1:ufnbus.obj
 0001:0002b5bc       ?PowerDown@DefaultBusDriver@@UAAHXZ 1002c5bc f i usb_ufnmddbase_common_topaz_v1:ufnbus.obj
 0001:0002b5e4       ?Close@DefaultBusDriver@@UAAHXZ 1002c5e4 f i usb_ufnmddbase_common_topaz_v1:ufnbus.obj
 0001:0002b60c       ?IOControl@DefaultBusDriver@@UAAHKPAEK0KPAK@Z 1002c60c f i usb_ufnmddbase_common_topaz_v1:ufnbus.obj
 0001:0002b680       ?IsChildRemoved@DefaultBusDriver@@UAAHPBG@Z 1002c680 f i usb_ufnmddbase_common_topaz_v1:ufnbus.obj
 0001:0002b6a8       ??_GCUfnBus@@UAAPAXI@Z     1002c6a8 f i usb_ufnmddbase_common_topaz_v1:ufnbus.obj
 0001:0002b6a8       ??_ECUfnBus@@UAAPAXI@Z     1002c6a8 f i usb_ufnmddbase_common_topaz_v1:ufnbus.obj
 0001:0002b6ec       ?GetDeviceHandle@DefaultBusDriver@@QAAPAXXZ 1002c6ec f i usb_ufnmddbase_common_topaz_v1:ufnbus.obj
 0001:0002b71c       ResetEvent                 1002c71c f i usb_ufnmddbase_common_topaz_v1:ufnbus.obj
 0001:0002b754       SetEvent                   1002c754 f i usb_ufnmddbase_common_topaz_v1:ufnbus.obj
 0001:0002b78c       GetCurrentThread           1002c78c f i usb_ufnmddbase_common_topaz_v1:ufnbus.obj
 0001:0002b7a4       ?GetUfnName@CUfnBusDevice@@QAAPBGXZ 1002c7a4 f i usb_ufnmddbase_common_topaz_v1:ufnbus.obj
 0001:0002b7d0       ??0CFreeTransferList@@QAA@XZ 1002c7d0 f i usb_ufnmddbase_common_topaz_v1:ufnbus.obj
 0001:0002b808       ?Compact@CFreeTransferList@@QAAXXZ 1002c808 f i usb_ufnmddbase_common_topaz_v1:ufnbus.obj
 0001:0002b824       ?PddSupportsReusableEndpoints@@YAHPAUUFN_MDD_CONTEXT@@@Z 1002c824 f i usb_ufnmddbase_common_topaz_v1:ufnbus.obj
 0001:0002b8c4       ?DeRef@CRefObject@@QAAKXZ  1002c8c4 f i usb_ufnmddbase_common_topaz_v1:ufnbus.obj
 0001:0002b960       ?GetHKey@CRegistryEdit@@QAAPAUHKEY__@@XZ 1002c960 f i usb_ufnmddbase_common_topaz_v1:ufnbus.obj
 0001:0002b98c       ?IsClientPresent@CUfnBus@@IAAHXZ 1002c98c f i usb_ufnmddbase_common_topaz_v1:ufnbus.obj
 0001:0002b9e0       ?ChangeDeviceState@@YAXPAUUFN_MDD_CONTEXT@@W4DEVICE_STATE@@@Z 1002c9e0 f i usb_ufnmddbase_common_topaz_v1:ufnbus.obj
 0001:0002bac0       ??_GCFreeTransferList@@QAAPAXI@Z 1002cac0 f i usb_ufnmddbase_common_topaz_v1:ufnbus.obj
 0001:0002bb04       ??1CFreeTransferList@@QAA@XZ 1002cb04 f i usb_ufnmddbase_common_topaz_v1:ufnbus.obj
 0001:0002bb20       ??0?$CFreePool@$00V?$fixed_block_allocator@$07@ce@@Utransfer_funcs@@@@QAA@I@Z 1002cb20 f i usb_ufnmddbase_common_topaz_v1:ufnbus.obj
 0001:0002bb80       ??1?$CFreePool@$00V?$fixed_block_allocator@$07@ce@@Utransfer_funcs@@@@QAA@XZ 1002cb80 f i usb_ufnmddbase_common_topaz_v1:ufnbus.obj
 0001:0002bcd0       ?compact@?$CFreePool@$00V?$fixed_block_allocator@$07@ce@@Utransfer_funcs@@@@QAAXXZ 1002ccd0 f i usb_ufnmddbase_common_topaz_v1:ufnbus.obj
 0001:0002bdf0       ?init@?$CFreePool@$00V?$fixed_block_allocator@$07@ce@@Utransfer_funcs@@@@IAAXI@Z 1002cdf0 f i usb_ufnmddbase_common_topaz_v1:ufnbus.obj
 0001:0002be88       ??0?$fixed_block_allocator@$07@ce@@QAA@XZ 1002ce88 f i usb_ufnmddbase_common_topaz_v1:ufnbus.obj
 0001:0002bebc       ??1?$fixed_block_allocator@$07@ce@@QAA@XZ 1002cebc f i usb_ufnmddbase_common_topaz_v1:ufnbus.obj
 0001:0002bf64       ?compact@?$fixed_block_allocator@$07@ce@@QBAXXZ 1002cf64 f i usb_ufnmddbase_common_topaz_v1:ufnbus.obj
 0001:0002bf9c       ??0?$interlocked_stack@PAXV?$fixed_block_allocator@$07@ce@@@@QAA@XZ 1002cf9c f i usb_ufnmddbase_common_topaz_v1:ufnbus.obj
 0001:0002bfe0       ??1?$interlocked_stack@PAXV?$fixed_block_allocator@$07@ce@@@@QAA@XZ 1002cfe0 f i usb_ufnmddbase_common_topaz_v1:ufnbus.obj
 0001:0002bffc       ?_Initialize@?$fixed_block_allocator@$07@ce@@IAAXI@Z 1002cffc f i usb_ufnmddbase_common_topaz_v1:ufnbus.obj
 0001:0002c058       ?GetDeviceStateName@@YAPBGW4DEVICE_STATE@@@Z 1002d058 f   usb_ufnmddbase_common_topaz_v1:enum.obj
 0001:0002c0e4       ?UfnMdd_Notify@@YAHPAXKK@Z 1002d0e4 f   usb_ufnmddbase_common_topaz_v1:enum.obj
 0001:0002fcb0       ?SetConfiguration@CDescriptors@@QAAKW4_UFN_BUS_SPEED@@K@Z 10030cb0 f i usb_ufnmddbase_common_topaz_v1:enum.obj
 0001:0002fd00       ?SetConfiguration@CDevice@@QAAKK@Z 10030d00 f i usb_ufnmddbase_common_topaz_v1:enum.obj
 0001:0002fd98       ?ResetInterfaces@CConfiguration@@QAAXXZ 10030d98 f i usb_ufnmddbase_common_topaz_v1:enum.obj
 0001:0002fdfc       ?GetDefaultInterfaceCount@CConfiguration@@QBAKXZ 10030dfc f i usb_ufnmddbase_common_topaz_v1:enum.obj
 0001:0002fea8       ?SetInterface@CConfiguration@@QAAKKK@Z 10030ea8 f i usb_ufnmddbase_common_topaz_v1:enum.obj
 0001:0002ff4c       ?SetInterface@CInterface@@QAAXK@Z 10030f4c f i usb_ufnmddbase_common_topaz_v1:enum.obj
 0001:0002ffc8       ?GetTotalConfigurationDescriptorByValue@CDescriptors@@QAAPBU_USB_CONFIGURATION_DESCRIPTOR@@W4_UFN_BUS_SPEED@@K@Z 10030fc8 f i usb_ufnmddbase_common_topaz_v1:enum.obj
 0001:00030020       ?GetTotalConfigurationDescriptorByValue@CDevice@@QAAPBU_USB_CONFIGURATION_DESCRIPTOR@@K@Z 10031020 f i usb_ufnmddbase_common_topaz_v1:enum.obj
 0001:00030084       ?GetDefaultInterfaceCount@CDescriptors@@QAAKW4_UFN_BUS_SPEED@@@Z 10031084 f i usb_ufnmddbase_common_topaz_v1:enum.obj
 0001:000300d0       ?GetDefaultInterfaceCount@CDevice@@QBAKXZ 100310d0 f i usb_ufnmddbase_common_topaz_v1:enum.obj
 0001:00030130       ?SetInterface@CDescriptors@@QAAKW4_UFN_BUS_SPEED@@KK@Z 10031130 f i usb_ufnmddbase_common_topaz_v1:enum.obj
 0001:00030184       ?SetInterface@CDevice@@QAAKKK@Z 10031184 f i usb_ufnmddbase_common_topaz_v1:enum.obj
 0001:0003026c       FslUfnIsUSBKitlEnable      1003126c f   usb_usbfn_os_mx25_topaz_v1:i_os.obj
 0001:00030300       FslUfnGetUsbFnPdd          10031300 f   usb_usbfn_os_mx25_topaz_v1:i_os.obj
 0001:00030334       FslUfnRequestIrq           10031334 f   usb_usbfn_os_mx25_topaz_v1:i_os.obj
 0001:00030660       FslUfnGetDMABuffer         10031660 f   usb_usbfn_os_mx25_topaz_v1:i_os.obj
 0001:0003089c       FslUfnCreateThread         1003189c f   usb_usbfn_os_mx25_topaz_v1:i_os.obj
 0001:000309ac       FslUfnTrigIrq              100319ac f   usb_usbfn_os_mx25_topaz_v1:i_os.obj
 0001:000309d0       FslUfnDeinit               100319d0 f   usb_usbfn_os_mx25_topaz_v1:i_os.obj
 0001:00030c34       InterruptThread            10031c34 f   usb_usbfn_os_mx25_topaz_v1:i_os.obj
 0001:00031608       FslUfnGetPageNumber        10032608 f   usb_usbfn_os_mx25_topaz_v1:i_os.obj
 0001:00031690       FslUfnGetPageSize          10032690 f   usb_usbfn_os_mx25_topaz_v1:i_os.obj
 0001:000316b0       FslUfnGetPageShift         100326b0 f   usb_usbfn_os_mx25_topaz_v1:i_os.obj
 0001:000316d0       FslInitializeCriticalSection 100326d0 f   usb_usbfn_os_mx25_topaz_v1:i_os.obj
 0001:000316ec       FslEnterCriticalSection    100326ec f   usb_usbfn_os_mx25_topaz_v1:i_os.obj
 0001:00031708       FslLeaveCriticalSection    10032708 f   usb_usbfn_os_mx25_topaz_v1:i_os.obj
 0001:00031724       FslNKDbgPrintfW            10032724 f   usb_usbfn_os_mx25_topaz_v1:i_os.obj
 0001:00031760       svsutil_Initialize         10032760 f   ceosutil:utilmem.obj
 0001:000318c4       svsutil_DeInitialize       100328c4 f   ceosutil:utilmem.obj
 0001:00031988       svsutil_TotalAlloc         10032988 f   ceosutil:utilmem.obj
 0001:000319a8       svsutil_LogCallStack       100329a8 f   ceosutil:utilmem.obj
 0001:000319ac       svsutil_Alloc              100329ac f   ceosutil:utilmem.obj
 0001:00031b90       svsutil_ReAlloc            10032b90 f   ceosutil:utilmem.obj
 0001:00031e60       svsutil_Free               10032e60 f   ceosutil:utilmem.obj
 0001:0003216c       svsutil_SetAlloc           1003316c f   ceosutil:utilmem.obj
 0001:000321f0       svsutil_SetAllocData       100331f0 f   ceosutil:utilmem.obj
 0001:00032224       svsutil_AllocFixedMemDescrSynch 10033224 f   ceosutil:utilmemf.obj
 0001:00032370       svsutil_AllocFixedMemDescr 10033370 f   ceosutil:utilmemf.obj
 0001:000323ac       svsutil_IsFixedEmpty       100333ac f   ceosutil:utilmemf.obj
 0001:000323fc       svsutil_FixedBlockSize     100333fc f   ceosutil:utilmemf.obj
 0001:0003242c       svsutil_GetFixed           1003342c f   ceosutil:utilmemf.obj
 0001:000325e8       svsutil_FreeFixed          100335e8 f   ceosutil:utilmemf.obj
 0001:00032768       svsutil_ReleaseFixedNonEmpty 10033768 f   ceosutil:utilmemf.obj
 0001:00032840       svsutil_ReleaseFixedEmpty  10033840 f   ceosutil:utilmemf.obj
 0001:00032968       svsutil_CompactFixed       10033968 f   ceosutil:utilmemf.obj
 0001:00032f60       svsutil_GetFixedStats      10033f60 f   ceosutil:utilmemf.obj
 0001:0003307c       ?LocateLeftNeighbor@SVSTree@@QAAPAVSVSTNode@@K@Z 1003407c f i ceosutil:utilmemf.obj
 0001:000331ac       ?Prev@SVSTree@@QAAPAVSVSTNode@@PAV2@@Z 100341ac f i ceosutil:utilmemf.obj
 0001:000332cc       ?GetData@SVSTree@@SAPAXPAVSVSTNode@@@Z 100342cc f i ceosutil:utilmemf.obj
 0001:000332fc       ?SVSNewTree@@YAPAVSVSTree@@I@Z 100342fc f i ceosutil:utilmemf.obj
 0001:000333ec       ??2SVSAllocClass@@SAPAXI@Z 100343ec f i ceosutil:utilmemf.obj
 0001:00033478       ?IsTreeInitialized@SVSTree@@QAAHXZ 10034478 f i ceosutil:utilmemf.obj
 0001:000334c8       ??0SVSTree@@QAA@I@Z        100344c8 f i ceosutil:utilmemf.obj
 0001:000336a0       ?InitializeMembers@SVSTree@@IAAXXZ 100346a0 f i ceosutil:utilmemf.obj
 0001:00033704       ?EnumStart@SVSTree@@UAAKXZ 10034704 f i ceosutil:utilmemf.obj
 0001:00033738       ?Min@SVSTree@@QAAPAVSVSTNode@@XZ 10034738 f i ceosutil:utilmemf.obj
 0001:000337c8       ?EnumNext@SVSTree@@UAAKK@Z 100347c8 f i ceosutil:utilmemf.obj
 0001:00033800       ?Next@SVSTree@@QAAPAVSVSTNode@@PAV2@@Z 10034800 f i ceosutil:utilmemf.obj
 0001:00033920       ?EnumGetData@SVSTree@@UAAPAXK@Z 10034920 f i ceosutil:utilmemf.obj
 0001:00033954       ?EnumGetKey@SVSTree@@UAAKK@Z 10034954 f i ceosutil:utilmemf.obj
 0001:00033988       ?GetKey@SVSTree@@SAKPAVSVSTNode@@@Z 10034988 f i ceosutil:utilmemf.obj
 0001:000339b4       ??0SVSEnumClass@@QAA@XZ    100349b4 f i ceosutil:utilmemf.obj
 0001:000339ec       ??_GSVSTree@@QAAPAXI@Z     100349ec f i ceosutil:utilmemf.obj
 0001:00033a30       ??3SVSAllocClass@@SAXPAX@Z 10034a30 f i ceosutil:utilmemf.obj
 0001:00033a68       ??1SVSTree@@QAA@XZ         10034a68 f i ceosutil:utilmemf.obj
 0001:00033aec       ?Empty@SVSTree@@QAAXXZ     10034aec f i ceosutil:utilmemf.obj
 0001:00033b44       ?DeleteSubtree@SVSTree@@IAAXPAVSVSTNode@@@Z 10034b44 f i ceosutil:utilmemf.obj
 0001:00033c40       svsutil_AssertBroken       10034c40 f   ceosutil:svsutil.obj
 0001:00033c9c       svsutil_wcsdup             10034c9c f   ceosutil:svsutil.obj
 0001:00033d3c       svsutil_strdup             10034d3c f   ceosutil:svsutil.obj
 0001:00033dd4       svsutil_OpenAndReadFile    10034dd4 f   ceosutil:svsutil.obj
 0001:00033fd0       ?svsutil_ReportEventPrintf@@YAHPAXGPAGZZ 10034fd0 f   ceosutil:svsutil.obj
 0001:000340e8       ?svsutil_ReportEventPrintfRC@@YAHPAXPAUHINSTANCE__@@KGZZ 100350e8 f   ceosutil:svsutil.obj
 0001:00034240       ??$_vsnwprintf_s@$0IA@@@YAHAAY0IA@GIPBGPAD@Z 10035240 f i ceosutil:svsutil.obj
 0001:00034288       svsutil_GetTree            10035288 f   ceosutil:utiltree.obj
 0001:000342bc       svsutil_EmptyTree          100352bc f   ceosutil:utiltree.obj
 0001:00034310       svsutil_EmptyTreeWithCallback 10035310 f   ceosutil:utiltree.obj
 0001:00034378       svsutil_DestroyTree        10035378 f   ceosutil:utiltree.obj
 0001:00034404       svsutil_NextTreeNode       10035404 f   ceosutil:utiltree.obj
 0001:00034478       svsutil_PrevTreeNode       10035478 f   ceosutil:utiltree.obj
 0001:000344ec       svsutil_MinTreeNode        100354ec f   ceosutil:utiltree.obj
 0001:00034550       svsutil_MaxTreeNode        10035550 f   ceosutil:utiltree.obj
 0001:000345b4       svsutil_LocateTreeNode     100355b4 f   ceosutil:utiltree.obj
 0001:0003461c       svsutil_LocateLeftNeighborNode 1003561c f   ceosutil:utiltree.obj
 0001:00034684       ?svsutil_LocateRightNeighborNode@@YAPAVSVSTNode@@PAVSVSTree@@K@Z 10035684 f   ceosutil:utiltree.obj
 0001:000346ec       svsutil_TreeToArray        100356ec f   ceosutil:utiltree.obj
 0001:00034754       svsutil_GetTreeSize        10035754 f   ceosutil:utiltree.obj
 0001:000347b8       svsutil_InsertTreeNode     100357b8 f   ceosutil:utiltree.obj
 0001:00034824       svsutil_DeleteTreeNode     10035824 f   ceosutil:utiltree.obj
 0001:00034898       svsutil_GetTreeNodeData    10035898 f   ceosutil:utiltree.obj
 0001:000348fc       svsutil_GetTreeNodeKey     100358fc f   ceosutil:utiltree.obj
 0001:00034960       svsutil_CompactTree        10035960 f   ceosutil:utiltree.obj
 0001:000349b4       ?Insert@SVSTree@@QAAPAVSVSTNode@@KPAX@Z 100359b4 f   ceosutil:utiltree.obj
 0001:00034d5c       ?DeleteFixup@SVSTree@@IAAXPAVSVSTNode@@@Z 10035d5c f   ceosutil:utiltree.obj
 0001:0003514c       ?Delete@SVSTree@@QAAPAXPAVSVSTNode@@@Z 1003614c f   ceosutil:utiltree.obj
 0001:0003554c       ?RBTreeIntegrity@SVSTree@@IAAXXZ 1003654c f   ceosutil:utiltree.obj
 0001:00035968       ?CheckBlackHeight@SVSTree@@IAAHPAVSVSTNode@@@Z 10036968 f   ceosutil:utiltree.obj
 0001:00035ba8       ?InTree@SVSTree@@IAAHPAVSVSTNode@@@Z 10036ba8 f   ceosutil:utiltree.obj
 0001:00035c40       ?Empty@SVSTree@@QAAXP6AXPAX0@Z0@Z 10036c40 f i ceosutil:utiltree.obj
 0001:00035ca0       ?DeleteSubtree@SVSTree@@IAAXPAVSVSTNode@@P6AXPAX1@Z1@Z 10036ca0 f i ceosutil:utiltree.obj
 0001:00035d38       ?Max@SVSTree@@QAAPAVSVSTNode@@XZ 10036d38 f i ceosutil:utiltree.obj
 0001:00035dc8       ?Locate@SVSTree@@QAAPAVSVSTNode@@K@Z 10036dc8 f i ceosutil:utiltree.obj
 0001:00035e8c       ?LocateRightNeighbor@SVSTree@@QAAPAVSVSTNode@@K@Z 10036e8c f i ceosutil:utiltree.obj
 0001:00035fbc       ?ToArray@SVSTree@@QAAIPAPAX@Z 10036fbc f i ceosutil:utiltree.obj
 0001:00036000       ?SubtreeToArray@SVSTree@@IAAIPAVSVSTNode@@AAPAPAX@Z 10037000 f i ceosutil:utiltree.obj
 0001:0003610c       ?Size@SVSTree@@QAAIXZ      1003710c f i ceosutil:utiltree.obj
 0001:0003613c       ?Compact@SVSTree@@QAAXXZ   1003713c f i ceosutil:utiltree.obj
 0001:00036160       ?TreeInsert@SVSTree@@IAAXPAVSVSTNode@@@Z 10037160 f i ceosutil:utiltree.obj
 0001:00036290       ?LeftRotate@SVSTree@@IAAXPAVSVSTNode@@@Z 10037290 f i ceosutil:utiltree.obj
 0001:000363cc       ?RightRotate@SVSTree@@IAAXPAVSVSTNode@@@Z 100373cc f i ceosutil:utiltree.obj
 0001:00036508       ??0DeviceFolder@@QAA@PBG0KKKKPAXK0@Z 10037508 f   defbuslib:DefBus.obj
 0001:00036adc       ??1DeviceFolder@@UAA@XZ    10037adc f   defbuslib:DefBus.obj
 0001:00036c88       ?AddInitReg@DeviceFolder@@QAAHHPAU_REGINI@@@Z 10037c88 f   defbuslib:DefBus.obj
 0001:00036ff0       ?LoadDevice@DeviceFolder@@UAAHXZ 10037ff0 f   defbuslib:DefBus.obj
 0001:00037674       ?UnloadDevice@DeviceFolder@@UAAHXZ 10038674 f   defbuslib:DefBus.obj
 0001:0003773c       ?SetConfigurationData@DeviceFolder@@UAAHPAU_CE_BUS_DEVICE_CONFIGURATION_DATA@@@Z 1003873c f   defbuslib:DefBus.obj
 0001:00037854       ?GetConfigurationData@DeviceFolder@@UAAHPAU_CE_BUS_DEVICE_CONFIGURATION_DATA@@@Z 10038854 f   defbuslib:DefBus.obj
 0001:0003796c       ?DebugZoneChk@DeviceFolder@@UAAKK@Z 1003896c f   defbuslib:DefBus.obj
 0001:00037a38       ??0DefaultBusDriver@@QAA@PBG@Z 10038a38 f   defbuslib:DefBus.obj
 0001:00037b48       ?Init@DefaultBusDriver@@UAAHXZ 10038b48 f   defbuslib:DefBus.obj
 0001:00037bac       ??1DefaultBusDriver@@UAA@XZ 10038bac f   defbuslib:DefBus.obj
 0001:00037ce4       ?TranslateChildBusAddr@DefaultBusDriver@@UAAHPAU_CE_BUS_TRANSLATE_BUS_ADDR@@@Z 10038ce4 f   defbuslib:DefBus.obj
 0001:00037d90       ?TranslateChildSystemAddr@DefaultBusDriver@@UAAHPAU_CE_BUS_TRANSLATE_SYSTEM_ADDR@@@Z 10038d90 f   defbuslib:DefBus.obj
 0001:00037e2c       ?SetChildDeviceConfigurationData@DefaultBusDriver@@UAAHPAU_CE_BUS_DEVICE_CONFIGURATION_DATA@@PAPAVDeviceFolder@@@Z 10038e2c f   defbuslib:DefBus.obj
 0001:00037edc       ?GetChildDeviceConfigurationData@DefaultBusDriver@@UAAHPAU_CE_BUS_DEVICE_CONFIGURATION_DATA@@PAPAVDeviceFolder@@@Z 10038edc f   defbuslib:DefBus.obj
 0001:00037f8c       ?SetChildDevicePowerState@DefaultBusDriver@@UAAHPAU_CE_BUS_POWER_STATE@@PAPAVDeviceFolder@@@Z 10038f8c f   defbuslib:DefBus.obj
 0001:0003806c       ?GetChildDevicePowerState@DefaultBusDriver@@UAAHPAU_CE_BUS_POWER_STATE@@PAPAVDeviceFolder@@@Z 1003906c f   defbuslib:DefBus.obj
 0001:00038150       ?ActivateChild@DefaultBusDriver@@UAAHPBG@Z 10039150 f   defbuslib:DefBus.obj
 0001:000381ec       ?DeactivateChild@DefaultBusDriver@@UAAHPBG@Z 100391ec f   defbuslib:DefBus.obj
 0001:00038288       ?GetBusNamePrefix@DefaultBusDriver@@UAAKPAGK@Z 10039288 f   defbuslib:DefBus.obj
 0001:00038334       ?FastIOControl@DefaultBusDriver@@UAAHKPAEK0KPAKPAPAVDeviceFolder@@@Z 10039334 f   defbuslib:DefBus.obj
 0001:00038abc       ?GetChildByName@DefaultBusDriver@@UAAPAVDeviceFolder@@PBGPAPAV2@@Z 10039abc f   defbuslib:DefBus.obj
 0001:00038d14       ?InsertChild@DefaultBusDriver@@UAAHPAVDeviceFolder@@@Z 10039d14 f   defbuslib:DefBus.obj
 0001:00038df0       ?RemoveChildByName@DefaultBusDriver@@UAAHPBG@Z 10039df0 f   defbuslib:DefBus.obj
 0001:00038e9c       ?RemoveChildByFolder@DefaultBusDriver@@UAAHPAVDeviceFolder@@@Z 10039e9c f   defbuslib:DefBus.obj
 0001:00038fb4       ?Open@DefaultBusDriver@@UAAHKK@Z 10039fb4 f   defbuslib:DefBus.obj
 0001:00038ffc       ??0CLockObject@@QAA@XZ     10039ffc f i defbuslib:DefBus.obj
 0001:0003902c       ??0CRefObject@@QAA@XZ      1003a02c f i defbuslib:DefBus.obj
 0001:00039074       ??_ECRefObject@@UAAPAXI@Z  1003a074 f i defbuslib:DefBus.obj
 0001:00039074       ??_GCRefObject@@UAAPAXI@Z  1003a074 f i defbuslib:DefBus.obj
 0001:000390b8       ??1CRefObject@@UAA@XZ      1003a0b8 f i defbuslib:DefBus.obj
 0001:000390dc       ??0CRegistryEdit@@QAA@PAUHKEY__@@PBG@Z 1003a0dc f i defbuslib:DefBus.obj
 0001:00039154       ?GetRegValue@CRegistryEdit@@QAAHPBGPAEK@Z 1003a154 f i defbuslib:DefBus.obj
 0001:000391d8       ?IsKeyOpened@CRegistryEdit@@QAAHXZ 1003a1d8 f i defbuslib:DefBus.obj
 0001:00039224       ??_EDeviceFolder@@UAAPAXI@Z 1003a224 f i defbuslib:DefBus.obj
 0001:00039224       ??_GDeviceFolder@@UAAPAXI@Z 1003a224 f i defbuslib:DefBus.obj
 0001:00039268       ??1CLockObject@@QAA@XZ     1003a268 f i defbuslib:DefBus.obj
 0001:00039284       ??1CRegistryEdit@@QAA@XZ   1003a284 f i defbuslib:DefBus.obj
 0001:000392b4       ?GetLoadFlag@DeviceFolder@@QAAKXZ 1003a2b4 f i defbuslib:DefBus.obj
 0001:000392e4       ?PostInit@DefaultBusDriver@@UAAHXZ 1003a2e4 f i defbuslib:DefBus.obj
 0001:0003930c       ??_GDefaultBusDriver@@UAAPAXI@Z 1003a30c f i defbuslib:DefBus.obj
 0001:0003930c       ??_EDefaultBusDriver@@UAAPAXI@Z 1003a30c f i defbuslib:DefBus.obj
 0001:00039350       ?GetNextDeviceFolder@DeviceFolder@@QAAPAV1@XZ 1003a350 f i defbuslib:DefBus.obj
 0001:00039380       ?TakeWriteLock@DefaultBusDriver@@QAAXXZ 1003a380 f i defbuslib:DefBus.obj
 0001:000393d8       ?Lock@CLockObject@@QAAXXZ  1003a3d8 f i defbuslib:DefBus.obj
 0001:000393f4       ?Unlock@CLockObject@@QAAXXZ 1003a3f4 f i defbuslib:DefBus.obj
 0001:00039410       ?LeaveWriteLock@DefaultBusDriver@@QAAXXZ 1003a410 f i defbuslib:DefBus.obj
 0001:00039430       ?TranslateBusAddr@DefaultBusDriver@@QAAHW4_INTERFACE_TYPE@@KT_LARGE_INTEGER@@PAKPAT3@@Z 1003a430 f i defbuslib:DefBus.obj
 0001:000394e4       ?TranslateSystemAddr@DefaultBusDriver@@QAAHW4_INTERFACE_TYPE@@KT_LARGE_INTEGER@@PAT3@@Z 1003a4e4 f i defbuslib:DefBus.obj
 0001:00039588       ?AddRef@CRefObject@@QAAKXZ 1003a588 f i defbuslib:DefBus.obj
 0001:000395c0       ?GetDeviceBusName@DeviceFolder@@QAAPBGXZ 1003a5c0 f i defbuslib:DefBus.obj
 0001:000395f0       ?TakeReadLock@DefaultBusDriver@@QAAXXZ 1003a5f0 f i defbuslib:DefBus.obj
 0001:00039638       ?LeaveReadLock@DefaultBusDriver@@QAAXXZ 1003a638 f i defbuslib:DefBus.obj
 0001:00039694       ?SetNextDeviceFolder@DeviceFolder@@QAAXPAV1@@Z 1003a694 f i defbuslib:DefBus.obj
 0001:000396b8       BusChildIoControl          1003a6b8 f   ceddk:CEDDK.dll
 0001:000396c8       CreateBusAccessHandle      1003a6c8 f   ceddk:CEDDK.dll
 0001:000396d8       CloseBusAccessHandle       1003a6d8 f   ceddk:CEDDK.dll
 0001:000396e8       HalAllocateCommonBuffer    1003a6e8 f   ceddk:CEDDK.dll
 0001:000396f8       HalFreeCommonBuffer        1003a6f8 f   ceddk:CEDDK.dll
 0001:00039708       MmUnmapIoSpace             1003a708 f   ceddk:CEDDK.dll
 0001:00039718       SetDevicePowerState        1003a718 f   ceddk:CEDDK.dll
 0001:00039728       HalSetBusDataByOffset      1003a728 f   ceddk:CEDDK.dll
 0001:00039738       HalGetBusDataByOffset      1003a738 f   ceddk:CEDDK.dll
 0001:00039748       HalTranslateBusAddress     1003a748 f   ceddk:CEDDK.dll
 0001:00039758       TranslateBusAddr           1003a758 f   ceddk:CEDDK.dll
 0001:00039768       HalTranslateSystemAddress  1003a768 f   ceddk:CEDDK.dll
 0001:00039778       TranslateSystemAddr        1003a778 f   ceddk:CEDDK.dll
 0001:00039788       NKDbgPrintfW               1003a788 f   coredll:COREDLL.dll
 0001:00039798       Sleep                      1003a798 f   coredll:COREDLL.dll
 0001:000397a8       InterlockedCompareExchange 1003a7a8 f   coredll:COREDLL.dll
 0001:000397b8       GetLastError               1003a7b8 f   coredll:COREDLL.dll
 0001:000397c8       MapViewOfFile              1003a7c8 f   coredll:COREDLL.dll
 0001:000397d8       CreateFileMappingW         1003a7d8 f   coredll:COREDLL.dll
 0001:000397e8       CloseHandle                1003a7e8 f   coredll:COREDLL.dll
 0001:000397f8       UnmapViewOfFile            1003a7f8 f   coredll:COREDLL.dll
 0001:00039808       KernelIoControl            1003a808 f   coredll:COREDLL.dll
 0001:00039818       LeaveCriticalSection       1003a818 f   coredll:COREDLL.dll
 0001:00039828       EnterCriticalSection       1003a828 f   coredll:COREDLL.dll
 0001:00039838       CeLogData                  1003a838 f   coredll:COREDLL.dll
 0001:00039848       StringCchLengthW           1003a848 f   coredll:COREDLL.dll
 0001:00039858       StringCchVPrintfW          1003a858 f   coredll:COREDLL.dll
 0001:00039868       OpenDeviceKey              1003a868 f   coredll:COREDLL.dll
 0001:00039878       CreateEventW               1003a878 f   coredll:COREDLL.dll
 0001:00039888       InitializeCriticalSection  1003a888 f   coredll:COREDLL.dll
 0001:00039898       LocalAlloc                 1003a898 f   coredll:COREDLL.dll
 0001:000398a8       RegOpenKeyExW              1003a8a8 f   coredll:COREDLL.dll
 0001:000398b8       LocalFree                  1003a8b8 f   coredll:COREDLL.dll
 0001:000398c8       RegCloseKey                1003a8c8 f   coredll:COREDLL.dll
 0001:000398d8       DeleteCriticalSection      1003a8d8 f   coredll:COREDLL.dll
 0001:000398e8       SetLastError               1003a8e8 f   coredll:COREDLL.dll
 0001:000398f8       DisableThreadLibraryCalls  1003a8f8 f   coredll:COREDLL.dll
 0001:00039908       RegisterDbgZones           1003a908 f   coredll:COREDLL.dll
 0001:00039918       OutputDebugStringW         1003a918 f   coredll:COREDLL.dll
 0001:00039928       __GetUserKData             1003a928 f   coredll:COREDLL.dll
 0001:00039938       InterlockedIncrement       1003a938 f   coredll:COREDLL.dll
 0001:00039948       InterlockedDecrement       1003a948 f   coredll:COREDLL.dll
 0001:00039958       InterlockedExchange        1003a958 f   coredll:COREDLL.dll
 0001:00039968       StringCchCopyNW            1003a968 f   coredll:COREDLL.dll
 0001:00039978       StringCchCopyW             1003a978 f   coredll:COREDLL.dll
 0001:00039988       StringCchPrintfW           1003a988 f   coredll:COREDLL.dll
 0001:00039998       GetDeviceInformationByDeviceHandle 1003a998 f   coredll:COREDLL.dll
 0001:000399a8       EventModify                1003a9a8 f   coredll:COREDLL.dll
 0001:000399b8       LoadLibraryW               1003a9b8 f   coredll:COREDLL.dll
 0001:000399c8       RegQueryValueExW           1003a9c8 f   coredll:COREDLL.dll
 0001:000399d8       RegSetValueExW             1003a9d8 f   coredll:COREDLL.dll
 0001:000399e8       RegEnumKeyExW              1003a9e8 f   coredll:COREDLL.dll
 0001:000399f8       WaitForSingleObject        1003a9f8 f   coredll:COREDLL.dll
 0001:00039a08       InterruptInitialize        1003aa08 f   coredll:COREDLL.dll
 0001:00039a18       AllocPhysMem               1003aa18 f   coredll:COREDLL.dll
 0001:00039a28       CeSetThreadPriority        1003aa28 f   coredll:COREDLL.dll
 0001:00039a38       CreateThread               1003aa38 f   coredll:COREDLL.dll
 0001:00039a48       FreePhysMem                1003aa48 f   coredll:COREDLL.dll
 0001:00039a58       InterruptDisable           1003aa58 f   coredll:COREDLL.dll
 0001:00039a68       ExitThread                 1003aa68 f   coredll:COREDLL.dll
 0001:00039a78       InterruptDone              1003aa78 f   coredll:COREDLL.dll
 0001:00039a88       StringCchCatW              1003aa88 f   coredll:COREDLL.dll
 0001:00039a98       NKvDbgPrintfW              1003aa98 f   coredll:COREDLL.dll
 0001:00039aa8       ReadFile                   1003aaa8 f   coredll:COREDLL.dll
 0001:00039ab8       GetFileSize                1003aab8 f   coredll:COREDLL.dll
 0001:00039ac8       CreateFileW                1003aac8 f   coredll:COREDLL.dll
 0001:00039ad8       ReportEventW               1003aad8 f   coredll:COREDLL.dll
 0001:00039ae8       LoadStringW                1003aae8 f   coredll:COREDLL.dll
 0001:00039af8       FreeLibrary                1003aaf8 f   coredll:COREDLL.dll
 0001:00039b08       GetProcAddressW            1003ab08 f   coredll:COREDLL.dll
 0001:00039b18       LoadDriver                 1003ab18 f   coredll:COREDLL.dll
 0001:00039b28       ActivateDeviceEx           1003ab28 f   coredll:COREDLL.dll
 0001:00039b38       GetTickCount               1003ab38 f   coredll:COREDLL.dll
 0001:00039b48       DeactivateDevice           1003ab48 f   coredll:COREDLL.dll
 0001:00039b58       GetDeviceHandleFromContext 1003ab58 f   coredll:COREDLL.dll
 0001:00039b68       DDKClockSetGatingMode      1003ab68 f   cspddk:CSPDDK.dll
 0001:00039b78       DDKClockGetGatingMode      1003ab78 f   cspddk:CSPDDK.dll
 0001:00039b88       DDKClockConfigBaud         1003ab88 f   cspddk:CSPDDK.dll
 0001:00039b98       _DllEntryCRTStartup        1003ab98 f   corelib0:pegdentry.obj
 0001:00039c08       __security_init_cookie     1003ac08 f   corelib0:seccinit.obj
 0001:00039cd0       __GSHandlerCheck           1003acd0 f   corelib0:gshandler.obj
 0001:00039d18       __GSHandlerCheckCommon     1003ad18 f   corelib0:gshandler.obj
 0001:00039dc0       __security_check_cookie    1003adc0 f   corelib0:armsecgs.obj
 0001:00039dd4       __gsfailure                1003add4 f   corelib0:armsecgs.obj
 0001:00039e20       _onexit                    1003ae20 f   corelib0:onexit.obj
 0001:0003a124       atexit                     1003b124 f   corelib0:onexit.obj
 0001:0003a178       exit                       1003b178 f   corelib0:cexit.obj
 0001:0003a2f8       _exit                      1003b2f8 f   corelib0:cexit.obj
 0001:0003a31c       _cexit                     1003b31c f   corelib0:cexit.obj
 0001:0003a338       _c_exit                    1003b338 f   corelib0:cexit.obj
 0001:0003a354       GetCurrentProcess          1003b354 f i corelib0:cexit.obj
 0001:0003a36c       _initterm                  1003b36c f   corelib0:crt0dat.obj
 0001:0003a3c0       _cinit                     1003b3c0 f   corelib0:crt0dat.obj
 0001:0003a3f4       ??2@YAPAXI@Z               1003b3f4 f   corelib1:COREDLL.dll
 0001:0003a404       __C_specific_handler       1003b404 f   corelib1:COREDLL.dll
 0001:0003a414       ??3@YAXPAX@Z               1003b414 f   corelib1:COREDLL.dll
 0001:0003a424       memcpy                     1003b424 f   corelib1:COREDLL.dll
 0001:0003a434       _purecall                  1003b434 f   corelib1:COREDLL.dll
 0001:0003a444       memset                     1003b444 f   corelib1:COREDLL.dll
 0001:0003a454       wcslen                     1003b454 f   corelib1:COREDLL.dll
 0001:0003a464       ??_V@YAXPAX@Z              1003b464 f   corelib1:COREDLL.dll
 0001:0003a474       ??_U@YAPAXI@Z              1003b474 f   corelib1:COREDLL.dll
 0001:0003a484       malloc                     1003b484 f   corelib1:COREDLL.dll
 0001:0003a494       realloc                    1003b494 f   corelib1:COREDLL.dll
 0001:0003a4a4       free                       1003b4a4 f   corelib1:COREDLL.dll
 0001:0003a4b4       __rt_udiv                  1003b4b4 f   corelib1:COREDLL.dll
 0001:0003a4c4       strlen                     1003b4c4 f   corelib1:COREDLL.dll
 0001:0003a4d4       _vsnwprintf                1003b4d4 f   corelib1:COREDLL.dll
 0001:0003a4e4       _vsnwprintf_s              1003b4e4 f   corelib1:COREDLL.dll
 0001:0003a4f4       wcscpy                     1003b4f4 f   corelib1:COREDLL.dll
 0001:0003a504       _wcsdup                    1003b504 f   corelib1:COREDLL.dll
 0001:0003a514       wcsncpy                    1003b514 f   corelib1:COREDLL.dll
 0001:0003a524       _wcsicmp                   1003b524 f   corelib1:COREDLL.dll
 0001:0003a534       _wcsnicmp                  1003b534 f   corelib1:COREDLL.dll
 0001:0003a544       __security_gen_cookie2     1003b544 f   corelib1:COREDLL.dll
 0001:0003a554       __report_gsfailure         1003b554 f   corelib1:COREDLL.dll
 0001:0003a564       _msize                     1003b564 f   corelib1:COREDLL.dll
 0001:0003a574       DescriptorPhy              1003b574 f   usb_usbfn_mx25_topaz_v1:i_pdd.obj
 0001:0003a5cc       DescriptorVirtual          1003b5cc f   usb_usbfn_mx25_topaz_v1:i_pdd.obj
 0001:0003a624       ClearUsbstsUI              1003b624 f   usb_usbfn_mx25_topaz_v1:i_pdd.obj
 0001:0003a6a4       UfnPdd_PowerDown           1003b6a4 f   usb_usbfn_mx25_topaz_v1:i_pdd.obj
 0001:0003add8       UfnPdd_PowerUp             1003bdd8 f   usb_usbfn_mx25_topaz_v1:i_pdd.obj
 0001:0003b32c       UpdateDevicePower          1003c32c f   usb_usbfn_mx25_topaz_v1:i_pdd.obj
 0001:0003b638       SetupEvent                 1003c638 f   usb_usbfn_mx25_topaz_v1:i_pdd.obj
 0001:0003bda0       DumpDeviceState            1003cda0 f   usb_usbfn_mx25_topaz_v1:i_pdd.obj
 0001:0003c268       DumpInterruptSource        1003d268 f   usb_usbfn_mx25_topaz_v1:i_pdd.obj
 0001:0003c404       CopyFromUncachedBuffer     1003d404 f   usb_usbfn_mx25_topaz_v1:i_pdd.obj
 0001:0003c694       CheckEndpoint              1003d694 f   usb_usbfn_mx25_topaz_v1:i_pdd.obj
 0001:0003dc20       InterruptHandle            1003ec20 f   usb_usbfn_mx25_topaz_v1:i_pdd.obj
 0001:0003f164       UfnPdd_IssueTransfer       10040164 f   usb_usbfn_mx25_topaz_v1:i_pdd.obj
 0001:00040f5c       UfnPdd_AbortTransfer       10041f5c f   usb_usbfn_mx25_topaz_v1:i_pdd.obj
 0001:00041634       UfnPdd_StallEndpoint       10042634 f   usb_usbfn_mx25_topaz_v1:i_pdd.obj
 0001:000417f0       UfnPdd_ClearEndpointStall  100427f0 f   usb_usbfn_mx25_topaz_v1:i_pdd.obj
 0001:000419f4       UfnPdd_IsEndpointHalted    100429f4 f   usb_usbfn_mx25_topaz_v1:i_pdd.obj
 0001:00041bc4       UfnPdd_SendControlStatusHandshake 10042bc4 f   usb_usbfn_mx25_topaz_v1:i_pdd.obj
 0001:00042594       UfnPdd_InitiateRemoteWakeup 10043594 f   usb_usbfn_mx25_topaz_v1:i_pdd.obj
 0001:0004261c       SetPowerState              1004361c f   usb_usbfn_mx25_topaz_v1:i_pdd.obj
 0001:000429d8       UfnPdd_IOControl           100439d8 f   usb_usbfn_mx25_topaz_v1:i_pdd.obj
 0001:00042f60       UfnPdd_Deinit              10043f60 f   usb_usbfn_mx25_topaz_v1:i_pdd.obj
 0001:00042f90       UfnPdd_DeregisterDevice    10043f90 f   usb_usbfn_mx25_topaz_v1:i_pdd.obj
 0001:00042fb8       UfnPdd_Stop                10043fb8 f   usb_usbfn_mx25_topaz_v1:i_pdd.obj
 0001:000430e8       UfnPdd_DeinitEndpoint      100440e8 f   usb_usbfn_mx25_topaz_v1:i_pdd.obj
 0001:00043344       UfnPdd_InitEndpoint        10044344 f   usb_usbfn_mx25_topaz_v1:i_pdd.obj
 0001:000437cc       UfnPdd_SetAddress          100447cc f   usb_usbfn_mx25_topaz_v1:i_pdd.obj
 0001:00043840       UfnPdd_Start               10044840 f   usb_usbfn_mx25_topaz_v1:i_pdd.obj
 0001:00044524       UfnPdd_RegisterDevice      10045524 f   usb_usbfn_mx25_topaz_v1:i_pdd.obj
 0001:000449f8       UfnPdd_IsEndpointSupportable 100459f8 f   usb_usbfn_mx25_topaz_v1:i_pdd.obj
 0001:00044a94       UfnPdd_IsConfigurationSupportable 10045a94 f   usb_usbfn_mx25_topaz_v1:i_pdd.obj
 0001:00044dc0       UfnPdd_Init                10045dc0 f   usb_usbfn_mx25_topaz_v1:i_pdd.obj
 0001:00045614       UfnPdd_DllEntry            10046614 f   usb_usbfn_mx25_topaz_v1:i_pdd.obj
 0001:0004563c       GetDeviceRegistryParams    1004663c f   usb_usbfn_os_mx25_topaz_v1:i_registry.obj
 0001:000460f0       MmMapIoSpace               100470f0 f   ceddk:CEDDK.dll
 0001:00046100       TerminateProcess           10047100 f   coredll:COREDLL.dll
 0001:00046110       SetInterruptEvent          10047110 f   coredll:COREDLL.dll
 0001:00046120       CacheSync                  10047120 f   coredll:COREDLL.dll
 0001:00046130       UnlockPages                10047130 f   coredll:COREDLL.dll
 0001:00046140       CacheRangeFlush            10047140 f   coredll:COREDLL.dll
 0001:00046150       CeCloseCallerBuffer        10047150 f   coredll:COREDLL.dll
 0001:00046160       LockPages                  10047160 f   coredll:COREDLL.dll
 0001:00046170       CeOpenCallerBuffer         10047170 f   coredll:COREDLL.dll
 0001:00046180       wcstoul                    10047180 f   corelib1:COREDLL.dll
 0001:00046220       ??__Fcs@?1??get_lock@?$singleton@V?$free_list@$0GE@Vallocator@ce@@@ce@@$03V?$static_allocator@V?$free_list@$0GE@Vallocator@ce@@@ce@@$03@2@@ce@@KAAAVcritical_section@2@XZ@YAXXZ 10047220 f i usb_ufnmddbase_common_topaz_v1:ufnmdd.obj
 0001:0004636c       __IMPORT_DESCRIPTOR_CEDDK  1004736c     ceddk:CEDDK.dll
 0001:00046380       __IMPORT_DESCRIPTOR_COREDLL 10047380     coredll:COREDLL.dll
 0001:00046394       __IMPORT_DESCRIPTOR_CSPDDK 10047394     cspddk:CSPDDK.dll
 0001:000463a8       __NULL_IMPORT_DESCRIPTOR   100473a8     ceddk:CEDDK.dll
 0002:00000000       __imp_BusChildIoControl    10048000     ceddk:CEDDK.dll
 0002:00000004       __imp_CreateBusAccessHandle 10048004     ceddk:CEDDK.dll
 0002:00000008       __imp_CloseBusAccessHandle 10048008     ceddk:CEDDK.dll
 0002:0000000c       __imp_HalAllocateCommonBuffer 1004800c     ceddk:CEDDK.dll
 0002:00000010       __imp_HalFreeCommonBuffer  10048010     ceddk:CEDDK.dll
 0002:00000014       __imp_MmUnmapIoSpace       10048014     ceddk:CEDDK.dll
 0002:00000018       __imp_SetDevicePowerState  10048018     ceddk:CEDDK.dll
 0002:0000001c       __imp_HalSetBusDataByOffset 1004801c     ceddk:CEDDK.dll
 0002:00000020       __imp_HalGetBusDataByOffset 10048020     ceddk:CEDDK.dll
 0002:00000024       __imp_HalTranslateBusAddress 10048024     ceddk:CEDDK.dll
 0002:00000028       __imp_TranslateBusAddr     10048028     ceddk:CEDDK.dll
 0002:0000002c       __imp_HalTranslateSystemAddress 1004802c     ceddk:CEDDK.dll
 0002:00000030       __imp_TranslateSystemAddr  10048030     ceddk:CEDDK.dll
 0002:00000034       __imp_MmMapIoSpace         10048034     ceddk:CEDDK.dll
 0002:00000038       \177CEDDK_NULL_THUNK_DATA  10048038     ceddk:CEDDK.dll
 0002:0000003c       __imp_Sleep                1004803c     coredll:COREDLL.dll
 0002:00000040       __imp_InterlockedCompareExchange 10048040     coredll:COREDLL.dll
 0002:00000044       __imp_GetLastError         10048044     coredll:COREDLL.dll
 0002:00000048       __imp_MapViewOfFile        10048048     coredll:COREDLL.dll
 0002:0000004c       __imp_CreateFileMappingW   1004804c     coredll:COREDLL.dll
 0002:00000050       __imp_CloseHandle          10048050     coredll:COREDLL.dll
 0002:00000054       __imp_UnmapViewOfFile      10048054     coredll:COREDLL.dll
 0002:00000058       __imp_KernelIoControl      10048058     coredll:COREDLL.dll
 0002:0000005c       __imp_LeaveCriticalSection 1004805c     coredll:COREDLL.dll
 0002:00000060       __imp_EnterCriticalSection 10048060     coredll:COREDLL.dll
 0002:00000064       __imp_CeLogData            10048064     coredll:COREDLL.dll
 0002:00000068       __imp_StringCchLengthW     10048068     coredll:COREDLL.dll
 0002:0000006c       __imp_StringCchVPrintfW    1004806c     coredll:COREDLL.dll
 0002:00000070       __imp_OpenDeviceKey        10048070     coredll:COREDLL.dll
 0002:00000074       __imp_CreateEventW         10048074     coredll:COREDLL.dll
 0002:00000078       __imp_InitializeCriticalSection 10048078     coredll:COREDLL.dll
 0002:0000007c       __imp_LocalAlloc           1004807c     coredll:COREDLL.dll
 0002:00000080       __imp_RegOpenKeyExW        10048080     coredll:COREDLL.dll
 0002:00000084       __imp_LocalFree            10048084     coredll:COREDLL.dll
 0002:00000088       __imp_RegCloseKey          10048088     coredll:COREDLL.dll
 0002:0000008c       __imp_DeleteCriticalSection 1004808c     coredll:COREDLL.dll
 0002:00000090       __imp_SetLastError         10048090     coredll:COREDLL.dll
 0002:00000094       __imp_DisableThreadLibraryCalls 10048094     coredll:COREDLL.dll
 0002:00000098       __imp_RegisterDbgZones     10048098     coredll:COREDLL.dll
 0002:0000009c       __imp_OutputDebugStringW   1004809c     coredll:COREDLL.dll
 0002:000000a0       __imp___GetUserKData       100480a0     coredll:COREDLL.dll
 0002:000000a4       __imp_InterlockedIncrement 100480a4     coredll:COREDLL.dll
 0002:000000a8       __imp_InterlockedDecrement 100480a8     coredll:COREDLL.dll
 0002:000000ac       __imp_InterlockedExchange  100480ac     coredll:COREDLL.dll
 0002:000000b0       __imp_StringCchCopyNW      100480b0     coredll:COREDLL.dll
 0002:000000b4       __imp_StringCchCopyW       100480b4     coredll:COREDLL.dll
 0002:000000b8       __imp_StringCchPrintfW     100480b8     coredll:COREDLL.dll
 0002:000000bc       __imp_GetDeviceInformationByDeviceHandle 100480bc     coredll:COREDLL.dll
 0002:000000c0       __imp_EventModify          100480c0     coredll:COREDLL.dll
 0002:000000c4       __imp_LoadLibraryW         100480c4     coredll:COREDLL.dll
 0002:000000c8       __imp_RegQueryValueExW     100480c8     coredll:COREDLL.dll
 0002:000000cc       __imp_RegSetValueExW       100480cc     coredll:COREDLL.dll
 0002:000000d0       __imp_RegEnumKeyExW        100480d0     coredll:COREDLL.dll
 0002:000000d4       __imp_NKDbgPrintfW         100480d4     coredll:COREDLL.dll
 0002:000000d8       __imp_InterruptInitialize  100480d8     coredll:COREDLL.dll
 0002:000000dc       __imp_AllocPhysMem         100480dc     coredll:COREDLL.dll
 0002:000000e0       __imp_CeSetThreadPriority  100480e0     coredll:COREDLL.dll
 0002:000000e4       __imp_CreateThread         100480e4     coredll:COREDLL.dll
 0002:000000e8       __imp_FreePhysMem          100480e8     coredll:COREDLL.dll
 0002:000000ec       __imp_InterruptDisable     100480ec     coredll:COREDLL.dll
 0002:000000f0       __imp_ExitThread           100480f0     coredll:COREDLL.dll
 0002:000000f4       __imp_InterruptDone        100480f4     coredll:COREDLL.dll
 0002:000000f8       __imp_StringCchCatW        100480f8     coredll:COREDLL.dll
 0002:000000fc       __imp_NKvDbgPrintfW        100480fc     coredll:COREDLL.dll
 0002:00000100       __imp_ReadFile             10048100     coredll:COREDLL.dll
 0002:00000104       __imp_GetFileSize          10048104     coredll:COREDLL.dll
 0002:00000108       __imp_CreateFileW          10048108     coredll:COREDLL.dll
 0002:0000010c       __imp_ReportEventW         1004810c     coredll:COREDLL.dll
 0002:00000110       __imp_LoadStringW          10048110     coredll:COREDLL.dll
 0002:00000114       __imp_FreeLibrary          10048114     coredll:COREDLL.dll
 0002:00000118       __imp_GetProcAddressW      10048118     coredll:COREDLL.dll
 0002:0000011c       __imp_LoadDriver           1004811c     coredll:COREDLL.dll
 0002:00000120       __imp_ActivateDeviceEx     10048120     coredll:COREDLL.dll
 0002:00000124       __imp_GetTickCount         10048124     coredll:COREDLL.dll
 0002:00000128       __imp_DeactivateDevice     10048128     coredll:COREDLL.dll
 0002:0000012c       __imp_GetDeviceHandleFromContext 1004812c     coredll:COREDLL.dll
 0002:00000130       __imp_CeOpenCallerBuffer   10048130     coredll:COREDLL.dll
 0002:00000134       __imp_LockPages            10048134     coredll:COREDLL.dll
 0002:00000138       __imp_CeCloseCallerBuffer  10048138     coredll:COREDLL.dll
 0002:0000013c       __imp_CacheRangeFlush      1004813c     coredll:COREDLL.dll
 0002:00000140       __imp_??2@YAPAXI@Z         10048140     corelib1:COREDLL.dll
 0002:00000144       __imp___C_specific_handler 10048144     corelib1:COREDLL.dll
 0002:00000148       __imp_??3@YAXPAX@Z         10048148     corelib1:COREDLL.dll
 0002:0000014c       __imp_memcpy               1004814c     corelib1:COREDLL.dll
 0002:00000150       __imp__purecall            10048150     corelib1:COREDLL.dll
 0002:00000154       __imp_memset               10048154     corelib1:COREDLL.dll
 0002:00000158       __imp_wcslen               10048158     corelib1:COREDLL.dll
 0002:0000015c       __imp_??_V@YAXPAX@Z        1004815c     corelib1:COREDLL.dll
 0002:00000160       __imp_??_U@YAPAXI@Z        10048160     corelib1:COREDLL.dll
 0002:00000164       __imp_malloc               10048164     corelib1:COREDLL.dll
 0002:00000168       __imp_realloc              10048168     corelib1:COREDLL.dll
 0002:0000016c       __imp_free                 1004816c     corelib1:COREDLL.dll
 0002:00000170       __imp___rt_udiv            10048170     corelib1:COREDLL.dll
 0002:00000174       __imp_strlen               10048174     corelib1:COREDLL.dll
 0002:00000178       __imp__vsnwprintf          10048178     corelib1:COREDLL.dll
 0002:0000017c       __imp__vsnwprintf_s        1004817c     corelib1:COREDLL.dll
 0002:00000180       __imp_wcscpy               10048180     corelib1:COREDLL.dll
 0002:00000184       __imp__wcsdup              10048184     corelib1:COREDLL.dll
 0002:00000188       __imp_wcsncpy              10048188     corelib1:COREDLL.dll
 0002:0000018c       __imp__wcsicmp             1004818c     corelib1:COREDLL.dll
 0002:00000190       __imp__wcsnicmp            10048190     corelib1:COREDLL.dll
 0002:00000194       __imp___security_gen_cookie2 10048194     corelib1:COREDLL.dll
 0002:00000198       __imp___report_gsfailure   10048198     corelib1:COREDLL.dll
 0002:0000019c       __imp__msize               1004819c     corelib1:COREDLL.dll
 0002:000001a0       __imp_WaitForSingleObject  100481a0     coredll:COREDLL.dll
 0002:000001a4       __imp_TerminateProcess     100481a4     coredll:COREDLL.dll
 0002:000001a8       __imp_SetInterruptEvent    100481a8     coredll:COREDLL.dll
 0002:000001ac       __imp_CacheSync            100481ac     coredll:COREDLL.dll
 0002:000001b0       __imp_UnlockPages          100481b0     coredll:COREDLL.dll
 0002:000001b4       __imp_wcstoul              100481b4     corelib1:COREDLL.dll
 0002:000001b8       \177COREDLL_NULL_THUNK_DATA 100481b8     coredll:COREDLL.dll
 0002:000001bc       __imp_DDKClockGetGatingMode 100481bc     cspddk:CSPDDK.dll
 0002:000001c0       __imp_DDKClockSetGatingMode 100481c0     cspddk:CSPDDK.dll
 0002:000001c4       __imp_DDKClockConfigBaud   100481c4     cspddk:CSPDDK.dll
 0002:000001c8       \177CSPDDK_NULL_THUNK_DATA 100481c8     cspddk:CSPDDK.dll
 0002:000001d0       dpCurSettings              100481d0     usb_usbfn_os_mx25_topaz_v1:i_os.obj
 0002:00000614       g_funcAlloc                10048614     ceosutil:utilmem.obj
 0002:00000618       g_funcFree                 10048618     ceosutil:utilmem.obj
 0002:0000061c       g_funcRealloc              1004861c     ceosutil:utilmem.obj
 0002:00000620       g_funcDebugOut             10048620     ceosutil:svsutil.obj
 0002:00000624       __security_cookie          10048624     corelib0:seccinit.obj
 0002:00000628       __security_cookie_complement 10048628     corelib0:seccinit.obj
 0002:00000640       m_hUSBClockGatingHandle    10048640     i_usbclock.obj
 0002:00000644       pUSBClkGating              10048644     i_usbclock.obj
 0002:00000650       ?s_rgbBuffer@?$CTransferQueue@VCUfnMddTransfer@@@@0PAEA 10048650     usb_ufnmddbase_common_topaz_v1:ufnmdd.obj
 0002:00000674       ?s_pListStructAllocator@?$CTransferQueue@VCUfnMddTransfer@@@@0PAV?$fixed_block_allocator@$0BE@@ce@@A 10048674     usb_ufnmddbase_common_topaz_v1:ufnmdd.obj
 0002:00000678       ?cs@?1??get_lock@?$singleton@V?$free_list@$0GE@Vallocator@ce@@@ce@@$03V?$static_allocator@V?$free_list@$0GE@Vallocator@ce@@@ce@@$03@2@@ce@@KAAAVcritical_section@3@XZ@4V43@A 10048678     usb_ufnmddbase_common_topaz_v1:ufnmdd.obj
 0002:0000068c       ??_B?1??get_lock@?$singleton@V?$free_list@$0GE@Vallocator@ce@@@ce@@$03V?$static_allocator@V?$free_list@$0GE@Vallocator@ce@@@ce@@$03@2@@ce@@KAAAVcritical_section@2@XZ@51 1004868c     usb_ufnmddbase_common_topaz_v1:ufnmdd.obj
 0002:00000690       ?_factory@?$singleton@V?$free_list@$0GE@Vallocator@ce@@@ce@@$03V?$static_allocator@V?$free_list@$0GE@Vallocator@ce@@@ce@@$03@2@@ce@@1Ulock_factory@12@A 10048690     usb_ufnmddbase_common_topaz_v1:ufnmdd.obj
 0002:00000694       g_pvAllocData              10048694     ceosutil:utilmem.obj
 0002:00000698       g_pvFreeData               10048698     ceosutil:utilmem.obj
 0002:000006b0       g_pvDebugData              100486b0     ceosutil:svsutil.obj
 0002:000006b8       _exitflag                  100486b8     corelib0:cexit.obj
 0002:000006c0       g_csRegister               100486c0     <common>
 0002:000006d4       __onexitend                100486d4     <common>
 0002:000006d8       __onexitbegin              100486d8     <common>
 0002:000006dc       g_pcsExit                  100486dc     <common>

 entry point at        0001:00039b98

 Static symbols

 0001:0000cd78       InitializeMux              1000dd78 f   hwinit.obj
 0001:0000cda0       SelectUSBCore              1000dda0 f   hwinit.obj
 0001:0000ce04       InitializeTransceiver      1000de04 f   hwinit.obj
 0001:0000d88c       USBClockSet                1000e88c f   i_usbclock.obj
 0001:0000e8d4       CeLogMsg                   1000f8d4 f   usb_ufnmddbase_common_topaz_v1:ufnmdd.obj
 0001:0000e9b0       ?ResetPipeStatusTable@@YAXPAUUFN_MDD_CONTEXT@@@Z 1000f9b0 f   usb_ufnmddbase_common_topaz_v1:ufnmdd.obj
 0001:00011eec       ?FreeContext@@YAXPAUUFN_MDD_CONTEXT@@@Z 10012eec f   usb_ufnmddbase_common_topaz_v1:ufnmdd.obj
 0001:000121e4       ?IsPddInterfaceInfoValid@@YAHPAU_UFN_PDD_INTERFACE_INFO@@@Z 100131e4 f   usb_ufnmddbase_common_topaz_v1:ufnmdd.obj
 0001:0001299c       ?ValidateBusContext@@YAXPAUUFN_MDD_BUS_OPEN_CONTEXT@@@Z 1001399c f   usb_ufnmddbase_common_topaz_v1:ufnmdd.obj
 0001:00016f54       CeLogMsg                   10017f54 f   usb_ufnmddbase_common_topaz_v1:pipe.obj
 0001:000208f4       CeLogMsg                   100218f4 f   usb_ufnmddbase_common_topaz_v1:descript.obj
 0001:00021348       ?FillBuffer@@YAKPAPAEPAKPBXK@Z 10022348 f   usb_ufnmddbase_common_topaz_v1:descript.obj
 0001:00024d80       ?CopyExtendedDesc@@YAKPAPAXPAKPAXK@Z 10025d80 f   usb_ufnmddbase_common_topaz_v1:descript.obj
 0001:00027104       CeLogMsg                   10028104 f   usb_ufnmddbase_common_topaz_v1:transfer.obj
 0001:00027be4       CeLogMsg                   10028be4 f   usb_ufnmddbase_common_topaz_v1:ufnbus.obj
 0001:0002887c       ?AllocEndpoints@@YAKPAUUFN_MDD_CONTEXT@@@Z 1002987c f   usb_ufnmddbase_common_topaz_v1:ufnbus.obj
 0001:0002a85c       ?GetUfnDescription@@YAHPAUHKEY__@@PAGK@Z 1002b85c f   usb_ufnmddbase_common_topaz_v1:ufnbus.obj
 0001:0002af28       ?FreePipes@@YAXPAUUFN_MDD_CONTEXT@@@Z 1002bf28 f   usb_ufnmddbase_common_topaz_v1:ufnbus.obj
 0001:0002d28c       CeLogMsg                   1002e28c f   usb_ufnmddbase_common_topaz_v1:enum.obj
 0001:0002d368       ?ProcessRequest@@YA?AW4CONTROL_RESPONSE@@PAUUFN_MDD_CONTEXT@@U_USB_DEVICE_REQUEST@@K@Z 1002e368 f   usb_ufnmddbase_common_topaz_v1:enum.obj
 0001:0002d6c0       ?ProcessGetDescriptor@@YA?AW4CONTROL_RESPONSE@@PAUUFN_MDD_CONTEXT@@U_USB_DEVICE_REQUEST@@K@Z 1002e6c0 f   usb_ufnmddbase_common_topaz_v1:enum.obj
 0001:0002d824       ?SetupTx@@YAXPAUUFN_MDD_CONTEXT@@PAXKK@Z 1002e824 f   usb_ufnmddbase_common_topaz_v1:enum.obj
 0001:0002da8c       ?EnumTransferComplete@@YAKPAX@Z 1002ea8c f   usb_ufnmddbase_common_topaz_v1:enum.obj
 0001:0002dd00       ?ProcessSetDescriptor@@YA?AW4CONTROL_RESPONSE@@PAUUFN_MDD_CONTEXT@@U_USB_DEVICE_REQUEST@@K@Z 1002ed00 f   usb_ufnmddbase_common_topaz_v1:enum.obj
 0001:0002dd28       ?ProcessGetConfiguration@@YA?AW4CONTROL_RESPONSE@@PAUUFN_MDD_CONTEXT@@U_USB_DEVICE_REQUEST@@K@Z 1002ed28 f   usb_ufnmddbase_common_topaz_v1:enum.obj
 0001:0002df74       ?ProcessGetInterface@@YA?AW4CONTROL_RESPONSE@@PAUUFN_MDD_CONTEXT@@U_USB_DEVICE_REQUEST@@K@Z 1002ef74 f   usb_ufnmddbase_common_topaz_v1:enum.obj
 0001:0002e1b0       ?ProcessGetStatus@@YA?AW4CONTROL_RESPONSE@@PAUUFN_MDD_CONTEXT@@U_USB_DEVICE_REQUEST@@K@Z 1002f1b0 f   usb_ufnmddbase_common_topaz_v1:enum.obj
 0001:0002e678       ?ProcessSetAddress@@YA?AW4CONTROL_RESPONSE@@PAUUFN_MDD_CONTEXT@@U_USB_DEVICE_REQUEST@@K@Z 1002f678 f   usb_ufnmddbase_common_topaz_v1:enum.obj
 0001:0002e8c4       ?ProcessSetConfiguration@@YA?AW4CONTROL_RESPONSE@@PAUUFN_MDD_CONTEXT@@U_USB_DEVICE_REQUEST@@K@Z 1002f8c4 f   usb_ufnmddbase_common_topaz_v1:enum.obj
 0001:0002eda0       ?ProcessSetInterface@@YA?AW4CONTROL_RESPONSE@@PAUUFN_MDD_CONTEXT@@U_USB_DEVICE_REQUEST@@K@Z 1002fda0 f   usb_ufnmddbase_common_topaz_v1:enum.obj
 0001:0002f150       ?ProcessClearFeature@@YA?AW4CONTROL_RESPONSE@@PAUUFN_MDD_CONTEXT@@U_USB_DEVICE_REQUEST@@K@Z 10030150 f   usb_ufnmddbase_common_topaz_v1:enum.obj
 0001:0002f454       ?ProcessSetFeature@@YA?AW4CONTROL_RESPONSE@@PAUUFN_MDD_CONTEXT@@U_USB_DEVICE_REQUEST@@K@Z 10030454 f   usb_ufnmddbase_common_topaz_v1:enum.obj
 0001:0002f9cc       ?ProcessSyncFrame@@YA?AW4CONTROL_RESPONSE@@PAUUFN_MDD_CONTEXT@@U_USB_DEVICE_REQUEST@@K@Z 100309cc f   usb_ufnmddbase_common_topaz_v1:enum.obj
 0001:0002f9f4       ?CloseAllPipesExceptEndpointZero@@YAXPAUUFN_MDD_CONTEXT@@@Z 100309f4 f   usb_ufnmddbase_common_topaz_v1:enum.obj
 0001:0002fb90       ?IgnoreNotification@@YAHPAUUFN_MDD_CONTEXT@@KK@Z 10030b90 f   usb_ufnmddbase_common_topaz_v1:enum.obj
 0001:0002fc40       ?IgnoreNotificationCheck@@YAHPAUUFN_MDD_CONTEXT@@@Z 10030c40 f   usb_ufnmddbase_common_topaz_v1:enum.obj
 0001:00030584       CeLogMsg                   10031584 f   usb_usbfn_os_mx25_topaz_v1:i_os.obj
 0001:000329c4       ?svsutil_CompactFixed_Worker@@YAXPAUFixedMemDescr@@@Z 100339c4 f   ceosutil:utilmemf.obj
 0001:00033bb8       ?svsutil_DebugOut@@YAHPAXPAGZZ 10034bb8 f   ceosutil:svsutil.obj
 0001:00039e7c       lockexit                   1003ae7c f   corelib0:onexit.obj
 0001:00039f18       unlockexit                 1003af18 f   corelib0:onexit.obj
 0001:00039f44       _onexit_nolock             1003af44 f   corelib0:onexit.obj
 0001:0003a19c       doexit                     1003b19c f   corelib0:cexit.obj
 0001:0003acfc       CeLogMsg                   1003bcfc f   usb_usbfn_mx25_topaz_v1:i_pdd.obj
 0001:0003b974       GetSetupPacket             1003c974 f   usb_usbfn_mx25_topaz_v1:i_pdd.obj
 0001:0003e87c       HandleUSBReset             1003f87c f   usb_usbfn_mx25_topaz_v1:i_pdd.obj
 0001:0003ed7c       DevStatEvent               1003fd7c f   usb_usbfn_mx25_topaz_v1:i_pdd.obj
 0001:0003ee44       USBControllerRun           1003fe44 f   usb_usbfn_mx25_topaz_v1:i_pdd.obj
 0001:00040778       BuildTdBufferList          10041778 f   usb_usbfn_mx25_topaz_v1:i_pdd.obj
 0001:000414c8       FlushEndpoint              100424c8 f   usb_usbfn_mx25_topaz_v1:i_pdd.obj
 0001:00041d50       PrimeQh0ForZeroTransfer    10042d50 f   usb_usbfn_mx25_topaz_v1:i_pdd.obj
 0001:00042770       SetDeviceTestMode          10043770 f   usb_usbfn_mx25_topaz_v1:i_pdd.obj
 0001:00043aec       InitQh0                    10044aec f   usb_usbfn_mx25_topaz_v1:i_pdd.obj
 0001:00044d38       Log2                       10045d38 f   usb_usbfn_mx25_topaz_v1:i_pdd.obj
 0001:000458fc       GetStringParam             100468fc f   usb_usbfn_os_mx25_topaz_v1:i_registry.obj
 0001:00045b78       GetDWordParam              10046b78 f   usb_usbfn_os_mx25_topaz_v1:i_registry.obj
 0001:00045c44       GetMultiDWordParam         10046c44 f   usb_usbfn_os_mx25_topaz_v1:i_registry.obj
 0001:00045f30       GetBinParam                10046f30 f   usb_usbfn_os_mx25_topaz_v1:i_registry.obj
 0001:00046190       ??__E?_factory@?$singleton@V?$free_list@$0GE@Vallocator@ce@@@ce@@$03V?$static_allocator@V?$free_list@$0GE@Vallocator@ce@@@ce@@$03@2@@ce@@1Ulock_factory@12@A@@YAXXZ 10047190 f   usb_ufnmddbase_common_topaz_v1:ufnmdd.obj
 0001:000461a8       ??__E?_factory@?$singleton@V?$free_list@$0GE@Vallocator@ce@@@ce@@$03V?$static_allocator@V?$free_list@$0GE@Vallocator@ce@@@ce@@$03@2@@ce@@1Ulock_factory@12@A@@YAXXZ 100471a8 f   usb_ufnmddbase_common_topaz_v1:pipe.obj
 0001:000461c0       ??__E?_factory@?$singleton@V?$free_list@$0GE@Vallocator@ce@@@ce@@$03V?$static_allocator@V?$free_list@$0GE@Vallocator@ce@@@ce@@$03@2@@ce@@1Ulock_factory@12@A@@YAXXZ 100471c0 f   usb_ufnmddbase_common_topaz_v1:descript.obj
 0001:000461d8       ??__E?_factory@?$singleton@V?$free_list@$0GE@Vallocator@ce@@@ce@@$03V?$static_allocator@V?$free_list@$0GE@Vallocator@ce@@@ce@@$03@2@@ce@@1Ulock_factory@12@A@@YAXXZ 100471d8 f   usb_ufnmddbase_common_topaz_v1:transfer.obj
 0001:000461f0       ??__E?_factory@?$singleton@V?$free_list@$0GE@Vallocator@ce@@@ce@@$03V?$static_allocator@V?$free_list@$0GE@Vallocator@ce@@@ce@@$03@2@@ce@@1Ulock_factory@12@A@@YAXXZ 100471f0 f   usb_ufnmddbase_common_topaz_v1:ufnbus.obj
 0001:00046208       ??__E?_factory@?$singleton@V?$free_list@$0GE@Vallocator@ce@@@ce@@$03V?$static_allocator@V?$free_list@$0GE@Vallocator@ce@@@ce@@$03@2@@ce@@1Ulock_factory@12@A@@YAXXZ 10047208 f   usb_ufnmddbase_common_topaz_v1:enum.obj
